Archive member included because of file (symbol)

c:/program files (x86)/microchip/xc32/v1.10/bin/../lib/gcc/pic32mx/4.5.1/../../../../pic32mx/lib/size\libmchp_peripheral.a(open_core_timer_lib.o)
                              build/default/production/_ext/365611741/system_services.o (OpenCoreTimer)
c:/program files (x86)/microchip/xc32/v1.10/bin/../lib/gcc/pic32mx/4.5.1/../../../../pic32mx/lib/size\libmchp_peripheral_32MX795F512L.a(soft_reset_lib.o)
                              build/default/production/_ext/365611741/system_services.o (SoftReset)
c:/program files (x86)/microchip/xc32/v1.10/bin/../lib/gcc/pic32mx/4.5.1/../../../../pic32mx/lib/size\libmchp_peripheral_32MX795F512L.a(pcache.o)
                              build/default/production/_ext/365611741/system_services.o (CheKseg0CacheOn)
c:/program files (x86)/microchip/xc32/v1.10/bin/../lib/gcc/pic32mx/4.5.1/../../../../pic32mx/lib/size\libmchp_peripheral_32MX795F512L.a(int_disable_interrupts_lib.o)
                              build/default/production/_ext/365611741/system_services.o (INTDisableInterrupts)
c:/program files (x86)/microchip/xc32/v1.10/bin/../lib/gcc/pic32mx/4.5.1/../../../../pic32mx/lib/size\libmchp_peripheral_32MX795F512L.a(int_restore_interrupts_lib.o)
                              build/default/production/_ext/365611741/system_services.o (INTRestoreInterrupts)
c:/program files (x86)/microchip/xc32/v1.10/bin/../lib/gcc/pic32mx/4.5.1/../../../../pic32mx/lib/size\libmchp_peripheral_32MX795F512L.a(int_enable_mv_int_lib.o)
                              build/default/production/_ext/365611741/system_services.o (INTEnableSystemMultiVectoredInt)
c:/program files (x86)/microchip/xc32/v1.10/bin/../lib/gcc/pic32mx/4.5.1/../../../../pic32mx/lib/size\libmchp_peripheral_32MX795F512L.a(int_tbl_lib.o)
                              build/default/production/_ext/365611741/system_services.o (INTClearFlag)
c:/program files (x86)/microchip/xc32/v1.10/bin/../lib/gcc/pic32mx/4.5.1/../../../../pic32mx/lib/size\libmchp_peripheral_32MX795F512L.a(rtcc_init_lib.o)
                              build/default/production/_ext/365611741/system_services.o (RtccInit)
c:/program files (x86)/microchip/xc32/v1.10/bin/../lib/gcc/pic32mx/4.5.1/../../../../pic32mx/lib/size\libmchp_peripheral_32MX795F512L.a(rtcc_open_lib.o)
                              build/default/production/_ext/365611741/system_services.o (RtccOpen)
c:/program files (x86)/microchip/xc32/v1.10/bin/../lib/gcc/pic32mx/4.5.1/../../../../pic32mx/lib/size\libmchp_peripheral_32MX795F512L.a(spi_chn_data_rdy_lib.o)
                              build/default/production/_ext/792872985/drv_spi.o (SpiChnDataRdy)
c:/program files (x86)/microchip/xc32/v1.10/bin/../lib/gcc/pic32mx/4.5.1/../../../../pic32mx/lib/size\libmchp_peripheral_32MX795F512L.a(spi_chn_getc_lib.o)
                              build/default/production/_ext/792872985/drv_spi.o (SpiChnReadC)
c:/program files (x86)/microchip/xc32/v1.10/bin/../lib/gcc/pic32mx/4.5.1/../../../../pic32mx/lib/size\libmchp_peripheral_32MX795F512L.a(spi_chn_open_lib.o)
                              build/default/production/_ext/792872985/drv_spi.o (SpiChnOpen)
c:/program files (x86)/microchip/xc32/v1.10/bin/../lib/gcc/pic32mx/4.5.1/../../../../pic32mx/lib/size\libmchp_peripheral_32MX795F512L.a(spi_chn_putc_lib.o)
                              build/default/production/_ext/792872985/drv_spi.o (SpiChnWriteC)
c:/program files (x86)/microchip/xc32/v1.10/bin/../lib/gcc/pic32mx/4.5.1/../../../../pic32mx/lib/size\libmchp_peripheral_32MX795F512L.a(spi_chn_tx_buff_empty_lib.o)
                              build/default/production/_ext/792872985/drv_spi.o (SpiChnTxBuffEmpty)
c:/program files (x86)/microchip/xc32/v1.10/bin/../lib/gcc/pic32mx/4.5.1/../../../../pic32mx/lib/size\libmchp_peripheral_32MX795F512L.a(spi_io_tbl_libp.o)
                              c:/program files (x86)/microchip/xc32/v1.10/bin/../lib/gcc/pic32mx/4.5.1/../../../../pic32mx/lib/size\libmchp_peripheral_32MX795F512L.a(spi_chn_open_lib.o) (_SpiIoTbl)
c:/program files (x86)/microchip/xc32/v1.10/bin/../lib/gcc/pic32mx/4.5.1/../../../../pic32mx/lib/size\libmchp_peripheral_32MX795F512L.a(spi_map_tbl_libp.o)
                              c:/program files (x86)/microchip/xc32/v1.10/bin/../lib/gcc/pic32mx/4.5.1/../../../../pic32mx/lib/size\libmchp_peripheral_32MX795F512L.a(spi_chn_data_rdy_lib.o) (_SpiMapTbl)
c:/program files (x86)/microchip/xc32/v1.10/bin/../lib/gcc/pic32mx/4.5.1/../../../../pic32mx/lib/size\libmchp_peripheral_32MX795F512L.a(port_set_pins_digital_in_lib.o)
                              c:/program files (x86)/microchip/xc32/v1.10/bin/../lib/gcc/pic32mx/4.5.1/../../../../pic32mx/lib/size\libmchp_peripheral_32MX795F512L.a(spi_chn_open_lib.o) (PORTSetPinsDigitalIn)
c:/program files (x86)/microchip/xc32/v1.10/bin/../lib/gcc/pic32mx/4.5.1/../../../../pic32mx/lib/size\libmchp_peripheral_32MX795F512L.a(port_set_pins_digital_out_lib.o)
                              c:/program files (x86)/microchip/xc32/v1.10/bin/../lib/gcc/pic32mx/4.5.1/../../../../pic32mx/lib/size\libmchp_peripheral_32MX795F512L.a(spi_chn_open_lib.o) (PORTSetPinsDigitalOut)
c:/program files (x86)/microchip/xc32/v1.10/bin/../lib/gcc/pic32mx/4.5.1/../../../../pic32mx/lib/size\libmchp_peripheral_32MX795F512L.a(_ports_tbl_libp.o)
                              c:/program files (x86)/microchip/xc32/v1.10/bin/../lib/gcc/pic32mx/4.5.1/../../../../pic32mx/lib/size\libmchp_peripheral_32MX795F512L.a(port_set_pins_digital_in_lib.o) (PortRegTbl)
c:/program files (x86)/microchip/xc32/v1.10/bin/../lib/gcc/pic32mx/4.5.1/../../../../pic32mx/lib/size\libmchp_peripheral_32MX795F512L.a(int_enable_interrupts_lib.o)
                              c:/program files (x86)/microchip/xc32/v1.10/bin/../lib/gcc/pic32mx/4.5.1/../../../../pic32mx/lib/size\libmchp_peripheral_32MX795F512L.a(int_enable_mv_int_lib.o) (INTEnableInterrupts)
c:/program files (x86)/microchip/xc32/v1.10/bin/../lib/gcc/pic32mx/4.5.1/../../../../pic32mx/lib/size\libmchp_peripheral_32MX795F512L.a(_rtcc_wait_clock_off_lib.o)
                              c:/program files (x86)/microchip/xc32/v1.10/bin/../lib/gcc/pic32mx/4.5.1/../../../../pic32mx/lib/size\libmchp_peripheral_32MX795F512L.a(rtcc_init_lib.o) (_RtccWaitClockOff)
c:/program files (x86)/microchip/xc32/v1.10/bin/../lib/gcc/pic32mx/4.5.1/../../../../pic32mx/lib/size\libmchp_peripheral_32MX795F512L.a(read_core_timer_lib.o)
                              c:/program files (x86)/microchip/xc32/v1.10/bin/../lib/gcc/pic32mx/4.5.1/../../../../pic32mx/lib/size\libmchp_peripheral_32MX795F512L.a(_rtcc_wait_clock_off_lib.o) (ReadCoreTimer)
c:/program files (x86)/microchip/xc32/v1.10/bin/../lib/gcc/pic32mx/4.5.1/size\libgcc.a(_udivdi3.o)
                              build/default/production/_ext/101875047/big_int.o (__udivdi3)
c:/program files (x86)/microchip/xc32/v1.10/bin/../lib/gcc/pic32mx/4.5.1/../../../../pic32mx/lib/size\libpic32.a(memcmp.o)
                              build/default/production/_ext/97638081/mpfs2.o (memcmp)
c:/program files (x86)/microchip/xc32/v1.10/bin/../lib/gcc/pic32mx/4.5.1/../../../../pic32mx/lib/size\libpic32.a(memcpy.o)
                              build/default/production/_ext/101875047/hashes.o (memcpy)
c:/program files (x86)/microchip/xc32/v1.10/bin/../lib/gcc/pic32mx/4.5.1/../../../../pic32mx/lib/size\libpic32.a(memset.o)
                              build/default/production/_ext/365611741/system_services.o (memset)
c:/program files (x86)/microchip/xc32/v1.10/bin/../lib/gcc/pic32mx/4.5.1/../../../../pic32mx/lib/size\libpic32.a(strcmp.o)
                              build/default/production/_ext/365611741/system_command.o (strcmp)
c:/program files (x86)/microchip/xc32/v1.10/bin/../lib/gcc/pic32mx/4.5.1/../../../../pic32mx/lib/size\libpic32.a(strcpy.o)
                              build/default/production/_ext/365611741/system_command.o (strcpy)
c:/program files (x86)/microchip/xc32/v1.10/bin/../lib/gcc/pic32mx/4.5.1/../../../../pic32mx/lib/size\libpic32.a(strlen.o)
                              build/default/production/_ext/101875047/helpers.o (strlen)
c:/program files (x86)/microchip/xc32/v1.10/bin/../lib/gcc/pic32mx/4.5.1/../../../../pic32mx/lib/size\libpic32.a(default-bootstrap-exception-handler.o)
                              c:/program files (x86)/microchip/xc32/v1.10/bin/../lib/gcc/pic32mx/4.5.1/../../../../pic32mx/lib/size/crt0.o (_bootstrap_exception_handler)
c:/program files (x86)/microchip/xc32/v1.10/bin/../lib/gcc/pic32mx/4.5.1/../../../../pic32mx/lib/size\libpic32.a(default-on-reset.o)
                              c:/program files (x86)/microchip/xc32/v1.10/bin/../lib/gcc/pic32mx/4.5.1/../../../../pic32mx/lib/size/crt0.o (_on_reset)
c:/program files (x86)/microchip/xc32/v1.10/bin/../lib/gcc/pic32mx/4.5.1/../../../../pic32mx/lib/size\libpic32.a(default-on-bootstrap.o)
                              c:/program files (x86)/microchip/xc32/v1.10/bin/../lib/gcc/pic32mx/4.5.1/../../../../pic32mx/lib/size/crt0.o (_on_bootstrap)
c:/program files (x86)/microchip/xc32/v1.10/bin/../lib/gcc/pic32mx/4.5.1/../../../../pic32mx/lib/size\libpic32.a(default-nmi-handler.o)
                              c:/program files (x86)/microchip/xc32/v1.10/bin/../lib/gcc/pic32mx/4.5.1/../../../../pic32mx/lib/size/crt0.o (_nmi_handler)
c:/program files (x86)/microchip/xc32/v1.10/bin/../lib/gcc/pic32mx/4.5.1/../../../../pic32mx/lib/size\libpic32.a(errno.o)
                              build/default/production/_ext/97638081/sys_fs.o (errno)
c:/program files (x86)/microchip/xc32/v1.10/bin/../lib/gcc/pic32mx/4.5.1/../../../../pic32mx/lib/size\libpic32.a(general-exception.o)
                              c:/program files (x86)/microchip/xc32/v1.10/bin/../lib/gcc/pic32mx/4.5.1/../../../../pic32mx/lib/size/crt0.o (_general_exception_context)
c:/program files (x86)/microchip/xc32/v1.10/bin/../lib/gcc/pic32mx/4.5.1/../../../../pic32mx/lib/size\libc.a(atoi.o)
                              build/default/production/_ext/334706090/wf_commands.o (atoi)
c:/program files (x86)/microchip/xc32/v1.10/bin/../lib/gcc/pic32mx/4.5.1/../../../../pic32mx/lib/size\libc.a(atol.o)
                              build/default/production/_ext/427700826/http2.o (atol)
c:/program files (x86)/microchip/xc32/v1.10/bin/../lib/gcc/pic32mx/4.5.1/../../../../pic32mx/lib/size\libc.a(ctype.o)
                              build/default/production/_ext/427700826/tcpip_helpers.o (_ctype)
c:/program files (x86)/microchip/xc32/v1.10/bin/../lib/gcc/pic32mx/4.5.1/../../../../pic32mx/lib/size\libc.a(malloc.o)
                              build/default/production/_ext/365611741/system_services.o (malloc)
c:/program files (x86)/microchip/xc32/v1.10/bin/../lib/gcc/pic32mx/4.5.1/../../../../pic32mx/lib/size\libc.a(rand.o)
                              build/default/production/_ext/427700826/dhcp.o (rand)
c:/program files (x86)/microchip/xc32/v1.10/bin/../lib/gcc/pic32mx/4.5.1/../../../../pic32mx/lib/size\libc.a(strcat.o)
                              build/default/production/_ext/1472/ping_demo.o (strcat)
c:/program files (x86)/microchip/xc32/v1.10/bin/../lib/gcc/pic32mx/4.5.1/../../../../pic32mx/lib/size\libc.a(strchr.o)
                              build/default/production/_ext/97638081/sys_fs.o (strchr)
c:/program files (x86)/microchip/xc32/v1.10/bin/../lib/gcc/pic32mx/4.5.1/../../../../pic32mx/lib/size\libc.a(strncat.o)
                              build/default/production/_ext/1472/tcp6_demo_app.o (strncat)
c:/program files (x86)/microchip/xc32/v1.10/bin/../lib/gcc/pic32mx/4.5.1/../../../../pic32mx/lib/size\libc.a(strncmp.o)
                              build/default/production/_ext/97638081/sys_fs.o (strncmp)
c:/program files (x86)/microchip/xc32/v1.10/bin/../lib/gcc/pic32mx/4.5.1/../../../../pic32mx/lib/size\libc.a(strncpy.o)
                              build/default/production/_ext/101875047/helpers.o (strncpy)
c:/program files (x86)/microchip/xc32/v1.10/bin/../lib/gcc/pic32mx/4.5.1/../../../../pic32mx/lib/size\libc.a(strrchr.o)
                              build/default/production/_ext/97638081/sys_fs.o (strrchr)
c:/program files (x86)/microchip/xc32/v1.10/bin/../lib/gcc/pic32mx/4.5.1/../../../../pic32mx/lib/size\libc.a(strstr.o)
                              build/default/production/_ext/97638081/sys_fs.o (strstr)
c:/program files (x86)/microchip/xc32/v1.10/bin/../lib/gcc/pic32mx/4.5.1/../../../../pic32mx/lib/size\libc.a(strtol.o)
                              build/default/production/_ext/1472/tcp6_demo_app.o (strtol)
c:/program files (x86)/microchip/xc32/v1.10/bin/../lib/gcc/pic32mx/4.5.1/../../../../pic32mx/lib/size\libc.a(snprintf_cdnopsuxX.eo)
                              build/default/production/_ext/365611741/system_debug.o (_snprintf_cdnopsuxX)
c:/program files (x86)/microchip/xc32/v1.10/bin/../lib/gcc/pic32mx/4.5.1/../../../../pic32mx/lib/size\libc.a(sprintf_cdnopsuxX.eo)
                              build/default/production/_ext/334706090/wf_configData.o (_sprintf_cdnopsuxX)
c:/program files (x86)/microchip/xc32/v1.10/bin/../lib/gcc/pic32mx/4.5.1/../../../../pic32mx/lib/size\libc.a(sprintf_cdnopuxX.eo)
                              build/default/production/_ext/427700826/tcpip_helpers.o (_sprintf_cdnopuxX)
c:/program files (x86)/microchip/xc32/v1.10/bin/../lib/gcc/pic32mx/4.5.1/../../../../pic32mx/lib/size\libc.a(vsnprintf_cdnopsuxX.eo)
                              c:/program files (x86)/microchip/xc32/v1.10/bin/../lib/gcc/pic32mx/4.5.1/../../../../pic32mx/lib/size\libc.a(snprintf_cdnopsuxX.eo) (_vsnprintf_cdnopsuxX)
c:/program files (x86)/microchip/xc32/v1.10/bin/../lib/gcc/pic32mx/4.5.1/../../../../pic32mx/lib/size\libc.a(vsnprintf.o)
                              build/default/production/_ext/365611741/system_debug.o (vsnprintf)
c:/program files (x86)/microchip/xc32/v1.10/bin/../lib/gcc/pic32mx/4.5.1/../../../../pic32mx/lib/size\libc.a(ctypef.o)
                              c:/program files (x86)/microchip/xc32/v1.10/bin/../lib/gcc/pic32mx/4.5.1/../../../../pic32mx/lib/size\libc.a(strtol.o) (toupper)
c:/program files (x86)/microchip/xc32/v1.10/bin/../lib/gcc/pic32mx/4.5.1/../../../../pic32mx/lib/size\libc.a(doprnt_cdnopsuxX.eo)
                              c:/program files (x86)/microchip/xc32/v1.10/bin/../lib/gcc/pic32mx/4.5.1/../../../../pic32mx/lib/size\libc.a(sprintf_cdnopsuxX.eo) (_vfprintf_cdnopsuxX)
c:/program files (x86)/microchip/xc32/v1.10/bin/../lib/gcc/pic32mx/4.5.1/../../../../pic32mx/lib/size\libc.a(doprnt_cdnopuxX.eo)
                              c:/program files (x86)/microchip/xc32/v1.10/bin/../lib/gcc/pic32mx/4.5.1/../../../../pic32mx/lib/size\libc.a(sprintf_cdnopuxX.eo) (_vfprintf_cdnopuxX)
c:/program files (x86)/microchip/xc32/v1.10/bin/../lib/gcc/pic32mx/4.5.1/../../../../pic32mx/lib/size\libc.a(doprnt.o)
                              c:/program files (x86)/microchip/xc32/v1.10/bin/../lib/gcc/pic32mx/4.5.1/../../../../pic32mx/lib/size\libc.a(vsnprintf.o) (vfprintf)
c:/program files (x86)/microchip/xc32/v1.10/bin/../lib/gcc/pic32mx/4.5.1/../../../../pic32mx/lib/size\libc.a(_fputc_simple.o)
                              c:/program files (x86)/microchip/xc32/v1.10/bin/../lib/gcc/pic32mx/4.5.1/../../../../pic32mx/lib/size\libc.a(doprnt_cdnopsuxX.eo) (fputc)
c:/program files (x86)/microchip/xc32/v1.10/bin/../lib/gcc/pic32mx/4.5.1/../../../../pic32mx/lib/size\libc.a(powersf.o)
                              c:/program files (x86)/microchip/xc32/v1.10/bin/../lib/gcc/pic32mx/4.5.1/../../../../pic32mx/lib/size\libc.a(doprnt.o) (_powers_f)
c:/program files (x86)/microchip/xc32/v1.10/bin/../lib/gcc/pic32mx/4.5.1/../../../../pic32mx/lib/size\libc.a(_iob.o)
                              c:/program files (x86)/microchip/xc32/v1.10/bin/../lib/gcc/pic32mx/4.5.1/../../../../pic32mx/lib/size\libc.a(_fputc_simple.o) (_outdone)
c:/program files (x86)/microchip/xc32/v1.10/bin/../lib/gcc/pic32mx/4.5.1/../../../../pic32mx/lib/size\libc.a(_flsbuf_simple.o)
                              c:/program files (x86)/microchip/xc32/v1.10/bin/../lib/gcc/pic32mx/4.5.1/../../../../pic32mx/lib/size\libc.a(_fputc_simple.o) (_flsbuf)
c:/program files (x86)/microchip/xc32/v1.10/bin/../lib/gcc/pic32mx/4.5.1/../../../../pic32mx/lib/size\libpic32.a(sbrk.o)
                              c:/program files (x86)/microchip/xc32/v1.10/bin/../lib/gcc/pic32mx/4.5.1/../../../../pic32mx/lib/size\libc.a(malloc.o) (sbrk)
c:/program files (x86)/microchip/xc32/v1.10/bin/../lib/gcc/pic32mx/4.5.1/../../../../pic32mx/lib/size\libpic32.a(write.o)
                              c:/program files (x86)/microchip/xc32/v1.10/bin/../lib/gcc/pic32mx/4.5.1/../../../../pic32mx/lib/size\libc.a(_fputc_simple.o) (write)
c:/program files (x86)/microchip/xc32/v1.10/bin/../lib/gcc/pic32mx/4.5.1/../../../../pic32mx/lib/size\libpic32.a(_mon_putc.o)
                              c:/program files (x86)/microchip/xc32/v1.10/bin/../lib/gcc/pic32mx/4.5.1/../../../../pic32mx/lib/size\libpic32.a(write.o) (_mon_putc)
c:/program files (x86)/microchip/xc32/v1.10/bin/../lib/gcc/pic32mx/4.5.1/../../../../pic32mx/lib/size\libpic32.a(xc32_uart.o)
                              c:/program files (x86)/microchip/xc32/v1.10/bin/../lib/gcc/pic32mx/4.5.1/../../../../pic32mx/lib/size\libpic32.a(_mon_putc.o) (__XC_UART)
c:/program files (x86)/microchip/xc32/v1.10/bin/../lib/gcc/pic32mx/4.5.1/../../../../pic32mx/lib/size\libm.a(fpmod32.o)
                              c:/program files (x86)/microchip/xc32/v1.10/bin/../lib/gcc/pic32mx/4.5.1/../../../../pic32mx/lib/size\libc.a(doprnt.o) (frexpf)
c:/program files (x86)/microchip/xc32/v1.10/bin/../lib/gcc/pic32mx/4.5.1/../../../../pic32mx/lib/size\libm.a(fp32.o)
                              c:/program files (x86)/microchip/xc32/v1.10/bin/../lib/gcc/pic32mx/4.5.1/../../../../pic32mx/lib/size\libc.a(doprnt.o) (fpsub)
c:/program files (x86)/microchip/xc32/v1.10/bin/../lib/gcc/pic32mx/4.5.1/../../../../pic32mx/lib/size\libe.a(_floatdisf.o)
                              c:/program files (x86)/microchip/xc32/v1.10/bin/../lib/gcc/pic32mx/4.5.1/../../../../pic32mx/lib/size\libc.a(doprnt.o) (__floatdisf)
c:/program files (x86)/microchip/xc32/v1.10/bin/../lib/gcc/pic32mx/4.5.1/size\libgcc.a(_lshrdi3.o)
                              c:/program files (x86)/microchip/xc32/v1.10/bin/../lib/gcc/pic32mx/4.5.1/../../../../pic32mx/lib/size\libc.a(doprnt_cdnopsuxX.eo) (__lshrdi3)
c:/program files (x86)/microchip/xc32/v1.10/bin/../lib/gcc/pic32mx/4.5.1/size\libgcc.a(_floatundisf.o)
                              c:/program files (x86)/microchip/xc32/v1.10/bin/../lib/gcc/pic32mx/4.5.1/../../../../pic32mx/lib/size\libc.a(doprnt.o) (__floatundisf)
c:/program files (x86)/microchip/xc32/v1.10/bin/../lib/gcc/pic32mx/4.5.1/size\libgcc.a(_umoddi3.o)
                              c:/program files (x86)/microchip/xc32/v1.10/bin/../lib/gcc/pic32mx/4.5.1/../../../../pic32mx/lib/size\libc.a(doprnt_cdnopsuxX.eo) (__umoddi3)
c:/program files (x86)/microchip/xc32/v1.10/bin/../lib/gcc/pic32mx/4.5.1/size\libgcc.a(floatunsisf.o)
                              c:/program files (x86)/microchip/xc32/v1.10/bin/../lib/gcc/pic32mx/4.5.1/../../../../pic32mx/lib/size\libc.a(doprnt.o) (__floatunsisf)

Allocating common symbols
Common symbol       size              file

g_savedPsPollContext
                    0x6               build/default/production/_ext/334706090/wf_power_save.o
myb64               0x80              build/default/production/_ext/1472/tcp6_demo_app.o
RawWindowState      0x2               build/default/production/_ext/334706090/wf_driver_raw_24g.o
mySocketInfo        0x28              build/default/production/_ext/1472/tcp6_demo_app.o
pNetIf              0x4               build/default/production/_ext/1472/ping_demo.o
g_softAPEvent       0x8               build/default/production/_ext/334706090/wf_event_handler.o
httpTransaction     0x4b0             build/default/production/_ext/1472/tcp6_demo_app.o
pingCount           0x1               build/default/production/_ext/1472/ping_demo.o
myNetHandle         0x4               build/default/production/_ext/1472/tcp6_demo_app.o
mac_addr_ptr        0x4               build/default/production/_ext/1472/tcp6_demo_app.o
dnsRes              0x4               build/default/production/_ext/1472/tcp6_demo_app.o
HTTPReplyDelay      0x4               build/default/production/_ext/1472/tcp6_demo_app.o
targetAddressIPv4   0x4               build/default/production/_ext/1472/ping_demo.o
hMac_softap_connect
                    0x4               build/default/production/_ext/334706090/wf_scan.o
iwconfigCb          0x3               build/default/production/_ext/334706090/wf_commands.o
g_gratArpContext    0x8               build/default/production/_ext/334706090/wf_mac_24g.o
g_pNetIf            0x4               build/default/production/_ext/334706090/wf_mac_24g.o
TCPInBuffer         0x1000            build/default/production/_ext/1472/tcp6_demo_app.o
TCPInBufPtr         0x4               build/default/production/_ext/1472/tcp6_demo_app.o
mysrc               0x80              build/default/production/_ext/1472/tcp6_demo_app.o
pingTimer           0x4               build/default/production/_ext/1472/ping_demo.o
RawMoveState        0x2               build/default/production/_ext/334706090/wf_driver_com_24g.o
myResourceState     0x64              build/default/production/_ext/1472/tcp6_demo_app.o
serverIP            0x4               build/default/production/_ext/1472/tcp6_demo_app.o
g_powerSaveState    0x1               build/default/production/_ext/334706090/wf_driver_com_24g.o
i                   0x4               build/default/production/_ext/1472/tcp6_demo_app.o
wifi_ConfigData     0x8a              build/default/production/_ext/334706090/wf_configData.o
mac_addr            0x6               build/default/production/_ext/1472/tcp6_demo_app.o
temp                0x20              build/default/production/_ext/1472/tcp6_demo_app.o
firstHopAddress     0x4               build/default/production/_ext/1472/ping_demo.o
lastBlock           0x40              build/default/production/_ext/101875047/hashes.o
clientTimer         0x4               build/default/production/_ext/1472/tcp6_demo_app.o
stackNotifyHandle   0x4               build/default/production/_ext/1472/main_demo.o
TCPReadByte         0x1               build/default/production/_ext/1472/tcp6_demo_app.o
remoteNode          0xa               build/default/production/_ext/427700826/tcpip_manager.o
targetHostName      0x4               build/default/production/_ext/1472/ping_demo.o
mac_addr_string     0x10              build/default/production/_ext/1472/tcp6_demo_app.o
j                   0x4               build/default/production/_ext/1472/tcp6_demo_app.o
g_easyConfigCtx     0x98              build/default/production/_ext/334706090/wf_easy_config.o
TCPInBufferIndex    0x4               build/default/production/_ext/1472/tcp6_demo_app.o
targetMACAddr       0x6               build/default/production/_ext/1472/ping_demo.o
toggleLed           0x4               build/default/production/_ext/1472/tcp6_demo_app.o
OutString           0x200             build/default/production/_ext/1472/tcp6_demo_app.o
HTTPReplyLineCnt    0x4               build/default/production/_ext/1472/tcp6_demo_app.o
g_rxBufferLength    0x2               build/default/production/_ext/334706090/wf_mac_24g.o
TCPIsPutReadyCnt    0x2               build/default/production/_ext/1472/tcp6_demo_app.o
TCPOutBuffer        0x200             build/default/production/_ext/1472/tcp6_demo_app.o
serverPort          0x2               build/default/production/_ext/1472/tcp6_demo_app.o
LCDText             0x21              build/default/production/_ext/792872985/lcd.o

Microchip PIC32 Memory-Usage Report

kseg0 Program-Memory Usage
section                    address  length [bytes]      (dec)  Description
-------                 ----------  -------------------------  -----------
.text.HTTPProcess       0x9d000020         0x1804        6148   
.text._TcpHandleSeg     0x9d001824         0x17e0        6112   
.text.vfprintf          0x9d003004         0x15b4        5556   
.text.DNSClientTask     0x9d0045b8         0x1144        4420   
.rodata                 0x9d0056fc         0x1088        4232  Read-only const 
.text.tcp6_demo_app_tas 0x9d006784          0xfd8        4056   
.text.DHCPTask          0x9d00775c          0xa74        2676   
.text._TcpSend          0x9d0081d0          0xa50        2640   
.text.TCPAdjustFIFOSize 0x9d008c20          0x974        2420   
.rodata                 0x9d009594          0x8f4        2292  Read-only const 
.text                   0x9d009e88          0x8ec        2284  App's exec code 
.text._vfprintf_cdnopsu 0x9d00a774          0x8c4        2244   
.text.TCPTick           0x9d00b038          0x8b8        2232   
.rodata                 0x9d00b8f0          0x7d4        2004  Read-only const 
.text._DHCPReceive      0x9d00c0c4          0x748        1864   
.dinit                  0x9d00c80c          0x748        1864   
.text.NBNSTask          0x9d00cf54          0x740        1856   
.text.HTTPPrint         0x9d00d694          0x6ac        1708   
.text.HTTPPostConfig    0x9d00dd40          0x694        1684   
.text._DHCPSend         0x9d00e3d4          0x5c8        1480   
.text.TCPFindArray      0x9d00e99c          0x578        1400   
.text.SHA1HashBlock     0x9d00ef14          0x4fc        1276   
.text.SYS_Initialize    0x9d00f410          0x4f0        1264   
.text.TCPIP_ANNOUNCE_Se 0x9d00f900          0x490        1168   
.text._TCPIP_HEAP_Free  0x9d00fd90          0x490        1168   
.text.TCPIP_STACK_Init  0x9d010220          0x468        1128   
.text                   0x9d010688          0x8ac        2220  App's exec code 
.rodata                 0x9d010f34          0x43c        1084  Read-only const 
.text.TCPIP_STACK_Bring 0x9d011370          0x438        1080   
.text.CommandHelp       0x9d0117a8          0x428        1064   
.text.TCPOpen           0x9d011bd0          0x420        1056   
.text.HTTPExecuteGet    0x9d011ff0          0x414        1044   
.text.HTTPMPFSUpload    0x9d012404          0x410        1040   
.text.MPFSSeek          0x9d012814          0x400        1024   
.rodata                 0x9d012c14          0x3f8        1016  Read-only const 
.text.ARPInitialize     0x9d01300c          0x3f4        1012   
.text._TcpFindMatchingS 0x9d013400          0x3e8        1000   
.text                   0x9d0137e8          0x3dc         988  App's exec code 
.text.TCPIP_HELPER_Stri 0x9d013bc4          0x3b8         952   
.text.WFProcessMgmtIndi 0x9d013f7c          0x3b0         944   
.text.FindMatchingSocke 0x9d01432c          0x3a0         928   
.text.TCPIP_Helper_Base 0x9d0146cc          0x394         916   
.text.OutputSecurityMod 0x9d014a60          0x38c         908   
.text.TCPIP_STACK_Task  0x9d014dec          0x35c         860   
.text._SYS_COMMAND_TASK 0x9d015148          0x354         852   
.text.HTTPPostMD5       0x9d01549c          0x340         832   
.text.UDPOpen           0x9d0157dc          0x334         820   
.text.main              0x9d015b10          0x328         808   
.text.MPFSOpen          0x9d015e38          0x31c         796   
.text.OutputConnectionF 0x9d016154          0x31c         796   
.text.HTTPInit          0x9d016470          0x318         792   
.text.UDPInit           0x9d016788          0x318         792   
.text.ARPTask           0x9d016aa0          0x310         784   
.text.TCPIP_IPV4_PutArr 0x9d016db0          0x310         784   
.text.SYS_FS_mount      0x9d0170c0          0x2e0         736   
.text.tcp6_demo_app_ini 0x9d0173a0          0x2d8         728   
.text.MD5HashBlock      0x9d017678          0x2c8         712   
.text.ProcessEscSequenc 0x9d017940          0x2c8         712   
.text.DoWrite           0x9d017c08          0x2c4         708   
.text.HTTPReadTo        0x9d017ecc          0x2c4         708   
.text.MPFSGetArray      0x9d018190          0x2bc         700   
.text.ICMPProcess       0x9d01844c          0x2ac         684   
.text.MD5Calculate      0x9d0186f8          0x2a8         680   
.text.TCPPutArray       0x9d0189a0          0x2a8         680   
.text.ParseCmdBuffer    0x9d018c48          0x2a4         676   
.text.DRV_MEDIA_Open    0x9d018eec          0x294         660   
.rodata                 0x9d019180          0x28c         652  Read-only const 
.text.Wifi_Connect      0x9d01940c          0x284         644   
.text.UDPProcessIPv4    0x9d019690          0x27c         636   
.text.SyncENCPtrRAWStat 0x9d01990c          0x278         632   
.text.GetMaxSegSizeOpti 0x9d019b84          0x274         628   
.text.MPFSGet           0x9d019df8          0x270         624   
.text.WriteAnalogRegist 0x9d01a068          0x270         624   
.text.XEEReadArray      0x9d01a2d8          0x268         616   
.text.TCPIP_IPV4_Calcul 0x9d01a540          0x268         616   
.text.HTTPSendFile      0x9d01a7a8          0x264         612   
.text.TCPGetArray       0x9d01aa0c          0x264         612   
.text.SYS_GENERATE_RAND 0x9d01ac70          0x25c         604   
.text.SYS_CLK_OscClockG 0x9d01aecc          0x258         600   
.text.TCPIP_IPV4_CopyTx 0x9d01b124          0x250         592   
.text                   0x9d01b374          0x248         584  App's exec code 
.text.LoadDefaultConfig 0x9d01b5bc          0x244         580   
.text.malloc            0x9d01b800          0x244         580   
.text.ProcessTCPIPMacEv 0x9d01ba44          0x240         576   
.rodata                 0x9d01bc84          0x238         568  Read-only const 
.text.LCD_UPDATE_OFFSET 0x9d01bebc          0x230         560   
.text.ARPEntryRemoveNet 0x9d01c0ec          0x224         548   
.text.TCPIP_IPV4_GetDat 0x9d01c310          0x224         548   
.text.__floatdisf       0x9d01c534          0x21c         540   
.text.HTTPHeaderParseCo 0x9d01c750          0x214         532   
.text.TCPInit           0x9d01c964          0x20c         524   
.text.DHCPInit          0x9d01cb70          0x204         516   
.text.HTTPIncFile       0x9d01cd74          0x200         512   
.text._TcpDisconnect    0x9d01cf74          0x200         512   
.text.UDPTask           0x9d01d174          0x200         512   
.text.SYS_USERIO_SetLED 0x9d01d374          0x1f8         504   
.text.TCPIP_ANNOUNCE_Ta 0x9d01d56c          0x1f8         504   
.text.SYS_FS_chdir      0x9d01d764          0x1f4         500   
.text.ARPProcess        0x9d01d958          0x1f4         500   
.text.TCPIP_IPV4_Flush  0x9d01db4c          0x1ec         492   
.text.SYS_FS_ExtractFir 0x9d01dd38          0x1e8         488   
.text.SYS_FS_initialize 0x9d01df20          0x1e8         488   
.rodata                 0x9d01e108          0x1e8         488  Read-only const 
.text._TCPIP_HEAP_Mallo 0x9d01e2f0          0x1e0         480   
.rodata                 0x9d01e4d0          0x1e0         480  Read-only const 
.text.StringToArgs      0x9d01e6b0          0x1dc         476   
.text.HTTPURLDecode     0x9d01e88c          0x1dc         476   
.text.TCPProcessIPv4    0x9d01ea68          0x1dc         476   
.text.TCPIP_IPV4_IsTxPu 0x9d01ec44          0x1d8         472   
.text.HTTPHeaderParseAu 0x9d01ee1c          0x1d4         468   
.text.UDPv4IsTxPutReady 0x9d01eff0          0x1d4         468   
.text._TCPIsPutReady    0x9d01f1c4          0x1cc         460   
.text.UDPDeInit         0x9d01f390          0x1cc         460   
.text.strtoul           0x9d01f55c          0x1cc         460   
.text.SYS_USERIO_ReadIO 0x9d01f728          0x1c8         456   
.text._TcpSocketSetIdle 0x9d01f8f0          0x1c8         456   
.text.HTTPPrint_ledSele 0x9d01fab8          0x1c4         452   
.text.TCPSetOptions     0x9d01fc7c          0x1b8         440   
.text.MRF24W_MACGetHead 0x9d01fe34          0x1b8         440   
.text.HTTPPrint_uploade 0x9d01ffec          0x1b8         440   
.text.WF_ProcessEvent   0x9d0201a4          0x1b4         436   
.text._SystemTickIntHan 0x9d020358          0x1b0         432   
.text.isNotifyApp       0x9d020508          0x1a8         424   
.text.DisplayNodeMsg    0x9d0206b0          0x1a0         416   
.text.HTTPPrint_led     0x9d020850          0x1a0         416   
.text                   0x9d0209f0          0x1a0         416  App's exec code 
.text._TcpCloseSocket   0x9d020b90          0x198         408   
.text.NBNSGetName       0x9d020d28          0x194         404   
.text._Sys_Ext1_Isr     0x9d020ebc          0x190         400   
.text._Sys_Ext3_Isr     0x9d02104c          0x190         400   
.text._Sys_CN_Isr       0x9d0211dc          0x190         400   
.text.MRF24W_ChipReset  0x9d02136c          0x190         400   
.text.RawMove           0x9d0214fc          0x190         400   
.text.TCPIP_HELPER_Stri 0x9d02168c          0x18c         396   
.text.WaitForRawMoveCom 0x9d021818          0x18c         396   
.text.DRV_MEDIA_Initial 0x9d0219a4          0x188         392   
.text.UDPGetArray       0x9d021b2c          0x188         392   
.text.OutputBeaconTimeo 0x9d021cb4          0x188         392   
.text.HTTPServer        0x9d021e3c          0x180         384   
.text._OAHashFindBkt    0x9d021fbc          0x180         384   
.text.ARPIsResolved     0x9d02213c          0x178         376   
.text.TCPIP_IPV4_Alloca 0x9d0222b4          0x178         376   
.text.TCPIP_HEAP_Create 0x9d02242c          0x178         376   
.text.HTTPPostLCD       0x9d0225a4          0x178         376   
.text.MPFSOpenID        0x9d02271c          0x174         372   
.text.SYS_FS_IsLegalDir 0x9d022890          0x170         368   
.text.LCD_INIT          0x9d022a00          0x170         368   
.text._ARPProbeAddress  0x9d022b70          0x170         368   
.text.SpiChnOpen        0x9d022ce0          0x170         368   
.text.stricmppgm2ram    0x9d022e50          0x16c         364   
.text.OAHashLookUpInser 0x9d022fbc          0x16c         364   
.text.UDPv4Flush        0x9d023128          0x16c         364   
.text.WFHardwareInit    0x9d023294          0x168         360   
.text                   0x9d0233fc          0x2d0         720  App's exec code 
.text.USART_INIT        0x9d0236cc          0x164         356   
.text.XEEIsBusy         0x9d023830          0x164         356   
.text.RawSetIndex       0x9d023994          0x164         356   
.text.SYS_TICK_TimerDel 0x9d023af8          0x160         352   
.text.DRV_SPI_TxRx      0x9d023c58          0x160         352   
.text.DNSPutString      0x9d023db8          0x160         352   
.text.TCPIP_IPV4_Transm 0x9d023f18          0x160         352   
.text.UDPBind           0x9d024078          0x160         352   
.text.WFEintHandler     0x9d0241d8          0x160         352   
.text.encodeblock       0x9d024338          0x160         352   
.text.ARP_SendIfPkt     0x9d024498          0x15c         348   
.text.TCPIP_IPV4_GetHea 0x9d0245f4          0x15c         348   
.text.DRV_MEDIA_Read    0x9d024750          0x158         344   
.text.HTTPPrint_config_ 0x9d0248a8          0x158         344   
.text.ProcessInterruptS 0x9d024a00          0x154         340   
.rodata                 0x9d024b54          0x150         336  Read-only const 
.text._TCPIPStackIsLoca 0x9d024ca4          0x150         336   
.text.TCPIP_Helper_Calc 0x9d024df4          0x150         336   
.text.OutputChannelList 0x9d024f44          0x150         336   
.text.UDPSocketSetNet   0x9d025094          0x14c         332   
.text._sbrk_init        0x9d0251e0          0x14c         332   
.text._SYS_CMDIO_DELETE 0x9d02532c          0x148         328   
.text.TCPIP_STACK_DeIni 0x9d025474          0x148         328   
.text.OutputConnectionT 0x9d0255bc          0x148         328   
.text.OutputConnectionP 0x9d025704          0x148         328   
.text.SendMgmtMsg       0x9d02584c          0x148         328   
.text.OAHashLookUp      0x9d025994          0x144         324   
.text.scale             0x9d025ad8          0x144         324   
.rodata                 0x9d025c1c          0x140         320  Read-only const 
.text._WF_OutputConnect 0x9d025d5c          0x140         320   
.text.PowerSaveTask     0x9d025e9c          0x140         320   
.text.UDPIsGetReady     0x9d025fdc          0x13c         316   
.text.WF_SetMultiCastFi 0x9d026118          0x13c         316   
.text._ARPUpdateEntry   0x9d026254          0x138         312   
.text.TCPIP_IPV4_Queued 0x9d02638c          0x138         312   
.text.HTTPPrint_btn     0x9d0264c4          0x138         312   
.text._general_exceptio 0x9d0265fc          0x134         308   
.text.SYS_USERIO_Initia 0x9d026730          0x134         308   
.text.SYS_FS_FSFromAbsP 0x9d026864          0x134         308   
.text.TCPIP_IPV4_Insert 0x9d026998          0x134         308   
.text.SetSecurity       0x9d026acc          0x134         308   
.text.fputc             0x9d026c00          0x134         308   
.text.DRV_MEDIA_Write   0x9d026d34          0x130         304   
.text.UDPSetBcastIPV4Ad 0x9d026e64          0x130         304   
.text.realloc           0x9d026f94          0x130         304   
.text.uitoa             0x9d0270c4          0x12c         300   
.text.WF_ConfigDataLoad 0x9d0271f0          0x12c         300   
.text.DNSBeginUsage     0x9d02731c          0x128         296   
.text.HTTPDeInit        0x9d027444          0x124         292   
.text.TCPIP_IPV4_Initia 0x9d027568          0x124         292   
.text._TCPSendWinIncUpd 0x9d02768c          0x124         292   
.text.UDPOpenServer     0x9d0277b0          0x124         292   
.text.WaitForMgmtRespon 0x9d0278d4          0x124         292   
.text.strtol            0x9d0279f8          0x124         292   
.text.TCPIP_IPV4_QueueP 0x9d027b1c          0x120         288   
.text.TCPOpenServer     0x9d027c3c          0x120         288   
.text                   0x9d027d5c          0x120         288  App's exec code 
.text.fround            0x9d027e7c          0x120         288   
.text.SHA1AddData       0x9d027f9c          0x11c         284   
.text.b64_encode        0x9d0280b8          0x11c         284   
.text.BSP_Initialize    0x9d0281d4          0x114         276   
.text.TCPIP_IPV4_PutHea 0x9d0282e8          0x114         276   
.text.DisplayIPValue    0x9d0283fc          0x114         276   
.text.MD5AddData        0x9d028510          0x110         272   
.text.WiFiAsyncTask     0x9d028620          0x110         272   
.text.WF_PsPollEnable   0x9d028730          0x110         272   
.text._flsbuf           0x9d028840          0x110         272   
.text._TcpSwapHeader    0x9d028950          0x10c         268   
.text.TCPIP_STACK_Bring 0x9d028a5c          0x108         264   
.text.OutputNetworkType 0x9d028b64          0x108         264   
.text._DHCPClose        0x9d028c6c          0x104         260   
.text.WF_ScanContextGet 0x9d028d70          0x104         260   
.rodata                 0x9d028e74          0x208         520  Read-only const 
.text.hexatob           0x9d02907c          0x100         256   
.text.MPFSGetFilename   0x9d02917c           0xfc         252   
.text.WaitForMgmtRespon 0x9d029278           0xfc         252   
.text.HTTPExecutePost   0x9d029374           0xfc         252   
.text.SYS_FS_IsAbsolute 0x9d029470           0xf8         248   
.text._TCPIPStackAddres 0x9d029568           0xf8         248   
.text.SingleListRemoveN 0x9d029660           0xf8         248   
.text.WF_Init           0x9d029758           0xf8         248   
.text.SYS_USERIO_Device 0x9d029850           0xf4         244   
.text.UDPSetSourceIPAdd 0x9d029944           0xf4         244   
.text.UDPSetDestination 0x9d029a38           0xf4         244   
.text.WF_SecurityGet    0x9d029b2c           0xf4         244   
.text.MRF24W_MACInitial 0x9d029c20           0xf4         244   
.text._ARPAddCompleteEn 0x9d029d14           0xf0         240   
.text.UDPDiscard        0x9d029e04           0xf0         240   
.text.WF_ScanContextSet 0x9d029ef4           0xf0         240   
.text.NBNSPutName       0x9d029fe4           0xec         236   
.text.TCPIsPutReady     0x9d02a0d0           0xec         236   
.text._TCPIP_HEAP_Callo 0x9d02a1bc           0xec         236   
.text.AllocateDataTxBuf 0x9d02a2a8           0xec         236   
.text.HTTPReadPostValue 0x9d02a394           0xe8         232   
.text.DNSIsResolved     0x9d02a47c           0xe8         232   
.text.TCPIP_IPV4_PutUpp 0x9d02a564           0xe8         232   
.text.UDPSetRxOffset    0x9d02a64c           0xe8         232   
.text.ProcessTCPIPTickE 0x9d02a734           0xe8         232   
.text.WF_GetDeviceInfo  0x9d02a81c           0xe8         232   
.rodata                 0x9d02a904            0x4           4  Read-only const 
.rodata                 0x9d02a908           0xe8         232  Read-only const 
.text.LCD_WRITE         0x9d02a9f0           0xe4         228   
.text.TCPIP_IPV4_ResetT 0x9d02aad4           0xe4         228   
.text.TCPIP_IPV4_Alloca 0x9d02abb8           0xe4         228   
.text.TCPDeInit         0x9d02ac9c           0xe4         228   
.text.TCPIP_HEAP_Delete 0x9d02ad80           0xe4         228   
.text.SYS_TICK_TimerCre 0x9d02ae64           0xe0         224   
.text._SYS_CMDIO_ADD    0x9d02af44           0xe0         224   
.text._ARPSetEntry      0x9d02b024           0xe0         224   
.text.ARPResolve        0x9d02b104           0xe0         224   
.text.UDPOpenClient     0x9d02b1e4           0xe0         224   
.text.UDPPutArray       0x9d02b2c4           0xe0         224   
.text.TCPIPMacEventCB   0x9d02b3a4           0xe0         224   
.text._SYS_ERROR_PRINT  0x9d02b484           0xdc         220   
.text.HTTPHeaderParseCo 0x9d02b560           0xdc         220   
.text.ARPHashDeleteEntr 0x9d02b63c           0xdc         220   
.text.DHCPConnectionHan 0x9d02b718           0xdc         220   
.text._TcpCleanup       0x9d02b7f4           0xdc         220   
.text.TCPOpenClient     0x9d02b8d0           0xdc         220   
.text.TcpAllocateEpheme 0x9d02b9ac           0xdc         220   
.text.UdpAllocateEpheme 0x9d02ba88           0xdc         220   
.text.OutputTxMode      0x9d02bb64           0xdc         220   
.text.MACIFService      0x9d02bc40           0xdc         220   
.text.DHCPEnable        0x9d02bd1c           0xd8         216   
.text.TCPIP_IPV4_GetPse 0x9d02bdf4           0xd8         216   
.text._TcpAbort         0x9d02becc           0xd8         216   
.text._TCPIP_HEAP_Mallo 0x9d02bfa4           0xd8         216   
.text._SYS_RANDOM_INIT  0x9d02c07c           0xd4         212   
.text.TCPIP_ANNOUNCE_In 0x9d02c150           0xd4         212   
.text.TCPClose          0x9d02c224           0xd4         212   
.text.OutputDomain      0x9d02c2f8           0xd4         212   
.text.AllocateMgmtTxBuf 0x9d02c3cc           0xd4         212   
.text                   0x9d02c4a0           0xd4         212  App's exec code 
.text._LoadFATRecord    0x9d02c574           0xd0         208   
.text.HTTPGetArg        0x9d02c644           0xd0         208   
.text._ARPDeleteResourc 0x9d02c714           0xd0         208   
.text.fnv_32_hash       0x9d02c7e4           0xd0         208   
.text._TcpSocketInitial 0x9d02c8b4           0xd0         208   
.text.UDPSetOptions     0x9d02c984           0xd0         208   
.text.TCPIP_STACK_Regis 0x9d02ca54           0xd0         208   
.text.DhcpConfigTask    0x9d02cb24           0xd0         208   
.text.OutputDeviceInfo  0x9d02cbf4           0xd0         208   
.text.MRF24W_MACPutHead 0x9d02ccc4           0xd0         208   
.text.general_exception 0x9d02cd94           0xd0         208   
.rodata                 0x9d02ce68           0xd0         208  Read-only const 
.text.DRV_MEDIA_WriteSe 0x9d02cf38           0xcc         204   
.text.HTTPSetMediaWrite 0x9d02d004           0xcc         204   
.text.TCPIP_IPV4_SetPay 0x9d02d0d0           0xcc         204   
.text.MPFSInit          0x9d02d19c           0xc8         200   
.text.DNSRetry          0x9d02d264           0xc8         200   
.text.DNSDiscardName    0x9d02d32c           0xc8         200   
.text.UDPClose          0x9d02d3f4           0xc8         200   
.text.UDPSetTxOffset    0x9d02d4bc           0xc8         200   
.text.InitNetConfig     0x9d02d584           0xc8         200   
.text.TCPIP_Helper_Form 0x9d02d64c           0xc8         200   
.text.OutputDemoHeader  0x9d02d714           0xc8         200   
.text.HostInterruptRegI 0x9d02d7dc           0xc8         200   
.text.HTTPPrintIP       0x9d02d8a4           0xc8         200   
.text.CmdAddHead        0x9d02d96c           0xc4         196   
.text._DHCPEnable       0x9d02da30           0xc4         196   
.text.MRF24W_MACGetArra 0x9d02daf4           0xc4         196   
.text.SYS_TICK_Initiali 0x9d02dbb8           0xc0         192   
.text.LowLevel_CPGetEle 0x9d02dc78           0xc0         192   
.text.ProcessMgmtRxMsg  0x9d02dd38           0xc0         192   
.text.SYS_INT_DynamicRe 0x9d02ddf8           0xbc         188   
.text._SYS_COMMAND_INIT 0x9d02deb4           0xbc         188   
.text.MPFSGetEndAddr    0x9d02df70           0xbc         188   
.text._ARPRemoveEntry   0x9d02e02c           0xbc         188   
.text.OAHashRemoveAll   0x9d02e0e8           0xbc         188   
.text.UDPDiscardNet     0x9d02e1a4           0xbc         188   
.text.TCPIP_Helper_Stri 0x9d02e260           0xbc         188   
.text.LowLevel_CAGetEle 0x9d02e31c           0xbc         188   
.text.MRF24W_MACEventSe 0x9d02e3d8           0xbc         188   
.text.OutputMacAddress  0x9d02e494           0xbc         188   
.text._SYS_DEBUG_INIT   0x9d02e550           0xb8         184   
.text._SYS_CONSOLE_INIT 0x9d02e608           0xb8         184   
.text.XEEInit           0x9d02e6c0           0xb8         184   
.text.TCPv4AllocateTxPa 0x9d02e778           0xb8         184   
.text._TCPIsGetReady    0x9d02e830           0xb8         184   
.text.UDPGetTxCount     0x9d02e8e8           0xb8         184   
.text.OutputScanType    0x9d02e9a0           0xb8         184   
.text.RawGetByte        0x9d02ea58           0xb8         184   
.text.RawSetByte        0x9d02eb10           0xb8         184   
.text.MPFSGetFlags      0x9d02ebc8           0xb4         180   
.text.MPFSGetSize       0x9d02ec7c           0xb4         180   
.text.MPFSGetStartAddr  0x9d02ed30           0xb4         180   
.text._TcpMac2RamCopy   0x9d02ede4           0xb4         180   
.text.UDPv4AllocateTxPa 0x9d02ee98           0xb4         180   
.text.UDPIsTxPutReady   0x9d02ef4c           0xb4         180   
.text.WF_SsidSet        0x9d02f000           0xb4         180   
.text.MRF24W_MACEventIn 0x9d02f0b4           0xb4         180   
.text._mon_putc         0x9d02f168           0xb4         180   
.text.CommandQuit       0x9d02f21c           0xb0         176   
.text.CmdRemoveTail     0x9d02f2cc           0xb0         176   
.text.Delay10us         0x9d02f37c           0xb0         176   
.text.TCPIP_ANNOUNCE_De 0x9d02f42c           0xb0         176   
.text._ARPRemoveCacheEn 0x9d02f4dc           0xb0         176   
.text._ARPNotifyClients 0x9d02f58c           0xb0         176   
.text._Tcpv4AckFnc      0x9d02f63c           0xb0         176   
.text._TCPIPStackSetNet 0x9d02f6ec           0xb0         176   
.text._TCPIPStackIsBcas 0x9d02f79c           0xb0         176   
.text.HostInterrupt2Reg 0x9d02f84c           0xb0         176   
.rodata                 0x9d02f8fc           0xac         172  Read-only const 
.text.TCPIsConnected    0x9d02f9a8           0xac         172   
.text.HTTPPrint_cookien 0x9d02fa54           0xac         172   
.text._SYS_ERROR        0x9d02fb00           0xa8         168   
.text.ARPDeinitialize   0x9d02fba8           0xa8         168   
.text._TCPIPStackString 0x9d02fc50           0xa8         168   
.text.WFConfigureLowPow 0x9d02fcf8           0xa8         168   
.text.WF_OutputConnecti 0x9d02fda0           0xa8         168   
.text                   0x9d02fe48           0xa8         168  App's exec code 
.text._Validate         0x9d02fef0           0xa4         164   
.text.XEEWriteArray     0x9d02ff94           0xa4         164   
.text.DNSResolve        0x9d030038           0xa4         164   
.text._ICMPAllocateTxPa 0x9d0300dc           0xa4         164   
.text.TCPIP_IPV4_DeInit 0x9d030180           0xa4         164   
.text._UdpSocketDcpt    0x9d030224           0xa4         164   
.text._TCPIPStackNetByA 0x9d0302c8           0xa4         164   
.text.WF_ReconnectModeS 0x9d03036c           0xa4         164   
.text.WF_LibInitialize  0x9d030410           0xa4         164   
.text.HTTPPrint_helloms 0x9d0304b4           0xa4         164   
.text._sbrk             0x9d030558           0xa4         164   
.text.USART_GETS        0x9d0305fc           0xa0         160   
.text.XEEWrite          0x9d03069c           0xa0         160   
.text._DHCPDiscard      0x9d03073c           0xa0         160   
.text._DHCPNotifyClient 0x9d0307dc           0xa0         160   
.text.HTTPPrint_buildda 0x9d03087c           0xa0         160   
.rodata                 0x9d03091c           0xa0         160  Read-only const 
.text.strupr            0x9d0309bc           0x9c         156   
.text.MPFSDeinit        0x9d030a58           0x9c         156   
.text.ANNOUNCE_Notify   0x9d030af4           0x9c         156   
.text.DHCPRegisterHandl 0x9d030b90           0x9c         156   
.text._TcpSocketKill    0x9d030c2c           0x9c         156   
.text.TCPIsAvailablePor 0x9d030cc8           0x9c         156   
.text.UdpIsAvailablePor 0x9d030d64           0x9c         156   
.text._TCPIPStackMacIdT 0x9d030e00           0x9c         156   
.text.SingleListRemoveH 0x9d030e9c           0x9c         156   
.text.SetWpsSecurity    0x9d030f38           0x9c         156   
.text.WF_SpiTxRx        0x9d030fd4           0x9c         156   
.text.OutputIpAddress   0x9d031070           0x9c         156   
.text.GetSpiPortWithBit 0x9d03110c           0x9c         156   
.text.HTTPPrint_ddns_st 0x9d0311a8           0x9c         156   
.text._SYS_DEBUG_OPEN   0x9d031244           0x98         152   
.text._SYS_ASSERT       0x9d0312dc           0x98         152   
.text._SYS_CONSOLE_OPEN 0x9d031374           0x98         152   
.text.DelayMs           0x9d03140c           0x98         152   
.text.TCPIP_STACK_Verif 0x9d0314a4           0x98         152   
.text.WF_ReconnectModeG 0x9d03153c           0x98         152   
.text.WF_ChannelListGet 0x9d0315d4           0x98         152   
.text                   0x9d03166c           0x98         152  App's exec code 
.text.HTTPHeaderParseLo 0x9d031704           0x94         148   
.text.TCPWasReset       0x9d031798           0x94         148   
.text.TCP_PutArray      0x9d03182c           0x94         148   
.text.SingleListAddTail 0x9d0318c0           0x94         148   
.text.LowLevel_CPSetEle 0x9d031954           0x94         148   
.text.MRF24W_SetUserEve 0x9d0319e8           0x94         148   
.text.RawMountRxBuffer  0x9d031a7c           0x94         148   
.text.MRF24W_MACCalcRxC 0x9d031b10           0x94         148   
.text.USART_PRINT       0x9d031ba4           0x90         144   
.text._HttpCleanup      0x9d031c34           0x90         144   
.text.DHCPIsBound       0x9d031cc4           0x90         144   
.text.TCPIP_IPV4_FreePa 0x9d031d54           0x90         144   
.text.NBNSDeInit        0x9d031de4           0x90         144   
.text.TCPDiscard        0x9d031e74           0x90         144   
.text.TCP_SetPayload    0x9d031f04           0x90         144   
.text.UDPRemoteBind     0x9d031f94           0x90         144   
.text._TCPIPStackIsNetB 0x9d032024           0x90         144   
.text.OutputSsid        0x9d0320b4           0x90         144   
.text.ReadWFArray       0x9d032144           0x90         144   
.text.SendGetParamMsg   0x9d0321d4           0x90         144   
.text.atol              0x9d032264           0x90         144   
.text.HTTPReadPostName  0x9d0322f4           0x8c         140   
.text.SwapARPPacket     0x9d032380           0x8c         140   
.text.DHCPDisable       0x9d03240c           0x8c         140   
.text.DNSClientInit     0x9d032498           0x8c         140   
.text.SwapIPV4Header    0x9d032524           0x8c         140   
.text.UDPFlush          0x9d0325b0           0x8c         140   
.text.LowLevel_CASetEle 0x9d03263c           0x8c         140   
.text.HTTPNeedsAuth     0x9d0326c8           0x8c         140   
.text.HTTPPrint_status_ 0x9d032754           0x8c         140   
.text.HTTPPrint_status_ 0x9d0327e0           0x8c         140   
.text.write             0x9d03286c           0x8c         140   
.text.SHA1Initialize    0x9d0328f8           0x88         136   
.text._SysGetCDevEntry  0x9d032980           0x88         136   
.text.DHCPDeInit        0x9d032a08           0x88         136   
.text.TCP_IsTxPutReady  0x9d032a90           0x88         136   
.text.TCP_PutHeader     0x9d032b18           0x88         136   
.text._TCPIPStackIpAddT 0x9d032ba0           0x88         136   
.text._TCPIPStackMACIdT 0x9d032c28           0x88         136   
.text.TCPIP_STACK_NetBc 0x9d032cb0           0x88         136   
.text.WF_EintInit       0x9d032d38           0x88         136   
.text.Read16BitWFRegist 0x9d032dc0           0x88         136   
.text.Write16BitWFRegis 0x9d032e48           0x88         136   
.text.WriteWFArray      0x9d032ed0           0x88         136   
.text.SendSetParamMsg   0x9d032f58           0x88         136   
.text.LFSRSeedRand      0x9d032fe0           0x84         132   
.text._SYS_CONSOLE_PRIN 0x9d033064           0x84         132   
.text.DRV_MEDIA_ReadSet 0x9d0330e8           0x84         132   
.text.OAHashInit        0x9d03316c           0x84         132   
.text._TCPIP_HEAP_Callo 0x9d0331f0           0x84         132   
.text.TcpipStackFindMod 0x9d033274           0x84         132   
.text.TcpipStackFindMac 0x9d0332f8           0x84         132   
.text.mrf24w_MACPowerMo 0x9d03337c           0x84         132   
.text.MRF24W_ISR        0x9d033400           0x84         132   
.rodata                 0x9d033484           0x84         132  Read-only const 
.text.HTTPCheckAuth     0x9d033508           0x84         132   
.text.atoi              0x9d03358c           0x84         132   
.text.TCPIP_IPV4_FlushD 0x9d033610           0x80         128   
.text.TCPDisconnect     0x9d033690           0x80         128   
.text.TCP_IsTxReady     0x9d033710           0x80         128   
.text.TCP_CopyTxPacketS 0x9d033790           0x80         128   
.text._Udpv4AckFnc      0x9d033810           0x80         128   
.text.SetWpaSecurity    0x9d033890           0x80         128   
.text.ValidateConfig    0x9d033910           0x80         128   
.text.ScratchMount      0x9d033990           0x80         128   
.text.ProcessNotificati 0x9d033a10           0x80         128   
.text._SYS_CMDIO_GET_HA 0x9d033a90           0x7c         124   
.text.SYS_FS_setdefdir  0x9d033b0c           0x7c         124   
.text.TCPFind           0x9d033b88           0x7c         124   
.text.TCP_Flush         0x9d033c04           0x7c         124   
.text._TCPIPStackAddres 0x9d033c80           0x7c         124   
.text.MRF24W_MACGetConf 0x9d033cfc           0x7c         124   
.text.DeallocateDataRxB 0x9d033d78           0x7c         124   
.text.HTTPPrint_config_ 0x9d033df4           0x7c         124   
.text.LFSRRand          0x9d033e70           0x78         120   
.text.SYS_TICK_TimerSet 0x9d033ee8           0x78         120   
.text.DHCPDeRegisterHan 0x9d033f60           0x78         120   
.text.DNSClientDeInit   0x9d033fd8           0x78         120   
.text.SetWepSecurity    0x9d034050           0x78         120   
.text.ResetPll          0x9d0340c8           0x78         120   
.text.SendRAWDataFrame  0x9d034140           0x78         120   
.text.MRF24W_MACFlush   0x9d0341b8           0x78         120   
.text.SoftReset         0x9d034230           0x78         120   
.text.rand              0x9d0342a8           0x78         120   
.text.strstr            0x9d034320           0x78         120   
.text.MD5Initialize     0x9d034398           0x74         116   
.text.SYS_RANDOM_ADD    0x9d03440c           0x74         116   
.text.CommandCleanup    0x9d034480           0x74         116   
.text.SYS_FS_IsLegalDir 0x9d0344f4           0x74         116   
.text.TCPIP_IPV4_SetTxB 0x9d034568           0x74         116   
.text.TCP_GetUpperLayer 0x9d0345dc           0x74         116   
.text.TCP_IsPacketQueue 0x9d034650           0x74         116   
.text.TCP_ResetTransmit 0x9d0346c4           0x74         116   
.text._TCPIP_HEAP_FreeD 0x9d034738           0x74         116   
.text.UDPIsConnected    0x9d0347ac           0x74         116   
.text._TCPIPStackIsAddr 0x9d034820           0x74         116   
.text.WF_PsPollDisable  0x9d034894           0x74         116   
.text.EnsureWFisAwake   0x9d034908           0x74         116   
.text.RawRead           0x9d03497c           0x74         116   
.text.RawWrite          0x9d0349f0           0x74         116   
.text.RawInit           0x9d034a64           0x74         116   
.text.HTTPPrint_pot     0x9d034ad8           0x74         116   
.text.HTTPPrint_config_ 0x9d034b4c           0x74         116   
.text.SYS_INT_SourceRes 0x9d034bc0           0x70         112   
.text._sys_CONSOLE_PRIN 0x9d034c30           0x70         112   
.text._ARPDeleteCache   0x9d034ca0           0x70         112   
.text.ICMPInitialize    0x9d034d10           0x70         112   
.text.TCPIP_IPV4_Single 0x9d034d80           0x70         112   
.text.NBNSInit          0x9d034df0           0x70         112   
.text.TCPPutString      0x9d034e60           0x70         112   
.text.WF_Connect        0x9d034ed0           0x70         112   
.text.MRF24W_MACOpen    0x9d034f40           0x70         112   
.text.Write8BitWFRegist 0x9d034fb0           0x70         112   
.text.HTTPPrint_config_ 0x9d035020           0x70         112   
.text.HTTPPrint_config_ 0x9d035090           0x70         112   
.text.HTTPPrint_config_ 0x9d035100           0x70         112   
.text.HTTPPrint_config_ 0x9d035170           0x70         112   
.text.HTTPPrint_config_ 0x9d0351e0           0x70         112   
.text.CommandReset      0x9d035250           0x6c         108   
.text.MPFSGetPosition   0x9d0352bc           0x6c         108   
.text._ARPRefreshEntry  0x9d035328           0x6c         108   
.text._TCPGetRxFIFOFree 0x9d035394           0x6c         108   
.text.TcpClientIpv4Remo 0x9d035400           0x6c         108   
.text.TCPIP_HEAP_FreeSi 0x9d03546c           0x6c         108   
.rodata                 0x9d0354d8           0x6c         108  Read-only const 
.text.ProcessTCPIPMacGe 0x9d035544           0x6c         108   
.text.TCPIP_STACK_NetGa 0x9d0355b0           0x6c         108   
.text.TCPIP_STACK_NetPr 0x9d03561c           0x6c         108   
.text.TCPIP_STACK_NetSe 0x9d035688           0x6c         108   
.text.TCPIP_STACK_NetBI 0x9d0356f4           0x6c         108   
.text.TCPIP_STACK_Filte 0x9d035760           0x6c         108   
.text.TCPIP_Notificatio 0x9d0357cc           0x6c         108   
.text.SendPowerModeMsg  0x9d035838           0x6c         108   
.text.Read8BitWFRegiste 0x9d0358a4           0x6c         108   
.text.MRF24W_MACInit    0x9d035910           0x6c         108   
.text.MPFSClose         0x9d03597c           0x68         104   
.text.OAHashGetEntry    0x9d0359e4           0x68         104   
.text.TCPIP_IPV4_FreePa 0x9d035a4c           0x68         104   
.text._TcpSocketBind    0x9d035ab4           0x68         104   
.text._TcpSocketChk     0x9d035b1c           0x68         104   
.text._TcpFlush         0x9d035b84           0x68         104   
.text.TCPIsGetReady     0x9d035bec           0x68         104   
.text.TCPGetRxFIFOFree  0x9d035c54           0x68         104   
.text._UdpSocketBind    0x9d035cbc           0x68         104   
.text.MACPutHeader      0x9d035d24           0x68         104   
.text.TCPIP_STACK_IxToN 0x9d035d8c           0x68         104   
.text.TCPIP_STACK_NetNa 0x9d035df4           0x68         104   
.text.TCPIP_Notificatio 0x9d035e5c           0x68         104   
.rodata                 0x9d035ec4           0x68         104  Read-only const 
.text.MRF24W_MACEventDe 0x9d035f2c           0x68         104   
.text.RawCalculateCheck 0x9d035f94           0x68         104   
.text.MRF24W_MACPutArra 0x9d035ffc           0x68         104   
.rodata                 0x9d036064           0x68         104  Read-only const 
.text.btohexa_high      0x9d0360cc           0x64         100   
.text.btohexa_low       0x9d036130           0x64         100   
.text.DRV_MEDIA_ReadByt 0x9d036194           0x64         100   
.text.DHCPIsEnabled     0x9d0361f8           0x64         100   
.text.TCPIP_IPV4_GetDat 0x9d03625c           0x64         100   
.text.TCPSocketGetNet   0x9d0362c0           0x64         100   
.text._TCPIPStackIsNetL 0x9d036324           0x64         100   
.text.TCPIP_Notificatio 0x9d036388           0x64         100   
.text.WF_CPCreate       0x9d0363ec           0x64         100   
.text.MRF24W_MACEventSe 0x9d036450           0x64         100   
.text._sprintf_cdnopsux 0x9d0364b4           0x64         100   
.text.SYS_DRIVERS_Initi 0x9d036518           0x60          96   
.text.USART_PUTC        0x9d036578           0x60          96   
.text.HTTPReleaseMedia  0x9d0365d8           0x60          96   
.text.ICMPDeinitialize  0x9d036638           0x60          96   
.text.TCPIP_IPV4_SetRxB 0x9d036698           0x60          96   
.text.TCP_FreePacket    0x9d0366f8           0x60          96   
.text.MACCalcRxChecksum 0x9d036758           0x60          96   
.rodata                 0x9d0367b8           0x60          96  Read-only const 
.text.MRF24W_MACDeiniti 0x9d036818           0x60          96   
.text.mrf24w_MACSetRXHa 0x9d036878           0x60          96   
.text.WiFi_EintTask     0x9d0368d8           0x60          96   
.text.HTTPPrint_reboota 0x9d036938           0x60          96   
.text.SYS_INT_SourceDis 0x9d036998           0x5c          92   
.text.SYS_INT_PriorityS 0x9d0369f4           0x5c          92   
.text.SYS_INT_Subpriori 0x9d036a50           0x5c          92   
.text.MPFSGetLong       0x9d036aac           0x5c          92   
.text.USART_OPEN        0x9d036b08           0x5c          92   
.text._DHCPCleanup      0x9d036b64           0x5c          92   
.text.OAHashRemoveEntry 0x9d036bc0           0x5c          92   
.text.TCPFlush          0x9d036c1c           0x5c          92   
.text.MACGetArray       0x9d036c78           0x5c          92   
.text.MACPutArray       0x9d036cd4           0x5c          92   
.text.MACEventSetNotify 0x9d036d30           0x5c          92   
.text._TCPIPStackNetAdd 0x9d036d8c           0x5c          92   
.text._TCPIPStackNetMas 0x9d036de8           0x5c          92   
.text._TCPIPStackNetMac 0x9d036e44           0x5c          92   
.text.SetListenInterval 0x9d036ea0           0x5c          92   
.text.SetDtimInterval   0x9d036efc           0x5c          92   
.text.WF_SecurityWepSet 0x9d036f58           0x5c          92   
.text.WF_SecurityWpaSet 0x9d036fb4           0x5c          92   
.text.WF_SecurityWpsSet 0x9d037010           0x5c          92   
.text.WF_EintIsPending  0x9d03706c           0x5c          92   
.text.ConfigureSpiMRF24 0x9d0370c8           0x5c          92   
.text.mrf24w_MACPutHead 0x9d037124           0x5c          92   
.text.SignalWiFiConnect 0x9d037180           0x5c          92   
.text.WF_StartGratuitou 0x9d0371dc           0x5c          92   
.text.MRF24W_MACIsTxRea 0x9d037238           0x5c          92   
.text.SYS_INT_SourceEna 0x9d037294           0x58          88   
.text.USART_GETC        0x9d0372ec           0x58          88   
.text.LCD_ERASE         0x9d037344           0x58          88   
.text.WaitForDataByte   0x9d03739c           0x58          88   
.text._XEEFlashInit     0x9d0373f4           0x58          88   
.text.ARPHashKeyHash    0x9d03744c           0x58          88   
.text._TcpipHeapHandleT 0x9d0374a4           0x58          88   
.text._TCPIPStackIsNetU 0x9d0374fc           0x58          88   
.text.WF_NetworkTypeSet 0x9d037554           0x58          88   
.text.mrf24w_MACCalcRxC 0x9d0375ac           0x58          88   
.text.MRF24W_MACCalcIPB 0x9d037604           0x58          88   
.text.HTTPPrint_ddns_st 0x9d03765c           0x58          88   
.text.HTTPPrint_smtps_e 0x9d0376b4           0x58          88   
.text.HTTPPrint_snmp_en 0x9d03770c           0x58          88   
.text.SYS_INT_SourceSta 0x9d037764           0x54          84   
.text._SYS_CONSOLE_PUTC 0x9d0377b8           0x54          84   
.text._SYS_OUT_MESSAGE_ 0x9d03780c           0x54          84   
.text._ICMPAckPacket    0x9d037860           0x54          84   
.text._TcpDiscardTx     0x9d0378b4           0x54          84   
.text.TCPPut            0x9d037908           0x54          84   
.text._UdpSocketInit    0x9d03795c           0x54          84   
.text.UDPPut            0x9d0379b0           0x54          84   
.text.MACGetHeader      0x9d037a04           0x54          84   
.text.MACSetReadPtrInRx 0x9d037a58           0x54          84   
.text.MACCalcIPBufferCh 0x9d037aac           0x54          84   
.text.MACEventSetNotify 0x9d037b00           0x54          84   
.text.MACEventAck       0x9d037b54           0x54          84   
.text._TCPIPStackAddres 0x9d037ba8           0x54          84   
.text._TCPIPStackAddres 0x9d037bfc           0x54          84   
.text.mrf24w_MACDeiniti 0x9d037c50           0x54          84   
.text.GratuitousArpHand 0x9d037ca4           0x54          84   
.text.HTTPPrint_version 0x9d037cf8           0x54          84   
.rodata                 0x9d037d4c           0x54          84  Read-only const 
.text._vsnprintf_cdnops 0x9d037da0           0x54          84   
.text.vsnprintf         0x9d037df4           0x54          84   
.text._SYS_CONSOLE_MESS 0x9d037e48           0x50          80   
.text._TCPIP_AnnounceCl 0x9d037e98           0x50          80   
.text.HTTPPrint_        0x9d037ee8           0x50          80   
.text.ARPHashKeyCompare 0x9d037f38           0x50          80   
.text._DNSReleaseSocket 0x9d037f88           0x50          80   
.text.WF_SpiInit        0x9d037fd8           0x50          80   
.text.mrf24w_MACEventSe 0x9d038028           0x50          80   
.text.MRF24W_GetTraffic 0x9d038078           0x50          80   
.text.MRF24W_GetMgmtEve 0x9d0380c8           0x50          80   
.text.SignalDHCPSuccess 0x9d038118           0x50          80   
.text.InitGratuitousArp 0x9d038168           0x50          80   
.text.MRF24W_MACSetWrit 0x9d0381b8           0x50          80   
.text.MRF24W_MACSetRead 0x9d038208           0x50          80   
.text.MRF24W_MACSetBase 0x9d038258           0x50          80   
.text.StackNotification 0x9d0382a8           0x50          80   
.text.DRV_SPI_Initializ 0x9d0382f8           0x4c          76   
.text.TCPGet            0x9d038344           0x4c          76   
.text.UDPGet            0x9d038390           0x4c          76   
.text.MACSetWritePtr    0x9d0383dc           0x4c          76   
.text.MACSetReadPtr     0x9d038428           0x4c          76   
.text.MACEventGetPendin 0x9d038474           0x4c          76   
.text.WF_ChannelListSet 0x9d0384c0           0x4c          76   
.text.WF_EintEnable     0x9d03850c           0x4c          76   
.text.DhcpEventHandler  0x9d038558           0x4c          76   
.rodata                 0x9d0385a4           0x4c          76  Read-only const 
.text.mrf24w_MACPutArra 0x9d0385f0           0x4c          76   
.text.mrf24w_MACGetArra 0x9d03863c           0x4c          76   
.text.MRF24W_MACEventAc 0x9d038688           0x4c          76   
.text.SendRAWManagement 0x9d0386d4           0x4c          76   
.text.ScratchUnmount    0x9d038720           0x4c          76   
.text.MRF24W_MACSetRead 0x9d03876c           0x4c          76   
.text.WiFiMemory_write  0x9d0387b8           0x4c          76   
.text.INTEnable         0x9d038804           0x4c          76   
.text.strncat           0x9d038850           0x4c          76   
.text                   0x9d03889c           0x4c          76  App's exec code 
.text.SYS_CLK_Periphera 0x9d0388e8           0x48          72   
.text._SYS_CONSOLE_DATA 0x9d038930           0x48          72   
.text._SYS_CONSOLE_GETC 0x9d038978           0x48          72   
.text._SYS_OUT_MESSAGE_ 0x9d0389c0           0x48          72   
.rodata                 0x9d038a08           0x48          72  Read-only const 
.text.MPFSGetID         0x9d038a50           0x48          72   
.text.HTTPCurConnection 0x9d038a98           0x48          72   
.text.ARPHashKeyCopy    0x9d038ae0           0x48          72   
.text.DNSEndUsage       0x9d038b28           0x48          72   
.text.TCPIP_IPV4_SetSou 0x9d038b70           0x48          72   
.text.TCPIP_STACK_NetAd 0x9d038bb8           0x48          72   
.text.TCPIP_STACK_NetMa 0x9d038c00           0x48          72   
.text.TCPIP_STACK_NetMa 0x9d038c48           0x48          72   
.text.isEventNotifyBitS 0x9d038c90           0x48          72   
.text.mrf24w_MACCalcIPB 0x9d038cd8           0x48          72   
.text.mrf24w_MACEventSe 0x9d038d20           0x48          72   
.text.mrf24w_MACEventCl 0x9d038d68           0x48          72   
.text.mrf24w_MACEventAc 0x9d038db0           0x48          72   
.text.MRF24W_MACEventCl 0x9d038df8           0x48          72   
.text.OutputPowerSaveMo 0x9d038e40           0x48          72   
.text.WFEnableMRF24WMod 0x9d038e88           0x48          72   
.text.strncpy           0x9d038ed0           0x48          72   
.text.sbrk              0x9d038f18           0x48          72   
.text.SYS_CLK_ClockGet  0x9d038f60           0x44          68   
.text._SYS_OUT_MESSAGE  0x9d038fa4           0x44          68   
.text._sys_CONSOLE_PUTC 0x9d038fe8           0x44          68   
.text.USART_DATA_RDY    0x9d03902c           0x44          68   
.text.TCPIP_IPV4_SetPac 0x9d039070           0x44          68   
.text.MACClose          0x9d0390b4           0x44          68   
.text.MACDiscardRx      0x9d0390f8           0x44          68   
.text.MACIsTxReady      0x9d03913c           0x44          68   
.text.MACFlush          0x9d039180           0x44          68   
.text.MACCheckLink      0x9d0391c4           0x44          68   
.text.MACGetTxBaseAddr  0x9d039208           0x44          68   
.text.TCPIP_STACK_NetHa 0x9d03924c           0x44          68   
.text._TCPIPStackNetIx  0x9d039290           0x44          68   
.text._TCPIPStackSetGat 0x9d0392d4           0x44          68   
.text._TCPIPStackSetPri 0x9d039318           0x44          68   
.text._TCPIPStackSetSec 0x9d03935c           0x44          68   
.text._TCPIPStackNetToM 0x9d0393a0           0x44          68   
.text.SingleListInit    0x9d0393e4           0x44          68   
.text.WF_ConnectContext 0x9d039428           0x44          68   
.rodata                 0x9d03946c           0x44          68  Read-only const 
.text.WF_NetworkTypeGet 0x9d0394b0           0x44          68   
.text.WF_WepKeyTypeGet  0x9d0394f4           0x44          68   
.text.mrf24w_MACGetHead 0x9d039538           0x44          68   
.text.mrf24w_MACSetRead 0x9d03957c           0x44          68   
.text.WiFi_GratuitousAr 0x9d0395c0           0x44          68   
.text.MRF24W_MACProcess 0x9d039604           0x44          68   
.text.RawGetMgmtRxBuffe 0x9d039648           0x44          68   
.text.WF_SetWPATimeout  0x9d03968c           0x44          68   
.text.WF_SetTxMode      0x9d0396d0           0x44          68   
.text.WF_SetTxDataConfi 0x9d039714           0x44          68   
.text.WiFiMemory_read   0x9d039758           0x44          68   
.text.strncmp           0x9d03979c           0x44          68   
.text                   0x9d0397e0           0x44          68  App's exec code 
.text.XEEEndWrite       0x9d039824           0x40          64   
.text.HTTPCurConnection 0x9d039864           0x40          64   
.text.HTTPCurConnection 0x9d0398a4           0x40          64   
.text.TCPIP_IPV4_Task   0x9d0398e4           0x40          64   
.text.UDPResetHeader    0x9d039924           0x40          64   
.text.WF_CASetEventNoti 0x9d039964           0x40          64   
.text.WF_SecurityOpenSe 0x9d0399a4           0x40          64   
.text.WF_ConfigDataSave 0x9d0399e4           0x40          64   
.text.MRF24W_MACConnect 0x9d039a24           0x40          64   
.text.mrf24w_MACEventGe 0x9d039a64           0x40          64   
.text.DeallocateMgmtRxB 0x9d039aa4           0x40          64   
.text.MRF24W_MACDiscard 0x9d039ae4           0x40          64   
.text.WF_GetTxMode      0x9d039b24           0x40          64   
.text.WF_MacAddressSet  0x9d039b64           0x40          64   
.text.WF_MacAddressGet  0x9d039ba4           0x40          64   
.text.WF_RegionalDomain 0x9d039be4           0x40          64   
.text.SpiChnDataRdy     0x9d039c24           0x40          64   
.text._sys_CONSOLE_MESS 0x9d039c64           0x3c          60   
.text.DRV_MEDIA_WriteFl 0x9d039ca0           0x3c          60   
.text.HTTPCurConnection 0x9d039cdc           0x3c          60   
.text.HTTPCurConnection 0x9d039d18           0x3c          60   
.text._ARPDeleteClients 0x9d039d54           0x3c          60   
.text.ARPTmoHandler     0x9d039d90           0x3c          60   
.text.TCPIP_IPV4_GetUpp 0x9d039dcc           0x3c          60   
.text.TCPIP_IPV4_GetPay 0x9d039e08           0x3c          60   
.rodata                 0x9d039e44           0x3c          60  Read-only const 
.text.WifiAsyncSetEvent 0x9d039e80           0x3c          60   
.text.mrf24w_MACSetWrit 0x9d039ebc           0x3c          60   
.text.mrf24w_MACSetRead 0x9d039ef8           0x3c          60   
.text.mrf24w_MACSetBase 0x9d039f34           0x3c          60   
.text.PORTSetPinsDigita 0x9d039f70           0x3c          60   
.text.PORTSetPinsDigita 0x9d039fac           0x3c          60   
.text                   0x9d039fe8           0x38          56  App's exec code 
.text.SYS_Tasks         0x9d03a020           0x38          56   
.text._SYS_OUT_INIT     0x9d03a058           0x38          56   
.text.DRV_MEDIA_Close   0x9d03a090           0x38          56   
.text._OAHashProbeStep  0x9d03a0c8           0x38          56   
.rodata                 0x9d03a100           0x38          56  Read-only const 
.text.RenewDhcp         0x9d03a138           0x38          56   
.text.mrf24w_MACClose   0x9d03a170           0x38          56   
.rodata                 0x9d03a1a8           0x70         112  Read-only const 
.text.INTSetVectorPrior 0x9d03a218           0x38          56   
.text.INTSetVectorSubPr 0x9d03a250           0x38          56   
.text._sys_CONSOLE_DATA 0x9d03a288           0x34          52   
.text._sys_CONSOLE_GETC 0x9d03a2bc           0x34          52   
.text.XEEBeginWrite     0x9d03a2f0           0x34          52   
.text.DRV_MEDIA_ClientS 0x9d03a324           0x34          52   
.text.HTTPCurConnection 0x9d03a358           0x34          52   
.text.HTTPCurConnection 0x9d03a38c           0x34          52   
.text.HTTPCurConnection 0x9d03a3c0           0x34          52   
.text.HTTPCurConnection 0x9d03a3f4           0x34          52   
.text.HTTPCurConnection 0x9d03a428           0x34          52   
.text.TCPIP_IPV4_SetDes 0x9d03a45c           0x34          52   
.text.TCPIP_IPV4_GetDes 0x9d03a490           0x34          52   
.text.TCPIP_IPV4_GetSou 0x9d03a4c4           0x34          52   
.text.ProcessTCPIPMacEr 0x9d03a4f8           0x34          52   
.rodata                 0x9d03a52c           0x34          52  Read-only const 
.text.WF_EintIsDisabled 0x9d03a560           0x34          52   
.text.WF_DeInit         0x9d03a594           0x34          52   
.text.WF_SpiDisableChip 0x9d03a5c8           0x34          52   
.text.mrf24w_MACGetRead 0x9d03a5fc           0x34          52   
.text.mrf24w_MACIsTxRea 0x9d03a630           0x34          52   
.text.mrf24w_MACFlush   0x9d03a664           0x34          52   
.text.mrf24w_MACDiscard 0x9d03a698           0x34          52   
.text.mrf24w_MACCheckLi 0x9d03a6cc           0x34          52   
.text.SetNetworkConfig  0x9d03a700           0x34          52   
.rodata                 0x9d03a734           0x34          52  Read-only const 
.text.HTTPPrint_reboot  0x9d03a768           0x34          52   
.text.INTEnableSystemMu 0x9d03a79c           0x34          52   
.text.SYS_USERIO_Tasks  0x9d03a7d0           0x30          48   
.text.SYS_FS_mpfs2fs_In 0x9d03a800           0x30          48   
.text.TCPIP_IPV4_TmoHan 0x9d03a830           0x30          48   
.text._TcpTmoHandler    0x9d03a860           0x30          48   
.text.TCPIP_STACK_TickH 0x9d03a890           0x30          48   
.text.SetEventNotificat 0x9d03a8c0           0x30          48   
.text.SetLogicalConnect 0x9d03a8f0           0x30          48   
.text.SetAppPowerSaveMo 0x9d03a920           0x30          48   
.text.WF_GetPowerSaveSt 0x9d03a950           0x30          48   
.text.SetPowerSaveState 0x9d03a980           0x30          48   
.text.WF_SpiEnableChipS 0x9d03a9b0           0x30          48   
.rodata                 0x9d03a9e0           0x30          48  Read-only const 
.text.MRF24W_MACCheckLi 0x9d03aa10           0x30          48   
.text.strcat            0x9d03aa40           0x30          48   
.text.SYS_WDT_Clear     0x9d03aa70           0x2c          44   
.text.TCPIP_ANNOUNCE_Ta 0x9d03aa9c           0x2c          44   
.text.ARPTaskPending    0x9d03aac8           0x2c          44   
.text.TCPIP_IPV4_TaskPe 0x9d03aaf4           0x2c          44   
.text.TCPTaskPending    0x9d03ab20           0x2c          44   
.text.WF_EintDisable    0x9d03ab4c           0x2c          44   
.text.WiFiAsyncTaskPend 0x9d03ab78           0x2c          44   
.rodata                 0x9d03aba4           0x2c          44  Read-only const 
.text.MRF24W_MACEventGe 0x9d03abd0           0x2c          44   
.text.HTTPPrint_read_co 0x9d03abfc           0x2c          44   
.text.HTTPPrint_write_c 0x9d03ac28           0x2c          44   
.text.HTTPPrint_ddns_se 0x9d03ac54           0x2c          44   
.text.strchr            0x9d03ac80           0x2c          44   
.text._stub_sbd_memlayo 0x9d03acac           0x2c          44   
.text.SYS_FS_GenError   0x9d03acd8           0x28          40   
.rodata                 0x9d03ad00           0x28          40  Read-only const 
.text.DHCPServerDisable 0x9d03ad28           0x28          40   
.text.DHCPServerEnable  0x9d03ad50           0x28          40   
.text.ZCLLEnable        0x9d03ad78           0x28          40   
.text.SetSleepNeeded    0x9d03ada0           0x28          40   
.text.mrf24w_MACGetTxBa 0x9d03adc8           0x28          40   
.text.WF_OutputConnecti 0x9d03adf0           0x28          40   
.text.SetDhcpProgressSt 0x9d03ae18           0x28          40   
.text.SignalMgmtConfirm 0x9d03ae40           0x28          40   
.text.INTClearFlag      0x9d03ae68           0x28          40   
.text.TCPIP_STACK_GetDe 0x9d03ae90           0x24          36   
.text.TCPIP_STACK_Netwo 0x9d03aeb4           0x24          36   
.text.GetEventNotificat 0x9d03aed8           0x24          36   
.text.WFisConnected     0x9d03aefc           0x24          36   
.text.GetWiFiNetworkTyp 0x9d03af20           0x24          36   
.text.WifiAsyncClearAll 0x9d03af44           0x24          36   
.text.isSleepNeeded     0x9d03af68           0x24          36   
.text.ClearSleepNeeded  0x9d03af8c           0x24          36   
.text.GetAppPowerSaveMo 0x9d03afb0           0x24          36   
.text.InitPowerSaveTask 0x9d03afd4           0x24          36   
.text.isDhcpInProgress  0x9d03aff8           0x24          36   
.text.GetReadPtrRawWind 0x9d03b01c           0x24          36   
.text.GetNetworkConfig  0x9d03b040           0x24          36   
.text.MRF24W_MACGetRead 0x9d03b064           0x24          36   
.text.HTTPPrint_lcdtext 0x9d03b088           0x24          36   
.text.HTTPPrint_ddns_us 0x9d03b0ac           0x24          36   
.text.HTTPPrint_ddns_pa 0x9d03b0d0           0x24          36   
.text.HTTPPrint_ddns_ho 0x9d03b0f4           0x24          36   
.text.free              0x9d03b118           0x24          36   
.text._snprintf_cdnopsu 0x9d03b13c           0x24          36   
.text.toupper           0x9d03b160           0x24          36   
.rodata                 0x9d03b184           0x20          32  Read-only const 
.text.SetEapSecurity    0x9d03b1a4           0x20          32   
.text.MRF24W_MACPowerDo 0x9d03b1c4           0x20          32   
.text.MRF24W_MACPowerUp 0x9d03b1e4           0x20          32   
.text.SpiChnReadC       0x9d03b204           0x20          32   
.text.SpiChnWriteC      0x9d03b224           0x20          32   
.text.SpiChnTxBuffEmpty 0x9d03b244           0x20          32   
.text.INTRestoreInterru 0x9d03b264           0x1c          28   
.text.srand             0x9d03b280           0x1c          28   
.text.SYS_Reboot        0x9d03b29c           0x18          24   
.text.CheKseg0CacheOn   0x9d03b2b4           0x18          24   
.text                   0x9d03b2cc           0x18          24  App's exec code 
.rodata                 0x9d03b2e4           0x34          52  Read-only const 
.text.OpenCoreTimer     0x9d03b318            0xc          12   
.text._bootstrap_except 0x9d03b324            0xc          12   
.text.INTDisableInterru 0x9d03b330            0x8           8   
.text.INTEnableInterrup 0x9d03b338            0x8           8   
.text._on_reset         0x9d03b340            0x8           8   
.text._on_bootstrap     0x9d03b348            0x8           8   
.rodata                 0x9d03b350            0x8           8  Read-only const 
      Total kseg0_program_mem used  :     0x3b334      242484  46.3% of 0x80000

kseg0 Boot-Memory Usage
section                    address  length [bytes]      (dec)  Description
-------                 ----------  -------------------------  -----------
         Total kseg0_boot_mem used  :           0           0  <1% of 0x970

Exception-Memory Usage 
section                    address  length [bytes]      (dec)  Description
-------                 ----------  -------------------------  -----------
.app_excpt              0x9fc01180           0x10          16  General-Exception 
.vector_0               0x9fc01200            0x8           8  Interrupt Vector 0 
.vector_7               0x9fc012e0            0x8           8  Interrupt Vector 7 
.vector_15              0x9fc013e0            0x8           8  Interrupt Vector 15 
.vector_26              0x9fc01540            0x8           8  Interrupt Vector 26 
          Total exception_mem used  :        0x30          48  1.2% of 0x1000

kseg1 Boot-Memory Usage
section                    address  length [bytes]      (dec)  Description
-------                 ----------  -------------------------  -----------
.reset                  0xbfc00000          0x1f4         500  Reset handler 
.bev_excpt              0xbfc00380           0x10          16  BEV-Exception 
         Total kseg1_boot_mem used  :       0x204         516  44.2% of 0x490
        --------------------------------------------------------------------------
         Total Program Memory used  :     0x3b568      243048  45.7% of 0x81e00
        --------------------------------------------------------------------------


kseg1 Data-Memory Usage
section                    address  length [bytes]      (dec)  Description
-------                 ----------  -------------------------  -----------
.eh_frame               0xa0000000           0x30          48   
.sdata                  0xa0000030          0x1e8         488  Small init data 
.sbss                   0xa0000218          0x410        1040  Small uninit data 
.bss                    0xa0000628         0x1b68        7016  Uninitialized data 
.bss                    0xa0002190          0x210         528  Uninitialized data 
.data                   0xa00023a0          0x174         372  Initialized data 
.bss                    0xa0002514          0x248         584  Uninitialized data 
.data                   0xa000275c           0x44          68  Initialized data 
.bss                    0xa00027a0           0x6c         108  Uninitialized data 
.bss                    0xa0002810           0x10          16  Uninitialized data 
         Total kseg1_data_mem used  :      0x281c       10268  7.8% of 0x20000
        --------------------------------------------------------------------------
            Total Data Memory used  :      0x281c       10268  7.8% of 0x20000
        --------------------------------------------------------------------------


Dynamic Data-Memory Reservation
section                    address  length [bytes]      (dec)  Description
-------                 ----------  -------------------------  -----------
heap                    0xa0002828         0x5208       21000  Reserved for heap 
stack                   0xa0007a48        0x185b0       99760  Reserved for stack 

        --------------------------------------------------------------------------

Discarded input sections

 .data          0x00000000        0x0 c:/program files (x86)/microchip/xc32/v1.10/bin/../lib/gcc/pic32mx/4.5.1/../../../../pic32mx/lib/size/crt0.o
 .bss           0x00000000        0x0 c:/program files (x86)/microchip/xc32/v1.10/bin/../lib/gcc/pic32mx/4.5.1/../../../../pic32mx/lib/size/crt0.o
 .pdr           0x00000000       0xa0 c:/program files (x86)/microchip/xc32/v1.10/bin/../lib/gcc/pic32mx/4.5.1/../../../../pic32mx/lib/size/crt0.o
 .text          0x00000000        0x0 build/default/production/_ext/1293749816/bsp.o
 .data          0x00000000        0x0 build/default/production/_ext/1293749816/bsp.o
 .bss           0x00000000        0x0 build/default/production/_ext/1293749816/bsp.o
 .reginfo       0x00000000       0x18 build/default/production/_ext/1293749816/bsp.o
 .pdr           0x00000000       0x20 build/default/production/_ext/1293749816/bsp.o
 .text          0x00000000        0x0 build/default/production/_ext/101875047/hashes.o
 .data          0x00000000        0x0 build/default/production/_ext/101875047/hashes.o
 .bss           0x00000000        0x0 build/default/production/_ext/101875047/hashes.o
 .reginfo       0x00000000       0x18 build/default/production/_ext/101875047/hashes.o
 .pdr           0x00000000      0x120 build/default/production/_ext/101875047/hashes.o
 .text.HashAddData
                0x00000000       0x94 build/default/production/_ext/101875047/hashes.o
 .text.SHA1Calculate
                0x00000000      0x4b8 build/default/production/_ext/101875047/hashes.o
 .text          0x00000000        0x0 build/default/production/_ext/101875047/lfsr.o
 .data          0x00000000        0x0 build/default/production/_ext/101875047/lfsr.o
 .bss           0x00000000        0x0 build/default/production/_ext/101875047/lfsr.o
 .reginfo       0x00000000       0x18 build/default/production/_ext/101875047/lfsr.o
 .pdr           0x00000000       0x40 build/default/production/_ext/101875047/lfsr.o
 .text          0x00000000        0x0 build/default/production/_ext/101875047/big_int.o
 .data          0x00000000        0x0 build/default/production/_ext/101875047/big_int.o
 .bss           0x00000000        0x0 build/default/production/_ext/101875047/big_int.o
 .reginfo       0x00000000       0x18 build/default/production/_ext/101875047/big_int.o
 .pdr           0x00000000      0x1a0 build/default/production/_ext/101875047/big_int.o
 .text.BigInt   0x00000000       0x70 build/default/production/_ext/101875047/big_int.o
 .text.BigIntZero
                0x00000000       0x68 build/default/production/_ext/101875047/big_int.o
 .text.BigIntMod
                0x00000000      0x220 build/default/production/_ext/101875047/big_int.o
 .text.BigIntCompare
                0x00000000      0x16c build/default/production/_ext/101875047/big_int.o
 .text.BigIntMagnitudeDifference
                0x00000000       0x58 build/default/production/_ext/101875047/big_int.o
 .text.BigIntMagnitude
                0x00000000       0x50 build/default/production/_ext/101875047/big_int.o
 .text.BigIntMSB
                0x00000000       0xac build/default/production/_ext/101875047/big_int.o
 .text.BigIntMultiply
                0x00000000       0x94 build/default/production/_ext/101875047/big_int.o
 .text.BigIntSquare
                0x00000000       0x74 build/default/production/_ext/101875047/big_int.o
 .text.BigIntAdd
                0x00000000       0x74 build/default/production/_ext/101875047/big_int.o
 .text.BigIntSubtract
                0x00000000       0x74 build/default/production/_ext/101875047/big_int.o
 .text.BigIntCopy
                0x00000000       0x70 build/default/production/_ext/101875047/big_int.o
 .text.BigIntSwapEndianness
                0x00000000       0x9c build/default/production/_ext/101875047/big_int.o
 .text          0x00000000      0x400 build/default/production/_ext/101875047/big_int_helper_c32.o
 .data          0x00000000        0x0 build/default/production/_ext/101875047/big_int_helper_c32.o
 .bss           0x00000000       0x20 build/default/production/_ext/101875047/big_int_helper_c32.o
 .reginfo       0x00000000       0x18 build/default/production/_ext/101875047/big_int_helper_c32.o
 .pdr           0x00000000      0x100 build/default/production/_ext/101875047/big_int_helper_c32.o
 .text          0x00000000        0x0 build/default/production/_ext/101875047/helpers.o
 .data          0x00000000        0x0 build/default/production/_ext/101875047/helpers.o
 .bss           0x00000000        0x0 build/default/production/_ext/101875047/helpers.o
 .reginfo       0x00000000       0x18 build/default/production/_ext/101875047/helpers.o
 .pdr           0x00000000      0x100 build/default/production/_ext/101875047/helpers.o
 .text.strnchr  0x00000000       0xb4 build/default/production/_ext/101875047/helpers.o
 .text.strncpy_m
                0x00000000      0x10c build/default/production/_ext/101875047/helpers.o
 .text          0x00000000        0x0 build/default/production/_ext/1472/berkeley_tcp_client_demo.o
 .data          0x00000000        0x0 build/default/production/_ext/1472/berkeley_tcp_client_demo.o
 .bss           0x00000000        0x0 build/default/production/_ext/1472/berkeley_tcp_client_demo.o
 .reginfo       0x00000000       0x18 build/default/production/_ext/1472/berkeley_tcp_client_demo.o
 .pdr           0x00000000        0x0 build/default/production/_ext/1472/berkeley_tcp_client_demo.o
 .text          0x00000000        0x0 build/default/production/_ext/1472/berkeley_tcp_server_demo.o
 .data          0x00000000        0x0 build/default/production/_ext/1472/berkeley_tcp_server_demo.o
 .bss           0x00000000        0x0 build/default/production/_ext/1472/berkeley_tcp_server_demo.o
 .reginfo       0x00000000       0x18 build/default/production/_ext/1472/berkeley_tcp_server_demo.o
 .pdr           0x00000000        0x0 build/default/production/_ext/1472/berkeley_tcp_server_demo.o
 .text          0x00000000        0x0 build/default/production/_ext/1472/berkeley_udp_client_demo.o
 .data          0x00000000        0x0 build/default/production/_ext/1472/berkeley_udp_client_demo.o
 .bss           0x00000000        0x0 build/default/production/_ext/1472/berkeley_udp_client_demo.o
 .reginfo       0x00000000       0x18 build/default/production/_ext/1472/berkeley_udp_client_demo.o
 .pdr           0x00000000        0x0 build/default/production/_ext/1472/berkeley_udp_client_demo.o
 .text          0x00000000        0x0 build/default/production/_ext/1472/generic_tcp_client.o
 .data          0x00000000        0x0 build/default/production/_ext/1472/generic_tcp_client.o
 .bss           0x00000000        0x0 build/default/production/_ext/1472/generic_tcp_client.o
 .reginfo       0x00000000       0x18 build/default/production/_ext/1472/generic_tcp_client.o
 .pdr           0x00000000        0x0 build/default/production/_ext/1472/generic_tcp_client.o
 .text          0x00000000        0x0 build/default/production/_ext/1472/generic_tcp_server.o
 .data          0x00000000        0x0 build/default/production/_ext/1472/generic_tcp_server.o
 .bss           0x00000000        0x0 build/default/production/_ext/1472/generic_tcp_server.o
 .reginfo       0x00000000       0x18 build/default/production/_ext/1472/generic_tcp_server.o
 .pdr           0x00000000        0x0 build/default/production/_ext/1472/generic_tcp_server.o
 .text          0x00000000        0x0 build/default/production/_ext/1472/ping_demo.o
 .data          0x00000000        0x0 build/default/production/_ext/1472/ping_demo.o
 .bss           0x00000000        0x0 build/default/production/_ext/1472/ping_demo.o
 .reginfo       0x00000000       0x18 build/default/production/_ext/1472/ping_demo.o
 .pdr           0x00000000       0x60 build/default/production/_ext/1472/ping_demo.o
 .sbss          0x00000000        0x8 build/default/production/_ext/1472/ping_demo.o
 .sdata         0x00000000        0x4 build/default/production/_ext/1472/ping_demo.o
 .text.Ping4    0x00000000       0x90 build/default/production/_ext/1472/ping_demo.o
 .text.PingDemoTask
                0x00000000       0x20 build/default/production/_ext/1472/ping_demo.o
 .rodata        0x00000000        0xc build/default/production/_ext/1472/ping_demo.o
 .text.PingProcessIPv4
                0x00000000      0x19c build/default/production/_ext/1472/ping_demo.o
 .text          0x00000000        0x0 build/default/production/_ext/1472/smtp_demo.o
 .data          0x00000000        0x0 build/default/production/_ext/1472/smtp_demo.o
 .bss           0x00000000        0x0 build/default/production/_ext/1472/smtp_demo.o
 .reginfo       0x00000000       0x18 build/default/production/_ext/1472/smtp_demo.o
 .pdr           0x00000000        0x0 build/default/production/_ext/1472/smtp_demo.o
 .text          0x00000000        0x0 build/default/production/_ext/365611741/system_services.o
 .data          0x00000000        0x0 build/default/production/_ext/365611741/system_services.o
 .bss           0x00000000        0x0 build/default/production/_ext/365611741/system_services.o
 .reginfo       0x00000000       0x18 build/default/production/_ext/365611741/system_services.o
 .pdr           0x00000000      0x420 build/default/production/_ext/365611741/system_services.o
 .text.SYS_RTCC_Initialize
                0x00000000       0xf4 build/default/production/_ext/365611741/system_services.o
 .text.SYS_RTCC_DateGet
                0x00000000       0x4c build/default/production/_ext/365611741/system_services.o
 .text.SYS_RTCC_TimeGet
                0x00000000       0x4c build/default/production/_ext/365611741/system_services.o
 .text.SYS_TICK_MsDelay
                0x00000000       0x88 build/default/production/_ext/365611741/system_services.o
 .text.SYS_TICK_UsDelay
                0x00000000       0x88 build/default/production/_ext/365611741/system_services.o
 .text.SYS_TICK_NsDelay
                0x00000000       0xa0 build/default/production/_ext/365611741/system_services.o
 .text          0x00000000        0x0 build/default/production/_ext/365611741/system_debug.o
 .data          0x00000000        0x0 build/default/production/_ext/365611741/system_debug.o
 .bss           0x00000000        0x0 build/default/production/_ext/365611741/system_debug.o
 .reginfo       0x00000000       0x18 build/default/production/_ext/365611741/system_debug.o
 .pdr           0x00000000      0x2c0 build/default/production/_ext/365611741/system_debug.o
 .text.__sys_assert
                0x00000000       0x3c build/default/production/_ext/365611741/system_debug.o
 .text._SYS_PRINT
                0x00000000       0xcc build/default/production/_ext/365611741/system_debug.o
 .text._SYS_CONSOLE_GETLINE
                0x00000000       0x58 build/default/production/_ext/365611741/system_debug.o
 .text.SYS_OUT_GET_LCD_MESSAGE
                0x00000000       0x28 build/default/production/_ext/365611741/system_debug.o
 .text          0x00000000        0x0 build/default/production/_ext/365611741/system_random.o
 .data          0x00000000        0x0 build/default/production/_ext/365611741/system_random.o
 .reginfo       0x00000000       0x18 build/default/production/_ext/365611741/system_random.o
 .pdr           0x00000000       0xa0 build/default/production/_ext/365611741/system_random.o
 .text.SYS_RANDOM_GET
                0x00000000       0x84 build/default/production/_ext/365611741/system_random.o
 .text._SYS_RANDOM_DE_INIT
                0x00000000       0x20 build/default/production/_ext/365611741/system_random.o
 .text          0x00000000        0x0 build/default/production/_ext/365611741/system_command.o
 .data          0x00000000        0x0 build/default/production/_ext/365611741/system_command.o
 .reginfo       0x00000000       0x18 build/default/production/_ext/365611741/system_command.o
 .pdr           0x00000000      0x2a0 build/default/production/_ext/365611741/system_command.o
 .text._SYS_COMMAND_ADDGRP
                0x00000000      0x1b4 build/default/production/_ext/365611741/system_command.o
 .text          0x00000000        0x0 build/default/production/_ext/365611741/system_userio.o
 .data          0x00000000        0x0 build/default/production/_ext/365611741/system_userio.o
 .reginfo       0x00000000       0x18 build/default/production/_ext/365611741/system_userio.o
 .pdr           0x00000000      0x100 build/default/production/_ext/365611741/system_userio.o
 .text.SYS_USERIO_ButtonGetBitMap
                0x00000000       0x68 build/default/production/_ext/365611741/system_userio.o
 .text.SYS_USERIO_ButtonGet
                0x00000000      0x140 build/default/production/_ext/365611741/system_userio.o
 .text.SYS_USERIO_ButtonsTest
                0x00000000       0xa8 build/default/production/_ext/365611741/system_userio.o
 .text          0x00000000        0x0 build/default/production/_ext/97638081/sys_fs.o
 .data          0x00000000        0x0 build/default/production/_ext/97638081/sys_fs.o
 .reginfo       0x00000000       0x18 build/default/production/_ext/97638081/sys_fs.o
 .pdr           0x00000000      0x8a0 build/default/production/_ext/97638081/sys_fs.o
 .text.SYS_FS_mpfs2fs_Deinit
                0x00000000       0x30 build/default/production/_ext/97638081/sys_fs.o
 .text.SYS_FS_mpfs2fs_Open
                0x00000000       0x3c build/default/production/_ext/97638081/sys_fs.o
 .text.SYS_FS_mpfs2fs_OpenID
                0x00000000       0x40 build/default/production/_ext/97638081/sys_fs.o
 .text.SYS_FS_mpfs2fs_Close
                0x00000000       0x40 build/default/production/_ext/97638081/sys_fs.o
 .text.SYS_FS_mpfs2fs_Get
                0x00000000       0x48 build/default/production/_ext/97638081/sys_fs.o
 .text.SYS_FS_mpfs2fs_ArrayGet
                0x00000000       0x50 build/default/production/_ext/97638081/sys_fs.o
 .text.SYS_FS_mpfs2fs_LongGet
                0x00000000       0x48 build/default/production/_ext/97638081/sys_fs.o
 .text.SYS_FS_mpfs2fs_Seek
                0x00000000       0x50 build/default/production/_ext/97638081/sys_fs.o
 .text.SYS_FS_mpfs2fs_Format
                0x00000000       0x30 build/default/production/_ext/97638081/sys_fs.o
 .text.SYS_FS_mpfs2fs_ArrayPut
                0x00000000       0x50 build/default/production/_ext/97638081/sys_fs.o
 .text.SYS_FS_mpfs2fs_PutEnd
                0x00000000       0x50 build/default/production/_ext/97638081/sys_fs.o
 .text.SYS_FS_mpfs2fs_TimestampGet
                0x00000000       0x40 build/default/production/_ext/97638081/sys_fs.o
 .text.SYS_FS_mpfs2fs_MicrotimeGet
                0x00000000       0x40 build/default/production/_ext/97638081/sys_fs.o
 .text.SYS_FS_mpfs2fs_FlagsGet
                0x00000000       0x40 build/default/production/_ext/97638081/sys_fs.o
 .text.SYS_FS_mpfs2fs_SizeGet
                0x00000000       0x40 build/default/production/_ext/97638081/sys_fs.o
 .text.SYS_FS_mpfs2fs_BytesRemGet
                0x00000000       0x40 build/default/production/_ext/97638081/sys_fs.o
 .text.SYS_FS_mpfs2fs_StartAddrGet
                0x00000000       0x40 build/default/production/_ext/97638081/sys_fs.o
 .text.SYS_FS_mpfs2fs_EndAddrGet
                0x00000000       0x40 build/default/production/_ext/97638081/sys_fs.o
 .text.SYS_FS_mpfs2fs_FilenameGet
                0x00000000       0x58 build/default/production/_ext/97638081/sys_fs.o
 .text.SYS_FS_mpfs2fs_PositionGet
                0x00000000       0x40 build/default/production/_ext/97638081/sys_fs.o
 .text.SYS_FS_mpfs2fs_IDGet
                0x00000000       0x40 build/default/production/_ext/97638081/sys_fs.o
 .text.SYS_FS_IsLegalFileString
                0x00000000      0x144 build/default/production/_ext/97638081/sys_fs.o
 .text.SYS_FS_IsLegalFileChar
                0x00000000       0x7c build/default/production/_ext/97638081/sys_fs.o
 .text.SYS_FS_ExtractFilename
                0x00000000      0x104 build/default/production/_ext/97638081/sys_fs.o
 .text.SYS_FS_IsBadString
                0x00000000       0xd8 build/default/production/_ext/97638081/sys_fs.o
 .text.SYS_FS_ExtractPathname
                0x00000000      0x198 build/default/production/_ext/97638081/sys_fs.o
 .text.SYS_FS_createMBR
                0x00000000       0x64 build/default/production/_ext/97638081/sys_fs.o
 .text.SYS_FS_format
                0x00000000       0x6c build/default/production/_ext/97638081/sys_fs.o
 .text.SYS_FS_open
                0x00000000      0x374 build/default/production/_ext/97638081/sys_fs.o
 .text.SYS_FS_close
                0x00000000      0x198 build/default/production/_ext/97638081/sys_fs.o
 .text.SYS_FS_Loc2SysDesc
                0x00000000       0x74 build/default/production/_ext/97638081/sys_fs.o
 .text.SYS_FS_Sys2LocDesc
                0x00000000       0x90 build/default/production/_ext/97638081/sys_fs.o
 .text.SYS_FS_NextDescriptorGet
                0x00000000      0x150 build/default/production/_ext/97638081/sys_fs.o
 .text.SYS_FS_DescriptorIndexGet
                0x00000000      0x158 build/default/production/_ext/97638081/sys_fs.o
 .text.SYS_FS_DescriptorNameGet
                0x00000000      0x150 build/default/production/_ext/97638081/sys_fs.o
 .text.SYS_FS_fsize
                0x00000000       0xe0 build/default/production/_ext/97638081/sys_fs.o
 .text.SYS_FS_ftell
                0x00000000       0xe0 build/default/production/_ext/97638081/sys_fs.o
 .text.SYS_FS_fgetname
                0x00000000      0x11c build/default/production/_ext/97638081/sys_fs.o
 .text.SYS_FS_fstat
                0x00000000      0x114 build/default/production/_ext/97638081/sys_fs.o
 .text.SYS_FS_read
                0x00000000      0x18c build/default/production/_ext/97638081/sys_fs.o
 .text.SYS_FS_write
                0x00000000      0x134 build/default/production/_ext/97638081/sys_fs.o
 .text.SYS_FS_FSFromMountName
                0x00000000       0xe8 build/default/production/_ext/97638081/sys_fs.o
 .text.SYS_FS_FileTypeGet
                0x00000000       0xcc build/default/production/_ext/97638081/sys_fs.o
 .text.FS_MountRecGet
                0x00000000       0xf4 build/default/production/_ext/97638081/sys_fs.o
 .text.SYS_FS_fclose
                0x00000000       0x28 build/default/production/_ext/97638081/sys_fs.o
 .text.SYS_FS_fflush
                0x00000000       0x28 build/default/production/_ext/97638081/sys_fs.o
 .text.SYS_FS_fread
                0x00000000       0x34 build/default/production/_ext/97638081/sys_fs.o
 .text.SYS_FS_fwrite
                0x00000000       0x34 build/default/production/_ext/97638081/sys_fs.o
 .text.SYS_FS_remove
                0x00000000       0x28 build/default/production/_ext/97638081/sys_fs.o
 .text.SYS_FS_deinitialize
                0x00000000      0x128 build/default/production/_ext/97638081/sys_fs.o
 .text.SYS_FS_reinitialize
                0x00000000       0x58 build/default/production/_ext/97638081/sys_fs.o
 .text.SYS_FS_mkdir
                0x00000000       0xe0 build/default/production/_ext/97638081/sys_fs.o
 .text.SYS_FS_rmdir
                0x00000000       0xe8 build/default/production/_ext/97638081/sys_fs.o
 .text.SYS_FS_getcwd
                0x00000000       0x64 build/default/production/_ext/97638081/sys_fs.o
 .text.SYS_FS_lseek
                0x00000000      0x150 build/default/production/_ext/97638081/sys_fs.o
 .text.SYS_FS_unmount
                0x00000000       0x28 build/default/production/_ext/97638081/sys_fs.o
 .text.SYS_FS_error
                0x00000000       0x24 build/default/production/_ext/97638081/sys_fs.o
 .text.SYS_FS_clearerror
                0x00000000       0x24 build/default/production/_ext/97638081/sys_fs.o
 .text          0x00000000        0x0 build/default/production/_ext/97638081/mpfs2.o
 .data          0x00000000        0x0 build/default/production/_ext/97638081/mpfs2.o
 .reginfo       0x00000000       0x18 build/default/production/_ext/97638081/mpfs2.o
 .pdr           0x00000000      0x300 build/default/production/_ext/97638081/mpfs2.o
 .text.MPFSFormat
                0x00000000       0xe0 build/default/production/_ext/97638081/mpfs2.o
 .text.MPFSPutArray
                0x00000000       0x68 build/default/production/_ext/97638081/mpfs2.o
 .text.MPFSPutEnd
                0x00000000       0x94 build/default/production/_ext/97638081/mpfs2.o
 .text.MPFSGetTimestamp
                0x00000000       0xb4 build/default/production/_ext/97638081/mpfs2.o
 .text.MPFSGetMicrotime
                0x00000000       0xb4 build/default/production/_ext/97638081/mpfs2.o
 .text.MPFSGetBytesRem
                0x00000000       0x9c build/default/production/_ext/97638081/mpfs2.o
 .text          0x00000000        0x0 build/default/production/_ext/792872985/usart.o
 .data          0x00000000        0x0 build/default/production/_ext/792872985/usart.o
 .bss           0x00000000        0x0 build/default/production/_ext/792872985/usart.o
 .reginfo       0x00000000       0x18 build/default/production/_ext/792872985/usart.o
 .pdr           0x00000000       0xe0 build/default/production/_ext/792872985/usart.o
 .text          0x00000000        0x0 build/default/production/_ext/792872985/lcd.o
 .data          0x00000000        0x0 build/default/production/_ext/792872985/lcd.o
 .bss           0x00000000        0x0 build/default/production/_ext/792872985/lcd.o
 .reginfo       0x00000000       0x18 build/default/production/_ext/792872985/lcd.o
 .pdr           0x00000000       0xc0 build/default/production/_ext/792872985/lcd.o
 .text          0x00000000        0x0 build/default/production/_ext/792872985/drv_spi.o
 .data          0x00000000        0x0 build/default/production/_ext/792872985/drv_spi.o
 .bss           0x00000000        0x0 build/default/production/_ext/792872985/drv_spi.o
 .reginfo       0x00000000       0x18 build/default/production/_ext/792872985/drv_spi.o
 .pdr           0x00000000       0x60 build/default/production/_ext/792872985/drv_spi.o
 .text          0x00000000        0x0 build/default/production/_ext/792872985/db_appio.o
 .data          0x00000000        0x0 build/default/production/_ext/792872985/db_appio.o
 .bss           0x00000000        0x0 build/default/production/_ext/792872985/db_appio.o
 .reginfo       0x00000000       0x18 build/default/production/_ext/792872985/db_appio.o
 .pdr           0x00000000        0x0 build/default/production/_ext/792872985/db_appio.o
 .text          0x00000000        0x0 build/default/production/_ext/792872985/spi_ram.o
 .data          0x00000000        0x0 build/default/production/_ext/792872985/spi_ram.o
 .bss           0x00000000        0x0 build/default/production/_ext/792872985/spi_ram.o
 .reginfo       0x00000000       0x18 build/default/production/_ext/792872985/spi_ram.o
 .pdr           0x00000000        0x0 build/default/production/_ext/792872985/spi_ram.o
 .text          0x00000000        0x0 build/default/production/_ext/792872985/spi_eeprom.o
 .data          0x00000000        0x0 build/default/production/_ext/792872985/spi_eeprom.o
 .bss           0x00000000        0x0 build/default/production/_ext/792872985/spi_eeprom.o
 .reginfo       0x00000000       0x18 build/default/production/_ext/792872985/spi_eeprom.o
 .pdr           0x00000000      0x160 build/default/production/_ext/792872985/spi_eeprom.o
 .text.XEEBeginRead
                0x00000000       0x34 build/default/production/_ext/792872985/spi_eeprom.o
 .text.XEERead  0x00000000       0x8c build/default/production/_ext/792872985/spi_eeprom.o
 .text.XEEEndRead
                0x00000000       0x24 build/default/production/_ext/792872985/spi_eeprom.o
 .text          0x00000000        0x0 build/default/production/_ext/792872985/spi_flash.o
 .data          0x00000000        0x0 build/default/production/_ext/792872985/spi_flash.o
 .bss           0x00000000        0x0 build/default/production/_ext/792872985/spi_flash.o
 .reginfo       0x00000000       0x18 build/default/production/_ext/792872985/spi_flash.o
 .pdr           0x00000000        0x0 build/default/production/_ext/792872985/spi_flash.o
 .text          0x00000000        0x0 build/default/production/_ext/792872985/drv_media.o
 .data          0x00000000        0x0 build/default/production/_ext/792872985/drv_media.o
 .bss           0x00000000        0x0 build/default/production/_ext/792872985/drv_media.o
 .reginfo       0x00000000       0x18 build/default/production/_ext/792872985/drv_media.o
 .pdr           0x00000000      0x1e0 build/default/production/_ext/792872985/drv_media.o
 .text.DRV_MEDIA_Deinitialize
                0x00000000       0x34 build/default/production/_ext/792872985/drv_media.o
 .text.DRV_MEDIA_ClientSizeGet
                0x00000000       0x40 build/default/production/_ext/792872985/drv_media.o
 .text.DRV_MEDIA_ClientRangeSet
                0x00000000       0xfc build/default/production/_ext/792872985/drv_media.o
 .text.DRV_MEDIA_WriteByte
                0x00000000       0xec build/default/production/_ext/792872985/drv_media.o
 .text          0x00000000        0x0 build/default/production/_ext/427700826/tcpip_announce.o
 .data          0x00000000        0x0 build/default/production/_ext/427700826/tcpip_announce.o
 .bss           0x00000000        0x0 build/default/production/_ext/427700826/tcpip_announce.o
 .reginfo       0x00000000       0x18 build/default/production/_ext/427700826/tcpip_announce.o
 .pdr           0x00000000       0xe0 build/default/production/_ext/427700826/tcpip_announce.o
 .text          0x00000000        0x0 build/default/production/_ext/427700826/http2.o
 .data          0x00000000        0x0 build/default/production/_ext/427700826/http2.o
 .bss           0x00000000        0x0 build/default/production/_ext/427700826/http2.o
 .reginfo       0x00000000       0x18 build/default/production/_ext/427700826/http2.o
 .pdr           0x00000000      0x4a0 build/default/production/_ext/427700826/http2.o
 .text.HTTPCurConnectionCallbackPosGet
                0x00000000       0x34 build/default/production/_ext/427700826/http2.o
 .text.HTTPCurConnectionByteCountSet
                0x00000000       0x3c build/default/production/_ext/427700826/http2.o
 .text.HTTPCurConnectionIsAuthorizedGet
                0x00000000       0x34 build/default/production/_ext/427700826/http2.o
 .text.HTTPCurConnectionIsAuthorizedSet
                0x00000000       0x40 build/default/production/_ext/427700826/http2.o
 .text.HTTPCurConnectionUserDataSet
                0x00000000       0x3c build/default/production/_ext/427700826/http2.o
 .text.HTTPCurConnectionUserDataGet
                0x00000000       0x34 build/default/production/_ext/427700826/http2.o
 .text          0x00000000        0x0 build/default/production/_ext/427700826/arcfour.o
 .data          0x00000000        0x0 build/default/production/_ext/427700826/arcfour.o
 .bss           0x00000000        0x0 build/default/production/_ext/427700826/arcfour.o
 .reginfo       0x00000000       0x18 build/default/production/_ext/427700826/arcfour.o
 .pdr           0x00000000        0x0 build/default/production/_ext/427700826/arcfour.o
 .text          0x00000000        0x0 build/default/production/_ext/427700826/arp.o
 .data          0x00000000        0x0 build/default/production/_ext/427700826/arp.o
 .bss           0x00000000        0x0 build/default/production/_ext/427700826/arp.o
 .reginfo       0x00000000       0x18 build/default/production/_ext/427700826/arp.o
 .pdr           0x00000000      0x480 build/default/production/_ext/427700826/arp.o
 .text.ARPRegisterHandler
                0x00000000       0x9c build/default/production/_ext/427700826/arp.o
 .text.ARPDeRegisterHandler
                0x00000000       0x78 build/default/production/_ext/427700826/arp.o
 .text.ARPProbe
                0x00000000       0x5c build/default/production/_ext/427700826/arp.o
 .text.ARPEntrySet
                0x00000000      0x248 build/default/production/_ext/427700826/arp.o
 .text.ARPEntryGet
                0x00000000       0x7c build/default/production/_ext/427700826/arp.o
 .text.ARPEntryRemove
                0x00000000       0xd0 build/default/production/_ext/427700826/arp.o
 .text.ARPEntryRemoveAll
                0x00000000       0x90 build/default/production/_ext/427700826/arp.o
 .text.ARPEntryQuery
                0x00000000      0x1a8 build/default/production/_ext/427700826/arp.o
 .text.ARPCacheGetEntriesNo
                0x00000000      0x15c build/default/production/_ext/427700826/arp.o
 .text.ARPCacheSetThreshold
                0x00000000       0xc8 build/default/production/_ext/427700826/arp.o
 .text          0x00000000        0x0 build/default/production/_ext/427700826/berkeley_api.o
 .data          0x00000000        0x0 build/default/production/_ext/427700826/berkeley_api.o
 .bss           0x00000000        0x0 build/default/production/_ext/427700826/berkeley_api.o
 .reginfo       0x00000000       0x18 build/default/production/_ext/427700826/berkeley_api.o
 .pdr           0x00000000        0x0 build/default/production/_ext/427700826/berkeley_api.o
 .text          0x00000000        0x0 build/default/production/_ext/427700826/dhcp.o
 .data          0x00000000        0x0 build/default/production/_ext/427700826/dhcp.o
 .bss           0x00000000        0x0 build/default/production/_ext/427700826/dhcp.o
 .reginfo       0x00000000       0x18 build/default/production/_ext/427700826/dhcp.o
 .pdr           0x00000000      0x260 build/default/production/_ext/427700826/dhcp.o
 .text.DHCPIsServerDetected
                0x00000000       0x90 build/default/production/_ext/427700826/dhcp.o
 .text.DHCPSetRequestTimeout
                0x00000000       0x2c build/default/production/_ext/427700826/dhcp.o
 .text          0x00000000        0x0 build/default/production/_ext/427700826/dhcps.o
 .data          0x00000000        0x0 build/default/production/_ext/427700826/dhcps.o
 .bss           0x00000000        0x0 build/default/production/_ext/427700826/dhcps.o
 .reginfo       0x00000000       0x18 build/default/production/_ext/427700826/dhcps.o
 .pdr           0x00000000       0x60 build/default/production/_ext/427700826/dhcps.o
 .text.DHCPServerIsEnabled
                0x00000000       0x28 build/default/production/_ext/427700826/dhcps.o
 .text          0x00000000        0x0 build/default/production/_ext/427700826/dns.o
 .data          0x00000000        0x0 build/default/production/_ext/427700826/dns.o
 .bss           0x00000000        0x0 build/default/production/_ext/427700826/dns.o
 .reginfo       0x00000000       0x18 build/default/production/_ext/427700826/dns.o
 .pdr           0x00000000      0x160 build/default/production/_ext/427700826/dns.o
 .text          0x00000000        0x0 build/default/production/_ext/427700826/dnss.o
 .data          0x00000000        0x0 build/default/production/_ext/427700826/dnss.o
 .bss           0x00000000        0x0 build/default/production/_ext/427700826/dnss.o
 .reginfo       0x00000000       0x18 build/default/production/_ext/427700826/dnss.o
 .pdr           0x00000000        0x0 build/default/production/_ext/427700826/dnss.o
 .text          0x00000000        0x0 build/default/production/_ext/427700826/dyn_dns.o
 .data          0x00000000        0x0 build/default/production/_ext/427700826/dyn_dns.o
 .bss           0x00000000        0x0 build/default/production/_ext/427700826/dyn_dns.o
 .reginfo       0x00000000       0x18 build/default/production/_ext/427700826/dyn_dns.o
 .pdr           0x00000000        0x0 build/default/production/_ext/427700826/dyn_dns.o
 .text          0x00000000        0x0 build/default/production/_ext/427700826/enc28_mac.o
 .data          0x00000000        0x0 build/default/production/_ext/427700826/enc28_mac.o
 .bss           0x00000000        0x0 build/default/production/_ext/427700826/enc28_mac.o
 .reginfo       0x00000000       0x18 build/default/production/_ext/427700826/enc28_mac.o
 .pdr           0x00000000        0x0 build/default/production/_ext/427700826/enc28_mac.o
 .text          0x00000000        0x0 build/default/production/_ext/427700826/enc28j60.o
 .data          0x00000000        0x0 build/default/production/_ext/427700826/enc28j60.o
 .bss           0x00000000        0x0 build/default/production/_ext/427700826/enc28j60.o
 .reginfo       0x00000000       0x18 build/default/production/_ext/427700826/enc28j60.o
 .pdr           0x00000000        0x0 build/default/production/_ext/427700826/enc28j60.o
 .text          0x00000000        0x0 build/default/production/_ext/427700826/encs24j600.o
 .data          0x00000000        0x0 build/default/production/_ext/427700826/encs24j600.o
 .bss           0x00000000        0x0 build/default/production/_ext/427700826/encs24j600.o
 .reginfo       0x00000000       0x18 build/default/production/_ext/427700826/encs24j600.o
 .pdr           0x00000000        0x0 build/default/production/_ext/427700826/encs24j600.o
 .text          0x00000000        0x0 build/default/production/_ext/427700826/encx24_mac.o
 .data          0x00000000        0x0 build/default/production/_ext/427700826/encx24_mac.o
 .bss           0x00000000        0x0 build/default/production/_ext/427700826/encx24_mac.o
 .reginfo       0x00000000       0x18 build/default/production/_ext/427700826/encx24_mac.o
 .pdr           0x00000000        0x0 build/default/production/_ext/427700826/encx24_mac.o
 .text          0x00000000        0x0 build/default/production/_ext/427700826/eth_pic32_ext_phy.o
 .data          0x00000000        0x0 build/default/production/_ext/427700826/eth_pic32_ext_phy.o
 .bss           0x00000000        0x0 build/default/production/_ext/427700826/eth_pic32_ext_phy.o
 .reginfo       0x00000000       0x18 build/default/production/_ext/427700826/eth_pic32_ext_phy.o
 .pdr           0x00000000        0x0 build/default/production/_ext/427700826/eth_pic32_ext_phy.o
 .text          0x00000000        0x0 build/default/production/_ext/427700826/eth_pic32_ext_phy_dp83848.o
 .data          0x00000000        0x0 build/default/production/_ext/427700826/eth_pic32_ext_phy_dp83848.o
 .bss           0x00000000        0x0 build/default/production/_ext/427700826/eth_pic32_ext_phy_dp83848.o
 .reginfo       0x00000000       0x18 build/default/production/_ext/427700826/eth_pic32_ext_phy_dp83848.o
 .pdr           0x00000000        0x0 build/default/production/_ext/427700826/eth_pic32_ext_phy_dp83848.o
 .text          0x00000000        0x0 build/default/production/_ext/427700826/eth_pic32_int_mac.o
 .data          0x00000000        0x0 build/default/production/_ext/427700826/eth_pic32_int_mac.o
 .bss           0x00000000        0x0 build/default/production/_ext/427700826/eth_pic32_int_mac.o
 .reginfo       0x00000000       0x18 build/default/production/_ext/427700826/eth_pic32_int_mac.o
 .pdr           0x00000000        0x0 build/default/production/_ext/427700826/eth_pic32_int_mac.o
 .text          0x00000000        0x0 build/default/production/_ext/427700826/ftp.o
 .data          0x00000000        0x0 build/default/production/_ext/427700826/ftp.o
 .bss           0x00000000        0x0 build/default/production/_ext/427700826/ftp.o
 .reginfo       0x00000000       0x18 build/default/production/_ext/427700826/ftp.o
 .pdr           0x00000000        0x0 build/default/production/_ext/427700826/ftp.o
 .text          0x00000000        0x0 build/default/production/_ext/427700826/hash_fnv.o
 .data          0x00000000        0x0 build/default/production/_ext/427700826/hash_fnv.o
 .bss           0x00000000        0x0 build/default/production/_ext/427700826/hash_fnv.o
 .reginfo       0x00000000       0x18 build/default/production/_ext/427700826/hash_fnv.o
 .pdr           0x00000000       0x40 build/default/production/_ext/427700826/hash_fnv.o
 .text.fnv_32a_hash
                0x00000000       0xd0 build/default/production/_ext/427700826/hash_fnv.o
 .text          0x00000000        0x0 build/default/production/_ext/427700826/hash_tbl.o
 .data          0x00000000        0x0 build/default/production/_ext/427700826/hash_tbl.o
 .bss           0x00000000        0x0 build/default/production/_ext/427700826/hash_tbl.o
 .reginfo       0x00000000       0x18 build/default/production/_ext/427700826/hash_tbl.o
 .pdr           0x00000000      0x100 build/default/production/_ext/427700826/hash_tbl.o
 .text          0x00000000        0x0 build/default/production/_ext/427700826/icmp.o
 .data          0x00000000        0x0 build/default/production/_ext/427700826/icmp.o
 .bss           0x00000000        0x0 build/default/production/_ext/427700826/icmp.o
 .reginfo       0x00000000       0x18 build/default/production/_ext/427700826/icmp.o
 .pdr           0x00000000       0xe0 build/default/production/_ext/427700826/icmp.o
 .text.ICMPRegisterCallback
                0x00000000       0x28 build/default/production/_ext/427700826/icmp.o
 .text.ICMPDeRegisterCallback
                0x00000000       0x28 build/default/production/_ext/427700826/icmp.o
 .text          0x00000000        0x0 build/default/production/_ext/427700826/icmpv6.o
 .data          0x00000000        0x0 build/default/production/_ext/427700826/icmpv6.o
 .bss           0x00000000        0x0 build/default/production/_ext/427700826/icmpv6.o
 .reginfo       0x00000000       0x18 build/default/production/_ext/427700826/icmpv6.o
 .pdr           0x00000000        0x0 build/default/production/_ext/427700826/icmpv6.o
 .text          0x00000000        0x0 build/default/production/_ext/427700826/ipv4.o
 .data          0x00000000        0x0 build/default/production/_ext/427700826/ipv4.o
 .bss           0x00000000        0x0 build/default/production/_ext/427700826/ipv4.o
 .reginfo       0x00000000       0x18 build/default/production/_ext/427700826/ipv4.o
 .pdr           0x00000000      0x4e0 build/default/production/_ext/427700826/ipv4.o
 .text.TCPIP_IPV4_Put
                0x00000000       0x5c build/default/production/_ext/427700826/ipv4.o
 .text          0x00000000        0x0 build/default/production/_ext/427700826/ipv6.o
 .data          0x00000000        0x0 build/default/production/_ext/427700826/ipv6.o
 .bss           0x00000000        0x0 build/default/production/_ext/427700826/ipv6.o
 .reginfo       0x00000000       0x18 build/default/production/_ext/427700826/ipv6.o
 .pdr           0x00000000        0x0 build/default/production/_ext/427700826/ipv6.o
 .text          0x00000000        0x0 build/default/production/_ext/427700826/mac_events_pic32.o
 .data          0x00000000        0x0 build/default/production/_ext/427700826/mac_events_pic32.o
 .bss           0x00000000        0x0 build/default/production/_ext/427700826/mac_events_pic32.o
 .reginfo       0x00000000       0x18 build/default/production/_ext/427700826/mac_events_pic32.o
 .pdr           0x00000000        0x0 build/default/production/_ext/427700826/mac_events_pic32.o
 .text          0x00000000        0x0 build/default/production/_ext/427700826/nbns.o
 .data          0x00000000        0x0 build/default/production/_ext/427700826/nbns.o
 .bss           0x00000000        0x0 build/default/production/_ext/427700826/nbns.o
 .reginfo       0x00000000       0x18 build/default/production/_ext/427700826/nbns.o
 .pdr           0x00000000       0xa0 build/default/production/_ext/427700826/nbns.o
 .text          0x00000000        0x0 build/default/production/_ext/427700826/ndp.o
 .data          0x00000000        0x0 build/default/production/_ext/427700826/ndp.o
 .bss           0x00000000        0x0 build/default/production/_ext/427700826/ndp.o
 .reginfo       0x00000000       0x18 build/default/production/_ext/427700826/ndp.o
 .pdr           0x00000000        0x0 build/default/production/_ext/427700826/ndp.o
 .text          0x00000000        0x0 build/default/production/_ext/427700826/tcpip_reboot.o
 .data          0x00000000        0x0 build/default/production/_ext/427700826/tcpip_reboot.o
 .bss           0x00000000        0x0 build/default/production/_ext/427700826/tcpip_reboot.o
 .reginfo       0x00000000       0x18 build/default/production/_ext/427700826/tcpip_reboot.o
 .pdr           0x00000000        0x0 build/default/production/_ext/427700826/tcpip_reboot.o
 .text          0x00000000        0x0 build/default/production/_ext/427700826/rsa.o
 .data          0x00000000        0x0 build/default/production/_ext/427700826/rsa.o
 .bss           0x00000000        0x0 build/default/production/_ext/427700826/rsa.o
 .reginfo       0x00000000       0x18 build/default/production/_ext/427700826/rsa.o
 .pdr           0x00000000        0x0 build/default/production/_ext/427700826/rsa.o
 .text          0x00000000        0x0 build/default/production/_ext/427700826/smtp.o
 .data          0x00000000        0x0 build/default/production/_ext/427700826/smtp.o
 .bss           0x00000000        0x0 build/default/production/_ext/427700826/smtp.o
 .reginfo       0x00000000       0x18 build/default/production/_ext/427700826/smtp.o
 .pdr           0x00000000        0x0 build/default/production/_ext/427700826/smtp.o
 .text          0x00000000        0x0 build/default/production/_ext/427700826/snmp.o
 .data          0x00000000        0x0 build/default/production/_ext/427700826/snmp.o
 .bss           0x00000000        0x0 build/default/production/_ext/427700826/snmp.o
 .reginfo       0x00000000       0x18 build/default/production/_ext/427700826/snmp.o
 .pdr           0x00000000        0x0 build/default/production/_ext/427700826/snmp.o
 .text          0x00000000        0x0 build/default/production/_ext/427700826/snmpv3.o
 .data          0x00000000        0x0 build/default/production/_ext/427700826/snmpv3.o
 .bss           0x00000000        0x0 build/default/production/_ext/427700826/snmpv3.o
 .reginfo       0x00000000       0x18 build/default/production/_ext/427700826/snmpv3.o
 .pdr           0x00000000        0x0 build/default/production/_ext/427700826/snmpv3.o
 .text          0x00000000        0x0 build/default/production/_ext/427700826/snmpv3_usm.o
 .data          0x00000000        0x0 build/default/production/_ext/427700826/snmpv3_usm.o
 .bss           0x00000000        0x0 build/default/production/_ext/427700826/snmpv3_usm.o
 .reginfo       0x00000000       0x18 build/default/production/_ext/427700826/snmpv3_usm.o
 .pdr           0x00000000        0x0 build/default/production/_ext/427700826/snmpv3_usm.o
 .text          0x00000000        0x0 build/default/production/_ext/427700826/sntp.o
 .data          0x00000000        0x0 build/default/production/_ext/427700826/sntp.o
 .bss           0x00000000        0x0 build/default/production/_ext/427700826/sntp.o
 .reginfo       0x00000000       0x18 build/default/production/_ext/427700826/sntp.o
 .pdr           0x00000000        0x0 build/default/production/_ext/427700826/sntp.o
 .text          0x00000000        0x0 build/default/production/_ext/427700826/ssl.o
 .data          0x00000000        0x0 build/default/production/_ext/427700826/ssl.o
 .bss           0x00000000        0x0 build/default/production/_ext/427700826/ssl.o
 .reginfo       0x00000000       0x18 build/default/production/_ext/427700826/ssl.o
 .pdr           0x00000000        0x0 build/default/production/_ext/427700826/ssl.o
 .text          0x00000000        0x0 build/default/production/_ext/427700826/tcp.o
 .data          0x00000000        0x0 build/default/production/_ext/427700826/tcp.o
 .bss           0x00000000        0x0 build/default/production/_ext/427700826/tcp.o
 .reginfo       0x00000000       0x18 build/default/production/_ext/427700826/tcp.o
 .pdr           0x00000000      0x9c0 build/default/production/_ext/427700826/tcp.o
 .text.TCPSetConnectionMSS
                0x00000000       0x44 build/default/production/_ext/427700826/tcp.o
 .text.TCPAbort
                0x00000000       0x6c build/default/production/_ext/427700826/tcp.o
 .text.TCPGetSocketInfo
                0x00000000       0xfc build/default/production/_ext/427700826/tcp.o
 .text.TCPSocketsNo
                0x00000000       0x24 build/default/production/_ext/427700826/tcp.o
 .text.TCPGetTxFIFOFull
                0x00000000       0xa4 build/default/production/_ext/427700826/tcp.o
 .text.TCPPeekArray
                0x00000000      0x1ac build/default/production/_ext/427700826/tcp.o
 .text.TCPPeek  0x00000000       0x60 build/default/production/_ext/427700826/tcp.o
 .text.TCPSocketSetNet
                0x00000000       0x80 build/default/production/_ext/427700826/tcp.o
 .text.TCPBind  0x00000000      0x1c4 build/default/production/_ext/427700826/tcp.o
 .text.TCPRemoteBind
                0x00000000       0x9c build/default/production/_ext/427700826/tcp.o
 .text.TCPGetOptions
                0x00000000      0x1b8 build/default/production/_ext/427700826/tcp.o
 .text.TCPSetDestinationIPAddress
                0x00000000       0xc4 build/default/production/_ext/427700826/tcp.o
 .text.TCPSetSourceIPAddress
                0x00000000       0xc4 build/default/production/_ext/427700826/tcp.o
 .text          0x00000000        0x0 build/default/production/_ext/427700826/tcpip_heap_alloc.o
 .data          0x00000000        0x0 build/default/production/_ext/427700826/tcpip_heap_alloc.o
 .bss           0x00000000        0x0 build/default/production/_ext/427700826/tcpip_heap_alloc.o
 .reginfo       0x00000000       0x18 build/default/production/_ext/427700826/tcpip_heap_alloc.o
 .pdr           0x00000000      0x200 build/default/production/_ext/427700826/tcpip_heap_alloc.o
 .text.TCPIP_HEAP_Size
                0x00000000       0x60 build/default/production/_ext/427700826/tcpip_heap_alloc.o
 .text.TCPIP_HEAP_MaxSize
                0x00000000       0xb0 build/default/production/_ext/427700826/tcpip_heap_alloc.o
 .text.TCPIP_HEAP_LastError
                0x00000000       0x6c build/default/production/_ext/427700826/tcpip_heap_alloc.o
 .text.TCPIP_HEAP_SetNoMemHandler
                0x00000000       0x5c build/default/production/_ext/427700826/tcpip_heap_alloc.o
 .text.TCPIP_HEAP_TraceGetEntry
                0x00000000       0x30 build/default/production/_ext/427700826/tcpip_heap_alloc.o
 .text.TCPIP_HEAP_TraceGetEntriesNo
                0x00000000       0x30 build/default/production/_ext/427700826/tcpip_heap_alloc.o
 .text          0x00000000        0x0 build/default/production/_ext/427700826/tcpip_storage.o
 .data          0x00000000        0x0 build/default/production/_ext/427700826/tcpip_storage.o
 .bss           0x00000000        0x0 build/default/production/_ext/427700826/tcpip_storage.o
 .reginfo       0x00000000       0x18 build/default/production/_ext/427700826/tcpip_storage.o
 .pdr           0x00000000        0x0 build/default/production/_ext/427700826/tcpip_storage.o
 .text          0x00000000        0x0 build/default/production/_ext/427700826/telnet.o
 .data          0x00000000        0x0 build/default/production/_ext/427700826/telnet.o
 .bss           0x00000000        0x0 build/default/production/_ext/427700826/telnet.o
 .reginfo       0x00000000       0x18 build/default/production/_ext/427700826/telnet.o
 .pdr           0x00000000        0x0 build/default/production/_ext/427700826/telnet.o
 .text          0x00000000        0x0 build/default/production/_ext/427700826/tftpc.o
 .data          0x00000000        0x0 build/default/production/_ext/427700826/tftpc.o
 .bss           0x00000000        0x0 build/default/production/_ext/427700826/tftpc.o
 .reginfo       0x00000000       0x18 build/default/production/_ext/427700826/tftpc.o
 .pdr           0x00000000        0x0 build/default/production/_ext/427700826/tftpc.o
 .text          0x00000000        0x0 build/default/production/_ext/427700826/udp.o
 .data          0x00000000        0x0 build/default/production/_ext/427700826/udp.o
 .bss           0x00000000        0x0 build/default/production/_ext/427700826/udp.o
 .reginfo       0x00000000       0x18 build/default/production/_ext/427700826/udp.o
 .pdr           0x00000000      0x560 build/default/production/_ext/427700826/udp.o
 .text.UDPGetSocketInfo
                0x00000000      0x100 build/default/production/_ext/427700826/udp.o
 .text.UDPPutString
                0x00000000       0xa0 build/default/production/_ext/427700826/udp.o
 .text.UDPSocketGetNet
                0x00000000       0x68 build/default/production/_ext/427700826/udp.o
 .text.UDPGetOptions
                0x00000000       0xdc build/default/production/_ext/427700826/udp.o
 .text          0x00000000        0x0 build/default/production/_ext/427700826/tcpip_mac_object.o
 .data          0x00000000        0x0 build/default/production/_ext/427700826/tcpip_mac_object.o
 .bss           0x00000000        0x0 build/default/production/_ext/427700826/tcpip_mac_object.o
 .reginfo       0x00000000       0x18 build/default/production/_ext/427700826/tcpip_mac_object.o
 .pdr           0x00000000      0x300 build/default/production/_ext/427700826/tcpip_mac_object.o
 .text.MACGetReadPtrInRx
                0x00000000       0x44 build/default/production/_ext/427700826/tcpip_mac_object.o
 .text.MACSetBaseReadPtr
                0x00000000       0x4c build/default/production/_ext/427700826/tcpip_mac_object.o
 .text.MACSetRXHashTableEntry
                0x00000000       0x54 build/default/production/_ext/427700826/tcpip_mac_object.o
 .text.MACPowerMode
                0x00000000       0x4c build/default/production/_ext/427700826/tcpip_mac_object.o
 .text.MACEventClearNotifyEvents
                0x00000000       0x54 build/default/production/_ext/427700826/tcpip_mac_object.o
 .text          0x00000000        0x0 build/default/production/_ext/427700826/tcpip_manager.o
 .data          0x00000000        0x0 build/default/production/_ext/427700826/tcpip_manager.o
 .bss           0x00000000        0x0 build/default/production/_ext/427700826/tcpip_manager.o
 .reginfo       0x00000000       0x18 build/default/production/_ext/427700826/tcpip_manager.o
 .pdr           0x00000000      0xa00 build/default/production/_ext/427700826/tcpip_manager.o
 .text.TCPIP_STACK_NetUp
                0x00000000      0x1c0 build/default/production/_ext/427700826/tcpip_manager.o
 .text.TCPIP_STACK_NetDown
                0x00000000      0x134 build/default/production/_ext/427700826/tcpip_manager.o
 .text.TCPIP_STACK_SetDefaultNet
                0x00000000       0x70 build/default/production/_ext/427700826/tcpip_manager.o
 .text._TCPIPStackIpAddFromNet
                0x00000000       0xec build/default/production/_ext/427700826/tcpip_manager.o
 .text._TCPIPStackMacToNet
                0x00000000       0x88 build/default/production/_ext/427700826/tcpip_manager.o
 .text._TCPIPStackMacToNetIx
                0x00000000       0x88 build/default/production/_ext/427700826/tcpip_manager.o
 .text.TCPIP_STACK_NetIx
                0x00000000       0x48 build/default/production/_ext/427700826/tcpip_manager.o
 .text.TCPIP_STACK_SetNetAddress
                0x00000000       0x80 build/default/production/_ext/427700826/tcpip_manager.o
 .text.TCPIP_STACK_SetNetGatewayAddress
                0x00000000       0x5c build/default/production/_ext/427700826/tcpip_manager.o
 .text.TCPIP_STACK_SetNetPriDNSAddress
                0x00000000       0x5c build/default/production/_ext/427700826/tcpip_manager.o
 .text.TCPIP_STACK_SetNetSecondDNSAddress
                0x00000000       0x5c build/default/production/_ext/427700826/tcpip_manager.o
 .text.TCPIP_STACK_SetNetMacAddress
                0x00000000       0x7c build/default/production/_ext/427700826/tcpip_manager.o
 .text.TCPIP_STACK_SetNetBIOSName
                0x00000000       0x8c build/default/production/_ext/427700826/tcpip_manager.o
 .text.TCPIP_STACK_SetLocalMasksType
                0x00000000       0x98 build/default/production/_ext/427700826/tcpip_manager.o
 .text.TCPIP_STACK_SetLocalMasks
                0x00000000       0x70 build/default/production/_ext/427700826/tcpip_manager.o
 .text.TCPIP_STACK_NetMACId
                0x00000000       0x44 build/default/production/_ext/427700826/tcpip_manager.o
 .text.TCPIP_STACK_ModuleGetConfig
                0x00000000       0xc0 build/default/production/_ext/427700826/tcpip_manager.o
 .text.TCPIP_STACK_NetConfigGet
                0x00000000      0x10c build/default/production/_ext/427700826/tcpip_manager.o
 .text.NetConfigStringToBuffer
                0x00000000       0xf0 build/default/production/_ext/427700826/tcpip_manager.o
 .text.TCPIP_STACK_NetConfigSet
                0x00000000      0x4d8 build/default/production/_ext/427700826/tcpip_manager.o
 .text.TCPIP_STACK_IsNetUp
                0x00000000       0x48 build/default/production/_ext/427700826/tcpip_manager.o
 .text.TCPIP_STACK_IsNetLinked
                0x00000000       0x48 build/default/production/_ext/427700826/tcpip_manager.o
 .text.TCPIP_STACK_GetPendingEvents
                0x00000000       0x6c build/default/production/_ext/427700826/tcpip_manager.o
 .text.TCPIP_STACK_DeRegisterHandler
                0x00000000       0x7c build/default/production/_ext/427700826/tcpip_manager.o
 .text._TCPIPStackNetMacId
                0x00000000       0x44 build/default/production/_ext/427700826/tcpip_manager.o
 .text          0x00000000        0x0 build/default/production/_ext/427700826/tcpip_helpers.o
 .data          0x00000000        0x0 build/default/production/_ext/427700826/tcpip_helpers.o
 .bss           0x00000000        0x0 build/default/production/_ext/427700826/tcpip_helpers.o
 .reginfo       0x00000000       0x18 build/default/production/_ext/427700826/tcpip_helpers.o
 .pdr           0x00000000      0x340 build/default/production/_ext/427700826/tcpip_helpers.o
 .text.TCPIP_HELPER_IPAddressToString
                0x00000000       0xec build/default/production/_ext/427700826/tcpip_helpers.o
 .text.TCPIP_HELPER_MACAddressToString
                0x00000000       0xf4 build/default/production/_ext/427700826/tcpip_helpers.o
 .text.TCPIP_HELPER_PowerModeToString
                0x00000000       0x58 build/default/production/_ext/427700826/tcpip_helpers.o
 .text.TCPIP_Helper_FindCommonPrefix
                0x00000000      0x110 build/default/production/_ext/427700826/tcpip_helpers.o
 .text.SingleListAddHead
                0x00000000       0x74 build/default/production/_ext/427700826/tcpip_helpers.o
 .text.SingleListAddMid
                0x00000000       0x5c build/default/production/_ext/427700826/tcpip_helpers.o
 .text.SingleListRemoveNext
                0x00000000       0xb0 build/default/production/_ext/427700826/tcpip_helpers.o
 .text.SingleListAppendList
                0x00000000       0x64 build/default/production/_ext/427700826/tcpip_helpers.o
 .text.DoubleListInit
                0x00000000       0x44 build/default/production/_ext/427700826/tcpip_helpers.o
 .text.DoubleListAddHead
                0x00000000       0xbc build/default/production/_ext/427700826/tcpip_helpers.o
 .text.DoubleListAddTail
                0x00000000       0xbc build/default/production/_ext/427700826/tcpip_helpers.o
 .text.DoubleListAddMid
                0x00000000       0x78 build/default/production/_ext/427700826/tcpip_helpers.o
 .text.DoubleListRemoveHead
                0x00000000       0xa8 build/default/production/_ext/427700826/tcpip_helpers.o
 .text.DoubleListRemoveTail
                0x00000000       0xa8 build/default/production/_ext/427700826/tcpip_helpers.o
 .text.DoubleListRemoveMid
                0x00000000       0x64 build/default/production/_ext/427700826/tcpip_helpers.o
 .text.DoubleListRemoveNode
                0x00000000       0x90 build/default/production/_ext/427700826/tcpip_helpers.o
 .text          0x00000000        0x0 build/default/production/_ext/427700826/tcpip_commands.o
 .data          0x00000000        0x0 build/default/production/_ext/427700826/tcpip_commands.o
 .bss           0x00000000        0x0 build/default/production/_ext/427700826/tcpip_commands.o
 .reginfo       0x00000000       0x18 build/default/production/_ext/427700826/tcpip_commands.o
 .pdr           0x00000000        0x0 build/default/production/_ext/427700826/tcpip_commands.o
 .text          0x00000000        0x0 build/default/production/_ext/427700826/iperf.o
 .data          0x00000000        0x0 build/default/production/_ext/427700826/iperf.o
 .bss           0x00000000        0x0 build/default/production/_ext/427700826/iperf.o
 .reginfo       0x00000000       0x18 build/default/production/_ext/427700826/iperf.o
 .pdr           0x00000000        0x0 build/default/production/_ext/427700826/iperf.o
 .data          0x00000000        0x0 build/default/production/_ext/427700826/tcpip_helper_c32.o
 .bss           0x00000000        0x0 build/default/production/_ext/427700826/tcpip_helper_c32.o
 .reginfo       0x00000000       0x18 build/default/production/_ext/427700826/tcpip_helper_c32.o
 .pdr           0x00000000       0x60 build/default/production/_ext/427700826/tcpip_helper_c32.o
 .text          0x00000000        0x0 build/default/production/_ext/427700826/tcpip_notify.o
 .data          0x00000000        0x0 build/default/production/_ext/427700826/tcpip_notify.o
 .bss           0x00000000        0x0 build/default/production/_ext/427700826/tcpip_notify.o
 .reginfo       0x00000000       0x18 build/default/production/_ext/427700826/tcpip_notify.o
 .pdr           0x00000000       0x60 build/default/production/_ext/427700826/tcpip_notify.o
 .text          0x00000000        0x0 build/default/production/_ext/427700826/zero_conf_helper.o
 .data          0x00000000        0x0 build/default/production/_ext/427700826/zero_conf_helper.o
 .bss           0x00000000        0x0 build/default/production/_ext/427700826/zero_conf_helper.o
 .reginfo       0x00000000       0x18 build/default/production/_ext/427700826/zero_conf_helper.o
 .pdr           0x00000000        0x0 build/default/production/_ext/427700826/zero_conf_helper.o
 .text          0x00000000        0x0 build/default/production/_ext/427700826/zero_conf_link_local.o
 .data          0x00000000        0x0 build/default/production/_ext/427700826/zero_conf_link_local.o
 .bss           0x00000000        0x0 build/default/production/_ext/427700826/zero_conf_link_local.o
 .reginfo       0x00000000       0x18 build/default/production/_ext/427700826/zero_conf_link_local.o
 .pdr           0x00000000       0x60 build/default/production/_ext/427700826/zero_conf_link_local.o
 .text.ZCLLDisable
                0x00000000       0x28 build/default/production/_ext/427700826/zero_conf_link_local.o
 .text.ZCLLIsEnabled
                0x00000000       0x28 build/default/production/_ext/427700826/zero_conf_link_local.o
 .text          0x00000000        0x0 build/default/production/_ext/427700826/zero_conf_multicast_dns.o
 .data          0x00000000        0x0 build/default/production/_ext/427700826/zero_conf_multicast_dns.o
 .bss           0x00000000        0x0 build/default/production/_ext/427700826/zero_conf_multicast_dns.o
 .reginfo       0x00000000       0x18 build/default/production/_ext/427700826/zero_conf_multicast_dns.o
 .pdr           0x00000000        0x0 build/default/production/_ext/427700826/zero_conf_multicast_dns.o
 .text          0x00000000        0x0 build/default/production/_ext/334706090/wf_tx_power.o
 .data          0x00000000        0x0 build/default/production/_ext/334706090/wf_tx_power.o
 .bss           0x00000000        0x0 build/default/production/_ext/334706090/wf_tx_power.o
 .reginfo       0x00000000       0x18 build/default/production/_ext/334706090/wf_tx_power.o
 .pdr           0x00000000       0x60 build/default/production/_ext/334706090/wf_tx_power.o
 .rodata        0x00000000       0x30 build/default/production/_ext/334706090/wf_tx_power.o
 .text.WF_TxPowerSetMax
                0x00000000       0xb0 build/default/production/_ext/334706090/wf_tx_power.o
 .text.WF_TxPowerGetMax
                0x00000000       0x74 build/default/production/_ext/334706090/wf_tx_power.o
 .text.WF_TxPowerGetFactoryMax
                0x00000000       0x54 build/default/production/_ext/334706090/wf_tx_power.o
 .text          0x00000000        0x0 build/default/production/_ext/334706090/wf_connect.o
 .data          0x00000000        0x0 build/default/production/_ext/334706090/wf_connect.o
 .bss           0x00000000        0x0 build/default/production/_ext/334706090/wf_connect.o
 .reginfo       0x00000000       0x18 build/default/production/_ext/334706090/wf_connect.o
 .pdr           0x00000000       0xa0 build/default/production/_ext/334706090/wf_connect.o
 .text          0x00000000        0x0 build/default/production/_ext/334706090/wf_connection_algorithm.o
 .data          0x00000000        0x0 build/default/production/_ext/334706090/wf_connection_algorithm.o
 .bss           0x00000000        0x0 build/default/production/_ext/334706090/wf_connection_algorithm.o
 .reginfo       0x00000000       0x18 build/default/production/_ext/334706090/wf_connection_algorithm.o
 .pdr           0x00000000      0x240 build/default/production/_ext/334706090/wf_connection_algorithm.o
 .text.WF_RssiSet
                0x00000000       0x44 build/default/production/_ext/334706090/wf_connection_algorithm.o
 .text.WF_RssiGet
                0x00000000       0x44 build/default/production/_ext/334706090/wf_connection_algorithm.o
 .text.WF_CAGetEventNotificationAction
                0x00000000       0x40 build/default/production/_ext/334706090/wf_connection_algorithm.o
 .text.WF_AdhocContextSet
                0x00000000       0x84 build/default/production/_ext/334706090/wf_connection_algorithm.o
 .text.WF_AdhocContextGet
                0x00000000       0x98 build/default/production/_ext/334706090/wf_connection_algorithm.o
 .text          0x00000000        0x0 build/default/production/_ext/334706090/wf_connection_manager.o
 .data          0x00000000        0x0 build/default/production/_ext/334706090/wf_connection_manager.o
 .bss           0x00000000        0x0 build/default/production/_ext/334706090/wf_connection_manager.o
 .reginfo       0x00000000       0x18 build/default/production/_ext/334706090/wf_connection_manager.o
 .pdr           0x00000000       0xe0 build/default/production/_ext/334706090/wf_connection_manager.o
 .text.isDisconnectAllowed
                0x00000000       0x68 build/default/production/_ext/334706090/wf_connection_manager.o
 .text.WF_Disconnect
                0x00000000       0x8c build/default/production/_ext/334706090/wf_connection_manager.o
 .text.WF_ConnectionStateGet
                0x00000000       0xc8 build/default/production/_ext/334706090/wf_connection_manager.o
 .text          0x00000000        0x0 build/default/production/_ext/334706090/wf_connection_profile.o
 .data          0x00000000        0x0 build/default/production/_ext/334706090/wf_connection_profile.o
 .bss           0x00000000        0x0 build/default/production/_ext/334706090/wf_connection_profile.o
 .reginfo       0x00000000       0x18 build/default/production/_ext/334706090/wf_connection_profile.o
 .pdr           0x00000000      0x300 build/default/production/_ext/334706090/wf_connection_profile.o
 .text.WF_SsidGet
                0x00000000       0x98 build/default/production/_ext/334706090/wf_connection_profile.o
 .text.WF_BssidSet
                0x00000000       0x40 build/default/production/_ext/334706090/wf_connection_profile.o
 .text.WF_BssidGet
                0x00000000       0x44 build/default/production/_ext/334706090/wf_connection_profile.o
 .text.WF_CPSetWepKeyType
                0x00000000       0x50 build/default/production/_ext/334706090/wf_connection_profile.o
 .text.WF_WPSCredentialsGet
                0x00000000       0x48 build/default/production/_ext/334706090/wf_connection_profile.o
 .text.SetHiddenSsid
                0x00000000       0x48 build/default/production/_ext/334706090/wf_connection_profile.o
 .text.GetHiddenSsid
                0x00000000       0x48 build/default/production/_ext/334706090/wf_connection_profile.o
 .text.SetAdHocMode
                0x00000000       0x44 build/default/production/_ext/334706090/wf_connection_profile.o
 .text.GetAdHocMode
                0x00000000       0x48 build/default/production/_ext/334706090/wf_connection_profile.o
 .text          0x00000000        0x0 build/default/production/_ext/334706090/wf_easy_config.o
 .data          0x00000000        0x0 build/default/production/_ext/334706090/wf_easy_config.o
 .bss           0x00000000        0x0 build/default/production/_ext/334706090/wf_easy_config.o
 .reginfo       0x00000000       0x18 build/default/production/_ext/334706090/wf_easy_config.o
 .pdr           0x00000000       0x20 build/default/production/_ext/334706090/wf_easy_config.o
 .rodata        0x00000000       0x7c build/default/production/_ext/334706090/wf_easy_config.o
 .text.WFDisplayScanMgr
                0x00000000      0x308 build/default/production/_ext/334706090/wf_easy_config.o
 COMMON         0x00000000       0x98 build/default/production/_ext/334706090/wf_easy_config.o
 .text          0x00000000        0x0 build/default/production/_ext/334706090/wf_eint.o
 .data          0x00000000        0x0 build/default/production/_ext/334706090/wf_eint.o
 .bss           0x00000000        0x0 build/default/production/_ext/334706090/wf_eint.o
 .reginfo       0x00000000       0x18 build/default/production/_ext/334706090/wf_eint.o
 .pdr           0x00000000       0xa0 build/default/production/_ext/334706090/wf_eint.o
 .text          0x00000000        0x0 build/default/production/_ext/334706090/wf_event_handler.o
 .data          0x00000000        0x0 build/default/production/_ext/334706090/wf_event_handler.o
 .bss           0x00000000        0x0 build/default/production/_ext/334706090/wf_event_handler.o
 .reginfo       0x00000000       0x18 build/default/production/_ext/334706090/wf_event_handler.o
 .pdr           0x00000000      0x140 build/default/production/_ext/334706090/wf_event_handler.o
 .text.WF_GetSoftApEventInfo
                0x00000000       0x24 build/default/production/_ext/334706090/wf_event_handler.o
 .text          0x00000000        0x0 build/default/production/_ext/334706090/wf_init.o
 .data          0x00000000        0x0 build/default/production/_ext/334706090/wf_init.o
 .bss           0x00000000        0x0 build/default/production/_ext/334706090/wf_init.o
 .reginfo       0x00000000       0x18 build/default/production/_ext/334706090/wf_init.o
 .pdr           0x00000000       0xa0 build/default/production/_ext/334706090/wf_init.o
 .text          0x00000000        0x0 build/default/production/_ext/334706090/wf_power_save.o
 .data          0x00000000        0x0 build/default/production/_ext/334706090/wf_power_save.o
 .bss           0x00000000        0x0 build/default/production/_ext/334706090/wf_power_save.o
 .reginfo       0x00000000       0x18 build/default/production/_ext/334706090/wf_power_save.o
 .pdr           0x00000000      0x1e0 build/default/production/_ext/334706090/wf_power_save.o
 .text.WFisPsPollEnabled
                0x00000000       0x50 build/default/production/_ext/334706090/wf_power_save.o
 .text.WFIsPsPollActive
                0x00000000       0x24 build/default/production/_ext/334706090/wf_power_save.o
 .text.WF_HibernateEnable
                0x00000000       0x44 build/default/production/_ext/334706090/wf_power_save.o
 .text          0x00000000        0x0 build/default/production/_ext/334706090/wf_scan.o
 .data          0x00000000        0x0 build/default/production/_ext/334706090/wf_scan.o
 .bss           0x00000000        0x0 build/default/production/_ext/334706090/wf_scan.o
 .reginfo       0x00000000       0x18 build/default/production/_ext/334706090/wf_scan.o
 .pdr           0x00000000       0x60 build/default/production/_ext/334706090/wf_scan.o
 .text.isHostScanAllowed
                0x00000000       0x68 build/default/production/_ext/334706090/wf_scan.o
 .text.WF_Scan  0x00000000       0xb8 build/default/production/_ext/334706090/wf_scan.o
 .text.WF_ScanGetResult
                0x00000000       0xcc build/default/production/_ext/334706090/wf_scan.o
 .text          0x00000000        0x0 build/default/production/_ext/334706090/wf_spi.o
 .data          0x00000000        0x0 build/default/production/_ext/334706090/wf_spi.o
 .bss           0x00000000        0x0 build/default/production/_ext/334706090/wf_spi.o
 .reginfo       0x00000000       0x18 build/default/production/_ext/334706090/wf_spi.o
 .pdr           0x00000000       0xa0 build/default/production/_ext/334706090/wf_spi.o
 .text          0x00000000        0x0 build/default/production/_ext/334706090/mrf24w_mac_pic32.o
 .data          0x00000000        0x0 build/default/production/_ext/334706090/mrf24w_mac_pic32.o
 .bss           0x00000000        0x0 build/default/production/_ext/334706090/mrf24w_mac_pic32.o
 .reginfo       0x00000000       0x18 build/default/production/_ext/334706090/mrf24w_mac_pic32.o
 .pdr           0x00000000      0x3c0 build/default/production/_ext/334706090/mrf24w_mac_pic32.o
 .text          0x00000000        0x0 build/default/production/_ext/334706090/mrf24w_events.o
 .data          0x00000000        0x0 build/default/production/_ext/334706090/mrf24w_events.o
 .bss           0x00000000        0x0 build/default/production/_ext/334706090/mrf24w_events.o
 .reginfo       0x00000000       0x18 build/default/production/_ext/334706090/mrf24w_events.o
 .pdr           0x00000000      0x160 build/default/production/_ext/334706090/mrf24w_events.o
 .text          0x00000000        0x0 build/default/production/_ext/334706090/wf_debug_output.o
 .bss           0x00000000        0x0 build/default/production/_ext/334706090/wf_debug_output.o
 .reginfo       0x00000000       0x18 build/default/production/_ext/334706090/wf_debug_output.o
 .pdr           0x00000000      0x280 build/default/production/_ext/334706090/wf_debug_output.o
 .text          0x00000000        0x0 build/default/production/_ext/334706090/wf_commands.o
 .data          0x00000000        0x0 build/default/production/_ext/334706090/wf_commands.o
 .bss           0x00000000        0x0 build/default/production/_ext/334706090/wf_commands.o
 .reginfo       0x00000000       0x18 build/default/production/_ext/334706090/wf_commands.o
 .pdr           0x00000000      0x1e0 build/default/production/_ext/334706090/wf_commands.o
 .sbss          0x00000000        0x3 build/default/production/_ext/334706090/wf_commands.o
 .rodata        0x00000000      0x5d4 build/default/production/_ext/334706090/wf_commands.o
 .text.WIFICommandsInit
                0x00000000       0x6c build/default/production/_ext/334706090/wf_commands.o
 .text.CommandIwConfig
                0x00000000      0x4bc build/default/production/_ext/334706090/wf_commands.o
 .text.iwconfigUpdateCb
                0x00000000       0xf0 build/default/production/_ext/334706090/wf_commands.o
 .text.iwconfigDisplayStatus
                0x00000000      0x7f0 build/default/production/_ext/334706090/wf_commands.o
 .text.iwconfigSetSsid
                0x00000000      0x104 build/default/production/_ext/334706090/wf_commands.o
 .text.iwconfigSetMode
                0x00000000      0x2e0 build/default/production/_ext/334706090/wf_commands.o
 .text.iwconfigSetChannel
                0x00000000      0x2a8 build/default/production/_ext/334706090/wf_commands.o
 .text.iwconfigSetPower
                0x00000000      0x204 build/default/production/_ext/334706090/wf_commands.o
 .text.iwconfigSetRTS
                0x00000000       0xc4 build/default/production/_ext/334706090/wf_commands.o
 .text.CommandIw_eraseConfig
                0x00000000       0x68 build/default/production/_ext/334706090/wf_commands.o
 .text.CommandIw_saveConfig
                0x00000000       0x7c build/default/production/_ext/334706090/wf_commands.o
 .text.CommandIw_readConfig
                0x00000000       0x68 build/default/production/_ext/334706090/wf_commands.o
 .text.HexToBin
                0x00000000       0x9c build/default/production/_ext/334706090/wf_commands.o
 .text.ConvertASCIIHexToBinary
                0x00000000      0x144 build/default/production/_ext/334706090/wf_commands.o
 .text.convertAsciiToHexInPlace
                0x00000000      0x134 build/default/production/_ext/334706090/wf_commands.o
 .text          0x00000000        0x0 build/default/production/_ext/334706090/wf_pbkdf2.o
 .data          0x00000000        0x0 build/default/production/_ext/334706090/wf_pbkdf2.o
 .bss           0x00000000        0x0 build/default/production/_ext/334706090/wf_pbkdf2.o
 .reginfo       0x00000000       0x18 build/default/production/_ext/334706090/wf_pbkdf2.o
 .pdr           0x00000000        0x0 build/default/production/_ext/334706090/wf_pbkdf2.o
 .text          0x00000000        0x0 build/default/production/_ext/334706090/wf_driver_com_24g.o
 .data          0x00000000        0x0 build/default/production/_ext/334706090/wf_driver_com_24g.o
 .bss           0x00000000        0x0 build/default/production/_ext/334706090/wf_driver_com_24g.o
 .reginfo       0x00000000       0x18 build/default/production/_ext/334706090/wf_driver_com_24g.o
 .pdr           0x00000000      0x300 build/default/production/_ext/334706090/wf_driver_com_24g.o
 .text.ReenablePowerSaveMode
                0x00000000       0x28 build/default/production/_ext/334706090/wf_driver_com_24g.o
 .text          0x00000000        0x0 build/default/production/_ext/334706090/wf_driver_raw_24g.o
 .data          0x00000000        0x0 build/default/production/_ext/334706090/wf_driver_raw_24g.o
 .bss           0x00000000        0x0 build/default/production/_ext/334706090/wf_driver_raw_24g.o
 .reginfo       0x00000000       0x18 build/default/production/_ext/334706090/wf_driver_raw_24g.o
 .pdr           0x00000000      0x2a0 build/default/production/_ext/334706090/wf_driver_raw_24g.o
 .text.RawToRawCopy
                0x00000000       0x98 build/default/production/_ext/334706090/wf_driver_raw_24g.o
 .text.PushRawWindow
                0x00000000       0x4c build/default/production/_ext/334706090/wf_driver_raw_24g.o
 .text.PopRawWindow
                0x00000000       0x54 build/default/production/_ext/334706090/wf_driver_raw_24g.o
 .text.RawGetIndex
                0x00000000       0x60 build/default/production/_ext/334706090/wf_driver_raw_24g.o
 .text          0x00000000        0x0 build/default/production/_ext/334706090/wf_mac_24g.o
 .data          0x00000000        0x0 build/default/production/_ext/334706090/wf_mac_24g.o
 .bss           0x00000000        0x0 build/default/production/_ext/334706090/wf_mac_24g.o
 .reginfo       0x00000000       0x18 build/default/production/_ext/334706090/wf_mac_24g.o
 .pdr           0x00000000      0x3e0 build/default/production/_ext/334706090/wf_mac_24g.o
 .text.WF_StopGratuitousArp
                0x00000000       0x40 build/default/production/_ext/334706090/wf_mac_24g.o
 .text          0x00000000        0x0 build/default/production/_ext/334706090/wf_mgmt_msg_24g.o
 .data          0x00000000        0x0 build/default/production/_ext/334706090/wf_mgmt_msg_24g.o
 .bss           0x00000000        0x0 build/default/production/_ext/334706090/wf_mgmt_msg_24g.o
 .reginfo       0x00000000       0x18 build/default/production/_ext/334706090/wf_mgmt_msg_24g.o
 .pdr           0x00000000       0xa0 build/default/production/_ext/334706090/wf_mgmt_msg_24g.o
 .text.WFSetFuncState
                0x00000000       0x80 build/default/production/_ext/334706090/wf_mgmt_msg_24g.o
 .text          0x00000000        0x0 build/default/production/_ext/334706090/wf_param_msg_24g.o
 .data          0x00000000        0x0 build/default/production/_ext/334706090/wf_param_msg_24g.o
 .bss           0x00000000        0x0 build/default/production/_ext/334706090/wf_param_msg_24g.o
 .reginfo       0x00000000       0x18 build/default/production/_ext/334706090/wf_param_msg_24g.o
 .pdr           0x00000000      0x340 build/default/production/_ext/334706090/wf_param_msg_24g.o
 .text.WFEnableBroadcastProbeResponse
                0x00000000       0x48 build/default/production/_ext/334706090/wf_param_msg_24g.o
 .text.WF_SetLinkDownThreshold
                0x00000000       0x44 build/default/production/_ext/334706090/wf_param_msg_24g.o
 .text.WF_SetStackVersion
                0x00000000       0x7c build/default/production/_ext/334706090/wf_param_msg_24g.o
 .text.WF_GetWPATimeout
                0x00000000       0x44 build/default/production/_ext/334706090/wf_param_msg_24g.o
 .text.WF_GetMultiCastFilter
                0x00000000      0x120 build/default/production/_ext/334706090/wf_param_msg_24g.o
 .text.WF_MulticastSetConfig
                0x00000000      0x194 build/default/production/_ext/334706090/wf_param_msg_24g.o
 .text.WF_MulticastGetConfig
                0x00000000       0xf8 build/default/production/_ext/334706090/wf_param_msg_24g.o
 .text.WF_GetTxDataConfirm
                0x00000000       0x40 build/default/production/_ext/334706090/wf_param_msg_24g.o
 .text.WF_RtsThresholdSet
                0x00000000       0x88 build/default/production/_ext/334706090/wf_param_msg_24g.o
 .text.WF_RtsThresholdGet
                0x00000000       0x64 build/default/production/_ext/334706090/wf_param_msg_24g.o
 .text.WF_EnableSWMultiCastFilter
                0x00000000       0x48 build/default/production/_ext/334706090/wf_param_msg_24g.o
 .text.WF_GetMacStats
                0x00000000       0xac build/default/production/_ext/334706090/wf_param_msg_24g.o
 .text.WF_YieldPassphrase2Host
                0x00000000       0x48 build/default/production/_ext/334706090/wf_param_msg_24g.o
 .text.WF_SetPSK
                0x00000000       0x40 build/default/production/_ext/334706090/wf_param_msg_24g.o
 .text          0x00000000        0x0 build/default/production/_ext/334706090/wf_configData.o
 .data          0x00000000        0x0 build/default/production/_ext/334706090/wf_configData.o
 .bss           0x00000000        0x0 build/default/production/_ext/334706090/wf_configData.o
 .reginfo       0x00000000       0x18 build/default/production/_ext/334706090/wf_configData.o
 .pdr           0x00000000       0x80 build/default/production/_ext/334706090/wf_configData.o
 .rodata        0x00000000      0x190 build/default/production/_ext/334706090/wf_configData.o
 .text.WF_ConfigDataPrint
                0x00000000      0x4b8 build/default/production/_ext/334706090/wf_configData.o
 .text.WF_ConfigDataErase
                0x00000000       0x58 build/default/production/_ext/334706090/wf_configData.o
 .text          0x00000000        0x0 build/default/production/_ext/1472/main_demo.o
 .data          0x00000000        0x0 build/default/production/_ext/1472/main_demo.o
 .bss           0x00000000        0x0 build/default/production/_ext/1472/main_demo.o
 .reginfo       0x00000000       0x18 build/default/production/_ext/1472/main_demo.o
 .pdr           0x00000000       0x80 build/default/production/_ext/1472/main_demo.o
 .text          0x00000000        0x0 build/default/production/_ext/1472/custom_snmp_app.o
 .data          0x00000000        0x0 build/default/production/_ext/1472/custom_snmp_app.o
 .bss           0x00000000        0x0 build/default/production/_ext/1472/custom_snmp_app.o
 .reginfo       0x00000000       0x18 build/default/production/_ext/1472/custom_snmp_app.o
 .pdr           0x00000000        0x0 build/default/production/_ext/1472/custom_snmp_app.o
 .text          0x00000000        0x0 build/default/production/_ext/1472/custom_ssl_cert.o
 .data          0x00000000        0x0 build/default/production/_ext/1472/custom_ssl_cert.o
 .bss           0x00000000        0x0 build/default/production/_ext/1472/custom_ssl_cert.o
 .reginfo       0x00000000       0x18 build/default/production/_ext/1472/custom_ssl_cert.o
 .pdr           0x00000000        0x0 build/default/production/_ext/1472/custom_ssl_cert.o
 .text          0x00000000        0x0 build/default/production/_ext/1472/mpfs_img2.o
 .data          0x00000000        0x0 build/default/production/_ext/1472/mpfs_img2.o
 .bss           0x00000000        0x0 build/default/production/_ext/1472/mpfs_img2.o
 .reginfo       0x00000000       0x18 build/default/production/_ext/1472/mpfs_img2.o
 .pdr           0x00000000        0x0 build/default/production/_ext/1472/mpfs_img2.o
 .text          0x00000000        0x0 build/default/production/_ext/1472/wf_config.o
 .data          0x00000000        0x0 build/default/production/_ext/1472/wf_config.o
 .bss           0x00000000        0x0 build/default/production/_ext/1472/wf_config.o
 .reginfo       0x00000000       0x18 build/default/production/_ext/1472/wf_config.o
 .pdr           0x00000000       0x20 build/default/production/_ext/1472/wf_config.o
 .text          0x00000000        0x0 build/default/production/_ext/1472/custom_http_app.o
 .data          0x00000000        0x0 build/default/production/_ext/1472/custom_http_app.o
 .reginfo       0x00000000       0x18 build/default/production/_ext/1472/custom_http_app.o
 .pdr           0x00000000      0x500 build/default/production/_ext/1472/custom_http_app.o
 .text          0x00000000        0x0 build/default/production/_ext/1472/tcp6_demo_app.o
 .bss           0x00000000        0x0 build/default/production/_ext/1472/tcp6_demo_app.o
 .reginfo       0x00000000       0x18 build/default/production/_ext/1472/tcp6_demo_app.o
 .pdr           0x00000000       0x80 build/default/production/_ext/1472/tcp6_demo_app.o
 .text          0x00000000        0x0 c:/program files (x86)/microchip/xc32/v1.10/bin/../lib/gcc/pic32mx/4.5.1/../../../../pic32mx/lib/./proc/32MX795F512L\processor.o
 .data          0x00000000        0x0 c:/program files (x86)/microchip/xc32/v1.10/bin/../lib/gcc/pic32mx/4.5.1/../../../../pic32mx/lib/./proc/32MX795F512L\processor.o
 .bss           0x00000000        0x0 c:/program files (x86)/microchip/xc32/v1.10/bin/../lib/gcc/pic32mx/4.5.1/../../../../pic32mx/lib/./proc/32MX795F512L\processor.o
 .reginfo       0x00000000       0x18 c:/program files (x86)/microchip/xc32/v1.10/bin/../lib/gcc/pic32mx/4.5.1/../../../../pic32mx/lib/./proc/32MX795F512L\processor.o
 .pdr           0x00000000        0x0 c:/program files (x86)/microchip/xc32/v1.10/bin/../lib/gcc/pic32mx/4.5.1/../../../../pic32mx/lib/./proc/32MX795F512L\processor.o
 .text          0x00000000        0x0 c:/program files (x86)/microchip/xc32/v1.10/bin/../lib/gcc/pic32mx/4.5.1/../../../../pic32mx/lib/size\libmchp_peripheral.a(open_core_timer_lib.o)
 .data          0x00000000        0x0 c:/program files (x86)/microchip/xc32/v1.10/bin/../lib/gcc/pic32mx/4.5.1/../../../../pic32mx/lib/size\libmchp_peripheral.a(open_core_timer_lib.o)
 .bss           0x00000000        0x0 c:/program files (x86)/microchip/xc32/v1.10/bin/../lib/gcc/pic32mx/4.5.1/../../../../pic32mx/lib/size\libmchp_peripheral.a(open_core_timer_lib.o)
 .reginfo       0x00000000       0x18 c:/program files (x86)/microchip/xc32/v1.10/bin/../lib/gcc/pic32mx/4.5.1/../../../../pic32mx/lib/size\libmchp_peripheral.a(open_core_timer_lib.o)
 .pdr           0x00000000       0x20 c:/program files (x86)/microchip/xc32/v1.10/bin/../lib/gcc/pic32mx/4.5.1/../../../../pic32mx/lib/size\libmchp_peripheral.a(open_core_timer_lib.o)
 .text          0x00000000        0x0 c:/program files (x86)/microchip/xc32/v1.10/bin/../lib/gcc/pic32mx/4.5.1/../../../../pic32mx/lib/size\libmchp_peripheral_32MX795F512L.a(soft_reset_lib.o)
 .data          0x00000000        0x0 c:/program files (x86)/microchip/xc32/v1.10/bin/../lib/gcc/pic32mx/4.5.1/../../../../pic32mx/lib/size\libmchp_peripheral_32MX795F512L.a(soft_reset_lib.o)
 .bss           0x00000000        0x0 c:/program files (x86)/microchip/xc32/v1.10/bin/../lib/gcc/pic32mx/4.5.1/../../../../pic32mx/lib/size\libmchp_peripheral_32MX795F512L.a(soft_reset_lib.o)
 .reginfo       0x00000000       0x18 c:/program files (x86)/microchip/xc32/v1.10/bin/../lib/gcc/pic32mx/4.5.1/../../../../pic32mx/lib/size\libmchp_peripheral_32MX795F512L.a(soft_reset_lib.o)
 .pdr           0x00000000       0x20 c:/program files (x86)/microchip/xc32/v1.10/bin/../lib/gcc/pic32mx/4.5.1/../../../../pic32mx/lib/size\libmchp_peripheral_32MX795F512L.a(soft_reset_lib.o)
 .text          0x00000000        0x0 c:/program files (x86)/microchip/xc32/v1.10/bin/../lib/gcc/pic32mx/4.5.1/../../../../pic32mx/lib/size\libmchp_peripheral_32MX795F512L.a(pcache.o)
 .data          0x00000000        0x0 c:/program files (x86)/microchip/xc32/v1.10/bin/../lib/gcc/pic32mx/4.5.1/../../../../pic32mx/lib/size\libmchp_peripheral_32MX795F512L.a(pcache.o)
 .bss           0x00000000        0x0 c:/program files (x86)/microchip/xc32/v1.10/bin/../lib/gcc/pic32mx/4.5.1/../../../../pic32mx/lib/size\libmchp_peripheral_32MX795F512L.a(pcache.o)
 .reginfo       0x00000000       0x18 c:/program files (x86)/microchip/xc32/v1.10/bin/../lib/gcc/pic32mx/4.5.1/../../../../pic32mx/lib/size\libmchp_peripheral_32MX795F512L.a(pcache.o)
 .pdr           0x00000000       0x40 c:/program files (x86)/microchip/xc32/v1.10/bin/../lib/gcc/pic32mx/4.5.1/../../../../pic32mx/lib/size\libmchp_peripheral_32MX795F512L.a(pcache.o)
 .text.CheKseg0CacheOff
                0x00000000       0x18 c:/program files (x86)/microchip/xc32/v1.10/bin/../lib/gcc/pic32mx/4.5.1/../../../../pic32mx/lib/size\libmchp_peripheral_32MX795F512L.a(pcache.o)
 .text          0x00000000        0x0 c:/program files (x86)/microchip/xc32/v1.10/bin/../lib/gcc/pic32mx/4.5.1/../../../../pic32mx/lib/size\libmchp_peripheral_32MX795F512L.a(int_disable_interrupts_lib.o)
 .data          0x00000000        0x0 c:/program files (x86)/microchip/xc32/v1.10/bin/../lib/gcc/pic32mx/4.5.1/../../../../pic32mx/lib/size\libmchp_peripheral_32MX795F512L.a(int_disable_interrupts_lib.o)
 .bss           0x00000000        0x0 c:/program files (x86)/microchip/xc32/v1.10/bin/../lib/gcc/pic32mx/4.5.1/../../../../pic32mx/lib/size\libmchp_peripheral_32MX795F512L.a(int_disable_interrupts_lib.o)
 .reginfo       0x00000000       0x18 c:/program files (x86)/microchip/xc32/v1.10/bin/../lib/gcc/pic32mx/4.5.1/../../../../pic32mx/lib/size\libmchp_peripheral_32MX795F512L.a(int_disable_interrupts_lib.o)
 .pdr           0x00000000       0x20 c:/program files (x86)/microchip/xc32/v1.10/bin/../lib/gcc/pic32mx/4.5.1/../../../../pic32mx/lib/size\libmchp_peripheral_32MX795F512L.a(int_disable_interrupts_lib.o)
 .text          0x00000000        0x0 c:/program files (x86)/microchip/xc32/v1.10/bin/../lib/gcc/pic32mx/4.5.1/../../../../pic32mx/lib/size\libmchp_peripheral_32MX795F512L.a(int_restore_interrupts_lib.o)
 .data          0x00000000        0x0 c:/program files (x86)/microchip/xc32/v1.10/bin/../lib/gcc/pic32mx/4.5.1/../../../../pic32mx/lib/size\libmchp_peripheral_32MX795F512L.a(int_restore_interrupts_lib.o)
 .bss           0x00000000        0x0 c:/program files (x86)/microchip/xc32/v1.10/bin/../lib/gcc/pic32mx/4.5.1/../../../../pic32mx/lib/size\libmchp_peripheral_32MX795F512L.a(int_restore_interrupts_lib.o)
 .reginfo       0x00000000       0x18 c:/program files (x86)/microchip/xc32/v1.10/bin/../lib/gcc/pic32mx/4.5.1/../../../../pic32mx/lib/size\libmchp_peripheral_32MX795F512L.a(int_restore_interrupts_lib.o)
 .pdr           0x00000000       0x20 c:/program files (x86)/microchip/xc32/v1.10/bin/../lib/gcc/pic32mx/4.5.1/../../../../pic32mx/lib/size\libmchp_peripheral_32MX795F512L.a(int_restore_interrupts_lib.o)
 .text          0x00000000        0x0 c:/program files (x86)/microchip/xc32/v1.10/bin/../lib/gcc/pic32mx/4.5.1/../../../../pic32mx/lib/size\libmchp_peripheral_32MX795F512L.a(int_enable_mv_int_lib.o)
 .data          0x00000000        0x0 c:/program files (x86)/microchip/xc32/v1.10/bin/../lib/gcc/pic32mx/4.5.1/../../../../pic32mx/lib/size\libmchp_peripheral_32MX795F512L.a(int_enable_mv_int_lib.o)
 .bss           0x00000000        0x0 c:/program files (x86)/microchip/xc32/v1.10/bin/../lib/gcc/pic32mx/4.5.1/../../../../pic32mx/lib/size\libmchp_peripheral_32MX795F512L.a(int_enable_mv_int_lib.o)
 .reginfo       0x00000000       0x18 c:/program files (x86)/microchip/xc32/v1.10/bin/../lib/gcc/pic32mx/4.5.1/../../../../pic32mx/lib/size\libmchp_peripheral_32MX795F512L.a(int_enable_mv_int_lib.o)
 .pdr           0x00000000       0x20 c:/program files (x86)/microchip/xc32/v1.10/bin/../lib/gcc/pic32mx/4.5.1/../../../../pic32mx/lib/size\libmchp_peripheral_32MX795F512L.a(int_enable_mv_int_lib.o)
 .text          0x00000000        0x0 c:/program files (x86)/microchip/xc32/v1.10/bin/../lib/gcc/pic32mx/4.5.1/../../../../pic32mx/lib/size\libmchp_peripheral_32MX795F512L.a(int_tbl_lib.o)
 .data          0x00000000        0x0 c:/program files (x86)/microchip/xc32/v1.10/bin/../lib/gcc/pic32mx/4.5.1/../../../../pic32mx/lib/size\libmchp_peripheral_32MX795F512L.a(int_tbl_lib.o)
 .bss           0x00000000        0x0 c:/program files (x86)/microchip/xc32/v1.10/bin/../lib/gcc/pic32mx/4.5.1/../../../../pic32mx/lib/size\libmchp_peripheral_32MX795F512L.a(int_tbl_lib.o)
 .reginfo       0x00000000       0x18 c:/program files (x86)/microchip/xc32/v1.10/bin/../lib/gcc/pic32mx/4.5.1/../../../../pic32mx/lib/size\libmchp_peripheral_32MX795F512L.a(int_tbl_lib.o)
 .pdr           0x00000000      0x120 c:/program files (x86)/microchip/xc32/v1.10/bin/../lib/gcc/pic32mx/4.5.1/../../../../pic32mx/lib/size\libmchp_peripheral_32MX795F512L.a(int_tbl_lib.o)
 .text.INTSetFlag
                0x00000000       0x28 c:/program files (x86)/microchip/xc32/v1.10/bin/../lib/gcc/pic32mx/4.5.1/../../../../pic32mx/lib/size\libmchp_peripheral_32MX795F512L.a(int_tbl_lib.o)
 .text.INTGetFlag
                0x00000000       0x28 c:/program files (x86)/microchip/xc32/v1.10/bin/../lib/gcc/pic32mx/4.5.1/../../../../pic32mx/lib/size\libmchp_peripheral_32MX795F512L.a(int_tbl_lib.o)
 .text.INTGetEnable
                0x00000000       0x28 c:/program files (x86)/microchip/xc32/v1.10/bin/../lib/gcc/pic32mx/4.5.1/../../../../pic32mx/lib/size\libmchp_peripheral_32MX795F512L.a(int_tbl_lib.o)
 .text.INTGetVectorPriority
                0x00000000       0x2c c:/program files (x86)/microchip/xc32/v1.10/bin/../lib/gcc/pic32mx/4.5.1/../../../../pic32mx/lib/size\libmchp_peripheral_32MX795F512L.a(int_tbl_lib.o)
 .text.INTGetVectorSubPriority
                0x00000000       0x2c c:/program files (x86)/microchip/xc32/v1.10/bin/../lib/gcc/pic32mx/4.5.1/../../../../pic32mx/lib/size\libmchp_peripheral_32MX795F512L.a(int_tbl_lib.o)
 .text          0x00000000        0x0 c:/program files (x86)/microchip/xc32/v1.10/bin/../lib/gcc/pic32mx/4.5.1/../../../../pic32mx/lib/size\libmchp_peripheral_32MX795F512L.a(rtcc_init_lib.o)
 .data          0x00000000        0x0 c:/program files (x86)/microchip/xc32/v1.10/bin/../lib/gcc/pic32mx/4.5.1/../../../../pic32mx/lib/size\libmchp_peripheral_32MX795F512L.a(rtcc_init_lib.o)
 .bss           0x00000000        0x0 c:/program files (x86)/microchip/xc32/v1.10/bin/../lib/gcc/pic32mx/4.5.1/../../../../pic32mx/lib/size\libmchp_peripheral_32MX795F512L.a(rtcc_init_lib.o)
 .reginfo       0x00000000       0x18 c:/program files (x86)/microchip/xc32/v1.10/bin/../lib/gcc/pic32mx/4.5.1/../../../../pic32mx/lib/size\libmchp_peripheral_32MX795F512L.a(rtcc_init_lib.o)
 .pdr           0x00000000       0x20 c:/program files (x86)/microchip/xc32/v1.10/bin/../lib/gcc/pic32mx/4.5.1/../../../../pic32mx/lib/size\libmchp_peripheral_32MX795F512L.a(rtcc_init_lib.o)
 .text.RtccInit
                0x00000000      0x170 c:/program files (x86)/microchip/xc32/v1.10/bin/../lib/gcc/pic32mx/4.5.1/../../../../pic32mx/lib/size\libmchp_peripheral_32MX795F512L.a(rtcc_init_lib.o)
 .text          0x00000000        0x0 c:/program files (x86)/microchip/xc32/v1.10/bin/../lib/gcc/pic32mx/4.5.1/../../../../pic32mx/lib/size\libmchp_peripheral_32MX795F512L.a(rtcc_open_lib.o)
 .data          0x00000000        0x0 c:/program files (x86)/microchip/xc32/v1.10/bin/../lib/gcc/pic32mx/4.5.1/../../../../pic32mx/lib/size\libmchp_peripheral_32MX795F512L.a(rtcc_open_lib.o)
 .bss           0x00000000        0x0 c:/program files (x86)/microchip/xc32/v1.10/bin/../lib/gcc/pic32mx/4.5.1/../../../../pic32mx/lib/size\libmchp_peripheral_32MX795F512L.a(rtcc_open_lib.o)
 .reginfo       0x00000000       0x18 c:/program files (x86)/microchip/xc32/v1.10/bin/../lib/gcc/pic32mx/4.5.1/../../../../pic32mx/lib/size\libmchp_peripheral_32MX795F512L.a(rtcc_open_lib.o)
 .pdr           0x00000000       0x20 c:/program files (x86)/microchip/xc32/v1.10/bin/../lib/gcc/pic32mx/4.5.1/../../../../pic32mx/lib/size\libmchp_peripheral_32MX795F512L.a(rtcc_open_lib.o)
 .text.RtccOpen
                0x00000000      0x1b0 c:/program files (x86)/microchip/xc32/v1.10/bin/../lib/gcc/pic32mx/4.5.1/../../../../pic32mx/lib/size\libmchp_peripheral_32MX795F512L.a(rtcc_open_lib.o)
 .text          0x00000000        0x0 c:/program files (x86)/microchip/xc32/v1.10/bin/../lib/gcc/pic32mx/4.5.1/../../../../pic32mx/lib/size\libmchp_peripheral_32MX795F512L.a(spi_chn_data_rdy_lib.o)
 .data          0x00000000        0x0 c:/program files (x86)/microchip/xc32/v1.10/bin/../lib/gcc/pic32mx/4.5.1/../../../../pic32mx/lib/size\libmchp_peripheral_32MX795F512L.a(spi_chn_data_rdy_lib.o)
 .bss           0x00000000        0x0 c:/program files (x86)/microchip/xc32/v1.10/bin/../lib/gcc/pic32mx/4.5.1/../../../../pic32mx/lib/size\libmchp_peripheral_32MX795F512L.a(spi_chn_data_rdy_lib.o)
 .reginfo       0x00000000       0x18 c:/program files (x86)/microchip/xc32/v1.10/bin/../lib/gcc/pic32mx/4.5.1/../../../../pic32mx/lib/size\libmchp_peripheral_32MX795F512L.a(spi_chn_data_rdy_lib.o)
 .pdr           0x00000000       0x20 c:/program files (x86)/microchip/xc32/v1.10/bin/../lib/gcc/pic32mx/4.5.1/../../../../pic32mx/lib/size\libmchp_peripheral_32MX795F512L.a(spi_chn_data_rdy_lib.o)
 .text          0x00000000        0x0 c:/program files (x86)/microchip/xc32/v1.10/bin/../lib/gcc/pic32mx/4.5.1/../../../../pic32mx/lib/size\libmchp_peripheral_32MX795F512L.a(spi_chn_getc_lib.o)
 .data          0x00000000        0x0 c:/program files (x86)/microchip/xc32/v1.10/bin/../lib/gcc/pic32mx/4.5.1/../../../../pic32mx/lib/size\libmchp_peripheral_32MX795F512L.a(spi_chn_getc_lib.o)
 .bss           0x00000000        0x0 c:/program files (x86)/microchip/xc32/v1.10/bin/../lib/gcc/pic32mx/4.5.1/../../../../pic32mx/lib/size\libmchp_peripheral_32MX795F512L.a(spi_chn_getc_lib.o)
 .reginfo       0x00000000       0x18 c:/program files (x86)/microchip/xc32/v1.10/bin/../lib/gcc/pic32mx/4.5.1/../../../../pic32mx/lib/size\libmchp_peripheral_32MX795F512L.a(spi_chn_getc_lib.o)
 .pdr           0x00000000       0x40 c:/program files (x86)/microchip/xc32/v1.10/bin/../lib/gcc/pic32mx/4.5.1/../../../../pic32mx/lib/size\libmchp_peripheral_32MX795F512L.a(spi_chn_getc_lib.o)
 .text.SpiChnGetC
                0x00000000       0x54 c:/program files (x86)/microchip/xc32/v1.10/bin/../lib/gcc/pic32mx/4.5.1/../../../../pic32mx/lib/size\libmchp_peripheral_32MX795F512L.a(spi_chn_getc_lib.o)
 .text          0x00000000        0x0 c:/program files (x86)/microchip/xc32/v1.10/bin/../lib/gcc/pic32mx/4.5.1/../../../../pic32mx/lib/size\libmchp_peripheral_32MX795F512L.a(spi_chn_open_lib.o)
 .data          0x00000000        0x0 c:/program files (x86)/microchip/xc32/v1.10/bin/../lib/gcc/pic32mx/4.5.1/../../../../pic32mx/lib/size\libmchp_peripheral_32MX795F512L.a(spi_chn_open_lib.o)
 .bss           0x00000000        0x0 c:/program files (x86)/microchip/xc32/v1.10/bin/../lib/gcc/pic32mx/4.5.1/../../../../pic32mx/lib/size\libmchp_peripheral_32MX795F512L.a(spi_chn_open_lib.o)
 .reginfo       0x00000000       0x18 c:/program files (x86)/microchip/xc32/v1.10/bin/../lib/gcc/pic32mx/4.5.1/../../../../pic32mx/lib/size\libmchp_peripheral_32MX795F512L.a(spi_chn_open_lib.o)
 .pdr           0x00000000       0x20 c:/program files (x86)/microchip/xc32/v1.10/bin/../lib/gcc/pic32mx/4.5.1/../../../../pic32mx/lib/size\libmchp_peripheral_32MX795F512L.a(spi_chn_open_lib.o)
 .text          0x00000000        0x0 c:/program files (x86)/microchip/xc32/v1.10/bin/../lib/gcc/pic32mx/4.5.1/../../../../pic32mx/lib/size\libmchp_peripheral_32MX795F512L.a(spi_chn_putc_lib.o)
 .data          0x00000000        0x0 c:/program files (x86)/microchip/xc32/v1.10/bin/../lib/gcc/pic32mx/4.5.1/../../../../pic32mx/lib/size\libmchp_peripheral_32MX795F512L.a(spi_chn_putc_lib.o)
 .bss           0x00000000        0x0 c:/program files (x86)/microchip/xc32/v1.10/bin/../lib/gcc/pic32mx/4.5.1/../../../../pic32mx/lib/size\libmchp_peripheral_32MX795F512L.a(spi_chn_putc_lib.o)
 .reginfo       0x00000000       0x18 c:/program files (x86)/microchip/xc32/v1.10/bin/../lib/gcc/pic32mx/4.5.1/../../../../pic32mx/lib/size\libmchp_peripheral_32MX795F512L.a(spi_chn_putc_lib.o)
 .pdr           0x00000000       0x60 c:/program files (x86)/microchip/xc32/v1.10/bin/../lib/gcc/pic32mx/4.5.1/../../../../pic32mx/lib/size\libmchp_peripheral_32MX795F512L.a(spi_chn_putc_lib.o)
 .text.SpiChnPutC
                0x00000000       0x54 c:/program files (x86)/microchip/xc32/v1.10/bin/../lib/gcc/pic32mx/4.5.1/../../../../pic32mx/lib/size\libmchp_peripheral_32MX795F512L.a(spi_chn_putc_lib.o)
 .text.SpiChnBuffer
                0x00000000       0x1c c:/program files (x86)/microchip/xc32/v1.10/bin/../lib/gcc/pic32mx/4.5.1/../../../../pic32mx/lib/size\libmchp_peripheral_32MX795F512L.a(spi_chn_putc_lib.o)
 .text          0x00000000        0x0 c:/program files (x86)/microchip/xc32/v1.10/bin/../lib/gcc/pic32mx/4.5.1/../../../../pic32mx/lib/size\libmchp_peripheral_32MX795F512L.a(spi_chn_tx_buff_empty_lib.o)
 .data          0x00000000        0x0 c:/program files (x86)/microchip/xc32/v1.10/bin/../lib/gcc/pic32mx/4.5.1/../../../../pic32mx/lib/size\libmchp_peripheral_32MX795F512L.a(spi_chn_tx_buff_empty_lib.o)
 .bss           0x00000000        0x0 c:/program files (x86)/microchip/xc32/v1.10/bin/../lib/gcc/pic32mx/4.5.1/../../../../pic32mx/lib/size\libmchp_peripheral_32MX795F512L.a(spi_chn_tx_buff_empty_lib.o)
 .reginfo       0x00000000       0x18 c:/program files (x86)/microchip/xc32/v1.10/bin/../lib/gcc/pic32mx/4.5.1/../../../../pic32mx/lib/size\libmchp_peripheral_32MX795F512L.a(spi_chn_tx_buff_empty_lib.o)
 .pdr           0x00000000       0x20 c:/program files (x86)/microchip/xc32/v1.10/bin/../lib/gcc/pic32mx/4.5.1/../../../../pic32mx/lib/size\libmchp_peripheral_32MX795F512L.a(spi_chn_tx_buff_empty_lib.o)
 .text          0x00000000        0x0 c:/program files (x86)/microchip/xc32/v1.10/bin/../lib/gcc/pic32mx/4.5.1/../../../../pic32mx/lib/size\libmchp_peripheral_32MX795F512L.a(spi_io_tbl_libp.o)
 .data          0x00000000        0x0 c:/program files (x86)/microchip/xc32/v1.10/bin/../lib/gcc/pic32mx/4.5.1/../../../../pic32mx/lib/size\libmchp_peripheral_32MX795F512L.a(spi_io_tbl_libp.o)
 .bss           0x00000000        0x0 c:/program files (x86)/microchip/xc32/v1.10/bin/../lib/gcc/pic32mx/4.5.1/../../../../pic32mx/lib/size\libmchp_peripheral_32MX795F512L.a(spi_io_tbl_libp.o)
 .reginfo       0x00000000       0x18 c:/program files (x86)/microchip/xc32/v1.10/bin/../lib/gcc/pic32mx/4.5.1/../../../../pic32mx/lib/size\libmchp_peripheral_32MX795F512L.a(spi_io_tbl_libp.o)
 .pdr           0x00000000        0x0 c:/program files (x86)/microchip/xc32/v1.10/bin/../lib/gcc/pic32mx/4.5.1/../../../../pic32mx/lib/size\libmchp_peripheral_32MX795F512L.a(spi_io_tbl_libp.o)
 .text          0x00000000        0x0 c:/program files (x86)/microchip/xc32/v1.10/bin/../lib/gcc/pic32mx/4.5.1/../../../../pic32mx/lib/size\libmchp_peripheral_32MX795F512L.a(spi_map_tbl_libp.o)
 .data          0x00000000        0x0 c:/program files (x86)/microchip/xc32/v1.10/bin/../lib/gcc/pic32mx/4.5.1/../../../../pic32mx/lib/size\libmchp_peripheral_32MX795F512L.a(spi_map_tbl_libp.o)
 .bss           0x00000000        0x0 c:/program files (x86)/microchip/xc32/v1.10/bin/../lib/gcc/pic32mx/4.5.1/../../../../pic32mx/lib/size\libmchp_peripheral_32MX795F512L.a(spi_map_tbl_libp.o)
 .reginfo       0x00000000       0x18 c:/program files (x86)/microchip/xc32/v1.10/bin/../lib/gcc/pic32mx/4.5.1/../../../../pic32mx/lib/size\libmchp_peripheral_32MX795F512L.a(spi_map_tbl_libp.o)
 .pdr           0x00000000        0x0 c:/program files (x86)/microchip/xc32/v1.10/bin/../lib/gcc/pic32mx/4.5.1/../../../../pic32mx/lib/size\libmchp_peripheral_32MX795F512L.a(spi_map_tbl_libp.o)
 .text          0x00000000        0x0 c:/program files (x86)/microchip/xc32/v1.10/bin/../lib/gcc/pic32mx/4.5.1/../../../../pic32mx/lib/size\libmchp_peripheral_32MX795F512L.a(port_set_pins_digital_in_lib.o)
 .data          0x00000000        0x0 c:/program files (x86)/microchip/xc32/v1.10/bin/../lib/gcc/pic32mx/4.5.1/../../../../pic32mx/lib/size\libmchp_peripheral_32MX795F512L.a(port_set_pins_digital_in_lib.o)
 .bss           0x00000000        0x0 c:/program files (x86)/microchip/xc32/v1.10/bin/../lib/gcc/pic32mx/4.5.1/../../../../pic32mx/lib/size\libmchp_peripheral_32MX795F512L.a(port_set_pins_digital_in_lib.o)
 .reginfo       0x00000000       0x18 c:/program files (x86)/microchip/xc32/v1.10/bin/../lib/gcc/pic32mx/4.5.1/../../../../pic32mx/lib/size\libmchp_peripheral_32MX795F512L.a(port_set_pins_digital_in_lib.o)
 .pdr           0x00000000       0x20 c:/program files (x86)/microchip/xc32/v1.10/bin/../lib/gcc/pic32mx/4.5.1/../../../../pic32mx/lib/size\libmchp_peripheral_32MX795F512L.a(port_set_pins_digital_in_lib.o)
 .text          0x00000000        0x0 c:/program files (x86)/microchip/xc32/v1.10/bin/../lib/gcc/pic32mx/4.5.1/../../../../pic32mx/lib/size\libmchp_peripheral_32MX795F512L.a(port_set_pins_digital_out_lib.o)
 .data          0x00000000        0x0 c:/program files (x86)/microchip/xc32/v1.10/bin/../lib/gcc/pic32mx/4.5.1/../../../../pic32mx/lib/size\libmchp_peripheral_32MX795F512L.a(port_set_pins_digital_out_lib.o)
 .bss           0x00000000        0x0 c:/program files (x86)/microchip/xc32/v1.10/bin/../lib/gcc/pic32mx/4.5.1/../../../../pic32mx/lib/size\libmchp_peripheral_32MX795F512L.a(port_set_pins_digital_out_lib.o)
 .reginfo       0x00000000       0x18 c:/program files (x86)/microchip/xc32/v1.10/bin/../lib/gcc/pic32mx/4.5.1/../../../../pic32mx/lib/size\libmchp_peripheral_32MX795F512L.a(port_set_pins_digital_out_lib.o)
 .pdr           0x00000000       0x20 c:/program files (x86)/microchip/xc32/v1.10/bin/../lib/gcc/pic32mx/4.5.1/../../../../pic32mx/lib/size\libmchp_peripheral_32MX795F512L.a(port_set_pins_digital_out_lib.o)
 .text          0x00000000        0x0 c:/program files (x86)/microchip/xc32/v1.10/bin/../lib/gcc/pic32mx/4.5.1/../../../../pic32mx/lib/size\libmchp_peripheral_32MX795F512L.a(_ports_tbl_libp.o)
 .data          0x00000000        0x0 c:/program files (x86)/microchip/xc32/v1.10/bin/../lib/gcc/pic32mx/4.5.1/../../../../pic32mx/lib/size\libmchp_peripheral_32MX795F512L.a(_ports_tbl_libp.o)
 .bss           0x00000000        0x0 c:/program files (x86)/microchip/xc32/v1.10/bin/../lib/gcc/pic32mx/4.5.1/../../../../pic32mx/lib/size\libmchp_peripheral_32MX795F512L.a(_ports_tbl_libp.o)
 .reginfo       0x00000000       0x18 c:/program files (x86)/microchip/xc32/v1.10/bin/../lib/gcc/pic32mx/4.5.1/../../../../pic32mx/lib/size\libmchp_peripheral_32MX795F512L.a(_ports_tbl_libp.o)
 .pdr           0x00000000        0x0 c:/program files (x86)/microchip/xc32/v1.10/bin/../lib/gcc/pic32mx/4.5.1/../../../../pic32mx/lib/size\libmchp_peripheral_32MX795F512L.a(_ports_tbl_libp.o)
 .text          0x00000000        0x0 c:/program files (x86)/microchip/xc32/v1.10/bin/../lib/gcc/pic32mx/4.5.1/../../../../pic32mx/lib/size\libmchp_peripheral_32MX795F512L.a(int_enable_interrupts_lib.o)
 .data          0x00000000        0x0 c:/program files (x86)/microchip/xc32/v1.10/bin/../lib/gcc/pic32mx/4.5.1/../../../../pic32mx/lib/size\libmchp_peripheral_32MX795F512L.a(int_enable_interrupts_lib.o)
 .bss           0x00000000        0x0 c:/program files (x86)/microchip/xc32/v1.10/bin/../lib/gcc/pic32mx/4.5.1/../../../../pic32mx/lib/size\libmchp_peripheral_32MX795F512L.a(int_enable_interrupts_lib.o)
 .reginfo       0x00000000       0x18 c:/program files (x86)/microchip/xc32/v1.10/bin/../lib/gcc/pic32mx/4.5.1/../../../../pic32mx/lib/size\libmchp_peripheral_32MX795F512L.a(int_enable_interrupts_lib.o)
 .pdr           0x00000000       0x20 c:/program files (x86)/microchip/xc32/v1.10/bin/../lib/gcc/pic32mx/4.5.1/../../../../pic32mx/lib/size\libmchp_peripheral_32MX795F512L.a(int_enable_interrupts_lib.o)
 .text          0x00000000        0x0 c:/program files (x86)/microchip/xc32/v1.10/bin/../lib/gcc/pic32mx/4.5.1/../../../../pic32mx/lib/size\libmchp_peripheral_32MX795F512L.a(_rtcc_wait_clock_off_lib.o)
 .data          0x00000000        0x0 c:/program files (x86)/microchip/xc32/v1.10/bin/../lib/gcc/pic32mx/4.5.1/../../../../pic32mx/lib/size\libmchp_peripheral_32MX795F512L.a(_rtcc_wait_clock_off_lib.o)
 .bss           0x00000000        0x0 c:/program files (x86)/microchip/xc32/v1.10/bin/../lib/gcc/pic32mx/4.5.1/../../../../pic32mx/lib/size\libmchp_peripheral_32MX795F512L.a(_rtcc_wait_clock_off_lib.o)
 .reginfo       0x00000000       0x18 c:/program files (x86)/microchip/xc32/v1.10/bin/../lib/gcc/pic32mx/4.5.1/../../../../pic32mx/lib/size\libmchp_peripheral_32MX795F512L.a(_rtcc_wait_clock_off_lib.o)
 .pdr           0x00000000       0x40 c:/program files (x86)/microchip/xc32/v1.10/bin/../lib/gcc/pic32mx/4.5.1/../../../../pic32mx/lib/size\libmchp_peripheral_32MX795F512L.a(_rtcc_wait_clock_off_lib.o)
 .text._RtccWaitClockOff
                0x00000000       0xf8 c:/program files (x86)/microchip/xc32/v1.10/bin/../lib/gcc/pic32mx/4.5.1/../../../../pic32mx/lib/size\libmchp_peripheral_32MX795F512L.a(_rtcc_wait_clock_off_lib.o)
 .text._RtccSetClockWait
                0x00000000       0x14 c:/program files (x86)/microchip/xc32/v1.10/bin/../lib/gcc/pic32mx/4.5.1/../../../../pic32mx/lib/size\libmchp_peripheral_32MX795F512L.a(_rtcc_wait_clock_off_lib.o)
 .sdata         0x00000000        0x8 c:/program files (x86)/microchip/xc32/v1.10/bin/../lib/gcc/pic32mx/4.5.1/../../../../pic32mx/lib/size\libmchp_peripheral_32MX795F512L.a(_rtcc_wait_clock_off_lib.o)
 .text          0x00000000        0x0 c:/program files (x86)/microchip/xc32/v1.10/bin/../lib/gcc/pic32mx/4.5.1/../../../../pic32mx/lib/size\libmchp_peripheral_32MX795F512L.a(read_core_timer_lib.o)
 .data          0x00000000        0x0 c:/program files (x86)/microchip/xc32/v1.10/bin/../lib/gcc/pic32mx/4.5.1/../../../../pic32mx/lib/size\libmchp_peripheral_32MX795F512L.a(read_core_timer_lib.o)
 .bss           0x00000000        0x0 c:/program files (x86)/microchip/xc32/v1.10/bin/../lib/gcc/pic32mx/4.5.1/../../../../pic32mx/lib/size\libmchp_peripheral_32MX795F512L.a(read_core_timer_lib.o)
 .reginfo       0x00000000       0x18 c:/program files (x86)/microchip/xc32/v1.10/bin/../lib/gcc/pic32mx/4.5.1/../../../../pic32mx/lib/size\libmchp_peripheral_32MX795F512L.a(read_core_timer_lib.o)
 .pdr           0x00000000       0x20 c:/program files (x86)/microchip/xc32/v1.10/bin/../lib/gcc/pic32mx/4.5.1/../../../../pic32mx/lib/size\libmchp_peripheral_32MX795F512L.a(read_core_timer_lib.o)
 .text.ReadCoreTimer
                0x00000000        0x8 c:/program files (x86)/microchip/xc32/v1.10/bin/../lib/gcc/pic32mx/4.5.1/../../../../pic32mx/lib/size\libmchp_peripheral_32MX795F512L.a(read_core_timer_lib.o)
 .data          0x00000000        0x0 c:/program files (x86)/microchip/xc32/v1.10/bin/../lib/gcc/pic32mx/4.5.1/size\libgcc.a(_udivdi3.o)
 .bss           0x00000000        0x0 c:/program files (x86)/microchip/xc32/v1.10/bin/../lib/gcc/pic32mx/4.5.1/size\libgcc.a(_udivdi3.o)
 .reginfo       0x00000000       0x18 c:/program files (x86)/microchip/xc32/v1.10/bin/../lib/gcc/pic32mx/4.5.1/size\libgcc.a(_udivdi3.o)
 .pdr           0x00000000       0x20 c:/program files (x86)/microchip/xc32/v1.10/bin/../lib/gcc/pic32mx/4.5.1/size\libgcc.a(_udivdi3.o)
 .data          0x00000000        0x0 c:/program files (x86)/microchip/xc32/v1.10/bin/../lib/gcc/pic32mx/4.5.1/../../../../pic32mx/lib/size\libpic32.a(memcmp.o)
 .bss           0x00000000        0x0 c:/program files (x86)/microchip/xc32/v1.10/bin/../lib/gcc/pic32mx/4.5.1/../../../../pic32mx/lib/size\libpic32.a(memcmp.o)
 .reginfo       0x00000000       0x18 c:/program files (x86)/microchip/xc32/v1.10/bin/../lib/gcc/pic32mx/4.5.1/../../../../pic32mx/lib/size\libpic32.a(memcmp.o)
 .pdr           0x00000000       0x20 c:/program files (x86)/microchip/xc32/v1.10/bin/../lib/gcc/pic32mx/4.5.1/../../../../pic32mx/lib/size\libpic32.a(memcmp.o)
 .data          0x00000000        0x0 c:/program files (x86)/microchip/xc32/v1.10/bin/../lib/gcc/pic32mx/4.5.1/../../../../pic32mx/lib/size\libpic32.a(memcpy.o)
 .bss           0x00000000        0x0 c:/program files (x86)/microchip/xc32/v1.10/bin/../lib/gcc/pic32mx/4.5.1/../../../../pic32mx/lib/size\libpic32.a(memcpy.o)
 .reginfo       0x00000000       0x18 c:/program files (x86)/microchip/xc32/v1.10/bin/../lib/gcc/pic32mx/4.5.1/../../../../pic32mx/lib/size\libpic32.a(memcpy.o)
 .pdr           0x00000000       0x20 c:/program files (x86)/microchip/xc32/v1.10/bin/../lib/gcc/pic32mx/4.5.1/../../../../pic32mx/lib/size\libpic32.a(memcpy.o)
 .data          0x00000000        0x0 c:/program files (x86)/microchip/xc32/v1.10/bin/../lib/gcc/pic32mx/4.5.1/../../../../pic32mx/lib/size\libpic32.a(memset.o)
 .bss           0x00000000        0x0 c:/program files (x86)/microchip/xc32/v1.10/bin/../lib/gcc/pic32mx/4.5.1/../../../../pic32mx/lib/size\libpic32.a(memset.o)
 .reginfo       0x00000000       0x18 c:/program files (x86)/microchip/xc32/v1.10/bin/../lib/gcc/pic32mx/4.5.1/../../../../pic32mx/lib/size\libpic32.a(memset.o)
 .pdr           0x00000000       0x20 c:/program files (x86)/microchip/xc32/v1.10/bin/../lib/gcc/pic32mx/4.5.1/../../../../pic32mx/lib/size\libpic32.a(memset.o)
 .data          0x00000000        0x0 c:/program files (x86)/microchip/xc32/v1.10/bin/../lib/gcc/pic32mx/4.5.1/../../../../pic32mx/lib/size\libpic32.a(strcmp.o)
 .bss           0x00000000        0x0 c:/program files (x86)/microchip/xc32/v1.10/bin/../lib/gcc/pic32mx/4.5.1/../../../../pic32mx/lib/size\libpic32.a(strcmp.o)
 .reginfo       0x00000000       0x18 c:/program files (x86)/microchip/xc32/v1.10/bin/../lib/gcc/pic32mx/4.5.1/../../../../pic32mx/lib/size\libpic32.a(strcmp.o)
 .pdr           0x00000000       0x20 c:/program files (x86)/microchip/xc32/v1.10/bin/../lib/gcc/pic32mx/4.5.1/../../../../pic32mx/lib/size\libpic32.a(strcmp.o)
 .data          0x00000000        0x0 c:/program files (x86)/microchip/xc32/v1.10/bin/../lib/gcc/pic32mx/4.5.1/../../../../pic32mx/lib/size\libpic32.a(strcpy.o)
 .bss           0x00000000        0x0 c:/program files (x86)/microchip/xc32/v1.10/bin/../lib/gcc/pic32mx/4.5.1/../../../../pic32mx/lib/size\libpic32.a(strcpy.o)
 .reginfo       0x00000000       0x18 c:/program files (x86)/microchip/xc32/v1.10/bin/../lib/gcc/pic32mx/4.5.1/../../../../pic32mx/lib/size\libpic32.a(strcpy.o)
 .pdr           0x00000000       0x20 c:/program files (x86)/microchip/xc32/v1.10/bin/../lib/gcc/pic32mx/4.5.1/../../../../pic32mx/lib/size\libpic32.a(strcpy.o)
 .data          0x00000000        0x0 c:/program files (x86)/microchip/xc32/v1.10/bin/../lib/gcc/pic32mx/4.5.1/../../../../pic32mx/lib/size\libpic32.a(strlen.o)
 .bss           0x00000000        0x0 c:/program files (x86)/microchip/xc32/v1.10/bin/../lib/gcc/pic32mx/4.5.1/../../../../pic32mx/lib/size\libpic32.a(strlen.o)
 .reginfo       0x00000000       0x18 c:/program files (x86)/microchip/xc32/v1.10/bin/../lib/gcc/pic32mx/4.5.1/../../../../pic32mx/lib/size\libpic32.a(strlen.o)
 .pdr           0x00000000       0x20 c:/program files (x86)/microchip/xc32/v1.10/bin/../lib/gcc/pic32mx/4.5.1/../../../../pic32mx/lib/size\libpic32.a(strlen.o)
 .text          0x00000000        0x0 c:/program files (x86)/microchip/xc32/v1.10/bin/../lib/gcc/pic32mx/4.5.1/../../../../pic32mx/lib/size\libpic32.a(default-bootstrap-exception-handler.o)
 .data          0x00000000        0x0 c:/program files (x86)/microchip/xc32/v1.10/bin/../lib/gcc/pic32mx/4.5.1/../../../../pic32mx/lib/size\libpic32.a(default-bootstrap-exception-handler.o)
 .bss           0x00000000        0x0 c:/program files (x86)/microchip/xc32/v1.10/bin/../lib/gcc/pic32mx/4.5.1/../../../../pic32mx/lib/size\libpic32.a(default-bootstrap-exception-handler.o)
 .reginfo       0x00000000       0x18 c:/program files (x86)/microchip/xc32/v1.10/bin/../lib/gcc/pic32mx/4.5.1/../../../../pic32mx/lib/size\libpic32.a(default-bootstrap-exception-handler.o)
 .pdr           0x00000000       0x20 c:/program files (x86)/microchip/xc32/v1.10/bin/../lib/gcc/pic32mx/4.5.1/../../../../pic32mx/lib/size\libpic32.a(default-bootstrap-exception-handler.o)
 .text          0x00000000        0x0 c:/program files (x86)/microchip/xc32/v1.10/bin/../lib/gcc/pic32mx/4.5.1/../../../../pic32mx/lib/size\libpic32.a(default-on-reset.o)
 .data          0x00000000        0x0 c:/program files (x86)/microchip/xc32/v1.10/bin/../lib/gcc/pic32mx/4.5.1/../../../../pic32mx/lib/size\libpic32.a(default-on-reset.o)
 .bss           0x00000000        0x0 c:/program files (x86)/microchip/xc32/v1.10/bin/../lib/gcc/pic32mx/4.5.1/../../../../pic32mx/lib/size\libpic32.a(default-on-reset.o)
 .reginfo       0x00000000       0x18 c:/program files (x86)/microchip/xc32/v1.10/bin/../lib/gcc/pic32mx/4.5.1/../../../../pic32mx/lib/size\libpic32.a(default-on-reset.o)
 .pdr           0x00000000       0x20 c:/program files (x86)/microchip/xc32/v1.10/bin/../lib/gcc/pic32mx/4.5.1/../../../../pic32mx/lib/size\libpic32.a(default-on-reset.o)
 .text          0x00000000        0x0 c:/program files (x86)/microchip/xc32/v1.10/bin/../lib/gcc/pic32mx/4.5.1/../../../../pic32mx/lib/size\libpic32.a(default-on-bootstrap.o)
 .data          0x00000000        0x0 c:/program files (x86)/microchip/xc32/v1.10/bin/../lib/gcc/pic32mx/4.5.1/../../../../pic32mx/lib/size\libpic32.a(default-on-bootstrap.o)
 .bss           0x00000000        0x0 c:/program files (x86)/microchip/xc32/v1.10/bin/../lib/gcc/pic32mx/4.5.1/../../../../pic32mx/lib/size\libpic32.a(default-on-bootstrap.o)
 .reginfo       0x00000000       0x18 c:/program files (x86)/microchip/xc32/v1.10/bin/../lib/gcc/pic32mx/4.5.1/../../../../pic32mx/lib/size\libpic32.a(default-on-bootstrap.o)
 .pdr           0x00000000       0x20 c:/program files (x86)/microchip/xc32/v1.10/bin/../lib/gcc/pic32mx/4.5.1/../../../../pic32mx/lib/size\libpic32.a(default-on-bootstrap.o)
 .data          0x00000000        0x0 c:/program files (x86)/microchip/xc32/v1.10/bin/../lib/gcc/pic32mx/4.5.1/../../../../pic32mx/lib/size\libpic32.a(default-nmi-handler.o)
 .bss           0x00000000        0x0 c:/program files (x86)/microchip/xc32/v1.10/bin/../lib/gcc/pic32mx/4.5.1/../../../../pic32mx/lib/size\libpic32.a(default-nmi-handler.o)
 .reginfo       0x00000000       0x18 c:/program files (x86)/microchip/xc32/v1.10/bin/../lib/gcc/pic32mx/4.5.1/../../../../pic32mx/lib/size\libpic32.a(default-nmi-handler.o)
 .pdr           0x00000000       0x20 c:/program files (x86)/microchip/xc32/v1.10/bin/../lib/gcc/pic32mx/4.5.1/../../../../pic32mx/lib/size\libpic32.a(default-nmi-handler.o)
 .text          0x00000000        0x0 c:/program files (x86)/microchip/xc32/v1.10/bin/../lib/gcc/pic32mx/4.5.1/../../../../pic32mx/lib/size\libpic32.a(errno.o)
 .data          0x00000000        0x0 c:/program files (x86)/microchip/xc32/v1.10/bin/../lib/gcc/pic32mx/4.5.1/../../../../pic32mx/lib/size\libpic32.a(errno.o)
 .bss           0x00000000        0x0 c:/program files (x86)/microchip/xc32/v1.10/bin/../lib/gcc/pic32mx/4.5.1/../../../../pic32mx/lib/size\libpic32.a(errno.o)
 .reginfo       0x00000000       0x18 c:/program files (x86)/microchip/xc32/v1.10/bin/../lib/gcc/pic32mx/4.5.1/../../../../pic32mx/lib/size\libpic32.a(errno.o)
 .pdr           0x00000000        0x0 c:/program files (x86)/microchip/xc32/v1.10/bin/../lib/gcc/pic32mx/4.5.1/../../../../pic32mx/lib/size\libpic32.a(errno.o)
 .text          0x00000000        0x0 c:/program files (x86)/microchip/xc32/v1.10/bin/../lib/gcc/pic32mx/4.5.1/../../../../pic32mx/lib/size\libpic32.a(general-exception.o)
 .data          0x00000000        0x0 c:/program files (x86)/microchip/xc32/v1.10/bin/../lib/gcc/pic32mx/4.5.1/../../../../pic32mx/lib/size\libpic32.a(general-exception.o)
 .bss           0x00000000        0x0 c:/program files (x86)/microchip/xc32/v1.10/bin/../lib/gcc/pic32mx/4.5.1/../../../../pic32mx/lib/size\libpic32.a(general-exception.o)
 .reginfo       0x00000000       0x18 c:/program files (x86)/microchip/xc32/v1.10/bin/../lib/gcc/pic32mx/4.5.1/../../../../pic32mx/lib/size\libpic32.a(general-exception.o)
 .pdr           0x00000000       0x20 c:/program files (x86)/microchip/xc32/v1.10/bin/../lib/gcc/pic32mx/4.5.1/../../../../pic32mx/lib/size\libpic32.a(general-exception.o)
 .text          0x00000000        0x0 c:/program files (x86)/microchip/xc32/v1.10/bin/../lib/gcc/pic32mx/4.5.1/../../../../pic32mx/lib/size\libc.a(atoi.o)
 .data          0x00000000        0x0 c:/program files (x86)/microchip/xc32/v1.10/bin/../lib/gcc/pic32mx/4.5.1/../../../../pic32mx/lib/size\libc.a(atoi.o)
 .bss           0x00000000        0x0 c:/program files (x86)/microchip/xc32/v1.10/bin/../lib/gcc/pic32mx/4.5.1/../../../../pic32mx/lib/size\libc.a(atoi.o)
 .reginfo       0x00000000       0x18 c:/program files (x86)/microchip/xc32/v1.10/bin/../lib/gcc/pic32mx/4.5.1/../../../../pic32mx/lib/size\libc.a(atoi.o)
 .pdr           0x00000000       0x20 c:/program files (x86)/microchip/xc32/v1.10/bin/../lib/gcc/pic32mx/4.5.1/../../../../pic32mx/lib/size\libc.a(atoi.o)
 .text          0x00000000        0x0 c:/program files (x86)/microchip/xc32/v1.10/bin/../lib/gcc/pic32mx/4.5.1/../../../../pic32mx/lib/size\libc.a(atol.o)
 .data          0x00000000        0x0 c:/program files (x86)/microchip/xc32/v1.10/bin/../lib/gcc/pic32mx/4.5.1/../../../../pic32mx/lib/size\libc.a(atol.o)
 .bss           0x00000000        0x0 c:/program files (x86)/microchip/xc32/v1.10/bin/../lib/gcc/pic32mx/4.5.1/../../../../pic32mx/lib/size\libc.a(atol.o)
 .reginfo       0x00000000       0x18 c:/program files (x86)/microchip/xc32/v1.10/bin/../lib/gcc/pic32mx/4.5.1/../../../../pic32mx/lib/size\libc.a(atol.o)
 .pdr           0x00000000       0x20 c:/program files (x86)/microchip/xc32/v1.10/bin/../lib/gcc/pic32mx/4.5.1/../../../../pic32mx/lib/size\libc.a(atol.o)
 .text          0x00000000        0x0 c:/program files (x86)/microchip/xc32/v1.10/bin/../lib/gcc/pic32mx/4.5.1/../../../../pic32mx/lib/size\libc.a(ctype.o)
 .data          0x00000000        0x0 c:/program files (x86)/microchip/xc32/v1.10/bin/../lib/gcc/pic32mx/4.5.1/../../../../pic32mx/lib/size\libc.a(ctype.o)
 .bss           0x00000000        0x0 c:/program files (x86)/microchip/xc32/v1.10/bin/../lib/gcc/pic32mx/4.5.1/../../../../pic32mx/lib/size\libc.a(ctype.o)
 .reginfo       0x00000000       0x18 c:/program files (x86)/microchip/xc32/v1.10/bin/../lib/gcc/pic32mx/4.5.1/../../../../pic32mx/lib/size\libc.a(ctype.o)
 .pdr           0x00000000        0x0 c:/program files (x86)/microchip/xc32/v1.10/bin/../lib/gcc/pic32mx/4.5.1/../../../../pic32mx/lib/size\libc.a(ctype.o)
 .text          0x00000000        0x0 c:/program files (x86)/microchip/xc32/v1.10/bin/../lib/gcc/pic32mx/4.5.1/../../../../pic32mx/lib/size\libc.a(malloc.o)
 .data          0x00000000        0x0 c:/program files (x86)/microchip/xc32/v1.10/bin/../lib/gcc/pic32mx/4.5.1/../../../../pic32mx/lib/size\libc.a(malloc.o)
 .reginfo       0x00000000       0x18 c:/program files (x86)/microchip/xc32/v1.10/bin/../lib/gcc/pic32mx/4.5.1/../../../../pic32mx/lib/size\libc.a(malloc.o)
 .pdr           0x00000000       0x60 c:/program files (x86)/microchip/xc32/v1.10/bin/../lib/gcc/pic32mx/4.5.1/../../../../pic32mx/lib/size\libc.a(malloc.o)
 .text          0x00000000        0x0 c:/program files (x86)/microchip/xc32/v1.10/bin/../lib/gcc/pic32mx/4.5.1/../../../../pic32mx/lib/size\libc.a(rand.o)
 .data          0x00000000        0x0 c:/program files (x86)/microchip/xc32/v1.10/bin/../lib/gcc/pic32mx/4.5.1/../../../../pic32mx/lib/size\libc.a(rand.o)
 .reginfo       0x00000000       0x18 c:/program files (x86)/microchip/xc32/v1.10/bin/../lib/gcc/pic32mx/4.5.1/../../../../pic32mx/lib/size\libc.a(rand.o)
 .pdr           0x00000000       0x40 c:/program files (x86)/microchip/xc32/v1.10/bin/../lib/gcc/pic32mx/4.5.1/../../../../pic32mx/lib/size\libc.a(rand.o)
 .text          0x00000000        0x0 c:/program files (x86)/microchip/xc32/v1.10/bin/../lib/gcc/pic32mx/4.5.1/../../../../pic32mx/lib/size\libc.a(strcat.o)
 .data          0x00000000        0x0 c:/program files (x86)/microchip/xc32/v1.10/bin/../lib/gcc/pic32mx/4.5.1/../../../../pic32mx/lib/size\libc.a(strcat.o)
 .bss           0x00000000        0x0 c:/program files (x86)/microchip/xc32/v1.10/bin/../lib/gcc/pic32mx/4.5.1/../../../../pic32mx/lib/size\libc.a(strcat.o)
 .reginfo       0x00000000       0x18 c:/program files (x86)/microchip/xc32/v1.10/bin/../lib/gcc/pic32mx/4.5.1/../../../../pic32mx/lib/size\libc.a(strcat.o)
 .pdr           0x00000000       0x20 c:/program files (x86)/microchip/xc32/v1.10/bin/../lib/gcc/pic32mx/4.5.1/../../../../pic32mx/lib/size\libc.a(strcat.o)
 .text          0x00000000        0x0 c:/program files (x86)/microchip/xc32/v1.10/bin/../lib/gcc/pic32mx/4.5.1/../../../../pic32mx/lib/size\libc.a(strchr.o)
 .data          0x00000000        0x0 c:/program files (x86)/microchip/xc32/v1.10/bin/../lib/gcc/pic32mx/4.5.1/../../../../pic32mx/lib/size\libc.a(strchr.o)
 .bss           0x00000000        0x0 c:/program files (x86)/microchip/xc32/v1.10/bin/../lib/gcc/pic32mx/4.5.1/../../../../pic32mx/lib/size\libc.a(strchr.o)
 .reginfo       0x00000000       0x18 c:/program files (x86)/microchip/xc32/v1.10/bin/../lib/gcc/pic32mx/4.5.1/../../../../pic32mx/lib/size\libc.a(strchr.o)
 .pdr           0x00000000       0x20 c:/program files (x86)/microchip/xc32/v1.10/bin/../lib/gcc/pic32mx/4.5.1/../../../../pic32mx/lib/size\libc.a(strchr.o)
 .text          0x00000000        0x0 c:/program files (x86)/microchip/xc32/v1.10/bin/../lib/gcc/pic32mx/4.5.1/../../../../pic32mx/lib/size\libc.a(strncat.o)
 .data          0x00000000        0x0 c:/program files (x86)/microchip/xc32/v1.10/bin/../lib/gcc/pic32mx/4.5.1/../../../../pic32mx/lib/size\libc.a(strncat.o)
 .bss           0x00000000        0x0 c:/program files (x86)/microchip/xc32/v1.10/bin/../lib/gcc/pic32mx/4.5.1/../../../../pic32mx/lib/size\libc.a(strncat.o)
 .reginfo       0x00000000       0x18 c:/program files (x86)/microchip/xc32/v1.10/bin/../lib/gcc/pic32mx/4.5.1/../../../../pic32mx/lib/size\libc.a(strncat.o)
 .pdr           0x00000000       0x20 c:/program files (x86)/microchip/xc32/v1.10/bin/../lib/gcc/pic32mx/4.5.1/../../../../pic32mx/lib/size\libc.a(strncat.o)
 .text          0x00000000        0x0 c:/program files (x86)/microchip/xc32/v1.10/bin/../lib/gcc/pic32mx/4.5.1/../../../../pic32mx/lib/size\libc.a(strncmp.o)
 .data          0x00000000        0x0 c:/program files (x86)/microchip/xc32/v1.10/bin/../lib/gcc/pic32mx/4.5.1/../../../../pic32mx/lib/size\libc.a(strncmp.o)
 .bss           0x00000000        0x0 c:/program files (x86)/microchip/xc32/v1.10/bin/../lib/gcc/pic32mx/4.5.1/../../../../pic32mx/lib/size\libc.a(strncmp.o)
 .reginfo       0x00000000       0x18 c:/program files (x86)/microchip/xc32/v1.10/bin/../lib/gcc/pic32mx/4.5.1/../../../../pic32mx/lib/size\libc.a(strncmp.o)
 .pdr           0x00000000       0x20 c:/program files (x86)/microchip/xc32/v1.10/bin/../lib/gcc/pic32mx/4.5.1/../../../../pic32mx/lib/size\libc.a(strncmp.o)
 .text          0x00000000        0x0 c:/program files (x86)/microchip/xc32/v1.10/bin/../lib/gcc/pic32mx/4.5.1/../../../../pic32mx/lib/size\libc.a(strncpy.o)
 .data          0x00000000        0x0 c:/program files (x86)/microchip/xc32/v1.10/bin/../lib/gcc/pic32mx/4.5.1/../../../../pic32mx/lib/size\libc.a(strncpy.o)
 .bss           0x00000000        0x0 c:/program files (x86)/microchip/xc32/v1.10/bin/../lib/gcc/pic32mx/4.5.1/../../../../pic32mx/lib/size\libc.a(strncpy.o)
 .reginfo       0x00000000       0x18 c:/program files (x86)/microchip/xc32/v1.10/bin/../lib/gcc/pic32mx/4.5.1/../../../../pic32mx/lib/size\libc.a(strncpy.o)
 .pdr           0x00000000       0x20 c:/program files (x86)/microchip/xc32/v1.10/bin/../lib/gcc/pic32mx/4.5.1/../../../../pic32mx/lib/size\libc.a(strncpy.o)
 .text          0x00000000        0x0 c:/program files (x86)/microchip/xc32/v1.10/bin/../lib/gcc/pic32mx/4.5.1/../../../../pic32mx/lib/size\libc.a(strrchr.o)
 .data          0x00000000        0x0 c:/program files (x86)/microchip/xc32/v1.10/bin/../lib/gcc/pic32mx/4.5.1/../../../../pic32mx/lib/size\libc.a(strrchr.o)
 .bss           0x00000000        0x0 c:/program files (x86)/microchip/xc32/v1.10/bin/../lib/gcc/pic32mx/4.5.1/../../../../pic32mx/lib/size\libc.a(strrchr.o)
 .reginfo       0x00000000       0x18 c:/program files (x86)/microchip/xc32/v1.10/bin/../lib/gcc/pic32mx/4.5.1/../../../../pic32mx/lib/size\libc.a(strrchr.o)
 .pdr           0x00000000       0x20 c:/program files (x86)/microchip/xc32/v1.10/bin/../lib/gcc/pic32mx/4.5.1/../../../../pic32mx/lib/size\libc.a(strrchr.o)
 .text.strrchr  0x00000000       0x4c c:/program files (x86)/microchip/xc32/v1.10/bin/../lib/gcc/pic32mx/4.5.1/../../../../pic32mx/lib/size\libc.a(strrchr.o)
 .text          0x00000000        0x0 c:/program files (x86)/microchip/xc32/v1.10/bin/../lib/gcc/pic32mx/4.5.1/../../../../pic32mx/lib/size\libc.a(strstr.o)
 .data          0x00000000        0x0 c:/program files (x86)/microchip/xc32/v1.10/bin/../lib/gcc/pic32mx/4.5.1/../../../../pic32mx/lib/size\libc.a(strstr.o)
 .bss           0x00000000        0x0 c:/program files (x86)/microchip/xc32/v1.10/bin/../lib/gcc/pic32mx/4.5.1/../../../../pic32mx/lib/size\libc.a(strstr.o)
 .reginfo       0x00000000       0x18 c:/program files (x86)/microchip/xc32/v1.10/bin/../lib/gcc/pic32mx/4.5.1/../../../../pic32mx/lib/size\libc.a(strstr.o)
 .pdr           0x00000000       0x20 c:/program files (x86)/microchip/xc32/v1.10/bin/../lib/gcc/pic32mx/4.5.1/../../../../pic32mx/lib/size\libc.a(strstr.o)
 .text          0x00000000        0x0 c:/program files (x86)/microchip/xc32/v1.10/bin/../lib/gcc/pic32mx/4.5.1/../../../../pic32mx/lib/size\libc.a(strtol.o)
 .data          0x00000000        0x0 c:/program files (x86)/microchip/xc32/v1.10/bin/../lib/gcc/pic32mx/4.5.1/../../../../pic32mx/lib/size\libc.a(strtol.o)
 .bss           0x00000000        0x0 c:/program files (x86)/microchip/xc32/v1.10/bin/../lib/gcc/pic32mx/4.5.1/../../../../pic32mx/lib/size\libc.a(strtol.o)
 .reginfo       0x00000000       0x18 c:/program files (x86)/microchip/xc32/v1.10/bin/../lib/gcc/pic32mx/4.5.1/../../../../pic32mx/lib/size\libc.a(strtol.o)
 .pdr           0x00000000       0x40 c:/program files (x86)/microchip/xc32/v1.10/bin/../lib/gcc/pic32mx/4.5.1/../../../../pic32mx/lib/size\libc.a(strtol.o)
 .text          0x00000000        0x0 c:/program files (x86)/microchip/xc32/v1.10/bin/../lib/gcc/pic32mx/4.5.1/../../../../pic32mx/lib/size\libc.a(snprintf_cdnopsuxX.eo)
 .data          0x00000000        0x0 c:/program files (x86)/microchip/xc32/v1.10/bin/../lib/gcc/pic32mx/4.5.1/../../../../pic32mx/lib/size\libc.a(snprintf_cdnopsuxX.eo)
 .bss           0x00000000        0x0 c:/program files (x86)/microchip/xc32/v1.10/bin/../lib/gcc/pic32mx/4.5.1/../../../../pic32mx/lib/size\libc.a(snprintf_cdnopsuxX.eo)
 .reginfo       0x00000000       0x18 c:/program files (x86)/microchip/xc32/v1.10/bin/../lib/gcc/pic32mx/4.5.1/../../../../pic32mx/lib/size\libc.a(snprintf_cdnopsuxX.eo)
 .pdr           0x00000000       0x20 c:/program files (x86)/microchip/xc32/v1.10/bin/../lib/gcc/pic32mx/4.5.1/../../../../pic32mx/lib/size\libc.a(snprintf_cdnopsuxX.eo)
 .text          0x00000000        0x0 c:/program files (x86)/microchip/xc32/v1.10/bin/../lib/gcc/pic32mx/4.5.1/../../../../pic32mx/lib/size\libc.a(sprintf_cdnopsuxX.eo)
 .data          0x00000000        0x0 c:/program files (x86)/microchip/xc32/v1.10/bin/../lib/gcc/pic32mx/4.5.1/../../../../pic32mx/lib/size\libc.a(sprintf_cdnopsuxX.eo)
 .bss           0x00000000        0x0 c:/program files (x86)/microchip/xc32/v1.10/bin/../lib/gcc/pic32mx/4.5.1/../../../../pic32mx/lib/size\libc.a(sprintf_cdnopsuxX.eo)
 .reginfo       0x00000000       0x18 c:/program files (x86)/microchip/xc32/v1.10/bin/../lib/gcc/pic32mx/4.5.1/../../../../pic32mx/lib/size\libc.a(sprintf_cdnopsuxX.eo)
 .pdr           0x00000000       0x20 c:/program files (x86)/microchip/xc32/v1.10/bin/../lib/gcc/pic32mx/4.5.1/../../../../pic32mx/lib/size\libc.a(sprintf_cdnopsuxX.eo)
 .text          0x00000000        0x0 c:/program files (x86)/microchip/xc32/v1.10/bin/../lib/gcc/pic32mx/4.5.1/../../../../pic32mx/lib/size\libc.a(vsnprintf_cdnopsuxX.eo)
 .data          0x00000000        0x0 c:/program files (x86)/microchip/xc32/v1.10/bin/../lib/gcc/pic32mx/4.5.1/../../../../pic32mx/lib/size\libc.a(vsnprintf_cdnopsuxX.eo)
 .bss           0x00000000        0x0 c:/program files (x86)/microchip/xc32/v1.10/bin/../lib/gcc/pic32mx/4.5.1/../../../../pic32mx/lib/size\libc.a(vsnprintf_cdnopsuxX.eo)
 .reginfo       0x00000000       0x18 c:/program files (x86)/microchip/xc32/v1.10/bin/../lib/gcc/pic32mx/4.5.1/../../../../pic32mx/lib/size\libc.a(vsnprintf_cdnopsuxX.eo)
 .pdr           0x00000000       0x20 c:/program files (x86)/microchip/xc32/v1.10/bin/../lib/gcc/pic32mx/4.5.1/../../../../pic32mx/lib/size\libc.a(vsnprintf_cdnopsuxX.eo)
 .text          0x00000000        0x0 c:/program files (x86)/microchip/xc32/v1.10/bin/../lib/gcc/pic32mx/4.5.1/../../../../pic32mx/lib/size\libc.a(vsnprintf.o)
 .data          0x00000000        0x0 c:/program files (x86)/microchip/xc32/v1.10/bin/../lib/gcc/pic32mx/4.5.1/../../../../pic32mx/lib/size\libc.a(vsnprintf.o)
 .bss           0x00000000        0x0 c:/program files (x86)/microchip/xc32/v1.10/bin/../lib/gcc/pic32mx/4.5.1/../../../../pic32mx/lib/size\libc.a(vsnprintf.o)
 .reginfo       0x00000000       0x18 c:/program files (x86)/microchip/xc32/v1.10/bin/../lib/gcc/pic32mx/4.5.1/../../../../pic32mx/lib/size\libc.a(vsnprintf.o)
 .pdr           0x00000000       0x20 c:/program files (x86)/microchip/xc32/v1.10/bin/../lib/gcc/pic32mx/4.5.1/../../../../pic32mx/lib/size\libc.a(vsnprintf.o)
 .text          0x00000000        0x0 c:/program files (x86)/microchip/xc32/v1.10/bin/../lib/gcc/pic32mx/4.5.1/../../../../pic32mx/lib/size\libc.a(ctypef.o)
 .data          0x00000000        0x0 c:/program files (x86)/microchip/xc32/v1.10/bin/../lib/gcc/pic32mx/4.5.1/../../../../pic32mx/lib/size\libc.a(ctypef.o)
 .bss           0x00000000        0x0 c:/program files (x86)/microchip/xc32/v1.10/bin/../lib/gcc/pic32mx/4.5.1/../../../../pic32mx/lib/size\libc.a(ctypef.o)
 .reginfo       0x00000000       0x18 c:/program files (x86)/microchip/xc32/v1.10/bin/../lib/gcc/pic32mx/4.5.1/../../../../pic32mx/lib/size\libc.a(ctypef.o)
 .pdr           0x00000000      0x220 c:/program files (x86)/microchip/xc32/v1.10/bin/../lib/gcc/pic32mx/4.5.1/../../../../pic32mx/lib/size\libc.a(ctypef.o)
 .text.tolower  0x00000000       0x24 c:/program files (x86)/microchip/xc32/v1.10/bin/../lib/gcc/pic32mx/4.5.1/../../../../pic32mx/lib/size\libc.a(ctypef.o)
 .text.isalnum  0x00000000       0x18 c:/program files (x86)/microchip/xc32/v1.10/bin/../lib/gcc/pic32mx/4.5.1/../../../../pic32mx/lib/size\libc.a(ctypef.o)
 .text.isalpha  0x00000000       0x18 c:/program files (x86)/microchip/xc32/v1.10/bin/../lib/gcc/pic32mx/4.5.1/../../../../pic32mx/lib/size\libc.a(ctypef.o)
 .text.isascii  0x00000000        0x8 c:/program files (x86)/microchip/xc32/v1.10/bin/../lib/gcc/pic32mx/4.5.1/../../../../pic32mx/lib/size\libc.a(ctypef.o)
 .text.iscntrl  0x00000000       0x18 c:/program files (x86)/microchip/xc32/v1.10/bin/../lib/gcc/pic32mx/4.5.1/../../../../pic32mx/lib/size\libc.a(ctypef.o)
 .text.isdigit  0x00000000       0x18 c:/program files (x86)/microchip/xc32/v1.10/bin/../lib/gcc/pic32mx/4.5.1/../../../../pic32mx/lib/size\libc.a(ctypef.o)
 .text.isgraph  0x00000000       0x18 c:/program files (x86)/microchip/xc32/v1.10/bin/../lib/gcc/pic32mx/4.5.1/../../../../pic32mx/lib/size\libc.a(ctypef.o)
 .text.islower  0x00000000       0x18 c:/program files (x86)/microchip/xc32/v1.10/bin/../lib/gcc/pic32mx/4.5.1/../../../../pic32mx/lib/size\libc.a(ctypef.o)
 .text.isprint  0x00000000       0x18 c:/program files (x86)/microchip/xc32/v1.10/bin/../lib/gcc/pic32mx/4.5.1/../../../../pic32mx/lib/size\libc.a(ctypef.o)
 .text.ispunct  0x00000000       0x18 c:/program files (x86)/microchip/xc32/v1.10/bin/../lib/gcc/pic32mx/4.5.1/../../../../pic32mx/lib/size\libc.a(ctypef.o)
 .text.isspace  0x00000000       0x18 c:/program files (x86)/microchip/xc32/v1.10/bin/../lib/gcc/pic32mx/4.5.1/../../../../pic32mx/lib/size\libc.a(ctypef.o)
 .text.isupper  0x00000000       0x18 c:/program files (x86)/microchip/xc32/v1.10/bin/../lib/gcc/pic32mx/4.5.1/../../../../pic32mx/lib/size\libc.a(ctypef.o)
 .text.isxdigit
                0x00000000       0x18 c:/program files (x86)/microchip/xc32/v1.10/bin/../lib/gcc/pic32mx/4.5.1/../../../../pic32mx/lib/size\libc.a(ctypef.o)
 .text.toascii  0x00000000        0x8 c:/program files (x86)/microchip/xc32/v1.10/bin/../lib/gcc/pic32mx/4.5.1/../../../../pic32mx/lib/size\libc.a(ctypef.o)
 .text._tolower
                0x00000000        0x8 c:/program files (x86)/microchip/xc32/v1.10/bin/../lib/gcc/pic32mx/4.5.1/../../../../pic32mx/lib/size\libc.a(ctypef.o)
 .text._toupper
                0x00000000        0x8 c:/program files (x86)/microchip/xc32/v1.10/bin/../lib/gcc/pic32mx/4.5.1/../../../../pic32mx/lib/size\libc.a(ctypef.o)
 .text          0x00000000        0x0 c:/program files (x86)/microchip/xc32/v1.10/bin/../lib/gcc/pic32mx/4.5.1/../../../../pic32mx/lib/size\libc.a(doprnt_cdnopsuxX.eo)
 .data          0x00000000        0x0 c:/program files (x86)/microchip/xc32/v1.10/bin/../lib/gcc/pic32mx/4.5.1/../../../../pic32mx/lib/size\libc.a(doprnt_cdnopsuxX.eo)
 .bss           0x00000000        0x0 c:/program files (x86)/microchip/xc32/v1.10/bin/../lib/gcc/pic32mx/4.5.1/../../../../pic32mx/lib/size\libc.a(doprnt_cdnopsuxX.eo)
 .reginfo       0x00000000       0x18 c:/program files (x86)/microchip/xc32/v1.10/bin/../lib/gcc/pic32mx/4.5.1/../../../../pic32mx/lib/size\libc.a(doprnt_cdnopsuxX.eo)
 .pdr           0x00000000       0x20 c:/program files (x86)/microchip/xc32/v1.10/bin/../lib/gcc/pic32mx/4.5.1/../../../../pic32mx/lib/size\libc.a(doprnt_cdnopsuxX.eo)
 .text          0x00000000        0x0 c:/program files (x86)/microchip/xc32/v1.10/bin/../lib/gcc/pic32mx/4.5.1/../../../../pic32mx/lib/size\libc.a(doprnt.o)
 .data          0x00000000        0x0 c:/program files (x86)/microchip/xc32/v1.10/bin/../lib/gcc/pic32mx/4.5.1/../../../../pic32mx/lib/size\libc.a(doprnt.o)
 .bss           0x00000000        0x0 c:/program files (x86)/microchip/xc32/v1.10/bin/../lib/gcc/pic32mx/4.5.1/../../../../pic32mx/lib/size\libc.a(doprnt.o)
 .reginfo       0x00000000       0x18 c:/program files (x86)/microchip/xc32/v1.10/bin/../lib/gcc/pic32mx/4.5.1/../../../../pic32mx/lib/size\libc.a(doprnt.o)
 .pdr           0x00000000       0x60 c:/program files (x86)/microchip/xc32/v1.10/bin/../lib/gcc/pic32mx/4.5.1/../../../../pic32mx/lib/size\libc.a(doprnt.o)
 .text          0x00000000        0x0 c:/program files (x86)/microchip/xc32/v1.10/bin/../lib/gcc/pic32mx/4.5.1/../../../../pic32mx/lib/size\libc.a(_fputc_simple.o)
 .data          0x00000000        0x0 c:/program files (x86)/microchip/xc32/v1.10/bin/../lib/gcc/pic32mx/4.5.1/../../../../pic32mx/lib/size\libc.a(_fputc_simple.o)
 .bss           0x00000000        0x0 c:/program files (x86)/microchip/xc32/v1.10/bin/../lib/gcc/pic32mx/4.5.1/../../../../pic32mx/lib/size\libc.a(_fputc_simple.o)
 .reginfo       0x00000000       0x18 c:/program files (x86)/microchip/xc32/v1.10/bin/../lib/gcc/pic32mx/4.5.1/../../../../pic32mx/lib/size\libc.a(_fputc_simple.o)
 .pdr           0x00000000       0x20 c:/program files (x86)/microchip/xc32/v1.10/bin/../lib/gcc/pic32mx/4.5.1/../../../../pic32mx/lib/size\libc.a(_fputc_simple.o)
 .text          0x00000000        0x0 c:/program files (x86)/microchip/xc32/v1.10/bin/../lib/gcc/pic32mx/4.5.1/../../../../pic32mx/lib/size\libc.a(powersf.o)
 .data          0x00000000        0x0 c:/program files (x86)/microchip/xc32/v1.10/bin/../lib/gcc/pic32mx/4.5.1/../../../../pic32mx/lib/size\libc.a(powersf.o)
 .bss           0x00000000        0x0 c:/program files (x86)/microchip/xc32/v1.10/bin/../lib/gcc/pic32mx/4.5.1/../../../../pic32mx/lib/size\libc.a(powersf.o)
 .reginfo       0x00000000       0x18 c:/program files (x86)/microchip/xc32/v1.10/bin/../lib/gcc/pic32mx/4.5.1/../../../../pic32mx/lib/size\libc.a(powersf.o)
 .pdr           0x00000000        0x0 c:/program files (x86)/microchip/xc32/v1.10/bin/../lib/gcc/pic32mx/4.5.1/../../../../pic32mx/lib/size\libc.a(powersf.o)
 .text          0x00000000        0x0 c:/program files (x86)/microchip/xc32/v1.10/bin/../lib/gcc/pic32mx/4.5.1/../../../../pic32mx/lib/size\libc.a(_iob.o)
 .data          0x00000000       0xa0 c:/program files (x86)/microchip/xc32/v1.10/bin/../lib/gcc/pic32mx/4.5.1/../../../../pic32mx/lib/size\libc.a(_iob.o)
 .reginfo       0x00000000       0x18 c:/program files (x86)/microchip/xc32/v1.10/bin/../lib/gcc/pic32mx/4.5.1/../../../../pic32mx/lib/size\libc.a(_iob.o)
 .pdr           0x00000000        0x0 c:/program files (x86)/microchip/xc32/v1.10/bin/../lib/gcc/pic32mx/4.5.1/../../../../pic32mx/lib/size\libc.a(_iob.o)
 .sdata         0x00000000        0x4 c:/program files (x86)/microchip/xc32/v1.10/bin/../lib/gcc/pic32mx/4.5.1/../../../../pic32mx/lib/size\libc.a(_iob.o)
 .text          0x00000000        0x0 c:/program files (x86)/microchip/xc32/v1.10/bin/../lib/gcc/pic32mx/4.5.1/../../../../pic32mx/lib/size\libc.a(_flsbuf_simple.o)
 .data          0x00000000        0x0 c:/program files (x86)/microchip/xc32/v1.10/bin/../lib/gcc/pic32mx/4.5.1/../../../../pic32mx/lib/size\libc.a(_flsbuf_simple.o)
 .bss           0x00000000        0x0 c:/program files (x86)/microchip/xc32/v1.10/bin/../lib/gcc/pic32mx/4.5.1/../../../../pic32mx/lib/size\libc.a(_flsbuf_simple.o)
 .reginfo       0x00000000       0x18 c:/program files (x86)/microchip/xc32/v1.10/bin/../lib/gcc/pic32mx/4.5.1/../../../../pic32mx/lib/size\libc.a(_flsbuf_simple.o)
 .pdr           0x00000000       0x20 c:/program files (x86)/microchip/xc32/v1.10/bin/../lib/gcc/pic32mx/4.5.1/../../../../pic32mx/lib/size\libc.a(_flsbuf_simple.o)
 .text          0x00000000        0x0 c:/program files (x86)/microchip/xc32/v1.10/bin/../lib/gcc/pic32mx/4.5.1/../../../../pic32mx/lib/size\libpic32.a(sbrk.o)
 .data          0x00000000        0x0 c:/program files (x86)/microchip/xc32/v1.10/bin/../lib/gcc/pic32mx/4.5.1/../../../../pic32mx/lib/size\libpic32.a(sbrk.o)
 .reginfo       0x00000000       0x18 c:/program files (x86)/microchip/xc32/v1.10/bin/../lib/gcc/pic32mx/4.5.1/../../../../pic32mx/lib/size\libpic32.a(sbrk.o)
 .pdr           0x00000000       0xa0 c:/program files (x86)/microchip/xc32/v1.10/bin/../lib/gcc/pic32mx/4.5.1/../../../../pic32mx/lib/size\libpic32.a(sbrk.o)
 .text.getpagesize
                0x00000000        0x8 c:/program files (x86)/microchip/xc32/v1.10/bin/../lib/gcc/pic32mx/4.5.1/../../../../pic32mx/lib/size\libpic32.a(sbrk.o)
 .text          0x00000000        0x0 c:/program files (x86)/microchip/xc32/v1.10/bin/../lib/gcc/pic32mx/4.5.1/../../../../pic32mx/lib/size\libpic32.a(write.o)
 .data          0x00000000        0x0 c:/program files (x86)/microchip/xc32/v1.10/bin/../lib/gcc/pic32mx/4.5.1/../../../../pic32mx/lib/size\libpic32.a(write.o)
 .bss           0x00000000        0x0 c:/program files (x86)/microchip/xc32/v1.10/bin/../lib/gcc/pic32mx/4.5.1/../../../../pic32mx/lib/size\libpic32.a(write.o)
 .reginfo       0x00000000       0x18 c:/program files (x86)/microchip/xc32/v1.10/bin/../lib/gcc/pic32mx/4.5.1/../../../../pic32mx/lib/size\libpic32.a(write.o)
 .pdr           0x00000000       0x20 c:/program files (x86)/microchip/xc32/v1.10/bin/../lib/gcc/pic32mx/4.5.1/../../../../pic32mx/lib/size\libpic32.a(write.o)
 .text          0x00000000        0x0 c:/program files (x86)/microchip/xc32/v1.10/bin/../lib/gcc/pic32mx/4.5.1/../../../../pic32mx/lib/size\libpic32.a(_mon_putc.o)
 .data          0x00000000        0x0 c:/program files (x86)/microchip/xc32/v1.10/bin/../lib/gcc/pic32mx/4.5.1/../../../../pic32mx/lib/size\libpic32.a(_mon_putc.o)
 .bss           0x00000000        0x0 c:/program files (x86)/microchip/xc32/v1.10/bin/../lib/gcc/pic32mx/4.5.1/../../../../pic32mx/lib/size\libpic32.a(_mon_putc.o)
 .reginfo       0x00000000       0x18 c:/program files (x86)/microchip/xc32/v1.10/bin/../lib/gcc/pic32mx/4.5.1/../../../../pic32mx/lib/size\libpic32.a(_mon_putc.o)
 .pdr           0x00000000       0x20 c:/program files (x86)/microchip/xc32/v1.10/bin/../lib/gcc/pic32mx/4.5.1/../../../../pic32mx/lib/size\libpic32.a(_mon_putc.o)
 .text          0x00000000        0x0 c:/program files (x86)/microchip/xc32/v1.10/bin/../lib/gcc/pic32mx/4.5.1/../../../../pic32mx/lib/size\libpic32.a(xc32_uart.o)
 .data          0x00000000        0x0 c:/program files (x86)/microchip/xc32/v1.10/bin/../lib/gcc/pic32mx/4.5.1/../../../../pic32mx/lib/size\libpic32.a(xc32_uart.o)
 .bss           0x00000000        0x0 c:/program files (x86)/microchip/xc32/v1.10/bin/../lib/gcc/pic32mx/4.5.1/../../../../pic32mx/lib/size\libpic32.a(xc32_uart.o)
 .reginfo       0x00000000       0x18 c:/program files (x86)/microchip/xc32/v1.10/bin/../lib/gcc/pic32mx/4.5.1/../../../../pic32mx/lib/size\libpic32.a(xc32_uart.o)
 .pdr           0x00000000        0x0 c:/program files (x86)/microchip/xc32/v1.10/bin/../lib/gcc/pic32mx/4.5.1/../../../../pic32mx/lib/size\libpic32.a(xc32_uart.o)
 .data          0x00000000        0x0 c:/program files (x86)/microchip/xc32/v1.10/bin/../lib/gcc/pic32mx/4.5.1/../../../../pic32mx/lib/size\libm.a(fpmod32.o)
 .bss           0x00000000        0x0 c:/program files (x86)/microchip/xc32/v1.10/bin/../lib/gcc/pic32mx/4.5.1/../../../../pic32mx/lib/size\libm.a(fpmod32.o)
 .reginfo       0x00000000       0x18 c:/program files (x86)/microchip/xc32/v1.10/bin/../lib/gcc/pic32mx/4.5.1/../../../../pic32mx/lib/size\libm.a(fpmod32.o)
 .pdr           0x00000000        0x0 c:/program files (x86)/microchip/xc32/v1.10/bin/../lib/gcc/pic32mx/4.5.1/../../../../pic32mx/lib/size\libm.a(fpmod32.o)
 .data          0x00000000        0x0 c:/program files (x86)/microchip/xc32/v1.10/bin/../lib/gcc/pic32mx/4.5.1/../../../../pic32mx/lib/size\libm.a(fp32.o)
 .bss           0x00000000        0x0 c:/program files (x86)/microchip/xc32/v1.10/bin/../lib/gcc/pic32mx/4.5.1/../../../../pic32mx/lib/size\libm.a(fp32.o)
 .reginfo       0x00000000       0x18 c:/program files (x86)/microchip/xc32/v1.10/bin/../lib/gcc/pic32mx/4.5.1/../../../../pic32mx/lib/size\libm.a(fp32.o)
 .pdr           0x00000000        0x0 c:/program files (x86)/microchip/xc32/v1.10/bin/../lib/gcc/pic32mx/4.5.1/../../../../pic32mx/lib/size\libm.a(fp32.o)
 .text          0x00000000        0x0 c:/program files (x86)/microchip/xc32/v1.10/bin/../lib/gcc/pic32mx/4.5.1/../../../../pic32mx/lib/size\libe.a(_floatdisf.o)
 .data          0x00000000        0x0 c:/program files (x86)/microchip/xc32/v1.10/bin/../lib/gcc/pic32mx/4.5.1/../../../../pic32mx/lib/size\libe.a(_floatdisf.o)
 .bss           0x00000000        0x0 c:/program files (x86)/microchip/xc32/v1.10/bin/../lib/gcc/pic32mx/4.5.1/../../../../pic32mx/lib/size\libe.a(_floatdisf.o)
 .reginfo       0x00000000       0x18 c:/program files (x86)/microchip/xc32/v1.10/bin/../lib/gcc/pic32mx/4.5.1/../../../../pic32mx/lib/size\libe.a(_floatdisf.o)
 .pdr           0x00000000       0x20 c:/program files (x86)/microchip/xc32/v1.10/bin/../lib/gcc/pic32mx/4.5.1/../../../../pic32mx/lib/size\libe.a(_floatdisf.o)
 .data          0x00000000        0x0 c:/program files (x86)/microchip/xc32/v1.10/bin/../lib/gcc/pic32mx/4.5.1/size\libgcc.a(_lshrdi3.o)
 .bss           0x00000000        0x0 c:/program files (x86)/microchip/xc32/v1.10/bin/../lib/gcc/pic32mx/4.5.1/size\libgcc.a(_lshrdi3.o)
 .reginfo       0x00000000       0x18 c:/program files (x86)/microchip/xc32/v1.10/bin/../lib/gcc/pic32mx/4.5.1/size\libgcc.a(_lshrdi3.o)
 .pdr           0x00000000       0x20 c:/program files (x86)/microchip/xc32/v1.10/bin/../lib/gcc/pic32mx/4.5.1/size\libgcc.a(_lshrdi3.o)
 .data          0x00000000        0x0 c:/program files (x86)/microchip/xc32/v1.10/bin/../lib/gcc/pic32mx/4.5.1/size\libgcc.a(_floatundisf.o)
 .bss           0x00000000        0x0 c:/program files (x86)/microchip/xc32/v1.10/bin/../lib/gcc/pic32mx/4.5.1/size\libgcc.a(_floatundisf.o)
 .reginfo       0x00000000       0x18 c:/program files (x86)/microchip/xc32/v1.10/bin/../lib/gcc/pic32mx/4.5.1/size\libgcc.a(_floatundisf.o)
 .pdr           0x00000000       0x20 c:/program files (x86)/microchip/xc32/v1.10/bin/../lib/gcc/pic32mx/4.5.1/size\libgcc.a(_floatundisf.o)
 .data          0x00000000        0x0 c:/program files (x86)/microchip/xc32/v1.10/bin/../lib/gcc/pic32mx/4.5.1/size\libgcc.a(_umoddi3.o)
 .bss           0x00000000        0x0 c:/program files (x86)/microchip/xc32/v1.10/bin/../lib/gcc/pic32mx/4.5.1/size\libgcc.a(_umoddi3.o)
 .reginfo       0x00000000       0x18 c:/program files (x86)/microchip/xc32/v1.10/bin/../lib/gcc/pic32mx/4.5.1/size\libgcc.a(_umoddi3.o)
 .pdr           0x00000000       0x20 c:/program files (x86)/microchip/xc32/v1.10/bin/../lib/gcc/pic32mx/4.5.1/size\libgcc.a(_umoddi3.o)
 .data          0x00000000        0x0 c:/program files (x86)/microchip/xc32/v1.10/bin/../lib/gcc/pic32mx/4.5.1/size\libgcc.a(floatunsisf.o)
 .bss           0x00000000        0x0 c:/program files (x86)/microchip/xc32/v1.10/bin/../lib/gcc/pic32mx/4.5.1/size\libgcc.a(floatunsisf.o)
 .reginfo       0x00000000       0x18 c:/program files (x86)/microchip/xc32/v1.10/bin/../lib/gcc/pic32mx/4.5.1/size\libgcc.a(floatunsisf.o)
 .pdr           0x00000000       0x20 c:/program files (x86)/microchip/xc32/v1.10/bin/../lib/gcc/pic32mx/4.5.1/size\libgcc.a(floatunsisf.o)

Memory Configuration

Name             Origin             Length             Attributes
kseg0_program_mem 0x9d000000         0x00080000         xr
kseg0_boot_mem   0x9fc00490         0x00000970
exception_mem    0x9fc01000         0x00001000
kseg1_boot_mem   0xbfc00000         0x00000490
debug_exec_mem   0xbfc02000         0x00000ff0
config3          0xbfc02ff0         0x00000004
config2          0xbfc02ff4         0x00000004
config1          0xbfc02ff8         0x00000004
config0          0xbfc02ffc         0x00000004
kseg1_data_mem   0xa0000000         0x00020000         w !x
sfrs             0xbf800000         0x00100000
configsfrs       0xbfc02ff0         0x00000010
*default*        0x00000000         0xffffffff

Linker script and memory map

LOAD c:/program files (x86)/microchip/xc32/v1.10/bin/../lib/gcc/pic32mx/4.5.1/../../../../pic32mx/lib/size/crt0.o
LOAD build/default/production/_ext/1293749816/bsp.o
LOAD build/default/production/_ext/101875047/hashes.o
LOAD build/default/production/_ext/101875047/lfsr.o
LOAD build/default/production/_ext/101875047/big_int.o
LOAD build/default/production/_ext/101875047/big_int_helper_c32.o
LOAD build/default/production/_ext/101875047/helpers.o
LOAD build/default/production/_ext/1472/berkeley_tcp_client_demo.o
LOAD build/default/production/_ext/1472/berkeley_tcp_server_demo.o
LOAD build/default/production/_ext/1472/berkeley_udp_client_demo.o
LOAD build/default/production/_ext/1472/generic_tcp_client.o
LOAD build/default/production/_ext/1472/generic_tcp_server.o
LOAD build/default/production/_ext/1472/ping_demo.o
LOAD build/default/production/_ext/1472/smtp_demo.o
LOAD build/default/production/_ext/365611741/system_services.o
LOAD build/default/production/_ext/365611741/system_debug.o
LOAD build/default/production/_ext/365611741/system_random.o
LOAD build/default/production/_ext/365611741/system_command.o
LOAD build/default/production/_ext/365611741/system_userio.o
LOAD build/default/production/_ext/97638081/sys_fs.o
LOAD build/default/production/_ext/97638081/mpfs2.o
LOAD build/default/production/_ext/792872985/usart.o
LOAD build/default/production/_ext/792872985/lcd.o
LOAD build/default/production/_ext/792872985/drv_spi.o
LOAD build/default/production/_ext/792872985/db_appio.o
LOAD build/default/production/_ext/792872985/spi_ram.o
LOAD build/default/production/_ext/792872985/spi_eeprom.o
LOAD build/default/production/_ext/792872985/spi_flash.o
LOAD build/default/production/_ext/792872985/drv_media.o
LOAD build/default/production/_ext/427700826/tcpip_announce.o
LOAD build/default/production/_ext/427700826/http2.o
LOAD build/default/production/_ext/427700826/arcfour.o
LOAD build/default/production/_ext/427700826/arp.o
LOAD build/default/production/_ext/427700826/berkeley_api.o
LOAD build/default/production/_ext/427700826/dhcp.o
LOAD build/default/production/_ext/427700826/dhcps.o
LOAD build/default/production/_ext/427700826/dns.o
LOAD build/default/production/_ext/427700826/dnss.o
LOAD build/default/production/_ext/427700826/dyn_dns.o
LOAD build/default/production/_ext/427700826/enc28_mac.o
LOAD build/default/production/_ext/427700826/enc28j60.o
LOAD build/default/production/_ext/427700826/encs24j600.o
LOAD build/default/production/_ext/427700826/encx24_mac.o
LOAD build/default/production/_ext/427700826/eth_pic32_ext_phy.o
LOAD build/default/production/_ext/427700826/eth_pic32_ext_phy_dp83848.o
LOAD build/default/production/_ext/427700826/eth_pic32_int_mac.o
LOAD build/default/production/_ext/427700826/ftp.o
LOAD build/default/production/_ext/427700826/hash_fnv.o
LOAD build/default/production/_ext/427700826/hash_tbl.o
LOAD build/default/production/_ext/427700826/icmp.o
LOAD build/default/production/_ext/427700826/icmpv6.o
LOAD build/default/production/_ext/427700826/ipv4.o
LOAD build/default/production/_ext/427700826/ipv6.o
LOAD build/default/production/_ext/427700826/mac_events_pic32.o
LOAD build/default/production/_ext/427700826/nbns.o
LOAD build/default/production/_ext/427700826/ndp.o
LOAD build/default/production/_ext/427700826/tcpip_reboot.o
LOAD build/default/production/_ext/427700826/rsa.o
LOAD build/default/production/_ext/427700826/smtp.o
LOAD build/default/production/_ext/427700826/snmp.o
LOAD build/default/production/_ext/427700826/snmpv3.o
LOAD build/default/production/_ext/427700826/snmpv3_usm.o
LOAD build/default/production/_ext/427700826/sntp.o
LOAD build/default/production/_ext/427700826/ssl.o
LOAD build/default/production/_ext/427700826/tcp.o
LOAD build/default/production/_ext/427700826/tcpip_heap_alloc.o
LOAD build/default/production/_ext/427700826/tcpip_storage.o
LOAD build/default/production/_ext/427700826/telnet.o
LOAD build/default/production/_ext/427700826/tftpc.o
LOAD build/default/production/_ext/427700826/udp.o
LOAD build/default/production/_ext/427700826/tcpip_mac_object.o
LOAD build/default/production/_ext/427700826/tcpip_manager.o
LOAD build/default/production/_ext/427700826/tcpip_helpers.o
LOAD build/default/production/_ext/427700826/tcpip_commands.o
LOAD build/default/production/_ext/427700826/iperf.o
LOAD build/default/production/_ext/427700826/tcpip_helper_c32.o
LOAD build/default/production/_ext/427700826/tcpip_notify.o
LOAD build/default/production/_ext/427700826/zero_conf_helper.o
LOAD build/default/production/_ext/427700826/zero_conf_link_local.o
LOAD build/default/production/_ext/427700826/zero_conf_multicast_dns.o
LOAD build/default/production/_ext/334706090/wf_tx_power.o
LOAD build/default/production/_ext/334706090/wf_connect.o
LOAD build/default/production/_ext/334706090/wf_connection_algorithm.o
LOAD build/default/production/_ext/334706090/wf_connection_manager.o
LOAD build/default/production/_ext/334706090/wf_connection_profile.o
LOAD build/default/production/_ext/334706090/wf_easy_config.o
LOAD build/default/production/_ext/334706090/wf_eint.o
LOAD build/default/production/_ext/334706090/wf_event_handler.o
LOAD build/default/production/_ext/334706090/wf_init.o
LOAD build/default/production/_ext/334706090/wf_power_save.o
LOAD build/default/production/_ext/334706090/wf_scan.o
LOAD build/default/production/_ext/334706090/wf_spi.o
LOAD build/default/production/_ext/334706090/mrf24w_mac_pic32.o
LOAD build/default/production/_ext/334706090/mrf24w_events.o
LOAD build/default/production/_ext/334706090/wf_debug_output.o
LOAD build/default/production/_ext/334706090/wf_commands.o
LOAD build/default/production/_ext/334706090/wf_pbkdf2.o
LOAD build/default/production/_ext/334706090/wf_driver_com_24g.o
LOAD build/default/production/_ext/334706090/wf_driver_raw_24g.o
LOAD build/default/production/_ext/334706090/wf_mac_24g.o
LOAD build/default/production/_ext/334706090/wf_mgmt_msg_24g.o
LOAD build/default/production/_ext/334706090/wf_param_msg_24g.o
LOAD build/default/production/_ext/334706090/wf_configData.o
LOAD build/default/production/_ext/1472/main_demo.o
LOAD build/default/production/_ext/1472/custom_snmp_app.o
LOAD build/default/production/_ext/1472/custom_ssl_cert.o
LOAD build/default/production/_ext/1472/mpfs_img2.o
LOAD build/default/production/_ext/1472/wf_config.o
LOAD build/default/production/_ext/1472/custom_http_app.o
LOAD build/default/production/_ext/1472/tcp6_demo_app.o
                0x00000001                __MPLAB_BUILD = 0x1
                0x00005208                _min_heap_size = 0x5208
                0x00000800                _min_stack_size = 0x800
                0x00000400                PROVIDE (_min_stack_size, 0x400)
LOAD c:/program files (x86)/microchip/xc32/v1.10/bin/../lib/gcc/pic32mx/4.5.1/../../../../pic32mx/lib/./proc/32MX795F512L\processor.o
START GROUP
LOAD c:/program files (x86)/microchip/xc32/v1.10/bin/../lib/gcc/pic32mx/4.5.1/../../../../pic32mx/lib/size\libmchp_peripheral.a
END GROUP
START GROUP
LOAD c:/program files (x86)/microchip/xc32/v1.10/bin/../lib/gcc/pic32mx/4.5.1/../../../../pic32mx/lib/size\libmchp_peripheral_32MX795F512L.a
END GROUP
                0x00000001                PROVIDE (_vector_spacing, 0x1)
                0x9fc01000                _ebase_address = 0x9fc01000
                0xbfc00000                _RESET_ADDR = 0xbfc00000
                0xbfc00380                _BEV_EXCPT_ADDR = 0xbfc00380
                0xbfc00480                _DBG_EXCPT_ADDR = 0xbfc00480
                0xbfc02000                _DBG_CODE_ADDR = 0xbfc02000
                0x00000ff0                _DBG_CODE_SIZE = 0xff0
                0x9fc01180                _GEN_EXCPT_ADDR = (_ebase_address + 0x180)

.config_BFC02FF0
 *(.config_BFC02FF0)

.config_BFC02FF4
                0xbfc02ff4        0x4
 *(.config_BFC02FF4)
 .config_BFC02FF4
                0xbfc02ff4        0x4 build/default/production/_ext/1293749816/bsp.o

.config_BFC02FF8
                0xbfc02ff8        0x4
 *(.config_BFC02FF8)
 .config_BFC02FF8
                0xbfc02ff8        0x4 build/default/production/_ext/1293749816/bsp.o

.config_BFC02FFC
                0xbfc02ffc        0x4
 *(.config_BFC02FFC)
 .config_BFC02FFC
                0xbfc02ffc        0x4 build/default/production/_ext/1293749816/bsp.o
                0xbfc02000                PROVIDE (_DBG_CODE_ADDR, 0xbfc02000)
                0x00000ff0                PROVIDE (_DBG_CODE_SIZE, 0xff0)

.reset          0xbfc00000      0x1f4
 *(.reset)
 .reset         0xbfc00000       0x10 c:/program files (x86)/microchip/xc32/v1.10/bin/../lib/gcc/pic32mx/4.5.1/../../../../pic32mx/lib/size/crt0.o
                0xbfc00000                _reset
 *(.reset.startup)
 .reset.startup
                0xbfc00010      0x1e4 c:/program files (x86)/microchip/xc32/v1.10/bin/../lib/gcc/pic32mx/4.5.1/../../../../pic32mx/lib/size/crt0.o

.bev_excpt      0xbfc00380       0x10
 *(.bev_handler)
 .bev_handler   0xbfc00380       0x10 c:/program files (x86)/microchip/xc32/v1.10/bin/../lib/gcc/pic32mx/4.5.1/../../../../pic32mx/lib/size/crt0.o

.dbg_excpt      0xbfc00480        0x0
                0xbfc00480                . = (. + DEFINED (_DEBUGGER)?0x8:0x0)

.dbg_code       0xbfc02000        0x0
                0xbfc02000                . = (. + DEFINED (_DEBUGGER)?_DBG_CODE_SIZE:0x0)

.app_excpt      0x9fc01180       0x10
 *(.gen_handler)
 .gen_handler   0x9fc01180       0x10 c:/program files (x86)/microchip/xc32/v1.10/bin/../lib/gcc/pic32mx/4.5.1/../../../../pic32mx/lib/size/crt0.o

.vector_0       0x9fc01200        0x8
 *(.vector_0)
 .vector_0      0x9fc01200        0x8 build/default/production/_ext/365611741/system_services.o
                0x00000001                ASSERT (((_vector_spacing == 0x0) || (SIZEOF (.vector_0) <= (_vector_spacing << 0x5))), function at exception vector 0 too large)

.vector_1       0x9fc01220        0x0
 *(.vector_1)
                0x00000001                ASSERT (((_vector_spacing == 0x0) || (SIZEOF (.vector_1) <= (_vector_spacing << 0x5))), function at exception vector 1 too large)

.vector_2       0x9fc01240        0x0
 *(.vector_2)
                0x00000001                ASSERT (((_vector_spacing == 0x0) || (SIZEOF (.vector_2) <= (_vector_spacing << 0x5))), function at exception vector 2 too large)

.vector_3       0x9fc01260        0x0
 *(.vector_3)
                0x00000001                ASSERT (((_vector_spacing == 0x0) || (SIZEOF (.vector_3) <= (_vector_spacing << 0x5))), function at exception vector 3 too large)

.vector_4       0x9fc01280        0x0
 *(.vector_4)
                0x00000001                ASSERT (((_vector_spacing == 0x0) || (SIZEOF (.vector_4) <= (_vector_spacing << 0x5))), function at exception vector 4 too large)

.vector_5       0x9fc012a0        0x0
 *(.vector_5)
                0x00000001                ASSERT (((_vector_spacing == 0x0) || (SIZEOF (.vector_5) <= (_vector_spacing << 0x5))), function at exception vector 5 too large)

.vector_6       0x9fc012c0        0x0
 *(.vector_6)
                0x00000001                ASSERT (((_vector_spacing == 0x0) || (SIZEOF (.vector_6) <= (_vector_spacing << 0x5))), function at exception vector 6 too large)

.vector_7       0x9fc012e0        0x8
 *(.vector_7)
 .vector_7      0x9fc012e0        0x8 build/default/production/_ext/365611741/system_services.o
                0x00000001                ASSERT (((_vector_spacing == 0x0) || (SIZEOF (.vector_7) <= (_vector_spacing << 0x5))), function at exception vector 7 too large)

.vector_8       0x9fc01300        0x0
 *(.vector_8)
                0x00000001                ASSERT (((_vector_spacing == 0x0) || (SIZEOF (.vector_8) <= (_vector_spacing << 0x5))), function at exception vector 8 too large)

.vector_9       0x9fc01320        0x0
 *(.vector_9)
                0x00000001                ASSERT (((_vector_spacing == 0x0) || (SIZEOF (.vector_9) <= (_vector_spacing << 0x5))), function at exception vector 9 too large)

.vector_10      0x9fc01340        0x0
 *(.vector_10)
                0x00000001                ASSERT (((_vector_spacing == 0x0) || (SIZEOF (.vector_10) <= (_vector_spacing << 0x5))), function at exception vector 10 too large)

.vector_11      0x9fc01360        0x0
 *(.vector_11)
                0x00000001                ASSERT (((_vector_spacing == 0x0) || (SIZEOF (.vector_11) <= (_vector_spacing << 0x5))), function at exception vector 11 too large)

.vector_12      0x9fc01380        0x0
 *(.vector_12)
                0x00000001                ASSERT (((_vector_spacing == 0x0) || (SIZEOF (.vector_12) <= (_vector_spacing << 0x5))), function at exception vector 12 too large)

.vector_13      0x9fc013a0        0x0
 *(.vector_13)
                0x00000001                ASSERT (((_vector_spacing == 0x0) || (SIZEOF (.vector_13) <= (_vector_spacing << 0x5))), function at exception vector 13 too large)

.vector_14      0x9fc013c0        0x0
 *(.vector_14)
                0x00000001                ASSERT (((_vector_spacing == 0x0) || (SIZEOF (.vector_14) <= (_vector_spacing << 0x5))), function at exception vector 14 too large)

.vector_15      0x9fc013e0        0x8
 *(.vector_15)
 .vector_15     0x9fc013e0        0x8 build/default/production/_ext/365611741/system_services.o
                0x00000001                ASSERT (((_vector_spacing == 0x0) || (SIZEOF (.vector_15) <= (_vector_spacing << 0x5))), function at exception vector 15 too large)

.vector_16      0x9fc01400        0x0
 *(.vector_16)
                0x00000001                ASSERT (((_vector_spacing == 0x0) || (SIZEOF (.vector_16) <= (_vector_spacing << 0x5))), function at exception vector 16 too large)

.vector_17      0x9fc01420        0x0
 *(.vector_17)
                0x00000001                ASSERT (((_vector_spacing == 0x0) || (SIZEOF (.vector_17) <= (_vector_spacing << 0x5))), function at exception vector 17 too large)

.vector_18      0x9fc01440        0x0
 *(.vector_18)
                0x00000001                ASSERT (((_vector_spacing == 0x0) || (SIZEOF (.vector_18) <= (_vector_spacing << 0x5))), function at exception vector 18 too large)

.vector_19      0x9fc01460        0x0
 *(.vector_19)
                0x00000001                ASSERT (((_vector_spacing == 0x0) || (SIZEOF (.vector_19) <= (_vector_spacing << 0x5))), function at exception vector 19 too large)

.vector_20      0x9fc01480        0x0
 *(.vector_20)
                0x00000001                ASSERT (((_vector_spacing == 0x0) || (SIZEOF (.vector_20) <= (_vector_spacing << 0x5))), function at exception vector 20 too large)

.vector_21      0x9fc014a0        0x0
 *(.vector_21)
                0x00000001                ASSERT (((_vector_spacing == 0x0) || (SIZEOF (.vector_21) <= (_vector_spacing << 0x5))), function at exception vector 21 too large)

.vector_22      0x9fc014c0        0x0
 *(.vector_22)
                0x00000001                ASSERT (((_vector_spacing == 0x0) || (SIZEOF (.vector_22) <= (_vector_spacing << 0x5))), function at exception vector 22 too large)

.vector_23      0x9fc014e0        0x0
 *(.vector_23)
                0x00000001                ASSERT (((_vector_spacing == 0x0) || (SIZEOF (.vector_23) <= (_vector_spacing << 0x5))), function at exception vector 23 too large)

.vector_24      0x9fc01500        0x0
 *(.vector_24)
                0x00000001                ASSERT (((_vector_spacing == 0x0) || (SIZEOF (.vector_24) <= (_vector_spacing << 0x5))), function at exception vector 24 too large)

.vector_25      0x9fc01520        0x0
 *(.vector_25)
                0x00000001                ASSERT (((_vector_spacing == 0x0) || (SIZEOF (.vector_25) <= (_vector_spacing << 0x5))), function at exception vector 25 too large)

.vector_26      0x9fc01540        0x8
 *(.vector_26)
 .vector_26     0x9fc01540        0x8 build/default/production/_ext/365611741/system_services.o
                0x00000001                ASSERT (((_vector_spacing == 0x0) || (SIZEOF (.vector_26) <= (_vector_spacing << 0x5))), function at exception vector 26 too large)

.vector_27      0x9fc01560        0x0
 *(.vector_27)
                0x00000001                ASSERT (((_vector_spacing == 0x0) || (SIZEOF (.vector_27) <= (_vector_spacing << 0x5))), function at exception vector 27 too large)

.vector_28      0x9fc01580        0x0
 *(.vector_28)
                0x00000001                ASSERT (((_vector_spacing == 0x0) || (SIZEOF (.vector_28) <= (_vector_spacing << 0x5))), function at exception vector 28 too large)

.vector_29      0x9fc015a0        0x0
 *(.vector_29)
                0x00000001                ASSERT (((_vector_spacing == 0x0) || (SIZEOF (.vector_29) <= (_vector_spacing << 0x5))), function at exception vector 29 too large)

.vector_30      0x9fc015c0        0x0
 *(.vector_30)
                0x00000001                ASSERT (((_vector_spacing == 0x0) || (SIZEOF (.vector_30) <= (_vector_spacing << 0x5))), function at exception vector 30 too large)

.vector_31      0x9fc015e0        0x0
 *(.vector_31)
                0x00000001                ASSERT (((_vector_spacing == 0x0) || (SIZEOF (.vector_31) <= (_vector_spacing << 0x5))), function at exception vector 31 too large)

.vector_32      0x9fc01600        0x0
 *(.vector_32)
                0x00000001                ASSERT (((_vector_spacing == 0x0) || (SIZEOF (.vector_32) <= (_vector_spacing << 0x5))), function at exception vector 32 too large)

.vector_33      0x9fc01620        0x0
 *(.vector_33)
                0x00000001                ASSERT (((_vector_spacing == 0x0) || (SIZEOF (.vector_33) <= (_vector_spacing << 0x5))), function at exception vector 33 too large)

.vector_34      0x9fc01640        0x0
 *(.vector_34)
                0x00000001                ASSERT (((_vector_spacing == 0x0) || (SIZEOF (.vector_34) <= (_vector_spacing << 0x5))), function at exception vector 34 too large)

.vector_35      0x9fc01660        0x0
 *(.vector_35)
                0x00000001                ASSERT (((_vector_spacing == 0x0) || (SIZEOF (.vector_35) <= (_vector_spacing << 0x5))), function at exception vector 35 too large)

.vector_36      0x9fc01680        0x0
 *(.vector_36)
                0x00000001                ASSERT (((_vector_spacing == 0x0) || (SIZEOF (.vector_36) <= (_vector_spacing << 0x5))), function at exception vector 36 too large)

.vector_37      0x9fc016a0        0x0
 *(.vector_37)
                0x00000001                ASSERT (((_vector_spacing == 0x0) || (SIZEOF (.vector_37) <= (_vector_spacing << 0x5))), function at exception vector 37 too large)

.vector_38      0x9fc016c0        0x0
 *(.vector_38)
                0x00000001                ASSERT (((_vector_spacing == 0x0) || (SIZEOF (.vector_38) <= (_vector_spacing << 0x5))), function at exception vector 38 too large)

.vector_39      0x9fc016e0        0x0
 *(.vector_39)
                0x00000001                ASSERT (((_vector_spacing == 0x0) || (SIZEOF (.vector_39) <= (_vector_spacing << 0x5))), function at exception vector 39 too large)

.vector_40      0x9fc01700        0x0
 *(.vector_40)
                0x00000001                ASSERT (((_vector_spacing == 0x0) || (SIZEOF (.vector_40) <= (_vector_spacing << 0x5))), function at exception vector 40 too large)

.vector_41      0x9fc01720        0x0
 *(.vector_41)
                0x00000001                ASSERT (((_vector_spacing == 0x0) || (SIZEOF (.vector_41) <= (_vector_spacing << 0x5))), function at exception vector 41 too large)

.vector_42      0x9fc01740        0x0
 *(.vector_42)
                0x00000001                ASSERT (((_vector_spacing == 0x0) || (SIZEOF (.vector_42) <= (_vector_spacing << 0x5))), function at exception vector 42 too large)

.vector_43      0x9fc01760        0x0
 *(.vector_43)
                0x00000001                ASSERT (((_vector_spacing == 0x0) || (SIZEOF (.vector_43) <= (_vector_spacing << 0x5))), function at exception vector 43 too large)

.vector_44      0x9fc01780        0x0
 *(.vector_44)
                0x00000001                ASSERT (((_vector_spacing == 0x0) || (SIZEOF (.vector_44) <= (_vector_spacing << 0x5))), function at exception vector 44 too large)

.vector_45      0x9fc017a0        0x0
 *(.vector_45)
                0x00000001                ASSERT (((_vector_spacing == 0x0) || (SIZEOF (.vector_45) <= (_vector_spacing << 0x5))), function at exception vector 45 too large)

.vector_46      0x9fc017c0        0x0
 *(.vector_46)
                0x00000001                ASSERT (((_vector_spacing == 0x0) || (SIZEOF (.vector_46) <= (_vector_spacing << 0x5))), function at exception vector 46 too large)

.vector_47      0x9fc017e0        0x0
 *(.vector_47)
                0x00000001                ASSERT (((_vector_spacing == 0x0) || (SIZEOF (.vector_47) <= (_vector_spacing << 0x5))), function at exception vector 47 too large)

.vector_48      0x9fc01800        0x0
 *(.vector_48)
                0x00000001                ASSERT (((_vector_spacing == 0x0) || (SIZEOF (.vector_48) <= (_vector_spacing << 0x5))), function at exception vector 48 too large)

.vector_49      0x9fc01820        0x0
 *(.vector_49)
                0x00000001                ASSERT (((_vector_spacing == 0x0) || (SIZEOF (.vector_49) <= (_vector_spacing << 0x5))), function at exception vector 49 too large)

.vector_50      0x9fc01840        0x0
 *(.vector_50)
                0x00000001                ASSERT (((_vector_spacing == 0x0) || (SIZEOF (.vector_50) <= (_vector_spacing << 0x5))), function at exception vector 50 too large)

.vector_51      0x9fc01860        0x0
 *(.vector_51)
                0x00000001                ASSERT (((_vector_spacing == 0x0) || (SIZEOF (.vector_51) <= (_vector_spacing << 0x5))), function at exception vector 51 too large)

.vector_52      0x9fc01880        0x0
 *(.vector_52)
                0x00000001                ASSERT (((_vector_spacing == 0x0) || (SIZEOF (.vector_52) <= (_vector_spacing << 0x5))), function at exception vector 52 too large)

.vector_53      0x9fc018a0        0x0
 *(.vector_53)
                0x00000001                ASSERT (((_vector_spacing == 0x0) || (SIZEOF (.vector_53) <= (_vector_spacing << 0x5))), function at exception vector 53 too large)

.vector_54      0x9fc018c0        0x0
 *(.vector_54)
                0x00000001                ASSERT (((_vector_spacing == 0x0) || (SIZEOF (.vector_54) <= (_vector_spacing << 0x5))), function at exception vector 54 too large)

.vector_55      0x9fc018e0        0x0
 *(.vector_55)
                0x00000001                ASSERT (((_vector_spacing == 0x0) || (SIZEOF (.vector_55) <= (_vector_spacing << 0x5))), function at exception vector 55 too large)

.vector_56      0x9fc01900        0x0
 *(.vector_56)
                0x00000001                ASSERT (((_vector_spacing == 0x0) || (SIZEOF (.vector_56) <= (_vector_spacing << 0x5))), function at exception vector 56 too large)

.vector_57      0x9fc01920        0x0
 *(.vector_57)
                0x00000001                ASSERT (((_vector_spacing == 0x0) || (SIZEOF (.vector_57) <= (_vector_spacing << 0x5))), function at exception vector 57 too large)

.vector_58      0x9fc01940        0x0
 *(.vector_58)
                0x00000001                ASSERT (((_vector_spacing == 0x0) || (SIZEOF (.vector_58) <= (_vector_spacing << 0x5))), function at exception vector 58 too large)

.vector_59      0x9fc01960        0x0
 *(.vector_59)
                0x00000001                ASSERT (((_vector_spacing == 0x0) || (SIZEOF (.vector_59) <= (_vector_spacing << 0x5))), function at exception vector 59 too large)

.vector_60      0x9fc01980        0x0
 *(.vector_60)
                0x00000001                ASSERT (((_vector_spacing == 0x0) || (SIZEOF (.vector_60) <= (_vector_spacing << 0x5))), function at exception vector 60 too large)

.vector_61      0x9fc019a0        0x0
 *(.vector_61)
                0x00000001                ASSERT (((_vector_spacing == 0x0) || (SIZEOF (.vector_61) <= (_vector_spacing << 0x5))), function at exception vector 61 too large)

.vector_62      0x9fc019c0        0x0
 *(.vector_62)
                0x00000001                ASSERT (((_vector_spacing == 0x0) || (SIZEOF (.vector_62) <= (_vector_spacing << 0x5))), function at exception vector 62 too large)

.vector_63      0x9fc019e0        0x0
 *(.vector_63)
                0x00000001                ASSERT (((_vector_spacing == 0x0) || (SIZEOF (.vector_63) <= (_vector_spacing << 0x5))), function at exception vector 63 too large)

.startup
 *(.startup)

.text           0x9d000000        0x0
 *(.stub .gnu.linkonce.t.*)
 *(.text.*personality*)
 *(.mips16.fn.*)
 *(.mips16.call.*)
 *(.gnu.warning)
                0x9d000000                . = ALIGN (0x4)

.init           0x9d000000        0x0
 *crti.o(.init)
 *crtbegin.o(.init)
 *(EXCLUDE_FILE(*crtn.o *crtend?.o *crtend.o) .init)
 *crtend.o(.init)
 *crtn.o(.init)
                0x9d000000                . = ALIGN (0x4)

.fini           0x9d000000        0x0
 *(.fini)
                0x9d000000                . = ALIGN (0x4)

.preinit_array  0x9d000000        0x0
                0x9d000000                PROVIDE (__preinit_array_start, .)
 *(.preinit_array)
                0x9d000000                PROVIDE (__preinit_array_end, .)
                0x9d000000                . = ALIGN (0x4)

.init_array     0x9d000000        0x0
                0x9d000000                PROVIDE (__init_array_start, .)
 *(SORT(.init_array.*))
 *(.init_array)
                0x9d000000                PROVIDE (__init_array_end, .)
                0x9d000000                . = ALIGN (0x4)

.fini_array     0x9d000000        0x0
                0x9d000000                PROVIDE (__fini_array_start, .)
 *(SORT(.fini_array.*))
 *(.fini_array)
                0x9d000000                PROVIDE (__fini_array_end, .)
                0x9d000000                . = ALIGN (0x4)

.ctors          0x9d000000        0x0
 *crtbegin.o(.ctors)
 *crtbegin?.o(.ctors)
 *(EXCLUDE_FILE(*crtend?.o *crtend.o) .ctors)
 *(SORT(.ctors.*))
 *(.ctors)
                0x9d000000                . = ALIGN (0x4)

.dtors          0x9d000000        0x0
 *crtbegin.o(.dtors)
 *crtbegin?.o(.dtors)
 *(EXCLUDE_FILE(*crtend?.o *crtend.o) .dtors)
 *(SORT(.dtors.*))
 *(.dtors)
                0x9d000000                . = ALIGN (0x4)

.rodata         0x9d000000        0x0
 *(.gnu.linkonce.r.*)
 *(.rodata1)
                0x9d000000                . = ALIGN (0x4)

.sdata2         0x9fc00490        0x0
 *(.sdata2 .sdata2.* .gnu.linkonce.s2.*)
                0x9fc00490                . = ALIGN (0x4)

.sbss2          0x9fc00490        0x0
 *(.sbss2 .sbss2.* .gnu.linkonce.sb2.*)
                0x9fc00490                . = ALIGN (0x4)

.eh_frame_hdr
 *(.eh_frame_hdr)
                0x9fc00490                . = ALIGN (0x4)

.eh_frame
 *(.eh_frame)
                0x9fc00490                . = ALIGN (0x4)

.gcc_except_table
 *(.gcc_except_table .gcc_except_table.*)
                0x9fc00490                . = ALIGN (0x4)

.dbg_data       0xa0000000        0x0
                0xa0000000                . = (. + DEFINED (_DEBUGGER)?0x200:0x0)

.jcr            0xa0000000        0x0
 *(.jcr)
                0xa0000000                . = ALIGN (0x4)

.eh_frame       0xa0000000       0x30
 *(.eh_frame)
 .eh_frame      0xa0000000       0x20 c:/program files (x86)/microchip/xc32/v1.10/bin/../lib/gcc/pic32mx/4.5.1/size\libgcc.a(_udivdi3.o)
 .eh_frame      0xa0000020       0x10 c:/program files (x86)/microchip/xc32/v1.10/bin/../lib/gcc/pic32mx/4.5.1/size\libgcc.a(_umoddi3.o)
                0xa0000030                . = ALIGN (0x4)

.gcc_except_table
 *(.gcc_except_table .gcc_except_table.*)
                0xa0000030                . = ALIGN (0x4)

.persist        0xa0000030        0x0
                0xa0000030                _persist_begin = .
 *(.persist .persist.*)
 *(.pbss .pbss.*)
                0xa0000030                . = ALIGN (0x4)
                0xa0000030                _persist_end = .

.data           0xa0000030        0x0
 *(.gnu.linkonce.d.*)
 *(.data1)
                0xa0000030                . = ALIGN (0x4)
                0xa0000030                . = .
                0xa0008020                _gp = (ALIGN (0x10) + 0x7ff0)

.got            0xa0000030        0x0
 *(.got.plt)
 *(.got)
                0xa0000030                . = ALIGN (0x4)

.sdata          0xa0000030      0x1e8
                0xa0000030                _sdata_begin = .
 *(.sdata .sdata.* .gnu.linkonce.s.*)
 .sdata         0xa0000030        0x4 build/default/production/_ext/101875047/lfsr.o
 .sdata         0xa0000034       0x10 build/default/production/_ext/365611741/system_services.o
                0xa0000034                MEDIA_STORAGE_PARTITION_TABLE
 .sdata         0xa0000044       0x60 build/default/production/_ext/365611741/system_debug.o
 .sdata         0xa00000a4       0x1c build/default/production/_ext/792872985/usart.o
                0xa00000a4                _usart_cdev_obj
 .sdata         0xa00000c0       0x2c build/default/production/_ext/792872985/drv_media.o
 .sdata         0xa00000ec        0x8 build/default/production/_ext/427700826/arp.o
 .sdata         0xa00000f4        0x2 build/default/production/_ext/427700826/dns.o
 *fill*         0xa00000f6        0x2 00
 .sdata         0xa00000f8        0x4 build/default/production/_ext/427700826/tcpip_heap_alloc.o
 .sdata         0xa00000fc        0x1 build/default/production/_ext/334706090/wf_connection_algorithm.o
 .sdata         0xa00000fd        0x1 build/default/production/_ext/334706090/wf_power_save.o
 *fill*         0xa00000fe        0x2 00
 .sdata         0xa0000100        0xc build/default/production/_ext/334706090/mrf24w_mac_pic32.o
 .sdata         0xa000010c      0x100 build/default/production/_ext/334706090/wf_debug_output.o
                0xa000010c                connectionLostStrings
                0xa0000124                wpsState
                0xa0000160                wpsConfigErr
 .sdata         0xa000020c        0x4 build/default/production/_ext/334706090/wf_configData.o
                0xa000020c                p_wifi_ConfigData
 .sdata         0xa0000210        0x2 build/default/production/_ext/1472/tcp6_demo_app.o
                0xa0000210                mySocket
 *fill*         0xa0000212        0x2 00
 .sdata         0xa0000214        0x4 c:/program files (x86)/microchip/xc32/v1.10/bin/../lib/gcc/pic32mx/4.5.1/../../../../pic32mx/lib/size\libpic32.a(xc32_uart.o)
                0xa0000214                __XC_UART
                0xa0000218                . = ALIGN (0x4)
                0xa0000218                _sdata_end = .

.lit8
 *(.lit8)

.lit4
 *(.lit4)
                0xa0000218                . = ALIGN (0x4)
                0xa0000218                _data_end = .
                0xa0000218                _bss_begin = .

.sbss           0xa0000218      0x410
                0xa0000218                _sbss_begin = .
 *(.dynsbss)
 *(.sbss .sbss.* .gnu.linkonce.sb.*)
 .sbss          0xa0000218       0x34 build/default/production/_ext/365611741/system_services.o
                0xa0000218                _SystemTickCount
                0xa000021c                _SystemTickResolution
 .sbss          0xa000024c        0x8 build/default/production/_ext/365611741/system_debug.o
 .sbss          0xa0000254       0x18 build/default/production/_ext/365611741/system_random.o
 .sbss          0xa000026c       0x5c build/default/production/_ext/365611741/system_command.o
 .sbss          0xa00002c8       0x30 build/default/production/_ext/365611741/system_userio.o
 .sbss          0xa00002f8       0x10 build/default/production/_ext/97638081/sys_fs.o
 .sbss          0xa0000308       0x24 build/default/production/_ext/97638081/mpfs2.o
 .sbss          0xa000032c       0x28 build/default/production/_ext/792872985/spi_eeprom.o
 .sbss          0xa0000354       0x34 build/default/production/_ext/792872985/drv_media.o
 .sbss          0xa0000388       0x1c build/default/production/_ext/427700826/tcpip_announce.o
 .sbss          0xa00003a4       0x14 build/default/production/_ext/427700826/http2.o
 .sbss          0xa00003b8       0x3c build/default/production/_ext/427700826/arp.o
 .sbss          0xa00003f4       0x20 build/default/production/_ext/427700826/dhcp.o
 .sbss          0xa0000414       0x3c build/default/production/_ext/427700826/dns.o
 .sbss          0xa0000450        0x8 build/default/production/_ext/427700826/icmp.o
 .sbss          0xa0000458       0x20 build/default/production/_ext/427700826/ipv4.o
                0xa0000468                ipv4QueuedPackets
 .sbss          0xa0000478        0xc build/default/production/_ext/427700826/nbns.o
 .sbss          0xa0000484       0x20 build/default/production/_ext/427700826/tcp.o
 .sbss          0xa00004a4       0x18 build/default/production/_ext/427700826/udp.o
                0xa00004a4                UDPSocketDcpt
 .sbss          0xa00004bc       0x3c build/default/production/_ext/427700826/tcpip_manager.o
 .sbss          0xa00004f8        0x1 build/default/production/_ext/334706090/wf_connection_manager.o
 .sbss          0xa00004f9        0x1 build/default/production/_ext/334706090/wf_connection_profile.o
 .sbss          0xa00004fa        0x2 build/default/production/_ext/334706090/wf_event_handler.o
                0xa00004fa                g_DhcpRenew
                0xa00004fb                g_asyncTaskFlags
 .sbss          0xa00004fc        0x3 build/default/production/_ext/334706090/wf_power_save.o
 .sbss          0xa00004ff        0x1 build/default/production/_ext/334706090/wf_spi.o
 .sbss          0xa0000500       0x18 build/default/production/_ext/334706090/mrf24w_events.o
 .sbss          0xa0000518        0x1 build/default/production/_ext/334706090/wf_debug_output.o
                0xa0000518                g_outputConnectionContext
 *fill*         0xa0000519        0x3 00
 .sbss          0xa000051c       0x14 build/default/production/_ext/334706090/wf_driver_com_24g.o
                0xa0000529                g_DhcpSuccessful
                0xa000052a                g_WiFiConnectionChanged
                0xa000052b                g_WiFiConnection
                0xa000052c                g_dhcpInProgress
 .sbss          0xa0000530        0x2 build/default/production/_ext/334706090/wf_driver_raw_24g.o
                0xa0000530                g_HostRAWDataPacketReceived
                0xa0000531                g_RawIndexPastEnd
 *fill*         0xa0000532        0x2 00
 .sbss          0xa0000534        0xc build/default/production/_ext/334706090/wf_mac_24g.o
 .sbss          0xa0000540        0x3 build/default/production/_ext/334706090/wf_mgmt_msg_24g.o
                0xa0000541                g_WaitingForMgmtResponse
 *fill*         0xa0000543        0x1 00
 .sbss          0xa0000544       0x1c build/default/production/_ext/1472/main_demo.o
                0xa0000544                stackNotifyCnt
                0xa0000548                stackTotEvents
                0xa000054c                mrf_txEvents
                0xa000054e                mrf_txEventInfo
                0xa0000550                mrf_mgmtEvents
                0xa0000552                mrf_mgmtEventInfo
                0xa0000554                mrf_EventCnt
 .sbss          0xa0000560        0x2 build/default/production/_ext/1472/custom_http_app.o
 *fill*         0xa0000562        0x2 00
 .sbss          0xa0000564       0x10 build/default/production/_ext/1472/tcp6_demo_app.o
                0xa0000564                nAttempts
                0xa0000568                httpTransactionIndex
                0xa000056c                WaitDispatch2Timer
                0xa0000570                smMyDemoAppTasks
 .sbss          0xa0000574        0x4 c:/program files (x86)/microchip/xc32/v1.10/bin/../lib/gcc/pic32mx/4.5.1/../../../../pic32mx/lib/size\libpic32.a(errno.o)
                0xa0000574                errno
 .sbss          0xa0000578       0x10 c:/program files (x86)/microchip/xc32/v1.10/bin/../lib/gcc/pic32mx/4.5.1/../../../../pic32mx/lib/size\libc.a(malloc.o)
                0xa0000578                __allocp
                0xa000057c                __alloct
                0xa0000580                __allocx
 .sbss          0xa0000588        0x1 c:/program files (x86)/microchip/xc32/v1.10/bin/../lib/gcc/pic32mx/4.5.1/../../../../pic32mx/lib/size\libc.a(_iob.o)
                0xa0000588                _outdone
 *fill*         0xa0000589        0x3 00
 .sbss          0xa000058c        0x8 c:/program files (x86)/microchip/xc32/v1.10/bin/../lib/gcc/pic32mx/4.5.1/../../../../pic32mx/lib/size\libpic32.a(sbrk.o)
                0xa000058c                _minbrk
                0xa0000590                _maxbrk
 *(.scommon)
 .scommon       0xa0000594       0x1e build/default/production/_ext/1472/ping_demo.o
                0xa0000594                pNetIf
                0xa0000598                pingCount
                0xa000059c                targetAddressIPv4
                0xa00005a0                pingTimer
                0xa00005a4                firstHopAddress
                0xa00005a8                targetHostName
                0xa00005ac                targetMACAddr
 *fill*         0xa00005b2        0x2 00
 .scommon       0xa00005b4        0x8 build/default/production/_ext/334706090/wf_event_handler.o
                0xa00005b4                g_softAPEvent
 .scommon       0xa00005bc        0x6 build/default/production/_ext/334706090/wf_power_save.o
                0xa00005bc                g_savedPsPollContext
 *fill*         0xa00005c2        0x2 00
 .scommon       0xa00005c4        0x4 build/default/production/_ext/334706090/wf_scan.o
                0xa00005c4                hMac_softap_connect
 .scommon       0xa00005c8        0x3 build/default/production/_ext/334706090/wf_commands.o
                0xa00005c8                iwconfigCb
 *fill*         0xa00005cb        0x1 00
 .scommon       0xa00005cc        0x3 build/default/production/_ext/334706090/wf_driver_com_24g.o
                0xa00005cc                RawMoveState
                0xa00005ce                g_powerSaveState
 *fill*         0xa00005cf        0x1 00
 .scommon       0xa00005d0        0x2 build/default/production/_ext/334706090/wf_driver_raw_24g.o
                0xa00005d0                RawWindowState
 *fill*         0xa00005d2        0x2 00
 .scommon       0xa00005d4        0xe build/default/production/_ext/334706090/wf_mac_24g.o
                0xa00005d4                g_gratArpContext
                0xa00005dc                g_pNetIf
                0xa00005e0                g_rxBufferLength
 *fill*         0xa00005e2        0x2 00
 .scommon       0xa00005e4        0x4 build/default/production/_ext/1472/main_demo.o
                0xa00005e4                stackNotifyHandle
 .scommon       0xa00005e8       0x40 build/default/production/_ext/1472/tcp6_demo_app.o
                0xa00005e8                myNetHandle
                0xa00005ec                mac_addr_ptr
                0xa00005f0                dnsRes
                0xa00005f4                HTTPReplyDelay
                0xa00005f8                TCPInBufPtr
                0xa00005fc                serverIP
                0xa0000600                i
                0xa0000604                mac_addr
                0xa000060c                clientTimer
                0xa0000610                TCPReadByte
                0xa0000614                j
                0xa0000618                TCPInBufferIndex
                0xa000061c                toggleLed
                0xa0000620                HTTPReplyLineCnt
                0xa0000624                TCPIsPutReadyCnt
                0xa0000626                serverPort
                0xa0000628                _sbss_end = .
                0xa0000628                . = ALIGN (0x4)

.bss            0xa0000628     0x1b68
 *(.dynbss)
 *(COMMON)
 COMMON         0xa0000628       0x40 build/default/production/_ext/101875047/hashes.o
                0xa0000628                lastBlock
 COMMON         0xa0000668       0x21 build/default/production/_ext/792872985/lcd.o
                0xa0000668                LCDText
 *fill*         0xa0000689        0x3 00
 COMMON         0xa000068c        0xa build/default/production/_ext/427700826/tcpip_manager.o
                0xa000068c                remoteNode
 *fill*         0xa0000696        0x2 00
 COMMON         0xa0000698       0x8a build/default/production/_ext/334706090/wf_configData.o
                0xa0000698                wifi_ConfigData
 *fill*         0xa0000722        0x2 00
 COMMON         0xa0000724     0x1a6c build/default/production/_ext/1472/tcp6_demo_app.o
                0xa0000724                myb64
                0xa00007a4                mySocketInfo
                0xa00007cc                httpTransaction
                0xa0000c7c                TCPInBuffer
                0xa0001c7c                mysrc
                0xa0001cfc                myResourceState
                0xa0001d60                temp
                0xa0001d80                mac_addr_string
                0xa0001d90                OutString
                0xa0001f90                TCPOutBuffer
                0xa0002190                . = ALIGN ((. != 0x0)?0x4:0x1)
                0xa0002190                . = ALIGN (0x4)
                0xa0002190                _end = .
                0xa0002190                _bss_end = .
                0x00020000                _bmxdudba_address = 0x20000
                0x00020000                _bmxdupba_address = 0x20000

/DISCARD/
 *(.pdr)
 *(.rel.dyn)
 *(.note.GNU-stack)
 *(.note.GNU-stack)
 *(.gnu_debuglink)
 *(.gnu.lto_*)
 *(.discard)

.gptab.sdata
 *(.gptab.data)
 *(.gptab.sdata)

.gptab.sbss
 *(.gptab.bss)
 *(.gptab.sbss)

.mdebug.abi32   0xa0002190        0x0
 *(.mdebug.abi32)
 .mdebug.abi32  0xa0002190        0x0 build/default/production/_ext/1293749816/bsp.o
 .mdebug.abi32  0xa0002190        0x0 build/default/production/_ext/101875047/hashes.o
 .mdebug.abi32  0xa0002190        0x0 build/default/production/_ext/101875047/lfsr.o
 .mdebug.abi32  0xa0002190        0x0 build/default/production/_ext/101875047/big_int.o
 .mdebug.abi32  0xa0002190        0x0 build/default/production/_ext/101875047/helpers.o
 .mdebug.abi32  0xa0002190        0x0 build/default/production/_ext/1472/berkeley_tcp_client_demo.o
 .mdebug.abi32  0xa0002190        0x0 build/default/production/_ext/1472/berkeley_tcp_server_demo.o
 .mdebug.abi32  0xa0002190        0x0 build/default/production/_ext/1472/berkeley_udp_client_demo.o
 .mdebug.abi32  0xa0002190        0x0 build/default/production/_ext/1472/generic_tcp_client.o
 .mdebug.abi32  0xa0002190        0x0 build/default/production/_ext/1472/generic_tcp_server.o
 .mdebug.abi32  0xa0002190        0x0 build/default/production/_ext/1472/ping_demo.o
 .mdebug.abi32  0xa0002190        0x0 build/default/production/_ext/1472/smtp_demo.o
 .mdebug.abi32  0xa0002190        0x0 build/default/production/_ext/365611741/system_services.o
 .mdebug.abi32  0xa0002190        0x0 build/default/production/_ext/365611741/system_debug.o
 .mdebug.abi32  0xa0002190        0x0 build/default/production/_ext/365611741/system_random.o
 .mdebug.abi32  0xa0002190        0x0 build/default/production/_ext/365611741/system_command.o
 .mdebug.abi32  0xa0002190        0x0 build/default/production/_ext/365611741/system_userio.o
 .mdebug.abi32  0xa0002190        0x0 build/default/production/_ext/97638081/sys_fs.o
 .mdebug.abi32  0xa0002190        0x0 build/default/production/_ext/97638081/mpfs2.o
 .mdebug.abi32  0xa0002190        0x0 build/default/production/_ext/792872985/usart.o
 .mdebug.abi32  0xa0002190        0x0 build/default/production/_ext/792872985/lcd.o
 .mdebug.abi32  0xa0002190        0x0 build/default/production/_ext/792872985/drv_spi.o
 .mdebug.abi32  0xa0002190        0x0 build/default/production/_ext/792872985/db_appio.o
 .mdebug.abi32  0xa0002190        0x0 build/default/production/_ext/792872985/spi_ram.o
 .mdebug.abi32  0xa0002190        0x0 build/default/production/_ext/792872985/spi_eeprom.o
 .mdebug.abi32  0xa0002190        0x0 build/default/production/_ext/792872985/spi_flash.o
 .mdebug.abi32  0xa0002190        0x0 build/default/production/_ext/792872985/drv_media.o
 .mdebug.abi32  0xa0002190        0x0 build/default/production/_ext/427700826/tcpip_announce.o
 .mdebug.abi32  0xa0002190        0x0 build/default/production/_ext/427700826/http2.o
 .mdebug.abi32  0xa0002190        0x0 build/default/production/_ext/427700826/arcfour.o
 .mdebug.abi32  0xa0002190        0x0 build/default/production/_ext/427700826/arp.o
 .mdebug.abi32  0xa0002190        0x0 build/default/production/_ext/427700826/berkeley_api.o
 .mdebug.abi32  0xa0002190        0x0 build/default/production/_ext/427700826/dhcp.o
 .mdebug.abi32  0xa0002190        0x0 build/default/production/_ext/427700826/dhcps.o
 .mdebug.abi32  0xa0002190        0x0 build/default/production/_ext/427700826/dns.o
 .mdebug.abi32  0xa0002190        0x0 build/default/production/_ext/427700826/dnss.o
 .mdebug.abi32  0xa0002190        0x0 build/default/production/_ext/427700826/dyn_dns.o
 .mdebug.abi32  0xa0002190        0x0 build/default/production/_ext/427700826/enc28_mac.o
 .mdebug.abi32  0xa0002190        0x0 build/default/production/_ext/427700826/enc28j60.o
 .mdebug.abi32  0xa0002190        0x0 build/default/production/_ext/427700826/encs24j600.o
 .mdebug.abi32  0xa0002190        0x0 build/default/production/_ext/427700826/encx24_mac.o
 .mdebug.abi32  0xa0002190        0x0 build/default/production/_ext/427700826/eth_pic32_ext_phy.o
 .mdebug.abi32  0xa0002190        0x0 build/default/production/_ext/427700826/eth_pic32_ext_phy_dp83848.o
 .mdebug.abi32  0xa0002190        0x0 build/default/production/_ext/427700826/eth_pic32_int_mac.o
 .mdebug.abi32  0xa0002190        0x0 build/default/production/_ext/427700826/ftp.o
 .mdebug.abi32  0xa0002190        0x0 build/default/production/_ext/427700826/hash_fnv.o
 .mdebug.abi32  0xa0002190        0x0 build/default/production/_ext/427700826/hash_tbl.o
 .mdebug.abi32  0xa0002190        0x0 build/default/production/_ext/427700826/icmp.o
 .mdebug.abi32  0xa0002190        0x0 build/default/production/_ext/427700826/icmpv6.o
 .mdebug.abi32  0xa0002190        0x0 build/default/production/_ext/427700826/ipv4.o
 .mdebug.abi32  0xa0002190        0x0 build/default/production/_ext/427700826/ipv6.o
 .mdebug.abi32  0xa0002190        0x0 build/default/production/_ext/427700826/mac_events_pic32.o
 .mdebug.abi32  0xa0002190        0x0 build/default/production/_ext/427700826/nbns.o
 .mdebug.abi32  0xa0002190        0x0 build/default/production/_ext/427700826/ndp.o
 .mdebug.abi32  0xa0002190        0x0 build/default/production/_ext/427700826/tcpip_reboot.o
 .mdebug.abi32  0xa0002190        0x0 build/default/production/_ext/427700826/rsa.o
 .mdebug.abi32  0xa0002190        0x0 build/default/production/_ext/427700826/smtp.o
 .mdebug.abi32  0xa0002190        0x0 build/default/production/_ext/427700826/snmp.o
 .mdebug.abi32  0xa0002190        0x0 build/default/production/_ext/427700826/snmpv3.o
 .mdebug.abi32  0xa0002190        0x0 build/default/production/_ext/427700826/snmpv3_usm.o
 .mdebug.abi32  0xa0002190        0x0 build/default/production/_ext/427700826/sntp.o
 .mdebug.abi32  0xa0002190        0x0 build/default/production/_ext/427700826/ssl.o
 .mdebug.abi32  0xa0002190        0x0 build/default/production/_ext/427700826/tcp.o
 .mdebug.abi32  0xa0002190        0x0 build/default/production/_ext/427700826/tcpip_heap_alloc.o
 .mdebug.abi32  0xa0002190        0x0 build/default/production/_ext/427700826/tcpip_storage.o
 .mdebug.abi32  0xa0002190        0x0 build/default/production/_ext/427700826/telnet.o
 .mdebug.abi32  0xa0002190        0x0 build/default/production/_ext/427700826/tftpc.o
 .mdebug.abi32  0xa0002190        0x0 build/default/production/_ext/427700826/udp.o
 .mdebug.abi32  0xa0002190        0x0 build/default/production/_ext/427700826/tcpip_mac_object.o
 .mdebug.abi32  0xa0002190        0x0 build/default/production/_ext/427700826/tcpip_manager.o
 .mdebug.abi32  0xa0002190        0x0 build/default/production/_ext/427700826/tcpip_helpers.o
 .mdebug.abi32  0xa0002190        0x0 build/default/production/_ext/427700826/tcpip_commands.o
 .mdebug.abi32  0xa0002190        0x0 build/default/production/_ext/427700826/iperf.o
 .mdebug.abi32  0xa0002190        0x0 build/default/production/_ext/427700826/tcpip_notify.o
 .mdebug.abi32  0xa0002190        0x0 build/default/production/_ext/427700826/zero_conf_helper.o
 .mdebug.abi32  0xa0002190        0x0 build/default/production/_ext/427700826/zero_conf_link_local.o
 .mdebug.abi32  0xa0002190        0x0 build/default/production/_ext/427700826/zero_conf_multicast_dns.o
 .mdebug.abi32  0xa0002190        0x0 build/default/production/_ext/334706090/wf_tx_power.o
 .mdebug.abi32  0xa0002190        0x0 build/default/production/_ext/334706090/wf_connect.o
 .mdebug.abi32  0xa0002190        0x0 build/default/production/_ext/334706090/wf_connection_algorithm.o
 .mdebug.abi32  0xa0002190        0x0 build/default/production/_ext/334706090/wf_connection_manager.o
 .mdebug.abi32  0xa0002190        0x0 build/default/production/_ext/334706090/wf_connection_profile.o
 .mdebug.abi32  0xa0002190        0x0 build/default/production/_ext/334706090/wf_easy_config.o
 .mdebug.abi32  0xa0002190        0x0 build/default/production/_ext/334706090/wf_eint.o
 .mdebug.abi32  0xa0002190        0x0 build/default/production/_ext/334706090/wf_event_handler.o
 .mdebug.abi32  0xa0002190        0x0 build/default/production/_ext/334706090/wf_init.o
 .mdebug.abi32  0xa0002190        0x0 build/default/production/_ext/334706090/wf_power_save.o
 .mdebug.abi32  0xa0002190        0x0 build/default/production/_ext/334706090/wf_scan.o
 .mdebug.abi32  0xa0002190        0x0 build/default/production/_ext/334706090/wf_spi.o
 .mdebug.abi32  0xa0002190        0x0 build/default/production/_ext/334706090/mrf24w_mac_pic32.o
 .mdebug.abi32  0xa0002190        0x0 build/default/production/_ext/334706090/mrf24w_events.o
 .mdebug.abi32  0xa0002190        0x0 build/default/production/_ext/334706090/wf_debug_output.o
 .mdebug.abi32  0xa0002190        0x0 build/default/production/_ext/334706090/wf_commands.o
 .mdebug.abi32  0xa0002190        0x0 build/default/production/_ext/334706090/wf_pbkdf2.o
 .mdebug.abi32  0xa0002190        0x0 build/default/production/_ext/334706090/wf_driver_com_24g.o
 .mdebug.abi32  0xa0002190        0x0 build/default/production/_ext/334706090/wf_driver_raw_24g.o
 .mdebug.abi32  0xa0002190        0x0 build/default/production/_ext/334706090/wf_mac_24g.o
 .mdebug.abi32  0xa0002190        0x0 build/default/production/_ext/334706090/wf_mgmt_msg_24g.o
 .mdebug.abi32  0xa0002190        0x0 build/default/production/_ext/334706090/wf_param_msg_24g.o
 .mdebug.abi32  0xa0002190        0x0 build/default/production/_ext/334706090/wf_configData.o
 .mdebug.abi32  0xa0002190        0x0 build/default/production/_ext/1472/main_demo.o
 .mdebug.abi32  0xa0002190        0x0 build/default/production/_ext/1472/custom_snmp_app.o
 .mdebug.abi32  0xa0002190        0x0 build/default/production/_ext/1472/custom_ssl_cert.o
 .mdebug.abi32  0xa0002190        0x0 build/default/production/_ext/1472/mpfs_img2.o
 .mdebug.abi32  0xa0002190        0x0 build/default/production/_ext/1472/wf_config.o
 .mdebug.abi32  0xa0002190        0x0 build/default/production/_ext/1472/custom_http_app.o
 .mdebug.abi32  0xa0002190        0x0 build/default/production/_ext/1472/tcp6_demo_app.o
 .mdebug.abi32  0xa0002190        0x0 c:/program files (x86)/microchip/xc32/v1.10/bin/../lib/gcc/pic32mx/4.5.1/../../../../pic32mx/lib/size\libmchp_peripheral.a(open_core_timer_lib.o)
 .mdebug.abi32  0xa0002190        0x0 c:/program files (x86)/microchip/xc32/v1.10/bin/../lib/gcc/pic32mx/4.5.1/../../../../pic32mx/lib/size\libmchp_peripheral_32MX795F512L.a(soft_reset_lib.o)
 .mdebug.abi32  0xa0002190        0x0 c:/program files (x86)/microchip/xc32/v1.10/bin/../lib/gcc/pic32mx/4.5.1/../../../../pic32mx/lib/size\libmchp_peripheral_32MX795F512L.a(pcache.o)
 .mdebug.abi32  0xa0002190        0x0 c:/program files (x86)/microchip/xc32/v1.10/bin/../lib/gcc/pic32mx/4.5.1/../../../../pic32mx/lib/size\libmchp_peripheral_32MX795F512L.a(int_disable_interrupts_lib.o)
 .mdebug.abi32  0xa0002190        0x0 c:/program files (x86)/microchip/xc32/v1.10/bin/../lib/gcc/pic32mx/4.5.1/../../../../pic32mx/lib/size\libmchp_peripheral_32MX795F512L.a(int_restore_interrupts_lib.o)
 .mdebug.abi32  0xa0002190        0x0 c:/program files (x86)/microchip/xc32/v1.10/bin/../lib/gcc/pic32mx/4.5.1/../../../../pic32mx/lib/size\libmchp_peripheral_32MX795F512L.a(int_enable_mv_int_lib.o)
 .mdebug.abi32  0xa0002190        0x0 c:/program files (x86)/microchip/xc32/v1.10/bin/../lib/gcc/pic32mx/4.5.1/../../../../pic32mx/lib/size\libmchp_peripheral_32MX795F512L.a(int_tbl_lib.o)
 .mdebug.abi32  0xa0002190        0x0 c:/program files (x86)/microchip/xc32/v1.10/bin/../lib/gcc/pic32mx/4.5.1/../../../../pic32mx/lib/size\libmchp_peripheral_32MX795F512L.a(rtcc_init_lib.o)
 .mdebug.abi32  0xa0002190        0x0 c:/program files (x86)/microchip/xc32/v1.10/bin/../lib/gcc/pic32mx/4.5.1/../../../../pic32mx/lib/size\libmchp_peripheral_32MX795F512L.a(rtcc_open_lib.o)
 .mdebug.abi32  0xa0002190        0x0 c:/program files (x86)/microchip/xc32/v1.10/bin/../lib/gcc/pic32mx/4.5.1/../../../../pic32mx/lib/size\libmchp_peripheral_32MX795F512L.a(spi_chn_data_rdy_lib.o)
 .mdebug.abi32  0xa0002190        0x0 c:/program files (x86)/microchip/xc32/v1.10/bin/../lib/gcc/pic32mx/4.5.1/../../../../pic32mx/lib/size\libmchp_peripheral_32MX795F512L.a(spi_chn_getc_lib.o)
 .mdebug.abi32  0xa0002190        0x0 c:/program files (x86)/microchip/xc32/v1.10/bin/../lib/gcc/pic32mx/4.5.1/../../../../pic32mx/lib/size\libmchp_peripheral_32MX795F512L.a(spi_chn_open_lib.o)
 .mdebug.abi32  0xa0002190        0x0 c:/program files (x86)/microchip/xc32/v1.10/bin/../lib/gcc/pic32mx/4.5.1/../../../../pic32mx/lib/size\libmchp_peripheral_32MX795F512L.a(spi_chn_putc_lib.o)
 .mdebug.abi32  0xa0002190        0x0 c:/program files (x86)/microchip/xc32/v1.10/bin/../lib/gcc/pic32mx/4.5.1/../../../../pic32mx/lib/size\libmchp_peripheral_32MX795F512L.a(spi_chn_tx_buff_empty_lib.o)
 .mdebug.abi32  0xa0002190        0x0 c:/program files (x86)/microchip/xc32/v1.10/bin/../lib/gcc/pic32mx/4.5.1/../../../../pic32mx/lib/size\libmchp_peripheral_32MX795F512L.a(spi_io_tbl_libp.o)
 .mdebug.abi32  0xa0002190        0x0 c:/program files (x86)/microchip/xc32/v1.10/bin/../lib/gcc/pic32mx/4.5.1/../../../../pic32mx/lib/size\libmchp_peripheral_32MX795F512L.a(spi_map_tbl_libp.o)
 .mdebug.abi32  0xa0002190        0x0 c:/program files (x86)/microchip/xc32/v1.10/bin/../lib/gcc/pic32mx/4.5.1/../../../../pic32mx/lib/size\libmchp_peripheral_32MX795F512L.a(port_set_pins_digital_in_lib.o)
 .mdebug.abi32  0xa0002190        0x0 c:/program files (x86)/microchip/xc32/v1.10/bin/../lib/gcc/pic32mx/4.5.1/../../../../pic32mx/lib/size\libmchp_peripheral_32MX795F512L.a(port_set_pins_digital_out_lib.o)
 .mdebug.abi32  0xa0002190        0x0 c:/program files (x86)/microchip/xc32/v1.10/bin/../lib/gcc/pic32mx/4.5.1/../../../../pic32mx/lib/size\libmchp_peripheral_32MX795F512L.a(_ports_tbl_libp.o)
 .mdebug.abi32  0xa0002190        0x0 c:/program files (x86)/microchip/xc32/v1.10/bin/../lib/gcc/pic32mx/4.5.1/../../../../pic32mx/lib/size\libmchp_peripheral_32MX795F512L.a(int_enable_interrupts_lib.o)
 .mdebug.abi32  0xa0002190        0x0 c:/program files (x86)/microchip/xc32/v1.10/bin/../lib/gcc/pic32mx/4.5.1/../../../../pic32mx/lib/size\libmchp_peripheral_32MX795F512L.a(_rtcc_wait_clock_off_lib.o)
 .mdebug.abi32  0xa0002190        0x0 c:/program files (x86)/microchip/xc32/v1.10/bin/../lib/gcc/pic32mx/4.5.1/../../../../pic32mx/lib/size\libmchp_peripheral_32MX795F512L.a(read_core_timer_lib.o)
 .mdebug.abi32  0xa0002190        0x0 c:/program files (x86)/microchip/xc32/v1.10/bin/../lib/gcc/pic32mx/4.5.1/size\libgcc.a(_udivdi3.o)
 .mdebug.abi32  0xa0002190        0x0 c:/program files (x86)/microchip/xc32/v1.10/bin/../lib/gcc/pic32mx/4.5.1/../../../../pic32mx/lib/size\libpic32.a(default-bootstrap-exception-handler.o)
 .mdebug.abi32  0xa0002190        0x0 c:/program files (x86)/microchip/xc32/v1.10/bin/../lib/gcc/pic32mx/4.5.1/../../../../pic32mx/lib/size\libpic32.a(default-on-reset.o)
 .mdebug.abi32  0xa0002190        0x0 c:/program files (x86)/microchip/xc32/v1.10/bin/../lib/gcc/pic32mx/4.5.1/../../../../pic32mx/lib/size\libpic32.a(default-on-bootstrap.o)
 .mdebug.abi32  0xa0002190        0x0 c:/program files (x86)/microchip/xc32/v1.10/bin/../lib/gcc/pic32mx/4.5.1/../../../../pic32mx/lib/size\libpic32.a(errno.o)
 .mdebug.abi32  0xa0002190        0x0 c:/program files (x86)/microchip/xc32/v1.10/bin/../lib/gcc/pic32mx/4.5.1/../../../../pic32mx/lib/size\libc.a(atoi.o)
 .mdebug.abi32  0xa0002190        0x0 c:/program files (x86)/microchip/xc32/v1.10/bin/../lib/gcc/pic32mx/4.5.1/../../../../pic32mx/lib/size\libc.a(atol.o)
 .mdebug.abi32  0xa0002190        0x0 c:/program files (x86)/microchip/xc32/v1.10/bin/../lib/gcc/pic32mx/4.5.1/../../../../pic32mx/lib/size\libc.a(ctype.o)
 .mdebug.abi32  0xa0002190        0x0 c:/program files (x86)/microchip/xc32/v1.10/bin/../lib/gcc/pic32mx/4.5.1/../../../../pic32mx/lib/size\libc.a(malloc.o)
 .mdebug.abi32  0xa0002190        0x0 c:/program files (x86)/microchip/xc32/v1.10/bin/../lib/gcc/pic32mx/4.5.1/../../../../pic32mx/lib/size\libc.a(rand.o)
 .mdebug.abi32  0xa0002190        0x0 c:/program files (x86)/microchip/xc32/v1.10/bin/../lib/gcc/pic32mx/4.5.1/../../../../pic32mx/lib/size\libc.a(strcat.o)
 .mdebug.abi32  0xa0002190        0x0 c:/program files (x86)/microchip/xc32/v1.10/bin/../lib/gcc/pic32mx/4.5.1/../../../../pic32mx/lib/size\libc.a(strchr.o)
 .mdebug.abi32  0xa0002190        0x0 c:/program files (x86)/microchip/xc32/v1.10/bin/../lib/gcc/pic32mx/4.5.1/../../../../pic32mx/lib/size\libc.a(strncat.o)
 .mdebug.abi32  0xa0002190        0x0 c:/program files (x86)/microchip/xc32/v1.10/bin/../lib/gcc/pic32mx/4.5.1/../../../../pic32mx/lib/size\libc.a(strncmp.o)
 .mdebug.abi32  0xa0002190        0x0 c:/program files (x86)/microchip/xc32/v1.10/bin/../lib/gcc/pic32mx/4.5.1/../../../../pic32mx/lib/size\libc.a(strncpy.o)
 .mdebug.abi32  0xa0002190        0x0 c:/program files (x86)/microchip/xc32/v1.10/bin/../lib/gcc/pic32mx/4.5.1/../../../../pic32mx/lib/size\libc.a(strrchr.o)
 .mdebug.abi32  0xa0002190        0x0 c:/program files (x86)/microchip/xc32/v1.10/bin/../lib/gcc/pic32mx/4.5.1/../../../../pic32mx/lib/size\libc.a(strstr.o)
 .mdebug.abi32  0xa0002190        0x0 c:/program files (x86)/microchip/xc32/v1.10/bin/../lib/gcc/pic32mx/4.5.1/../../../../pic32mx/lib/size\libc.a(strtol.o)
 .mdebug.abi32  0xa0002190        0x0 c:/program files (x86)/microchip/xc32/v1.10/bin/../lib/gcc/pic32mx/4.5.1/../../../../pic32mx/lib/size\libc.a(snprintf_cdnopsuxX.eo)
 .mdebug.abi32  0xa0002190        0x0 c:/program files (x86)/microchip/xc32/v1.10/bin/../lib/gcc/pic32mx/4.5.1/../../../../pic32mx/lib/size\libc.a(sprintf_cdnopsuxX.eo)
 .mdebug.abi32  0xa0002190        0x0 c:/program files (x86)/microchip/xc32/v1.10/bin/../lib/gcc/pic32mx/4.5.1/../../../../pic32mx/lib/size\libc.a(vsnprintf_cdnopsuxX.eo)
 .mdebug.abi32  0xa0002190        0x0 c:/program files (x86)/microchip/xc32/v1.10/bin/../lib/gcc/pic32mx/4.5.1/../../../../pic32mx/lib/size\libc.a(vsnprintf.o)
 .mdebug.abi32  0xa0002190        0x0 c:/program files (x86)/microchip/xc32/v1.10/bin/../lib/gcc/pic32mx/4.5.1/../../../../pic32mx/lib/size\libc.a(ctypef.o)
 .mdebug.abi32  0xa0002190        0x0 c:/program files (x86)/microchip/xc32/v1.10/bin/../lib/gcc/pic32mx/4.5.1/../../../../pic32mx/lib/size\libc.a(doprnt_cdnopsuxX.eo)
 .mdebug.abi32  0xa0002190        0x0 c:/program files (x86)/microchip/xc32/v1.10/bin/../lib/gcc/pic32mx/4.5.1/../../../../pic32mx/lib/size\libc.a(doprnt.o)
 .mdebug.abi32  0xa0002190        0x0 c:/program files (x86)/microchip/xc32/v1.10/bin/../lib/gcc/pic32mx/4.5.1/../../../../pic32mx/lib/size\libc.a(_fputc_simple.o)
 .mdebug.abi32  0xa0002190        0x0 c:/program files (x86)/microchip/xc32/v1.10/bin/../lib/gcc/pic32mx/4.5.1/../../../../pic32mx/lib/size\libc.a(powersf.o)
 .mdebug.abi32  0xa0002190        0x0 c:/program files (x86)/microchip/xc32/v1.10/bin/../lib/gcc/pic32mx/4.5.1/../../../../pic32mx/lib/size\libc.a(_iob.o)
 .mdebug.abi32  0xa0002190        0x0 c:/program files (x86)/microchip/xc32/v1.10/bin/../lib/gcc/pic32mx/4.5.1/../../../../pic32mx/lib/size\libc.a(_flsbuf_simple.o)
 .mdebug.abi32  0xa0002190        0x0 c:/program files (x86)/microchip/xc32/v1.10/bin/../lib/gcc/pic32mx/4.5.1/../../../../pic32mx/lib/size\libpic32.a(sbrk.o)
 .mdebug.abi32  0xa0002190        0x0 c:/program files (x86)/microchip/xc32/v1.10/bin/../lib/gcc/pic32mx/4.5.1/../../../../pic32mx/lib/size\libpic32.a(write.o)
 .mdebug.abi32  0xa0002190        0x0 c:/program files (x86)/microchip/xc32/v1.10/bin/../lib/gcc/pic32mx/4.5.1/../../../../pic32mx/lib/size\libpic32.a(_mon_putc.o)
 .mdebug.abi32  0xa0002190        0x0 c:/program files (x86)/microchip/xc32/v1.10/bin/../lib/gcc/pic32mx/4.5.1/../../../../pic32mx/lib/size\libpic32.a(xc32_uart.o)
 .mdebug.abi32  0xa0002190        0x0 c:/program files (x86)/microchip/xc32/v1.10/bin/../lib/gcc/pic32mx/4.5.1/../../../../pic32mx/lib/size\libe.a(_floatdisf.o)
 .mdebug.abi32  0xa0002190        0x0 c:/program files (x86)/microchip/xc32/v1.10/bin/../lib/gcc/pic32mx/4.5.1/size\libgcc.a(_lshrdi3.o)
 .mdebug.abi32  0xa0002190        0x0 c:/program files (x86)/microchip/xc32/v1.10/bin/../lib/gcc/pic32mx/4.5.1/size\libgcc.a(_floatundisf.o)
 .mdebug.abi32  0xa0002190        0x0 c:/program files (x86)/microchip/xc32/v1.10/bin/../lib/gcc/pic32mx/4.5.1/size\libgcc.a(_umoddi3.o)
 .mdebug.abi32  0xa0002190        0x0 c:/program files (x86)/microchip/xc32/v1.10/bin/../lib/gcc/pic32mx/4.5.1/size\libgcc.a(floatunsisf.o)

.mdebug.abiN32
 *(.mdebug.abiN32)

.mdebug.abi64
 *(.mdebug.abi64)

.mdebug.abiO64
 *(.mdebug.abiO64)

.mdebug.eabi32
 *(.mdebug.eabi32)

.mdebug.eabi64
 *(.mdebug.eabi64)

.gcc_compiled_long32
 *(.gcc_compiled_long32)

.gcc_compiled_long64
 *(.gcc_compiled_long64)

.stab
 *(.stab)

.stabstr
 *(.stabstr)

.stab.excl
 *(.stab.excl)

.stab.exclstr
 *(.stab.exclstr)

.stab.index
 *(.stab.index)

.stab.indexstr
 *(.stab.indexstr)

.comment        0x00000000      0x2ca
 *(.comment)
 .comment       0x00000000       0x3c build/default/production/_ext/1293749816/bsp.o
                                 0x3d (size before relaxing)
 .comment       0x00000000       0x3d build/default/production/_ext/101875047/hashes.o
 .comment       0x00000000       0x3d build/default/production/_ext/101875047/lfsr.o
 .comment       0x00000000       0x3d build/default/production/_ext/101875047/big_int.o
 .comment       0x00000000       0x3d build/default/production/_ext/101875047/helpers.o
 .comment       0x00000000       0x3d build/default/production/_ext/1472/berkeley_tcp_client_demo.o
 .comment       0x00000000       0x3d build/default/production/_ext/1472/berkeley_tcp_server_demo.o
 .comment       0x00000000       0x3d build/default/production/_ext/1472/berkeley_udp_client_demo.o
 .comment       0x00000000       0x3d build/default/production/_ext/1472/generic_tcp_client.o
 .comment       0x00000000       0x3d build/default/production/_ext/1472/generic_tcp_server.o
 .comment       0x00000000       0x3d build/default/production/_ext/1472/ping_demo.o
 .comment       0x00000000       0x3d build/default/production/_ext/1472/smtp_demo.o
 .comment       0x00000000       0x3d build/default/production/_ext/365611741/system_services.o
 .comment       0x00000000       0x3d build/default/production/_ext/365611741/system_debug.o
 .comment       0x00000000       0x3d build/default/production/_ext/365611741/system_random.o
 .comment       0x00000000       0x3d build/default/production/_ext/365611741/system_command.o
 .comment       0x00000000       0x3d build/default/production/_ext/365611741/system_userio.o
 .comment       0x00000000       0x3d build/default/production/_ext/97638081/sys_fs.o
 .comment       0x00000000       0x3d build/default/production/_ext/97638081/mpfs2.o
 .comment       0x00000000       0x3d build/default/production/_ext/792872985/usart.o
 .comment       0x00000000       0x3d build/default/production/_ext/792872985/lcd.o
 .comment       0x00000000       0x3d build/default/production/_ext/792872985/drv_spi.o
 .comment       0x00000000       0x3d build/default/production/_ext/792872985/db_appio.o
 .comment       0x00000000       0x3d build/default/production/_ext/792872985/spi_ram.o
 .comment       0x00000000       0x3d build/default/production/_ext/792872985/spi_eeprom.o
 .comment       0x00000000       0x3d build/default/production/_ext/792872985/spi_flash.o
 .comment       0x00000000       0x3d build/default/production/_ext/792872985/drv_media.o
 .comment       0x00000000       0x3d build/default/production/_ext/427700826/tcpip_announce.o
 .comment       0x00000000       0x3d build/default/production/_ext/427700826/http2.o
 .comment       0x00000000       0x3d build/default/production/_ext/427700826/arcfour.o
 .comment       0x00000000       0x3d build/default/production/_ext/427700826/arp.o
 .comment       0x00000000       0x3d build/default/production/_ext/427700826/berkeley_api.o
 .comment       0x00000000       0x3d build/default/production/_ext/427700826/dhcp.o
 .comment       0x00000000       0x3d build/default/production/_ext/427700826/dhcps.o
 .comment       0x00000000       0x3d build/default/production/_ext/427700826/dns.o
 .comment       0x00000000       0x3d build/default/production/_ext/427700826/dnss.o
 .comment       0x00000000       0x3d build/default/production/_ext/427700826/dyn_dns.o
 .comment       0x00000000       0x3d build/default/production/_ext/427700826/enc28_mac.o
 .comment       0x00000000       0x3d build/default/production/_ext/427700826/enc28j60.o
 .comment       0x00000000       0x3d build/default/production/_ext/427700826/encs24j600.o
 .comment       0x00000000       0x3d build/default/production/_ext/427700826/encx24_mac.o
 .comment       0x00000000       0x3d build/default/production/_ext/427700826/eth_pic32_ext_phy.o
 .comment       0x00000000       0x3d build/default/production/_ext/427700826/eth_pic32_ext_phy_dp83848.o
 .comment       0x00000000       0x3d build/default/production/_ext/427700826/eth_pic32_int_mac.o
 .comment       0x00000000       0x3d build/default/production/_ext/427700826/ftp.o
 .comment       0x00000000       0x3d build/default/production/_ext/427700826/hash_fnv.o
 .comment       0x00000000       0x3d build/default/production/_ext/427700826/hash_tbl.o
 .comment       0x00000000       0x3d build/default/production/_ext/427700826/icmp.o
 .comment       0x00000000       0x3d build/default/production/_ext/427700826/icmpv6.o
 .comment       0x00000000       0x3d build/default/production/_ext/427700826/ipv4.o
 .comment       0x00000000       0x3d build/default/production/_ext/427700826/ipv6.o
 .comment       0x00000000       0x3d build/default/production/_ext/427700826/mac_events_pic32.o
 .comment       0x00000000       0x3d build/default/production/_ext/427700826/nbns.o
 .comment       0x00000000       0x3d build/default/production/_ext/427700826/ndp.o
 .comment       0x00000000       0x3d build/default/production/_ext/427700826/tcpip_reboot.o
 .comment       0x00000000       0x3d build/default/production/_ext/427700826/rsa.o
 .comment       0x00000000       0x3d build/default/production/_ext/427700826/smtp.o
 .comment       0x00000000       0x3d build/default/production/_ext/427700826/snmp.o
 .comment       0x00000000       0x3d build/default/production/_ext/427700826/snmpv3.o
 .comment       0x00000000       0x3d build/default/production/_ext/427700826/snmpv3_usm.o
 .comment       0x00000000       0x3d build/default/production/_ext/427700826/sntp.o
 .comment       0x00000000       0x3d build/default/production/_ext/427700826/ssl.o
 .comment       0x00000000       0x3d build/default/production/_ext/427700826/tcp.o
 .comment       0x00000000       0x3d build/default/production/_ext/427700826/tcpip_heap_alloc.o
 .comment       0x00000000       0x3d build/default/production/_ext/427700826/tcpip_storage.o
 .comment       0x00000000       0x3d build/default/production/_ext/427700826/telnet.o
 .comment       0x00000000       0x3d build/default/production/_ext/427700826/tftpc.o
 .comment       0x00000000       0x3d build/default/production/_ext/427700826/udp.o
 .comment       0x00000000       0x3d build/default/production/_ext/427700826/tcpip_mac_object.o
 .comment       0x00000000       0x3d build/default/production/_ext/427700826/tcpip_manager.o
 .comment       0x00000000       0x3d build/default/production/_ext/427700826/tcpip_helpers.o
 .comment       0x00000000       0x3d build/default/production/_ext/427700826/tcpip_commands.o
 .comment       0x00000000       0x3d build/default/production/_ext/427700826/iperf.o
 .comment       0x00000000       0x3d build/default/production/_ext/427700826/tcpip_notify.o
 .comment       0x00000000       0x3d build/default/production/_ext/427700826/zero_conf_helper.o
 .comment       0x00000000       0x3d build/default/production/_ext/427700826/zero_conf_link_local.o
 .comment       0x00000000       0x3d build/default/production/_ext/427700826/zero_conf_multicast_dns.o
 .comment       0x00000000       0x3d build/default/production/_ext/334706090/wf_tx_power.o
 .comment       0x00000000       0x3d build/default/production/_ext/334706090/wf_connect.o
 .comment       0x00000000       0x3d build/default/production/_ext/334706090/wf_connection_algorithm.o
 .comment       0x00000000       0x3d build/default/production/_ext/334706090/wf_connection_manager.o
 .comment       0x00000000       0x3d build/default/production/_ext/334706090/wf_connection_profile.o
 .comment       0x00000000       0x3d build/default/production/_ext/334706090/wf_easy_config.o
 .comment       0x00000000       0x3d build/default/production/_ext/334706090/wf_eint.o
 .comment       0x00000000       0x3d build/default/production/_ext/334706090/wf_event_handler.o
 .comment       0x00000000       0x3d build/default/production/_ext/334706090/wf_init.o
 .comment       0x00000000       0x3d build/default/production/_ext/334706090/wf_power_save.o
 .comment       0x00000000       0x3d build/default/production/_ext/334706090/wf_scan.o
 .comment       0x00000000       0x3d build/default/production/_ext/334706090/wf_spi.o
 .comment       0x00000000       0x3d build/default/production/_ext/334706090/mrf24w_mac_pic32.o
 .comment       0x00000000       0x3d build/default/production/_ext/334706090/mrf24w_events.o
 .comment       0x00000000       0x3d build/default/production/_ext/334706090/wf_debug_output.o
 .comment       0x00000000       0x3d build/default/production/_ext/334706090/wf_commands.o
 .comment       0x00000000       0x3d build/default/production/_ext/334706090/wf_pbkdf2.o
 .comment       0x00000000       0x3d build/default/production/_ext/334706090/wf_driver_com_24g.o
 .comment       0x00000000       0x3d build/default/production/_ext/334706090/wf_driver_raw_24g.o
 .comment       0x00000000       0x3d build/default/production/_ext/334706090/wf_mac_24g.o
 .comment       0x00000000       0x3d build/default/production/_ext/334706090/wf_mgmt_msg_24g.o
 .comment       0x00000000       0x3d build/default/production/_ext/334706090/wf_param_msg_24g.o
 .comment       0x00000000       0x3d build/default/production/_ext/334706090/wf_configData.o
 .comment       0x00000000       0x3d build/default/production/_ext/1472/main_demo.o
 .comment       0x00000000       0x3d build/default/production/_ext/1472/custom_snmp_app.o
 .comment       0x00000000       0x3d build/default/production/_ext/1472/custom_ssl_cert.o
 .comment       0x00000000       0x3d build/default/production/_ext/1472/mpfs_img2.o
 .comment       0x00000000       0x3d build/default/production/_ext/1472/wf_config.o
 .comment       0x00000000       0x3d build/default/production/_ext/1472/custom_http_app.o
 .comment       0x00000000       0x3d build/default/production/_ext/1472/tcp6_demo_app.o
 .comment       0x0000003c       0x51 c:/program files (x86)/microchip/xc32/v1.10/bin/../lib/gcc/pic32mx/4.5.1/../../../../pic32mx/lib/size\libmchp_peripheral.a(open_core_timer_lib.o)
                                 0x52 (size before relaxing)
 .comment       0x00000000       0x52 c:/program files (x86)/microchip/xc32/v1.10/bin/../lib/gcc/pic32mx/4.5.1/../../../../pic32mx/lib/size\libmchp_peripheral_32MX795F512L.a(soft_reset_lib.o)
 .comment       0x00000000       0x52 c:/program files (x86)/microchip/xc32/v1.10/bin/../lib/gcc/pic32mx/4.5.1/../../../../pic32mx/lib/size\libmchp_peripheral_32MX795F512L.a(pcache.o)
 .comment       0x00000000       0x52 c:/program files (x86)/microchip/xc32/v1.10/bin/../lib/gcc/pic32mx/4.5.1/../../../../pic32mx/lib/size\libmchp_peripheral_32MX795F512L.a(int_disable_interrupts_lib.o)
 .comment       0x00000000       0x52 c:/program files (x86)/microchip/xc32/v1.10/bin/../lib/gcc/pic32mx/4.5.1/../../../../pic32mx/lib/size\libmchp_peripheral_32MX795F512L.a(int_restore_interrupts_lib.o)
 .comment       0x00000000       0x52 c:/program files (x86)/microchip/xc32/v1.10/bin/../lib/gcc/pic32mx/4.5.1/../../../../pic32mx/lib/size\libmchp_peripheral_32MX795F512L.a(int_enable_mv_int_lib.o)
 .comment       0x00000000       0x52 c:/program files (x86)/microchip/xc32/v1.10/bin/../lib/gcc/pic32mx/4.5.1/../../../../pic32mx/lib/size\libmchp_peripheral_32MX795F512L.a(int_tbl_lib.o)
 .comment       0x00000000       0x52 c:/program files (x86)/microchip/xc32/v1.10/bin/../lib/gcc/pic32mx/4.5.1/../../../../pic32mx/lib/size\libmchp_peripheral_32MX795F512L.a(rtcc_init_lib.o)
 .comment       0x00000000       0x52 c:/program files (x86)/microchip/xc32/v1.10/bin/../lib/gcc/pic32mx/4.5.1/../../../../pic32mx/lib/size\libmchp_peripheral_32MX795F512L.a(rtcc_open_lib.o)
 .comment       0x00000000       0x52 c:/program files (x86)/microchip/xc32/v1.10/bin/../lib/gcc/pic32mx/4.5.1/../../../../pic32mx/lib/size\libmchp_peripheral_32MX795F512L.a(spi_chn_data_rdy_lib.o)
 .comment       0x00000000       0x52 c:/program files (x86)/microchip/xc32/v1.10/bin/../lib/gcc/pic32mx/4.5.1/../../../../pic32mx/lib/size\libmchp_peripheral_32MX795F512L.a(spi_chn_getc_lib.o)
 .comment       0x00000000       0x52 c:/program files (x86)/microchip/xc32/v1.10/bin/../lib/gcc/pic32mx/4.5.1/../../../../pic32mx/lib/size\libmchp_peripheral_32MX795F512L.a(spi_chn_open_lib.o)
 .comment       0x00000000       0x52 c:/program files (x86)/microchip/xc32/v1.10/bin/../lib/gcc/pic32mx/4.5.1/../../../../pic32mx/lib/size\libmchp_peripheral_32MX795F512L.a(spi_chn_putc_lib.o)
 .comment       0x00000000       0x52 c:/program files (x86)/microchip/xc32/v1.10/bin/../lib/gcc/pic32mx/4.5.1/../../../../pic32mx/lib/size\libmchp_peripheral_32MX795F512L.a(spi_chn_tx_buff_empty_lib.o)
 .comment       0x00000000       0x52 c:/program files (x86)/microchip/xc32/v1.10/bin/../lib/gcc/pic32mx/4.5.1/../../../../pic32mx/lib/size\libmchp_peripheral_32MX795F512L.a(spi_io_tbl_libp.o)
 .comment       0x00000000       0x52 c:/program files (x86)/microchip/xc32/v1.10/bin/../lib/gcc/pic32mx/4.5.1/../../../../pic32mx/lib/size\libmchp_peripheral_32MX795F512L.a(spi_map_tbl_libp.o)
 .comment       0x00000000       0x52 c:/program files (x86)/microchip/xc32/v1.10/bin/../lib/gcc/pic32mx/4.5.1/../../../../pic32mx/lib/size\libmchp_peripheral_32MX795F512L.a(port_set_pins_digital_in_lib.o)
 .comment       0x00000000       0x52 c:/program files (x86)/microchip/xc32/v1.10/bin/../lib/gcc/pic32mx/4.5.1/../../../../pic32mx/lib/size\libmchp_peripheral_32MX795F512L.a(port_set_pins_digital_out_lib.o)
 .comment       0x00000000       0x52 c:/program files (x86)/microchip/xc32/v1.10/bin/../lib/gcc/pic32mx/4.5.1/../../../../pic32mx/lib/size\libmchp_peripheral_32MX795F512L.a(_ports_tbl_libp.o)
 .comment       0x00000000       0x52 c:/program files (x86)/microchip/xc32/v1.10/bin/../lib/gcc/pic32mx/4.5.1/../../../../pic32mx/lib/size\libmchp_peripheral_32MX795F512L.a(int_enable_interrupts_lib.o)
 .comment       0x00000000       0x52 c:/program files (x86)/microchip/xc32/v1.10/bin/../lib/gcc/pic32mx/4.5.1/../../../../pic32mx/lib/size\libmchp_peripheral_32MX795F512L.a(_rtcc_wait_clock_off_lib.o)
 .comment       0x00000000       0x52 c:/program files (x86)/microchip/xc32/v1.10/bin/../lib/gcc/pic32mx/4.5.1/../../../../pic32mx/lib/size\libmchp_peripheral_32MX795F512L.a(read_core_timer_lib.o)
 .comment       0x00000000       0x3d c:/program files (x86)/microchip/xc32/v1.10/bin/../lib/gcc/pic32mx/4.5.1/size\libgcc.a(_udivdi3.o)
 .comment       0x0000008d       0x18 c:/program files (x86)/microchip/xc32/v1.10/bin/../lib/gcc/pic32mx/4.5.1/../../../../pic32mx/lib/size\libpic32.a(memcmp.o)
                                 0x19 (size before relaxing)
 .comment       0x000000a5       0x18 c:/program files (x86)/microchip/xc32/v1.10/bin/../lib/gcc/pic32mx/4.5.1/../../../../pic32mx/lib/size\libpic32.a(memset.o)
                                 0x19 (size before relaxing)
 .comment       0x000000bd       0x55 c:/program files (x86)/microchip/xc32/v1.10/bin/../lib/gcc/pic32mx/4.5.1/../../../../pic32mx/lib/size\libpic32.a(strcmp.o)
                                 0x56 (size before relaxing)
 .comment       0x00000112       0x19 c:/program files (x86)/microchip/xc32/v1.10/bin/../lib/gcc/pic32mx/4.5.1/../../../../pic32mx/lib/size\libpic32.a(strcpy.o)
                                 0x1a (size before relaxing)
 .comment       0x0000012b       0x19 c:/program files (x86)/microchip/xc32/v1.10/bin/../lib/gcc/pic32mx/4.5.1/../../../../pic32mx/lib/size\libpic32.a(strlen.o)
                                 0x1a (size before relaxing)
 .comment       0x00000000       0x3d c:/program files (x86)/microchip/xc32/v1.10/bin/../lib/gcc/pic32mx/4.5.1/../../../../pic32mx/lib/size\libpic32.a(default-bootstrap-exception-handler.o)
 .comment       0x00000000       0x3d c:/program files (x86)/microchip/xc32/v1.10/bin/../lib/gcc/pic32mx/4.5.1/../../../../pic32mx/lib/size\libpic32.a(default-on-reset.o)
 .comment       0x00000000       0x3d c:/program files (x86)/microchip/xc32/v1.10/bin/../lib/gcc/pic32mx/4.5.1/../../../../pic32mx/lib/size\libpic32.a(default-on-bootstrap.o)
 .comment       0x00000000       0x3d c:/program files (x86)/microchip/xc32/v1.10/bin/../lib/gcc/pic32mx/4.5.1/../../../../pic32mx/lib/size\libpic32.a(errno.o)
 .comment       0x00000000       0x3d c:/program files (x86)/microchip/xc32/v1.10/bin/../lib/gcc/pic32mx/4.5.1/../../../../pic32mx/lib/size\libc.a(atoi.o)
 .comment       0x00000000       0x3d c:/program files (x86)/microchip/xc32/v1.10/bin/../lib/gcc/pic32mx/4.5.1/../../../../pic32mx/lib/size\libc.a(atol.o)
 .comment       0x00000144       0x4e c:/program files (x86)/microchip/xc32/v1.10/bin/../lib/gcc/pic32mx/4.5.1/../../../../pic32mx/lib/size\libc.a(ctype.o)
                                 0x8b (size before relaxing)
 .comment       0x00000000       0x3d c:/program files (x86)/microchip/xc32/v1.10/bin/../lib/gcc/pic32mx/4.5.1/../../../../pic32mx/lib/size\libc.a(malloc.o)
 .comment       0x00000000       0x3d c:/program files (x86)/microchip/xc32/v1.10/bin/../lib/gcc/pic32mx/4.5.1/../../../../pic32mx/lib/size\libc.a(rand.o)
 .comment       0x00000000       0x3d c:/program files (x86)/microchip/xc32/v1.10/bin/../lib/gcc/pic32mx/4.5.1/../../../../pic32mx/lib/size\libc.a(strcat.o)
 .comment       0x00000000       0x3d c:/program files (x86)/microchip/xc32/v1.10/bin/../lib/gcc/pic32mx/4.5.1/../../../../pic32mx/lib/size\libc.a(strchr.o)
 .comment       0x00000000       0x3d c:/program files (x86)/microchip/xc32/v1.10/bin/../lib/gcc/pic32mx/4.5.1/../../../../pic32mx/lib/size\libc.a(strncat.o)
 .comment       0x00000000       0x3d c:/program files (x86)/microchip/xc32/v1.10/bin/../lib/gcc/pic32mx/4.5.1/../../../../pic32mx/lib/size\libc.a(strncmp.o)
 .comment       0x00000000       0x3d c:/program files (x86)/microchip/xc32/v1.10/bin/../lib/gcc/pic32mx/4.5.1/../../../../pic32mx/lib/size\libc.a(strncpy.o)
 .comment       0x00000000       0x3d c:/program files (x86)/microchip/xc32/v1.10/bin/../lib/gcc/pic32mx/4.5.1/../../../../pic32mx/lib/size\libc.a(strrchr.o)
 .comment       0x00000000       0x3d c:/program files (x86)/microchip/xc32/v1.10/bin/../lib/gcc/pic32mx/4.5.1/../../../../pic32mx/lib/size\libc.a(strstr.o)
 .comment       0x00000000       0x3d c:/program files (x86)/microchip/xc32/v1.10/bin/../lib/gcc/pic32mx/4.5.1/../../../../pic32mx/lib/size\libc.a(strtol.o)
 .comment       0x00000000       0x3d c:/program files (x86)/microchip/xc32/v1.10/bin/../lib/gcc/pic32mx/4.5.1/../../../../pic32mx/lib/size\libc.a(snprintf_cdnopsuxX.eo)
 .comment       0x00000000       0x3d c:/program files (x86)/microchip/xc32/v1.10/bin/../lib/gcc/pic32mx/4.5.1/../../../../pic32mx/lib/size\libc.a(sprintf_cdnopsuxX.eo)
 .comment       0x00000000       0x3d c:/program files (x86)/microchip/xc32/v1.10/bin/../lib/gcc/pic32mx/4.5.1/../../../../pic32mx/lib/size\libc.a(vsnprintf_cdnopsuxX.eo)
 .comment       0x00000000       0x3d c:/program files (x86)/microchip/xc32/v1.10/bin/../lib/gcc/pic32mx/4.5.1/../../../../pic32mx/lib/size\libc.a(vsnprintf.o)
 .comment       0x00000192       0x4f c:/program files (x86)/microchip/xc32/v1.10/bin/../lib/gcc/pic32mx/4.5.1/../../../../pic32mx/lib/size\libc.a(ctypef.o)
                                 0x8c (size before relaxing)
 .comment       0x00000000       0x3d c:/program files (x86)/microchip/xc32/v1.10/bin/../lib/gcc/pic32mx/4.5.1/../../../../pic32mx/lib/size\libc.a(doprnt_cdnopsuxX.eo)
 .comment       0x00000000       0x3d c:/program files (x86)/microchip/xc32/v1.10/bin/../lib/gcc/pic32mx/4.5.1/../../../../pic32mx/lib/size\libc.a(doprnt.o)
 .comment       0x00000000       0x3d c:/program files (x86)/microchip/xc32/v1.10/bin/../lib/gcc/pic32mx/4.5.1/../../../../pic32mx/lib/size\libc.a(_fputc_simple.o)
 .comment       0x00000000       0x3d c:/program files (x86)/microchip/xc32/v1.10/bin/../lib/gcc/pic32mx/4.5.1/../../../../pic32mx/lib/size\libc.a(powersf.o)
 .comment       0x00000000       0x3d c:/program files (x86)/microchip/xc32/v1.10/bin/../lib/gcc/pic32mx/4.5.1/../../../../pic32mx/lib/size\libc.a(_iob.o)
 .comment       0x00000000       0x3d c:/program files (x86)/microchip/xc32/v1.10/bin/../lib/gcc/pic32mx/4.5.1/../../../../pic32mx/lib/size\libc.a(_flsbuf_simple.o)
 .comment       0x000001e1       0x4b c:/program files (x86)/microchip/xc32/v1.10/bin/../lib/gcc/pic32mx/4.5.1/../../../../pic32mx/lib/size\libpic32.a(sbrk.o)
                                 0x88 (size before relaxing)
 .comment       0x00000000       0x3d c:/program files (x86)/microchip/xc32/v1.10/bin/../lib/gcc/pic32mx/4.5.1/../../../../pic32mx/lib/size\libpic32.a(write.o)
 .comment       0x00000000       0x3d c:/program files (x86)/microchip/xc32/v1.10/bin/../lib/gcc/pic32mx/4.5.1/../../../../pic32mx/lib/size\libpic32.a(_mon_putc.o)
 .comment       0x00000000       0x3d c:/program files (x86)/microchip/xc32/v1.10/bin/../lib/gcc/pic32mx/4.5.1/../../../../pic32mx/lib/size\libpic32.a(xc32_uart.o)
 .comment       0x0000022c       0x9e c:/program files (x86)/microchip/xc32/v1.10/bin/../lib/gcc/pic32mx/4.5.1/../../../../pic32mx/lib/size\libe.a(_floatdisf.o)
                                 0xdb (size before relaxing)
 .comment       0x00000000       0x3d c:/program files (x86)/microchip/xc32/v1.10/bin/../lib/gcc/pic32mx/4.5.1/size\libgcc.a(_lshrdi3.o)
 .comment       0x00000000       0x3d c:/program files (x86)/microchip/xc32/v1.10/bin/../lib/gcc/pic32mx/4.5.1/size\libgcc.a(_floatundisf.o)
 .comment       0x00000000       0x3d c:/program files (x86)/microchip/xc32/v1.10/bin/../lib/gcc/pic32mx/4.5.1/size\libgcc.a(_umoddi3.o)
 .comment       0x00000000       0x3d c:/program files (x86)/microchip/xc32/v1.10/bin/../lib/gcc/pic32mx/4.5.1/size\libgcc.a(floatunsisf.o)

.debug
 *(.debug)

.line
 *(.line)

.debug_srcinfo
 *(.debug_srcinfo)

.debug_sfnames
 *(.debug_sfnames)

.debug_aranges  0x00000000     0x2e60
 *(.debug_aranges)
 .debug_aranges
                0x00000000       0x20 build/default/production/_ext/1293749816/bsp.o
 .debug_aranges
                0x00000020       0x60 build/default/production/_ext/101875047/hashes.o
 .debug_aranges
                0x00000080       0x28 build/default/production/_ext/101875047/lfsr.o
 .debug_aranges
                0x000000a8       0x80 build/default/production/_ext/101875047/big_int.o
 .debug_aranges
                0x00000128       0x20 build/default/production/_ext/101875047/big_int_helper_c32.o
 .debug_aranges
                0x00000148       0x58 build/default/production/_ext/101875047/helpers.o
 .debug_aranges
                0x000001a0       0x30 build/default/production/_ext/1472/ping_demo.o
 .debug_aranges
                0x000001d0      0x100 build/default/production/_ext/365611741/system_services.o
 .debug_aranges
                0x000002d0       0xc8 build/default/production/_ext/365611741/system_debug.o
 .debug_aranges
                0x00000398       0x40 build/default/production/_ext/365611741/system_random.o
 .debug_aranges
                0x000003d8       0xc0 build/default/production/_ext/365611741/system_command.o
 .debug_aranges
                0x00000498       0x58 build/default/production/_ext/365611741/system_userio.o
 .debug_aranges
                0x000004f0      0x240 build/default/production/_ext/97638081/sys_fs.o
 .debug_aranges
                0x00000730       0xd8 build/default/production/_ext/97638081/mpfs2.o
 .debug_aranges
                0x00000808       0x50 build/default/production/_ext/792872985/usart.o
 .debug_aranges
                0x00000858       0x48 build/default/production/_ext/792872985/lcd.o
 .debug_aranges
                0x000008a0       0x30 build/default/production/_ext/792872985/drv_spi.o
 .debug_aranges
                0x000008d0       0x70 build/default/production/_ext/792872985/spi_eeprom.o
 .debug_aranges
                0x00000940       0x90 build/default/production/_ext/792872985/drv_media.o
 .debug_aranges
                0x000009d0       0x50 build/default/production/_ext/427700826/tcpip_announce.o
 .debug_aranges
                0x00000a20      0x140 build/default/production/_ext/427700826/http2.o
 .debug_aranges
                0x00000b60      0x138 build/default/production/_ext/427700826/arp.o
 .debug_aranges
                0x00000c98       0xb0 build/default/production/_ext/427700826/dhcp.o
 .debug_aranges
                0x00000d48       0x30 build/default/production/_ext/427700826/dhcps.o
 .debug_aranges
                0x00000d78       0x70 build/default/production/_ext/427700826/dns.o
 .debug_aranges
                0x00000de8       0x28 build/default/production/_ext/427700826/hash_fnv.o
 .debug_aranges
                0x00000e10       0x58 build/default/production/_ext/427700826/hash_tbl.o
 .debug_aranges
                0x00000e68       0x50 build/default/production/_ext/427700826/icmp.o
 .debug_aranges
                0x00000eb8      0x150 build/default/production/_ext/427700826/ipv4.o
 .debug_aranges
                0x00001008       0x40 build/default/production/_ext/427700826/nbns.o
 .debug_aranges
                0x00001048      0x288 build/default/production/_ext/427700826/tcp.o
 .debug_aranges
                0x000012d0       0x98 build/default/production/_ext/427700826/tcpip_heap_alloc.o
 .debug_aranges
                0x00001368      0x170 build/default/production/_ext/427700826/udp.o
 .debug_aranges
                0x000014d8       0xd8 build/default/production/_ext/427700826/tcpip_mac_object.o
 .debug_aranges
                0x000015b0      0x298 build/default/production/_ext/427700826/tcpip_manager.o
 .debug_aranges
                0x00001848       0xe8 build/default/production/_ext/427700826/tcpip_helpers.o
 .debug_aranges
                0x00001930       0x20 build/default/production/_ext/427700826/tcpip_helper_c32.o
 .debug_aranges
                0x00001950       0x30 build/default/production/_ext/427700826/tcpip_notify.o
 .debug_aranges
                0x00001980       0x30 build/default/production/_ext/427700826/zero_conf_link_local.o
 .debug_aranges
                0x000019b0       0x30 build/default/production/_ext/334706090/wf_tx_power.o
 .debug_aranges
                0x000019e0       0x40 build/default/production/_ext/334706090/wf_connect.o
 .debug_aranges
                0x00001a20       0xa8 build/default/production/_ext/334706090/wf_connection_algorithm.o
 .debug_aranges
                0x00001ac8       0x50 build/default/production/_ext/334706090/wf_connection_manager.o
 .debug_aranges
                0x00001b18       0xd8 build/default/production/_ext/334706090/wf_connection_profile.o
 .debug_aranges
                0x00001bf0       0x20 build/default/production/_ext/334706090/wf_easy_config.o
 .debug_aranges
                0x00001c10       0x40 build/default/production/_ext/334706090/wf_eint.o
 .debug_aranges
                0x00001c50       0x68 build/default/production/_ext/334706090/wf_event_handler.o
 .debug_aranges
                0x00001cb8       0x40 build/default/production/_ext/334706090/wf_init.o
 .debug_aranges
                0x00001cf8       0x90 build/default/production/_ext/334706090/wf_power_save.o
 .debug_aranges
                0x00001d88       0x30 build/default/production/_ext/334706090/wf_scan.o
 .debug_aranges
                0x00001db8       0x40 build/default/production/_ext/334706090/wf_spi.o
 .debug_aranges
                0x00001df8      0x108 build/default/production/_ext/334706090/mrf24w_mac_pic32.o
 .debug_aranges
                0x00001f00       0x70 build/default/production/_ext/334706090/mrf24w_events.o
 .debug_aranges
                0x00001f70       0xb8 build/default/production/_ext/334706090/wf_debug_output.o
 .debug_aranges
                0x00002028       0x90 build/default/production/_ext/334706090/wf_commands.o
 .debug_aranges
                0x000020b8       0xd8 build/default/production/_ext/334706090/wf_driver_com_24g.o
 .debug_aranges
                0x00002190       0xc0 build/default/production/_ext/334706090/wf_driver_raw_24g.o
 .debug_aranges
                0x00002250      0x110 build/default/production/_ext/334706090/wf_mac_24g.o
 .debug_aranges
                0x00002360       0x40 build/default/production/_ext/334706090/wf_mgmt_msg_24g.o
 .debug_aranges
                0x000023a0       0xe8 build/default/production/_ext/334706090/wf_param_msg_24g.o
 .debug_aranges
                0x00002488       0x38 build/default/production/_ext/334706090/wf_configData.o
 .debug_aranges
                0x000024c0       0x38 build/default/production/_ext/1472/main_demo.o
 .debug_aranges
                0x000024f8       0x20 build/default/production/_ext/1472/wf_config.o
 .debug_aranges
                0x00002518      0x158 build/default/production/_ext/1472/custom_http_app.o
 .debug_aranges
                0x00002670       0x38 build/default/production/_ext/1472/tcp6_demo_app.o
 .debug_aranges
                0x000026a8       0x20 c:/program files (x86)/microchip/xc32/v1.10/bin/../lib/gcc/pic32mx/4.5.1/../../../../pic32mx/lib/size\libmchp_peripheral.a(open_core_timer_lib.o)
 .debug_aranges
                0x000026c8       0x20 c:/program files (x86)/microchip/xc32/v1.10/bin/../lib/gcc/pic32mx/4.5.1/../../../../pic32mx/lib/size\libmchp_peripheral_32MX795F512L.a(soft_reset_lib.o)
 .debug_aranges
                0x000026e8       0x28 c:/program files (x86)/microchip/xc32/v1.10/bin/../lib/gcc/pic32mx/4.5.1/../../../../pic32mx/lib/size\libmchp_peripheral_32MX795F512L.a(pcache.o)
 .debug_aranges
                0x00002710       0x20 c:/program files (x86)/microchip/xc32/v1.10/bin/../lib/gcc/pic32mx/4.5.1/../../../../pic32mx/lib/size\libmchp_peripheral_32MX795F512L.a(int_disable_interrupts_lib.o)
 .debug_aranges
                0x00002730       0x20 c:/program files (x86)/microchip/xc32/v1.10/bin/../lib/gcc/pic32mx/4.5.1/../../../../pic32mx/lib/size\libmchp_peripheral_32MX795F512L.a(int_restore_interrupts_lib.o)
 .debug_aranges
                0x00002750       0x20 c:/program files (x86)/microchip/xc32/v1.10/bin/../lib/gcc/pic32mx/4.5.1/../../../../pic32mx/lib/size\libmchp_peripheral_32MX795F512L.a(int_enable_mv_int_lib.o)
 .debug_aranges
                0x00002770       0x60 c:/program files (x86)/microchip/xc32/v1.10/bin/../lib/gcc/pic32mx/4.5.1/../../../../pic32mx/lib/size\libmchp_peripheral_32MX795F512L.a(int_tbl_lib.o)
 .debug_aranges
                0x000027d0       0x20 c:/program files (x86)/microchip/xc32/v1.10/bin/../lib/gcc/pic32mx/4.5.1/../../../../pic32mx/lib/size\libmchp_peripheral_32MX795F512L.a(rtcc_init_lib.o)
 .debug_aranges
                0x000027f0       0x20 c:/program files (x86)/microchip/xc32/v1.10/bin/../lib/gcc/pic32mx/4.5.1/../../../../pic32mx/lib/size\libmchp_peripheral_32MX795F512L.a(rtcc_open_lib.o)
 .debug_aranges
                0x00002810       0x20 c:/program files (x86)/microchip/xc32/v1.10/bin/../lib/gcc/pic32mx/4.5.1/../../../../pic32mx/lib/size\libmchp_peripheral_32MX795F512L.a(spi_chn_data_rdy_lib.o)
 .debug_aranges
                0x00002830       0x28 c:/program files (x86)/microchip/xc32/v1.10/bin/../lib/gcc/pic32mx/4.5.1/../../../../pic32mx/lib/size\libmchp_peripheral_32MX795F512L.a(spi_chn_getc_lib.o)
 .debug_aranges
                0x00002858       0x20 c:/program files (x86)/microchip/xc32/v1.10/bin/../lib/gcc/pic32mx/4.5.1/../../../../pic32mx/lib/size\libmchp_peripheral_32MX795F512L.a(spi_chn_open_lib.o)
 .debug_aranges
                0x00002878       0x30 c:/program files (x86)/microchip/xc32/v1.10/bin/../lib/gcc/pic32mx/4.5.1/../../../../pic32mx/lib/size\libmchp_peripheral_32MX795F512L.a(spi_chn_putc_lib.o)
 .debug_aranges
                0x000028a8       0x20 c:/program files (x86)/microchip/xc32/v1.10/bin/../lib/gcc/pic32mx/4.5.1/../../../../pic32mx/lib/size\libmchp_peripheral_32MX795F512L.a(spi_chn_tx_buff_empty_lib.o)
 .debug_aranges
                0x000028c8       0x20 c:/program files (x86)/microchip/xc32/v1.10/bin/../lib/gcc/pic32mx/4.5.1/../../../../pic32mx/lib/size\libmchp_peripheral_32MX795F512L.a(port_set_pins_digital_in_lib.o)
 .debug_aranges
                0x000028e8       0x20 c:/program files (x86)/microchip/xc32/v1.10/bin/../lib/gcc/pic32mx/4.5.1/../../../../pic32mx/lib/size\libmchp_peripheral_32MX795F512L.a(port_set_pins_digital_out_lib.o)
 .debug_aranges
                0x00002908       0x20 c:/program files (x86)/microchip/xc32/v1.10/bin/../lib/gcc/pic32mx/4.5.1/../../../../pic32mx/lib/size\libmchp_peripheral_32MX795F512L.a(int_enable_interrupts_lib.o)
 .debug_aranges
                0x00002928       0x28 c:/program files (x86)/microchip/xc32/v1.10/bin/../lib/gcc/pic32mx/4.5.1/../../../../pic32mx/lib/size\libmchp_peripheral_32MX795F512L.a(_rtcc_wait_clock_off_lib.o)
 .debug_aranges
                0x00002950       0x20 c:/program files (x86)/microchip/xc32/v1.10/bin/../lib/gcc/pic32mx/4.5.1/../../../../pic32mx/lib/size\libmchp_peripheral_32MX795F512L.a(read_core_timer_lib.o)
 .debug_aranges
                0x00002970       0x20 c:/program files (x86)/microchip/xc32/v1.10/bin/../lib/gcc/pic32mx/4.5.1/size\libgcc.a(_udivdi3.o)
 .debug_aranges
                0x00002990       0x20 c:/program files (x86)/microchip/xc32/v1.10/bin/../lib/gcc/pic32mx/4.5.1/../../../../pic32mx/lib/size\libpic32.a(default-bootstrap-exception-handler.o)
 .debug_aranges
                0x000029b0       0x20 c:/program files (x86)/microchip/xc32/v1.10/bin/../lib/gcc/pic32mx/4.5.1/../../../../pic32mx/lib/size\libpic32.a(default-on-reset.o)
 .debug_aranges
                0x000029d0       0x20 c:/program files (x86)/microchip/xc32/v1.10/bin/../lib/gcc/pic32mx/4.5.1/../../../../pic32mx/lib/size\libpic32.a(default-on-bootstrap.o)
 .debug_aranges
                0x000029f0       0x20 c:/program files (x86)/microchip/xc32/v1.10/bin/../lib/gcc/pic32mx/4.5.1/../../../../pic32mx/lib/size\libc.a(atoi.o)
 .debug_aranges
                0x00002a10       0x20 c:/program files (x86)/microchip/xc32/v1.10/bin/../lib/gcc/pic32mx/4.5.1/../../../../pic32mx/lib/size\libc.a(atol.o)
 .debug_aranges
                0x00002a30       0x30 c:/program files (x86)/microchip/xc32/v1.10/bin/../lib/gcc/pic32mx/4.5.1/../../../../pic32mx/lib/size\libc.a(malloc.o)
 .debug_aranges
                0x00002a60       0x28 c:/program files (x86)/microchip/xc32/v1.10/bin/../lib/gcc/pic32mx/4.5.1/../../../../pic32mx/lib/size\libc.a(rand.o)
 .debug_aranges
                0x00002a88       0x20 c:/program files (x86)/microchip/xc32/v1.10/bin/../lib/gcc/pic32mx/4.5.1/../../../../pic32mx/lib/size\libc.a(strcat.o)
 .debug_aranges
                0x00002aa8       0x20 c:/program files (x86)/microchip/xc32/v1.10/bin/../lib/gcc/pic32mx/4.5.1/../../../../pic32mx/lib/size\libc.a(strchr.o)
 .debug_aranges
                0x00002ac8       0x20 c:/program files (x86)/microchip/xc32/v1.10/bin/../lib/gcc/pic32mx/4.5.1/../../../../pic32mx/lib/size\libc.a(strncat.o)
 .debug_aranges
                0x00002ae8       0x20 c:/program files (x86)/microchip/xc32/v1.10/bin/../lib/gcc/pic32mx/4.5.1/../../../../pic32mx/lib/size\libc.a(strncmp.o)
 .debug_aranges
                0x00002b08       0x20 c:/program files (x86)/microchip/xc32/v1.10/bin/../lib/gcc/pic32mx/4.5.1/../../../../pic32mx/lib/size\libc.a(strncpy.o)
 .debug_aranges
                0x00002b28       0x20 c:/program files (x86)/microchip/xc32/v1.10/bin/../lib/gcc/pic32mx/4.5.1/../../../../pic32mx/lib/size\libc.a(strrchr.o)
 .debug_aranges
                0x00002b48       0x20 c:/program files (x86)/microchip/xc32/v1.10/bin/../lib/gcc/pic32mx/4.5.1/../../../../pic32mx/lib/size\libc.a(strstr.o)
 .debug_aranges
                0x00002b68       0x28 c:/program files (x86)/microchip/xc32/v1.10/bin/../lib/gcc/pic32mx/4.5.1/../../../../pic32mx/lib/size\libc.a(strtol.o)
 .debug_aranges
                0x00002b90       0x20 c:/program files (x86)/microchip/xc32/v1.10/bin/../lib/gcc/pic32mx/4.5.1/../../../../pic32mx/lib/size\libc.a(snprintf_cdnopsuxX.eo)
 .debug_aranges
                0x00002bb0       0x20 c:/program files (x86)/microchip/xc32/v1.10/bin/../lib/gcc/pic32mx/4.5.1/../../../../pic32mx/lib/size\libc.a(sprintf_cdnopsuxX.eo)
 .debug_aranges
                0x00002bd0       0x20 c:/program files (x86)/microchip/xc32/v1.10/bin/../lib/gcc/pic32mx/4.5.1/../../../../pic32mx/lib/size\libc.a(vsnprintf_cdnopsuxX.eo)
 .debug_aranges
                0x00002bf0       0x20 c:/program files (x86)/microchip/xc32/v1.10/bin/../lib/gcc/pic32mx/4.5.1/../../../../pic32mx/lib/size\libc.a(vsnprintf.o)
 .debug_aranges
                0x00002c10       0xa0 c:/program files (x86)/microchip/xc32/v1.10/bin/../lib/gcc/pic32mx/4.5.1/../../../../pic32mx/lib/size\libc.a(ctypef.o)
 .debug_aranges
                0x00002cb0       0x20 c:/program files (x86)/microchip/xc32/v1.10/bin/../lib/gcc/pic32mx/4.5.1/../../../../pic32mx/lib/size\libc.a(doprnt_cdnopsuxX.eo)
 .debug_aranges
                0x00002cd0       0x30 c:/program files (x86)/microchip/xc32/v1.10/bin/../lib/gcc/pic32mx/4.5.1/../../../../pic32mx/lib/size\libc.a(doprnt.o)
 .debug_aranges
                0x00002d00       0x20 c:/program files (x86)/microchip/xc32/v1.10/bin/../lib/gcc/pic32mx/4.5.1/../../../../pic32mx/lib/size\libc.a(_fputc_simple.o)
 .debug_aranges
                0x00002d20       0x20 c:/program files (x86)/microchip/xc32/v1.10/bin/../lib/gcc/pic32mx/4.5.1/../../../../pic32mx/lib/size\libc.a(_flsbuf_simple.o)
 .debug_aranges
                0x00002d40       0x40 c:/program files (x86)/microchip/xc32/v1.10/bin/../lib/gcc/pic32mx/4.5.1/../../../../pic32mx/lib/size\libpic32.a(sbrk.o)
 .debug_aranges
                0x00002d80       0x20 c:/program files (x86)/microchip/xc32/v1.10/bin/../lib/gcc/pic32mx/4.5.1/../../../../pic32mx/lib/size\libpic32.a(write.o)
 .debug_aranges
                0x00002da0       0x20 c:/program files (x86)/microchip/xc32/v1.10/bin/../lib/gcc/pic32mx/4.5.1/../../../../pic32mx/lib/size\libpic32.a(_mon_putc.o)
 .debug_aranges
                0x00002dc0       0x20 c:/program files (x86)/microchip/xc32/v1.10/bin/../lib/gcc/pic32mx/4.5.1/../../../../pic32mx/lib/size\libe.a(_floatdisf.o)
 .debug_aranges
                0x00002de0       0x20 c:/program files (x86)/microchip/xc32/v1.10/bin/../lib/gcc/pic32mx/4.5.1/size\libgcc.a(_lshrdi3.o)
 .debug_aranges
                0x00002e00       0x20 c:/program files (x86)/microchip/xc32/v1.10/bin/../lib/gcc/pic32mx/4.5.1/size\libgcc.a(_floatundisf.o)
 .debug_aranges
                0x00002e20       0x20 c:/program files (x86)/microchip/xc32/v1.10/bin/../lib/gcc/pic32mx/4.5.1/size\libgcc.a(_umoddi3.o)
 .debug_aranges
                0x00002e40       0x20 c:/program files (x86)/microchip/xc32/v1.10/bin/../lib/gcc/pic32mx/4.5.1/size\libgcc.a(floatunsisf.o)

.debug_pubnames
                0x00000000     0x5d1b
 *(.debug_pubnames)
 .debug_pubnames
                0x00000000       0x25 build/default/production/_ext/1293749816/bsp.o
 .debug_pubnames
                0x00000025       0x97 build/default/production/_ext/101875047/hashes.o
 .debug_pubnames
                0x000000bc       0x30 build/default/production/_ext/101875047/lfsr.o
 .debug_pubnames
                0x000000ec       0xeb build/default/production/_ext/101875047/big_int.o
 .debug_pubnames
                0x000001d7       0x81 build/default/production/_ext/101875047/helpers.o
 .debug_pubnames
                0x00000258       0xc4 build/default/production/_ext/1472/ping_demo.o
 .debug_pubnames
                0x0000031c      0x393 build/default/production/_ext/365611741/system_services.o
 .debug_pubnames
                0x000006af      0x1e1 build/default/production/_ext/365611741/system_debug.o
 .debug_pubnames
                0x00000890       0x83 build/default/production/_ext/365611741/system_random.o
 .debug_pubnames
                0x00000913       0xab build/default/production/_ext/365611741/system_command.o
 .debug_pubnames
                0x000009be       0xc8 build/default/production/_ext/365611741/system_userio.o
 .debug_pubnames
                0x00000a86      0x575 build/default/production/_ext/97638081/sys_fs.o
 .debug_pubnames
                0x00000ffb      0x17e build/default/production/_ext/97638081/mpfs2.o
 .debug_pubnames
                0x00001179       0x94 build/default/production/_ext/792872985/usart.o
 .debug_pubnames
                0x0000120d       0x77 build/default/production/_ext/792872985/lcd.o
 .debug_pubnames
                0x00001284       0x3a build/default/production/_ext/792872985/drv_spi.o
 .debug_pubnames
                0x000012be       0xaa build/default/production/_ext/792872985/spi_eeprom.o
 .debug_pubnames
                0x00001368      0x169 build/default/production/_ext/792872985/drv_media.o
 .debug_pubnames
                0x000014d1       0x93 build/default/production/_ext/427700826/tcpip_announce.o
 .debug_pubnames
                0x00001564      0x2cc build/default/production/_ext/427700826/http2.o
 .debug_pubnames
                0x00001830      0x1ba build/default/production/_ext/427700826/arp.o
 .debug_pubnames
                0x000019ea       0xfb build/default/production/_ext/427700826/dhcp.o
 .debug_pubnames
                0x00001ae5       0x55 build/default/production/_ext/427700826/dhcps.o
 .debug_pubnames
                0x00001b3a       0x8d build/default/production/_ext/427700826/dns.o
 .debug_pubnames
                0x00001bc7       0x33 build/default/production/_ext/427700826/hash_fnv.o
 .debug_pubnames
                0x00001bfa       0x86 build/default/production/_ext/427700826/hash_tbl.o
 .debug_pubnames
                0x00001c80       0x7e build/default/production/_ext/427700826/icmp.o
 .debug_pubnames
                0x00001cfe      0x47f build/default/production/_ext/427700826/ipv4.o
 .debug_pubnames
                0x0000217d       0x3b build/default/production/_ext/427700826/nbns.o
 .debug_pubnames
                0x000021b8      0x2b3 build/default/production/_ext/427700826/tcp.o
 .debug_pubnames
                0x0000246b      0x18c build/default/production/_ext/427700826/tcpip_heap_alloc.o
 .debug_pubnames
                0x000025f7      0x25a build/default/production/_ext/427700826/udp.o
 .debug_pubnames
                0x00002851      0x1f9 build/default/production/_ext/427700826/tcpip_mac_object.o
 .debug_pubnames
                0x00002a4a      0x781 build/default/production/_ext/427700826/tcpip_manager.o
 .debug_pubnames
                0x000031cb      0x2e1 build/default/production/_ext/427700826/tcpip_helpers.o
 .debug_pubnames
                0x000034ac       0x69 build/default/production/_ext/427700826/tcpip_notify.o
 .debug_pubnames
                0x00003515       0x43 build/default/production/_ext/427700826/zero_conf_link_local.o
 .debug_pubnames
                0x00003558       0x58 build/default/production/_ext/334706090/wf_tx_power.o
 .debug_pubnames
                0x000035b0       0x23 build/default/production/_ext/334706090/wf_connect.o
 .debug_pubnames
                0x000035d3      0x175 build/default/production/_ext/334706090/wf_connection_algorithm.o
 .debug_pubnames
                0x00003748       0x96 build/default/production/_ext/334706090/wf_connection_manager.o
 .debug_pubnames
                0x000037de      0x1ad build/default/production/_ext/334706090/wf_connection_profile.o
 .debug_pubnames
                0x0000398b       0x3b build/default/production/_ext/334706090/wf_easy_config.o
 .debug_pubnames
                0x000039c6       0x72 build/default/production/_ext/334706090/wf_eint.o
 .debug_pubnames
                0x00003a38       0xf9 build/default/production/_ext/334706090/wf_event_handler.o
 .debug_pubnames
                0x00003b31       0x6d build/default/production/_ext/334706090/wf_init.o
 .debug_pubnames
                0x00003b9e      0x149 build/default/production/_ext/334706090/wf_power_save.o
 .debug_pubnames
                0x00003ce7       0x4b build/default/production/_ext/334706090/wf_scan.o
 .debug_pubnames
                0x00003d32       0x67 build/default/production/_ext/334706090/wf_spi.o
 .debug_pubnames
                0x00003d99       0x87 build/default/production/_ext/334706090/mrf24w_mac_pic32.o
 .debug_pubnames
                0x00003e20      0x142 build/default/production/_ext/334706090/mrf24w_events.o
 .debug_pubnames
                0x00003f62      0x139 build/default/production/_ext/334706090/wf_debug_output.o
 .debug_pubnames
                0x0000409b       0x8a build/default/production/_ext/334706090/wf_commands.o
 .debug_pubnames
                0x00004125      0x1f4 build/default/production/_ext/334706090/wf_driver_com_24g.o
 .debug_pubnames
                0x00004319      0x1ef build/default/production/_ext/334706090/wf_driver_raw_24g.o
 .debug_pubnames
                0x00004508      0x2ed build/default/production/_ext/334706090/wf_mac_24g.o
 .debug_pubnames
                0x000047f5       0xb0 build/default/production/_ext/334706090/wf_mgmt_msg_24g.o
 .debug_pubnames
                0x000048a5      0x26d build/default/production/_ext/334706090/wf_param_msg_24g.o
 .debug_pubnames
                0x00004b12       0x93 build/default/production/_ext/334706090/wf_configData.o
 .debug_pubnames
                0x00004ba5      0x1df build/default/production/_ext/1472/main_demo.o
 .debug_pubnames
                0x00004d84       0x26 build/default/production/_ext/1472/wf_config.o
 .debug_pubnames
                0x00004daa      0x3a2 build/default/production/_ext/1472/custom_http_app.o
 .debug_pubnames
                0x0000514c      0x298 build/default/production/_ext/1472/tcp6_demo_app.o
 .debug_pubnames
                0x000053e4       0x24 c:/program files (x86)/microchip/xc32/v1.10/bin/../lib/gcc/pic32mx/4.5.1/../../../../pic32mx/lib/size\libmchp_peripheral.a(open_core_timer_lib.o)
 .debug_pubnames
                0x00005408       0x20 c:/program files (x86)/microchip/xc32/v1.10/bin/../lib/gcc/pic32mx/4.5.1/../../../../pic32mx/lib/size\libmchp_peripheral_32MX795F512L.a(soft_reset_lib.o)
 .debug_pubnames
                0x00005428       0x3b c:/program files (x86)/microchip/xc32/v1.10/bin/../lib/gcc/pic32mx/4.5.1/../../../../pic32mx/lib/size\libmchp_peripheral_32MX795F512L.a(pcache.o)
 .debug_pubnames
                0x00005463       0x2b c:/program files (x86)/microchip/xc32/v1.10/bin/../lib/gcc/pic32mx/4.5.1/../../../../pic32mx/lib/size\libmchp_peripheral_32MX795F512L.a(int_disable_interrupts_lib.o)
 .debug_pubnames
                0x0000548e       0x2b c:/program files (x86)/microchip/xc32/v1.10/bin/../lib/gcc/pic32mx/4.5.1/../../../../pic32mx/lib/size\libmchp_peripheral_32MX795F512L.a(int_restore_interrupts_lib.o)
 .debug_pubnames
                0x000054b9       0x36 c:/program files (x86)/microchip/xc32/v1.10/bin/../lib/gcc/pic32mx/4.5.1/../../../../pic32mx/lib/size\libmchp_peripheral_32MX795F512L.a(int_enable_mv_int_lib.o)
 .debug_pubnames
                0x000054ef       0xca c:/program files (x86)/microchip/xc32/v1.10/bin/../lib/gcc/pic32mx/4.5.1/../../../../pic32mx/lib/size\libmchp_peripheral_32MX795F512L.a(int_tbl_lib.o)
 .debug_pubnames
                0x000055b9       0x1f c:/program files (x86)/microchip/xc32/v1.10/bin/../lib/gcc/pic32mx/4.5.1/../../../../pic32mx/lib/size\libmchp_peripheral_32MX795F512L.a(rtcc_init_lib.o)
 .debug_pubnames
                0x000055d8       0x1f c:/program files (x86)/microchip/xc32/v1.10/bin/../lib/gcc/pic32mx/4.5.1/../../../../pic32mx/lib/size\libmchp_peripheral_32MX795F512L.a(rtcc_open_lib.o)
 .debug_pubnames
                0x000055f7       0x24 c:/program files (x86)/microchip/xc32/v1.10/bin/../lib/gcc/pic32mx/4.5.1/../../../../pic32mx/lib/size\libmchp_peripheral_32MX795F512L.a(spi_chn_data_rdy_lib.o)
 .debug_pubnames
                0x0000561b       0x31 c:/program files (x86)/microchip/xc32/v1.10/bin/../lib/gcc/pic32mx/4.5.1/../../../../pic32mx/lib/size\libmchp_peripheral_32MX795F512L.a(spi_chn_getc_lib.o)
 .debug_pubnames
                0x0000564c       0x21 c:/program files (x86)/microchip/xc32/v1.10/bin/../lib/gcc/pic32mx/4.5.1/../../../../pic32mx/lib/size\libmchp_peripheral_32MX795F512L.a(spi_chn_open_lib.o)
 .debug_pubnames
                0x0000566d       0x43 c:/program files (x86)/microchip/xc32/v1.10/bin/../lib/gcc/pic32mx/4.5.1/../../../../pic32mx/lib/size\libmchp_peripheral_32MX795F512L.a(spi_chn_putc_lib.o)
 .debug_pubnames
                0x000056b0       0x28 c:/program files (x86)/microchip/xc32/v1.10/bin/../lib/gcc/pic32mx/4.5.1/../../../../pic32mx/lib/size\libmchp_peripheral_32MX795F512L.a(spi_chn_tx_buff_empty_lib.o)
 .debug_pubnames
                0x000056d8       0x2b c:/program files (x86)/microchip/xc32/v1.10/bin/../lib/gcc/pic32mx/4.5.1/../../../../pic32mx/lib/size\libmchp_peripheral_32MX795F512L.a(port_set_pins_digital_in_lib.o)
 .debug_pubnames
                0x00005703       0x2c c:/program files (x86)/microchip/xc32/v1.10/bin/../lib/gcc/pic32mx/4.5.1/../../../../pic32mx/lib/size\libmchp_peripheral_32MX795F512L.a(port_set_pins_digital_out_lib.o)
 .debug_pubnames
                0x0000572f       0x2a c:/program files (x86)/microchip/xc32/v1.10/bin/../lib/gcc/pic32mx/4.5.1/../../../../pic32mx/lib/size\libmchp_peripheral_32MX795F512L.a(int_enable_interrupts_lib.o)
 .debug_pubnames
                0x00005759       0x3e c:/program files (x86)/microchip/xc32/v1.10/bin/../lib/gcc/pic32mx/4.5.1/../../../../pic32mx/lib/size\libmchp_peripheral_32MX795F512L.a(_rtcc_wait_clock_off_lib.o)
 .debug_pubnames
                0x00005797       0x24 c:/program files (x86)/microchip/xc32/v1.10/bin/../lib/gcc/pic32mx/4.5.1/../../../../pic32mx/lib/size\libmchp_peripheral_32MX795F512L.a(read_core_timer_lib.o)
 .debug_pubnames
                0x000057bb       0x20 c:/program files (x86)/microchip/xc32/v1.10/bin/../lib/gcc/pic32mx/4.5.1/size\libgcc.a(_udivdi3.o)
 .debug_pubnames
                0x000057db       0x33 c:/program files (x86)/microchip/xc32/v1.10/bin/../lib/gcc/pic32mx/4.5.1/../../../../pic32mx/lib/size\libpic32.a(default-bootstrap-exception-handler.o)
 .debug_pubnames
                0x0000580e       0x20 c:/program files (x86)/microchip/xc32/v1.10/bin/../lib/gcc/pic32mx/4.5.1/../../../../pic32mx/lib/size\libpic32.a(default-on-reset.o)
 .debug_pubnames
                0x0000582e       0x24 c:/program files (x86)/microchip/xc32/v1.10/bin/../lib/gcc/pic32mx/4.5.1/../../../../pic32mx/lib/size\libpic32.a(default-on-bootstrap.o)
 .debug_pubnames
                0x00005852       0x1b c:/program files (x86)/microchip/xc32/v1.10/bin/../lib/gcc/pic32mx/4.5.1/../../../../pic32mx/lib/size\libc.a(atoi.o)
 .debug_pubnames
                0x0000586d       0x1b c:/program files (x86)/microchip/xc32/v1.10/bin/../lib/gcc/pic32mx/4.5.1/../../../../pic32mx/lib/size\libc.a(atol.o)
 .debug_pubnames
                0x00005888       0x32 c:/program files (x86)/microchip/xc32/v1.10/bin/../lib/gcc/pic32mx/4.5.1/../../../../pic32mx/lib/size\libc.a(malloc.o)
 .debug_pubnames
                0x000058ba       0x25 c:/program files (x86)/microchip/xc32/v1.10/bin/../lib/gcc/pic32mx/4.5.1/../../../../pic32mx/lib/size\libc.a(rand.o)
 .debug_pubnames
                0x000058df       0x1d c:/program files (x86)/microchip/xc32/v1.10/bin/../lib/gcc/pic32mx/4.5.1/../../../../pic32mx/lib/size\libc.a(strcat.o)
 .debug_pubnames
                0x000058fc       0x1d c:/program files (x86)/microchip/xc32/v1.10/bin/../lib/gcc/pic32mx/4.5.1/../../../../pic32mx/lib/size\libc.a(strchr.o)
 .debug_pubnames
                0x00005919       0x1e c:/program files (x86)/microchip/xc32/v1.10/bin/../lib/gcc/pic32mx/4.5.1/../../../../pic32mx/lib/size\libc.a(strncat.o)
 .debug_pubnames
                0x00005937       0x1e c:/program files (x86)/microchip/xc32/v1.10/bin/../lib/gcc/pic32mx/4.5.1/../../../../pic32mx/lib/size\libc.a(strncmp.o)
 .debug_pubnames
                0x00005955       0x1e c:/program files (x86)/microchip/xc32/v1.10/bin/../lib/gcc/pic32mx/4.5.1/../../../../pic32mx/lib/size\libc.a(strncpy.o)
 .debug_pubnames
                0x00005973       0x1e c:/program files (x86)/microchip/xc32/v1.10/bin/../lib/gcc/pic32mx/4.5.1/../../../../pic32mx/lib/size\libc.a(strrchr.o)
 .debug_pubnames
                0x00005991       0x1d c:/program files (x86)/microchip/xc32/v1.10/bin/../lib/gcc/pic32mx/4.5.1/../../../../pic32mx/lib/size\libc.a(strstr.o)
 .debug_pubnames
                0x000059ae       0x29 c:/program files (x86)/microchip/xc32/v1.10/bin/../lib/gcc/pic32mx/4.5.1/../../../../pic32mx/lib/size\libc.a(strtol.o)
 .debug_pubnames
                0x000059d7       0x2a c:/program files (x86)/microchip/xc32/v1.10/bin/../lib/gcc/pic32mx/4.5.1/../../../../pic32mx/lib/size\libc.a(snprintf_cdnopsuxX.eo)
 .debug_pubnames
                0x00005a01       0x29 c:/program files (x86)/microchip/xc32/v1.10/bin/../lib/gcc/pic32mx/4.5.1/../../../../pic32mx/lib/size\libc.a(sprintf_cdnopsuxX.eo)
 .debug_pubnames
                0x00005a2a       0x2b c:/program files (x86)/microchip/xc32/v1.10/bin/../lib/gcc/pic32mx/4.5.1/../../../../pic32mx/lib/size\libc.a(vsnprintf_cdnopsuxX.eo)
 .debug_pubnames
                0x00005a55       0x20 c:/program files (x86)/microchip/xc32/v1.10/bin/../lib/gcc/pic32mx/4.5.1/../../../../pic32mx/lib/size\libc.a(vsnprintf.o)
 .debug_pubnames
                0x00005a75       0xe1 c:/program files (x86)/microchip/xc32/v1.10/bin/../lib/gcc/pic32mx/4.5.1/../../../../pic32mx/lib/size\libc.a(ctypef.o)
 .debug_pubnames
                0x00005b56       0x2a c:/program files (x86)/microchip/xc32/v1.10/bin/../lib/gcc/pic32mx/4.5.1/../../../../pic32mx/lib/size\libc.a(doprnt_cdnopsuxX.eo)
 .debug_pubnames
                0x00005b80       0x1f c:/program files (x86)/microchip/xc32/v1.10/bin/../lib/gcc/pic32mx/4.5.1/../../../../pic32mx/lib/size\libc.a(doprnt.o)
 .debug_pubnames
                0x00005b9f       0x1c c:/program files (x86)/microchip/xc32/v1.10/bin/../lib/gcc/pic32mx/4.5.1/../../../../pic32mx/lib/size\libc.a(_fputc_simple.o)
 .debug_pubnames
                0x00005bbb       0x1e c:/program files (x86)/microchip/xc32/v1.10/bin/../lib/gcc/pic32mx/4.5.1/../../../../pic32mx/lib/size\libc.a(_flsbuf_simple.o)
 .debug_pubnames
                0x00005bd9       0x5c c:/program files (x86)/microchip/xc32/v1.10/bin/../lib/gcc/pic32mx/4.5.1/../../../../pic32mx/lib/size\libpic32.a(sbrk.o)
 .debug_pubnames
                0x00005c35       0x1c c:/program files (x86)/microchip/xc32/v1.10/bin/../lib/gcc/pic32mx/4.5.1/../../../../pic32mx/lib/size\libpic32.a(write.o)
 .debug_pubnames
                0x00005c51       0x20 c:/program files (x86)/microchip/xc32/v1.10/bin/../lib/gcc/pic32mx/4.5.1/../../../../pic32mx/lib/size\libpic32.a(_mon_putc.o)
 .debug_pubnames
                0x00005c71       0x22 c:/program files (x86)/microchip/xc32/v1.10/bin/../lib/gcc/pic32mx/4.5.1/../../../../pic32mx/lib/size\libe.a(_floatdisf.o)
 .debug_pubnames
                0x00005c93       0x20 c:/program files (x86)/microchip/xc32/v1.10/bin/../lib/gcc/pic32mx/4.5.1/size\libgcc.a(_lshrdi3.o)
 .debug_pubnames
                0x00005cb3       0x24 c:/program files (x86)/microchip/xc32/v1.10/bin/../lib/gcc/pic32mx/4.5.1/size\libgcc.a(_floatundisf.o)
 .debug_pubnames
                0x00005cd7       0x20 c:/program files (x86)/microchip/xc32/v1.10/bin/../lib/gcc/pic32mx/4.5.1/size\libgcc.a(_umoddi3.o)
 .debug_pubnames
                0x00005cf7       0x24 c:/program files (x86)/microchip/xc32/v1.10/bin/../lib/gcc/pic32mx/4.5.1/size\libgcc.a(floatunsisf.o)

.debug_info     0x00000000    0xb5a9d
 *(.debug_info .gnu.linkonce.wi.*)
 .debug_info    0x00000000     0x1699 build/default/production/_ext/1293749816/bsp.o
 .debug_info    0x00001699      0x844 build/default/production/_ext/101875047/hashes.o
 .debug_info    0x00001edd      0x23b build/default/production/_ext/101875047/lfsr.o
 .debug_info    0x00002118     0x1759 build/default/production/_ext/101875047/big_int.o
 .debug_info    0x00003871       0xd5 build/default/production/_ext/101875047/big_int_helper_c32.o
 .debug_info    0x00003946      0x52d build/default/production/_ext/101875047/helpers.o
 .debug_info    0x00003e73        0x0 build/default/production/_ext/1472/berkeley_tcp_client_demo.o
 .debug_info    0x00003e73        0x0 build/default/production/_ext/1472/berkeley_tcp_server_demo.o
 .debug_info    0x00003e73        0x0 build/default/production/_ext/1472/berkeley_udp_client_demo.o
 .debug_info    0x00003e73     0x11e8 build/default/production/_ext/1472/generic_tcp_client.o
 .debug_info    0x0000505b     0x11e8 build/default/production/_ext/1472/generic_tcp_server.o
 .debug_info    0x00006243     0x1a83 build/default/production/_ext/1472/ping_demo.o
 .debug_info    0x00007cc6        0x0 build/default/production/_ext/1472/smtp_demo.o
 .debug_info    0x00007cc6     0x3482 build/default/production/_ext/365611741/system_services.o
 .debug_info    0x0000b148     0x1752 build/default/production/_ext/365611741/system_debug.o
 .debug_info    0x0000c89a     0x1c6c build/default/production/_ext/365611741/system_random.o
 .debug_info    0x0000e506     0x1a8c build/default/production/_ext/365611741/system_command.o
 .debug_info    0x0000ff92     0x21e2 build/default/production/_ext/365611741/system_userio.o
 .debug_info    0x00012174     0x2c4a build/default/production/_ext/97638081/sys_fs.o
 .debug_info    0x00014dbe     0x1cbd build/default/production/_ext/97638081/mpfs2.o
 .debug_info    0x00016a7b     0x1688 build/default/production/_ext/792872985/usart.o
 .debug_info    0x00018103     0x1b60 build/default/production/_ext/792872985/lcd.o
 .debug_info    0x00019c63     0x16ae build/default/production/_ext/792872985/drv_spi.o
 .debug_info    0x0001b311        0x0 build/default/production/_ext/792872985/db_appio.o
 .debug_info    0x0001b311     0x11a5 build/default/production/_ext/792872985/spi_ram.o
 .debug_info    0x0001c4b6     0x1ffc build/default/production/_ext/792872985/spi_eeprom.o
 .debug_info    0x0001e4b2     0x11a7 build/default/production/_ext/792872985/spi_flash.o
 .debug_info    0x0001f659     0x230f build/default/production/_ext/792872985/drv_media.o
 .debug_info    0x00021968     0x2340 build/default/production/_ext/427700826/tcpip_announce.o
 .debug_info    0x00023ca8     0x3f0f build/default/production/_ext/427700826/http2.o
 .debug_info    0x00027bb7     0x13a6 build/default/production/_ext/427700826/arcfour.o
 .debug_info    0x00028f5d     0x3c72 build/default/production/_ext/427700826/arp.o
 .debug_info    0x0002cbcf     0x13ab build/default/production/_ext/427700826/berkeley_api.o
 .debug_info    0x0002df7a     0x3855 build/default/production/_ext/427700826/dhcp.o
 .debug_info    0x000317cf     0x1479 build/default/production/_ext/427700826/dhcps.o
 .debug_info    0x00032c48     0x29ef build/default/production/_ext/427700826/dns.o
 .debug_info    0x00035637     0x13a3 build/default/production/_ext/427700826/dnss.o
 .debug_info    0x000369da     0x13a6 build/default/production/_ext/427700826/dyn_dns.o
 .debug_info    0x00037d80     0x13a8 build/default/production/_ext/427700826/enc28_mac.o
 .debug_info    0x00039128     0x13a7 build/default/production/_ext/427700826/enc28j60.o
 .debug_info    0x0003a4cf     0x13a9 build/default/production/_ext/427700826/encs24j600.o
 .debug_info    0x0003b878     0x13a9 build/default/production/_ext/427700826/encx24_mac.o
 .debug_info    0x0003cc21     0x13b0 build/default/production/_ext/427700826/eth_pic32_ext_phy.o
 .debug_info    0x0003dfd1     0x13b8 build/default/production/_ext/427700826/eth_pic32_ext_phy_dp83848.o
 .debug_info    0x0003f389     0x13b0 build/default/production/_ext/427700826/eth_pic32_int_mac.o
 .debug_info    0x00040739     0x13a2 build/default/production/_ext/427700826/ftp.o
 .debug_info    0x00041adb      0x297 build/default/production/_ext/427700826/hash_fnv.o
 .debug_info    0x00041d72      0x7b5 build/default/production/_ext/427700826/hash_tbl.o
 .debug_info    0x00042527     0x27b7 build/default/production/_ext/427700826/icmp.o
 .debug_info    0x00044cde     0x13a5 build/default/production/_ext/427700826/icmpv6.o
 .debug_info    0x00046083     0x3bc7 build/default/production/_ext/427700826/ipv4.o
 .debug_info    0x00049c4a     0x13a3 build/default/production/_ext/427700826/ipv6.o
 .debug_info    0x0004afed     0x13af build/default/production/_ext/427700826/mac_events_pic32.o
 .debug_info    0x0004c39c     0x27e5 build/default/production/_ext/427700826/nbns.o
 .debug_info    0x0004eb81     0x13a2 build/default/production/_ext/427700826/ndp.o
 .debug_info    0x0004ff23     0x13ab build/default/production/_ext/427700826/tcpip_reboot.o
 .debug_info    0x000512ce     0x13a2 build/default/production/_ext/427700826/rsa.o
 .debug_info    0x00052670     0x13a3 build/default/production/_ext/427700826/smtp.o
 .debug_info    0x00053a13     0x13a3 build/default/production/_ext/427700826/snmp.o
 .debug_info    0x00054db6     0x13a5 build/default/production/_ext/427700826/snmpv3.o
 .debug_info    0x0005615b     0x13a9 build/default/production/_ext/427700826/snmpv3_usm.o
 .debug_info    0x00057504     0x13a3 build/default/production/_ext/427700826/sntp.o
 .debug_info    0x000588a7     0x13a2 build/default/production/_ext/427700826/ssl.o
 .debug_info    0x00059c49     0x58f3 build/default/production/_ext/427700826/tcp.o
 .debug_info    0x0005f53c     0x1f0b build/default/production/_ext/427700826/tcpip_heap_alloc.o
 .debug_info    0x00061447     0x13ac build/default/production/_ext/427700826/tcpip_storage.o
 .debug_info    0x000627f3     0x13a5 build/default/production/_ext/427700826/telnet.o
 .debug_info    0x00063b98     0x13a4 build/default/production/_ext/427700826/tftpc.o
 .debug_info    0x00064f3c     0x428f build/default/production/_ext/427700826/udp.o
 .debug_info    0x000691cb     0x223e build/default/production/_ext/427700826/tcpip_mac_object.o
 .debug_info    0x0006b409     0x52be build/default/production/_ext/427700826/tcpip_manager.o
 .debug_info    0x000706c7     0x2675 build/default/production/_ext/427700826/tcpip_helpers.o
 .debug_info    0x00072d3c     0x13ad build/default/production/_ext/427700826/tcpip_commands.o
 .debug_info    0x000740e9     0x13a4 build/default/production/_ext/427700826/iperf.o
 .debug_info    0x0007548d       0xd2 build/default/production/_ext/427700826/tcpip_helper_c32.o
 .debug_info    0x0007555f      0x3aa build/default/production/_ext/427700826/tcpip_notify.o
 .debug_info    0x00075909     0x13af build/default/production/_ext/427700826/zero_conf_helper.o
 .debug_info    0x00076cb8     0x1470 build/default/production/_ext/427700826/zero_conf_link_local.o
 .debug_info    0x00078128     0x13b6 build/default/production/_ext/427700826/zero_conf_multicast_dns.o
 .debug_info    0x000794de     0x191e build/default/production/_ext/334706090/wf_tx_power.o
 .debug_info    0x0007adfc     0x1b68 build/default/production/_ext/334706090/wf_connect.o
 .debug_info    0x0007c964     0x2188 build/default/production/_ext/334706090/wf_connection_algorithm.o
 .debug_info    0x0007eaec     0x246e build/default/production/_ext/334706090/wf_connection_manager.o
 .debug_info    0x00080f5a     0x2667 build/default/production/_ext/334706090/wf_connection_profile.o
 .debug_info    0x000835c1     0x17f1 build/default/production/_ext/334706090/wf_easy_config.o
 .debug_info    0x00084db2     0x2229 build/default/production/_ext/334706090/wf_eint.o
 .debug_info    0x00086fdb     0x1abb build/default/production/_ext/334706090/wf_event_handler.o
 .debug_info    0x00088a96     0x1cb2 build/default/production/_ext/334706090/wf_init.o
 .debug_info    0x0008a748     0x1f2b build/default/production/_ext/334706090/wf_power_save.o
 .debug_info    0x0008c673     0x209c build/default/production/_ext/334706090/wf_scan.o
 .debug_info    0x0008e70f     0x1bd2 build/default/production/_ext/334706090/wf_spi.o
 .debug_info    0x000902e1     0x3440 build/default/production/_ext/334706090/mrf24w_mac_pic32.o
 .debug_info    0x00093721     0x1df5 build/default/production/_ext/334706090/mrf24w_events.o
 .debug_info    0x00095516     0x2923 build/default/production/_ext/334706090/wf_debug_output.o
 .debug_info    0x00097e39     0x22a5 build/default/production/_ext/334706090/wf_commands.o
 .debug_info    0x0009a0de     0x13ad build/default/production/_ext/334706090/wf_pbkdf2.o
 .debug_info    0x0009b48b     0x26c8 build/default/production/_ext/334706090/wf_driver_com_24g.o
 .debug_info    0x0009db53     0x1de5 build/default/production/_ext/334706090/wf_driver_raw_24g.o
 .debug_info    0x0009f938     0x2721 build/default/production/_ext/334706090/wf_mac_24g.o
 .debug_info    0x000a2059     0x1eca build/default/production/_ext/334706090/wf_mgmt_msg_24g.o
 .debug_info    0x000a3f23     0x294b build/default/production/_ext/334706090/wf_param_msg_24g.o
 .debug_info    0x000a686e     0x1c82 build/default/production/_ext/334706090/wf_configData.o
 .debug_info    0x000a84f0     0x262f build/default/production/_ext/1472/main_demo.o
 .debug_info    0x000aab1f        0x0 build/default/production/_ext/1472/custom_snmp_app.o
 .debug_info    0x000aab1f        0x0 build/default/production/_ext/1472/custom_ssl_cert.o
 .debug_info    0x000aab1f     0x1188 build/default/production/_ext/1472/mpfs_img2.o
 .debug_info    0x000abca7     0x141e build/default/production/_ext/1472/wf_config.o
 .debug_info    0x000ad0c5     0x282d build/default/production/_ext/1472/custom_http_app.o
 .debug_info    0x000af8f2     0x24d2 build/default/production/_ext/1472/tcp6_demo_app.o
 .debug_info    0x000b1dc4       0xbf c:/program files (x86)/microchip/xc32/v1.10/bin/../lib/gcc/pic32mx/4.5.1/../../../../pic32mx/lib/size\libmchp_peripheral.a(open_core_timer_lib.o)
 .debug_info    0x000b1e83       0xc7 c:/program files (x86)/microchip/xc32/v1.10/bin/../lib/gcc/pic32mx/4.5.1/../../../../pic32mx/lib/size\libmchp_peripheral_32MX795F512L.a(soft_reset_lib.o)
 .debug_info    0x000b1f4a       0xd4 c:/program files (x86)/microchip/xc32/v1.10/bin/../lib/gcc/pic32mx/4.5.1/../../../../pic32mx/lib/size\libmchp_peripheral_32MX795F512L.a(pcache.o)
 .debug_info    0x000b201e       0xcb c:/program files (x86)/microchip/xc32/v1.10/bin/../lib/gcc/pic32mx/4.5.1/../../../../pic32mx/lib/size\libmchp_peripheral_32MX795F512L.a(int_disable_interrupts_lib.o)
 .debug_info    0x000b20e9       0xcb c:/program files (x86)/microchip/xc32/v1.10/bin/../lib/gcc/pic32mx/4.5.1/../../../../pic32mx/lib/size\libmchp_peripheral_32MX795F512L.a(int_restore_interrupts_lib.o)
 .debug_info    0x000b21b4       0xd1 c:/program files (x86)/microchip/xc32/v1.10/bin/../lib/gcc/pic32mx/4.5.1/../../../../pic32mx/lib/size\libmchp_peripheral_32MX795F512L.a(int_enable_mv_int_lib.o)
 .debug_info    0x000b2285      0x1ab c:/program files (x86)/microchip/xc32/v1.10/bin/../lib/gcc/pic32mx/4.5.1/../../../../pic32mx/lib/size\libmchp_peripheral_32MX795F512L.a(int_tbl_lib.o)
 .debug_info    0x000b2430      0x121 c:/program files (x86)/microchip/xc32/v1.10/bin/../lib/gcc/pic32mx/4.5.1/../../../../pic32mx/lib/size\libmchp_peripheral_32MX795F512L.a(rtcc_init_lib.o)
 .debug_info    0x000b2551      0x121 c:/program files (x86)/microchip/xc32/v1.10/bin/../lib/gcc/pic32mx/4.5.1/../../../../pic32mx/lib/size\libmchp_peripheral_32MX795F512L.a(rtcc_open_lib.o)
 .debug_info    0x000b2672       0xd1 c:/program files (x86)/microchip/xc32/v1.10/bin/../lib/gcc/pic32mx/4.5.1/../../../../pic32mx/lib/size\libmchp_peripheral_32MX795F512L.a(spi_chn_data_rdy_lib.o)
 .debug_info    0x000b2743       0xe4 c:/program files (x86)/microchip/xc32/v1.10/bin/../lib/gcc/pic32mx/4.5.1/../../../../pic32mx/lib/size\libmchp_peripheral_32MX795F512L.a(spi_chn_getc_lib.o)
 .debug_info    0x000b2827       0xb7 c:/program files (x86)/microchip/xc32/v1.10/bin/../lib/gcc/pic32mx/4.5.1/../../../../pic32mx/lib/size\libmchp_peripheral_32MX795F512L.a(spi_chn_open_lib.o)
 .debug_info    0x000b28de      0x100 c:/program files (x86)/microchip/xc32/v1.10/bin/../lib/gcc/pic32mx/4.5.1/../../../../pic32mx/lib/size\libmchp_peripheral_32MX795F512L.a(spi_chn_putc_lib.o)
 .debug_info    0x000b29de       0xc7 c:/program files (x86)/microchip/xc32/v1.10/bin/../lib/gcc/pic32mx/4.5.1/../../../../pic32mx/lib/size\libmchp_peripheral_32MX795F512L.a(spi_chn_tx_buff_empty_lib.o)
 .debug_info    0x000b2aa5        0x0 c:/program files (x86)/microchip/xc32/v1.10/bin/../lib/gcc/pic32mx/4.5.1/../../../../pic32mx/lib/size\libmchp_peripheral_32MX795F512L.a(spi_io_tbl_libp.o)
 .debug_info    0x000b2aa5        0x0 c:/program files (x86)/microchip/xc32/v1.10/bin/../lib/gcc/pic32mx/4.5.1/../../../../pic32mx/lib/size\libmchp_peripheral_32MX795F512L.a(spi_map_tbl_libp.o)
 .debug_info    0x000b2aa5       0xcf c:/program files (x86)/microchip/xc32/v1.10/bin/../lib/gcc/pic32mx/4.5.1/../../../../pic32mx/lib/size\libmchp_peripheral_32MX795F512L.a(port_set_pins_digital_in_lib.o)
 .debug_info    0x000b2b74       0xd1 c:/program files (x86)/microchip/xc32/v1.10/bin/../lib/gcc/pic32mx/4.5.1/../../../../pic32mx/lib/size\libmchp_peripheral_32MX795F512L.a(port_set_pins_digital_out_lib.o)
 .debug_info    0x000b2c45        0x0 c:/program files (x86)/microchip/xc32/v1.10/bin/../lib/gcc/pic32mx/4.5.1/../../../../pic32mx/lib/size\libmchp_peripheral_32MX795F512L.a(_ports_tbl_libp.o)
 .debug_info    0x000b2c45       0xc9 c:/program files (x86)/microchip/xc32/v1.10/bin/../lib/gcc/pic32mx/4.5.1/../../../../pic32mx/lib/size\libmchp_peripheral_32MX795F512L.a(int_enable_interrupts_lib.o)
 .debug_info    0x000b2d0e       0xfc c:/program files (x86)/microchip/xc32/v1.10/bin/../lib/gcc/pic32mx/4.5.1/../../../../pic32mx/lib/size\libmchp_peripheral_32MX795F512L.a(_rtcc_wait_clock_off_lib.o)
 .debug_info    0x000b2e0a       0xbf c:/program files (x86)/microchip/xc32/v1.10/bin/../lib/gcc/pic32mx/4.5.1/../../../../pic32mx/lib/size\libmchp_peripheral_32MX795F512L.a(read_core_timer_lib.o)
 .debug_info    0x000b2ec9      0x74f c:/program files (x86)/microchip/xc32/v1.10/bin/../lib/gcc/pic32mx/4.5.1/size\libgcc.a(_udivdi3.o)
 .debug_info    0x000b3618       0xdf c:/program files (x86)/microchip/xc32/v1.10/bin/../lib/gcc/pic32mx/4.5.1/../../../../pic32mx/lib/size\libpic32.a(default-bootstrap-exception-handler.o)
 .debug_info    0x000b36f7       0xb9 c:/program files (x86)/microchip/xc32/v1.10/bin/../lib/gcc/pic32mx/4.5.1/../../../../pic32mx/lib/size\libpic32.a(default-on-reset.o)
 .debug_info    0x000b37b0       0xc1 c:/program files (x86)/microchip/xc32/v1.10/bin/../lib/gcc/pic32mx/4.5.1/../../../../pic32mx/lib/size\libpic32.a(default-on-bootstrap.o)
 .debug_info    0x000b3871        0x0 c:/program files (x86)/microchip/xc32/v1.10/bin/../lib/gcc/pic32mx/4.5.1/../../../../pic32mx/lib/size\libpic32.a(errno.o)
 .debug_info    0x000b3871       0xaa c:/program files (x86)/microchip/xc32/v1.10/bin/../lib/gcc/pic32mx/4.5.1/../../../../pic32mx/lib/size\libc.a(atoi.o)
 .debug_info    0x000b391b       0xaa c:/program files (x86)/microchip/xc32/v1.10/bin/../lib/gcc/pic32mx/4.5.1/../../../../pic32mx/lib/size\libc.a(atol.o)
 .debug_info    0x000b39c5        0x0 c:/program files (x86)/microchip/xc32/v1.10/bin/../lib/gcc/pic32mx/4.5.1/../../../../pic32mx/lib/size\libc.a(ctype.o)
 .debug_info    0x000b39c5       0xd7 c:/program files (x86)/microchip/xc32/v1.10/bin/../lib/gcc/pic32mx/4.5.1/../../../../pic32mx/lib/size\libc.a(malloc.o)
 .debug_info    0x000b3a9c       0xbe c:/program files (x86)/microchip/xc32/v1.10/bin/../lib/gcc/pic32mx/4.5.1/../../../../pic32mx/lib/size\libc.a(rand.o)
 .debug_info    0x000b3b5a       0xae c:/program files (x86)/microchip/xc32/v1.10/bin/../lib/gcc/pic32mx/4.5.1/../../../../pic32mx/lib/size\libc.a(strcat.o)
 .debug_info    0x000b3c08       0xae c:/program files (x86)/microchip/xc32/v1.10/bin/../lib/gcc/pic32mx/4.5.1/../../../../pic32mx/lib/size\libc.a(strchr.o)
 .debug_info    0x000b3cb6       0xb0 c:/program files (x86)/microchip/xc32/v1.10/bin/../lib/gcc/pic32mx/4.5.1/../../../../pic32mx/lib/size\libc.a(strncat.o)
 .debug_info    0x000b3d66       0xb0 c:/program files (x86)/microchip/xc32/v1.10/bin/../lib/gcc/pic32mx/4.5.1/../../../../pic32mx/lib/size\libc.a(strncmp.o)
 .debug_info    0x000b3e16       0xb0 c:/program files (x86)/microchip/xc32/v1.10/bin/../lib/gcc/pic32mx/4.5.1/../../../../pic32mx/lib/size\libc.a(strncpy.o)
 .debug_info    0x000b3ec6       0xb0 c:/program files (x86)/microchip/xc32/v1.10/bin/../lib/gcc/pic32mx/4.5.1/../../../../pic32mx/lib/size\libc.a(strrchr.o)
 .debug_info    0x000b3f76       0xae c:/program files (x86)/microchip/xc32/v1.10/bin/../lib/gcc/pic32mx/4.5.1/../../../../pic32mx/lib/size\libc.a(strstr.o)
 .debug_info    0x000b4024       0xc4 c:/program files (x86)/microchip/xc32/v1.10/bin/../lib/gcc/pic32mx/4.5.1/../../../../pic32mx/lib/size\libc.a(strtol.o)
 .debug_info    0x000b40e8       0xbd c:/program files (x86)/microchip/xc32/v1.10/bin/../lib/gcc/pic32mx/4.5.1/../../../../pic32mx/lib/size\libc.a(snprintf_cdnopsuxX.eo)
 .debug_info    0x000b41a5       0xbb c:/program files (x86)/microchip/xc32/v1.10/bin/../lib/gcc/pic32mx/4.5.1/../../../../pic32mx/lib/size\libc.a(sprintf_cdnopsuxX.eo)
 .debug_info    0x000b4260       0xbf c:/program files (x86)/microchip/xc32/v1.10/bin/../lib/gcc/pic32mx/4.5.1/../../../../pic32mx/lib/size\libc.a(vsnprintf_cdnopsuxX.eo)
 .debug_info    0x000b431f       0xb4 c:/program files (x86)/microchip/xc32/v1.10/bin/../lib/gcc/pic32mx/4.5.1/../../../../pic32mx/lib/size\libc.a(vsnprintf.o)
 .debug_info    0x000b43d3      0x212 c:/program files (x86)/microchip/xc32/v1.10/bin/../lib/gcc/pic32mx/4.5.1/../../../../pic32mx/lib/size\libc.a(ctypef.o)
 .debug_info    0x000b45e5       0xbc c:/program files (x86)/microchip/xc32/v1.10/bin/../lib/gcc/pic32mx/4.5.1/../../../../pic32mx/lib/size\libc.a(doprnt_cdnopsuxX.eo)
 .debug_info    0x000b46a1       0xda c:/program files (x86)/microchip/xc32/v1.10/bin/../lib/gcc/pic32mx/4.5.1/../../../../pic32mx/lib/size\libc.a(doprnt.o)
 .debug_info    0x000b477b       0xac c:/program files (x86)/microchip/xc32/v1.10/bin/../lib/gcc/pic32mx/4.5.1/../../../../pic32mx/lib/size\libc.a(_fputc_simple.o)
 .debug_info    0x000b4827        0x0 c:/program files (x86)/microchip/xc32/v1.10/bin/../lib/gcc/pic32mx/4.5.1/../../../../pic32mx/lib/size\libc.a(powersf.o)
 .debug_info    0x000b4827        0x0 c:/program files (x86)/microchip/xc32/v1.10/bin/../lib/gcc/pic32mx/4.5.1/../../../../pic32mx/lib/size\libc.a(_iob.o)
 .debug_info    0x000b4827       0xaf c:/program files (x86)/microchip/xc32/v1.10/bin/../lib/gcc/pic32mx/4.5.1/../../../../pic32mx/lib/size\libc.a(_flsbuf_simple.o)
 .debug_info    0x000b48d6      0x112 c:/program files (x86)/microchip/xc32/v1.10/bin/../lib/gcc/pic32mx/4.5.1/../../../../pic32mx/lib/size\libpic32.a(sbrk.o)
 .debug_info    0x000b49e8       0xaa c:/program files (x86)/microchip/xc32/v1.10/bin/../lib/gcc/pic32mx/4.5.1/../../../../pic32mx/lib/size\libpic32.a(write.o)
 .debug_info    0x000b4a92       0xb2 c:/program files (x86)/microchip/xc32/v1.10/bin/../lib/gcc/pic32mx/4.5.1/../../../../pic32mx/lib/size\libpic32.a(_mon_putc.o)
 .debug_info    0x000b4b44        0x0 c:/program files (x86)/microchip/xc32/v1.10/bin/../lib/gcc/pic32mx/4.5.1/../../../../pic32mx/lib/size\libpic32.a(xc32_uart.o)
 .debug_info    0x000b4b44       0xc8 c:/program files (x86)/microchip/xc32/v1.10/bin/../lib/gcc/pic32mx/4.5.1/../../../../pic32mx/lib/size\libe.a(_floatdisf.o)
 .debug_info    0x000b4c0c      0x315 c:/program files (x86)/microchip/xc32/v1.10/bin/../lib/gcc/pic32mx/4.5.1/size\libgcc.a(_lshrdi3.o)
 .debug_info    0x000b4f21      0x29c c:/program files (x86)/microchip/xc32/v1.10/bin/../lib/gcc/pic32mx/4.5.1/size\libgcc.a(_floatundisf.o)
 .debug_info    0x000b51bd      0x78c c:/program files (x86)/microchip/xc32/v1.10/bin/../lib/gcc/pic32mx/4.5.1/size\libgcc.a(_umoddi3.o)
 .debug_info    0x000b5949      0x154 c:/program files (x86)/microchip/xc32/v1.10/bin/../lib/gcc/pic32mx/4.5.1/size\libgcc.a(floatunsisf.o)

.debug_abbrev   0x00000000     0xe134
 *(.debug_abbrev)
 .debug_abbrev  0x00000000      0x17d build/default/production/_ext/1293749816/bsp.o
 .debug_abbrev  0x0000017d      0x18e build/default/production/_ext/101875047/hashes.o
 .debug_abbrev  0x0000030b       0x65 build/default/production/_ext/101875047/lfsr.o
 .debug_abbrev  0x00000370      0x218 build/default/production/_ext/101875047/big_int.o
 .debug_abbrev  0x00000588       0x14 build/default/production/_ext/101875047/big_int_helper_c32.o
 .debug_abbrev  0x0000059c       0xfd build/default/production/_ext/101875047/helpers.o
 .debug_abbrev  0x00000699        0x1 build/default/production/_ext/1472/berkeley_tcp_client_demo.o
 .debug_abbrev  0x0000069a        0x1 build/default/production/_ext/1472/berkeley_tcp_server_demo.o
 .debug_abbrev  0x0000069b        0x1 build/default/production/_ext/1472/berkeley_udp_client_demo.o
 .debug_abbrev  0x0000069c      0x166 build/default/production/_ext/1472/generic_tcp_client.o
 .debug_abbrev  0x00000802      0x166 build/default/production/_ext/1472/generic_tcp_server.o
 .debug_abbrev  0x00000968      0x265 build/default/production/_ext/1472/ping_demo.o
 .debug_abbrev  0x00000bcd        0x1 build/default/production/_ext/1472/smtp_demo.o
 .debug_abbrev  0x00000bce      0x3dd build/default/production/_ext/365611741/system_services.o
 .debug_abbrev  0x00000fab      0x2dd build/default/production/_ext/365611741/system_debug.o
 .debug_abbrev  0x00001288      0x230 build/default/production/_ext/365611741/system_random.o
 .debug_abbrev  0x000014b8      0x2a8 build/default/production/_ext/365611741/system_command.o
 .debug_abbrev  0x00001760      0x26c build/default/production/_ext/365611741/system_userio.o
 .debug_abbrev  0x000019cc      0x329 build/default/production/_ext/97638081/sys_fs.o
 .debug_abbrev  0x00001cf5      0x27d build/default/production/_ext/97638081/mpfs2.o
 .debug_abbrev  0x00001f72      0x218 build/default/production/_ext/792872985/usart.o
 .debug_abbrev  0x0000218a      0x201 build/default/production/_ext/792872985/lcd.o
 .debug_abbrev  0x0000238b      0x1e1 build/default/production/_ext/792872985/drv_spi.o
 .debug_abbrev  0x0000256c        0x1 build/default/production/_ext/792872985/db_appio.o
 .debug_abbrev  0x0000256d      0x166 build/default/production/_ext/792872985/spi_ram.o
 .debug_abbrev  0x000026d3      0x289 build/default/production/_ext/792872985/spi_eeprom.o
 .debug_abbrev  0x0000295c      0x166 build/default/production/_ext/792872985/spi_flash.o
 .debug_abbrev  0x00002ac2      0x288 build/default/production/_ext/792872985/drv_media.o
 .debug_abbrev  0x00002d4a      0x36c build/default/production/_ext/427700826/tcpip_announce.o
 .debug_abbrev  0x000030b6      0x36a build/default/production/_ext/427700826/http2.o
 .debug_abbrev  0x00003420      0x18b build/default/production/_ext/427700826/arcfour.o
 .debug_abbrev  0x000035ab      0x3f8 build/default/production/_ext/427700826/arp.o
 .debug_abbrev  0x000039a3      0x18b build/default/production/_ext/427700826/berkeley_api.o
 .debug_abbrev  0x00003b2e      0x3a3 build/default/production/_ext/427700826/dhcp.o
 .debug_abbrev  0x00003ed1      0x1ba build/default/production/_ext/427700826/dhcps.o
 .debug_abbrev  0x0000408b      0x36c build/default/production/_ext/427700826/dns.o
 .debug_abbrev  0x000043f7      0x18b build/default/production/_ext/427700826/dnss.o
 .debug_abbrev  0x00004582      0x18b build/default/production/_ext/427700826/dyn_dns.o
 .debug_abbrev  0x0000470d      0x18b build/default/production/_ext/427700826/enc28_mac.o
 .debug_abbrev  0x00004898      0x18b build/default/production/_ext/427700826/enc28j60.o
 .debug_abbrev  0x00004a23      0x18b build/default/production/_ext/427700826/encs24j600.o
 .debug_abbrev  0x00004bae      0x18b build/default/production/_ext/427700826/encx24_mac.o
 .debug_abbrev  0x00004d39      0x18b build/default/production/_ext/427700826/eth_pic32_ext_phy.o
 .debug_abbrev  0x00004ec4      0x18b build/default/production/_ext/427700826/eth_pic32_ext_phy_dp83848.o
 .debug_abbrev  0x0000504f      0x18b build/default/production/_ext/427700826/eth_pic32_int_mac.o
 .debug_abbrev  0x000051da      0x18b build/default/production/_ext/427700826/ftp.o
 .debug_abbrev  0x00005365       0x8c build/default/production/_ext/427700826/hash_fnv.o
 .debug_abbrev  0x000053f1      0x1ca build/default/production/_ext/427700826/hash_tbl.o
 .debug_abbrev  0x000055bb      0x2ff build/default/production/_ext/427700826/icmp.o
 .debug_abbrev  0x000058ba      0x18b build/default/production/_ext/427700826/icmpv6.o
 .debug_abbrev  0x00005a45      0x3c7 build/default/production/_ext/427700826/ipv4.o
 .debug_abbrev  0x00005e0c      0x18b build/default/production/_ext/427700826/ipv6.o
 .debug_abbrev  0x00005f97      0x18b build/default/production/_ext/427700826/mac_events_pic32.o
 .debug_abbrev  0x00006122      0x2c2 build/default/production/_ext/427700826/nbns.o
 .debug_abbrev  0x000063e4      0x18b build/default/production/_ext/427700826/ndp.o
 .debug_abbrev  0x0000656f      0x18b build/default/production/_ext/427700826/tcpip_reboot.o
 .debug_abbrev  0x000066fa      0x18b build/default/production/_ext/427700826/rsa.o
 .debug_abbrev  0x00006885      0x18b build/default/production/_ext/427700826/smtp.o
 .debug_abbrev  0x00006a10      0x18b build/default/production/_ext/427700826/snmp.o
 .debug_abbrev  0x00006b9b      0x18b build/default/production/_ext/427700826/snmpv3.o
 .debug_abbrev  0x00006d26      0x18b build/default/production/_ext/427700826/snmpv3_usm.o
 .debug_abbrev  0x00006eb1      0x18b build/default/production/_ext/427700826/sntp.o
 .debug_abbrev  0x0000703c      0x18b build/default/production/_ext/427700826/ssl.o
 .debug_abbrev  0x000071c7      0x39d build/default/production/_ext/427700826/tcp.o
 .debug_abbrev  0x00007564      0x295 build/default/production/_ext/427700826/tcpip_heap_alloc.o
 .debug_abbrev  0x000077f9      0x18b build/default/production/_ext/427700826/tcpip_storage.o
 .debug_abbrev  0x00007984      0x18b build/default/production/_ext/427700826/telnet.o
 .debug_abbrev  0x00007b0f      0x18b build/default/production/_ext/427700826/tftpc.o
 .debug_abbrev  0x00007c9a      0x3ad build/default/production/_ext/427700826/udp.o
 .debug_abbrev  0x00008047      0x22e build/default/production/_ext/427700826/tcpip_mac_object.o
 .debug_abbrev  0x00008275      0x3d5 build/default/production/_ext/427700826/tcpip_manager.o
 .debug_abbrev  0x0000864a      0x28d build/default/production/_ext/427700826/tcpip_helpers.o
 .debug_abbrev  0x000088d7      0x18b build/default/production/_ext/427700826/tcpip_commands.o
 .debug_abbrev  0x00008a62      0x18b build/default/production/_ext/427700826/iperf.o
 .debug_abbrev  0x00008bed       0x14 build/default/production/_ext/427700826/tcpip_helper_c32.o
 .debug_abbrev  0x00008c01       0xd9 build/default/production/_ext/427700826/tcpip_notify.o
 .debug_abbrev  0x00008cda      0x18b build/default/production/_ext/427700826/zero_conf_helper.o
 .debug_abbrev  0x00008e65      0x1ba build/default/production/_ext/427700826/zero_conf_link_local.o
 .debug_abbrev  0x0000901f      0x18b build/default/production/_ext/427700826/zero_conf_multicast_dns.o
 .debug_abbrev  0x000091aa      0x1da build/default/production/_ext/334706090/wf_tx_power.o
 .debug_abbrev  0x00009384      0x267 build/default/production/_ext/334706090/wf_connect.o
 .debug_abbrev  0x000095eb      0x277 build/default/production/_ext/334706090/wf_connection_algorithm.o
 .debug_abbrev  0x00009862      0x263 build/default/production/_ext/334706090/wf_connection_manager.o
 .debug_abbrev  0x00009ac5      0x2d5 build/default/production/_ext/334706090/wf_connection_profile.o
 .debug_abbrev  0x00009d9a      0x1d2 build/default/production/_ext/334706090/wf_easy_config.o
 .debug_abbrev  0x00009f6c      0x1b9 build/default/production/_ext/334706090/wf_eint.o
 .debug_abbrev  0x0000a125      0x2a8 build/default/production/_ext/334706090/wf_event_handler.o
 .debug_abbrev  0x0000a3cd      0x284 build/default/production/_ext/334706090/wf_init.o
 .debug_abbrev  0x0000a651      0x29b build/default/production/_ext/334706090/wf_power_save.o
 .debug_abbrev  0x0000a8ec      0x21e build/default/production/_ext/334706090/wf_scan.o
 .debug_abbrev  0x0000ab0a      0x22a build/default/production/_ext/334706090/wf_spi.o
 .debug_abbrev  0x0000ad34      0x310 build/default/production/_ext/334706090/mrf24w_mac_pic32.o
 .debug_abbrev  0x0000b044      0x259 build/default/production/_ext/334706090/mrf24w_events.o
 .debug_abbrev  0x0000b29d      0x316 build/default/production/_ext/334706090/wf_debug_output.o
 .debug_abbrev  0x0000b5b3      0x2f8 build/default/production/_ext/334706090/wf_commands.o
 .debug_abbrev  0x0000b8ab      0x18b build/default/production/_ext/334706090/wf_pbkdf2.o
 .debug_abbrev  0x0000ba36      0x37a build/default/production/_ext/334706090/wf_driver_com_24g.o
 .debug_abbrev  0x0000bdb0      0x281 build/default/production/_ext/334706090/wf_driver_raw_24g.o
 .debug_abbrev  0x0000c031      0x356 build/default/production/_ext/334706090/wf_mac_24g.o
 .debug_abbrev  0x0000c387      0x24e build/default/production/_ext/334706090/wf_mgmt_msg_24g.o
 .debug_abbrev  0x0000c5d5      0x267 build/default/production/_ext/334706090/wf_param_msg_24g.o
 .debug_abbrev  0x0000c83c      0x271 build/default/production/_ext/334706090/wf_configData.o
 .debug_abbrev  0x0000caad      0x278 build/default/production/_ext/1472/main_demo.o
 .debug_abbrev  0x0000cd25        0x1 build/default/production/_ext/1472/custom_snmp_app.o
 .debug_abbrev  0x0000cd26        0x1 build/default/production/_ext/1472/custom_ssl_cert.o
 .debug_abbrev  0x0000cd27      0x166 build/default/production/_ext/1472/mpfs_img2.o
 .debug_abbrev  0x0000ce8d      0x1bc build/default/production/_ext/1472/wf_config.o
 .debug_abbrev  0x0000d049      0x28b build/default/production/_ext/1472/custom_http_app.o
 .debug_abbrev  0x0000d2d4      0x283 build/default/production/_ext/1472/tcp6_demo_app.o
 .debug_abbrev  0x0000d557       0x25 c:/program files (x86)/microchip/xc32/v1.10/bin/../lib/gcc/pic32mx/4.5.1/../../../../pic32mx/lib/size\libmchp_peripheral.a(open_core_timer_lib.o)
 .debug_abbrev  0x0000d57c       0x34 c:/program files (x86)/microchip/xc32/v1.10/bin/../lib/gcc/pic32mx/4.5.1/../../../../pic32mx/lib/size\libmchp_peripheral_32MX795F512L.a(soft_reset_lib.o)
 .debug_abbrev  0x0000d5b0       0x25 c:/program files (x86)/microchip/xc32/v1.10/bin/../lib/gcc/pic32mx/4.5.1/../../../../pic32mx/lib/size\libmchp_peripheral_32MX795F512L.a(pcache.o)
 .debug_abbrev  0x0000d5d5       0x25 c:/program files (x86)/microchip/xc32/v1.10/bin/../lib/gcc/pic32mx/4.5.1/../../../../pic32mx/lib/size\libmchp_peripheral_32MX795F512L.a(int_disable_interrupts_lib.o)
 .debug_abbrev  0x0000d5fa       0x25 c:/program files (x86)/microchip/xc32/v1.10/bin/../lib/gcc/pic32mx/4.5.1/../../../../pic32mx/lib/size\libmchp_peripheral_32MX795F512L.a(int_restore_interrupts_lib.o)
 .debug_abbrev  0x0000d61f       0x25 c:/program files (x86)/microchip/xc32/v1.10/bin/../lib/gcc/pic32mx/4.5.1/../../../../pic32mx/lib/size\libmchp_peripheral_32MX795F512L.a(int_enable_mv_int_lib.o)
 .debug_abbrev  0x0000d644       0x25 c:/program files (x86)/microchip/xc32/v1.10/bin/../lib/gcc/pic32mx/4.5.1/../../../../pic32mx/lib/size\libmchp_peripheral_32MX795F512L.a(int_tbl_lib.o)
 .debug_abbrev  0x0000d669       0x41 c:/program files (x86)/microchip/xc32/v1.10/bin/../lib/gcc/pic32mx/4.5.1/../../../../pic32mx/lib/size\libmchp_peripheral_32MX795F512L.a(rtcc_init_lib.o)
 .debug_abbrev  0x0000d6aa       0x41 c:/program files (x86)/microchip/xc32/v1.10/bin/../lib/gcc/pic32mx/4.5.1/../../../../pic32mx/lib/size\libmchp_peripheral_32MX795F512L.a(rtcc_open_lib.o)
 .debug_abbrev  0x0000d6eb       0x34 c:/program files (x86)/microchip/xc32/v1.10/bin/../lib/gcc/pic32mx/4.5.1/../../../../pic32mx/lib/size\libmchp_peripheral_32MX795F512L.a(spi_chn_data_rdy_lib.o)
 .debug_abbrev  0x0000d71f       0x34 c:/program files (x86)/microchip/xc32/v1.10/bin/../lib/gcc/pic32mx/4.5.1/../../../../pic32mx/lib/size\libmchp_peripheral_32MX795F512L.a(spi_chn_getc_lib.o)
 .debug_abbrev  0x0000d753       0x25 c:/program files (x86)/microchip/xc32/v1.10/bin/../lib/gcc/pic32mx/4.5.1/../../../../pic32mx/lib/size\libmchp_peripheral_32MX795F512L.a(spi_chn_open_lib.o)
 .debug_abbrev  0x0000d778       0x34 c:/program files (x86)/microchip/xc32/v1.10/bin/../lib/gcc/pic32mx/4.5.1/../../../../pic32mx/lib/size\libmchp_peripheral_32MX795F512L.a(spi_chn_putc_lib.o)
 .debug_abbrev  0x0000d7ac       0x25 c:/program files (x86)/microchip/xc32/v1.10/bin/../lib/gcc/pic32mx/4.5.1/../../../../pic32mx/lib/size\libmchp_peripheral_32MX795F512L.a(spi_chn_tx_buff_empty_lib.o)
 .debug_abbrev  0x0000d7d1        0x1 c:/program files (x86)/microchip/xc32/v1.10/bin/../lib/gcc/pic32mx/4.5.1/../../../../pic32mx/lib/size\libmchp_peripheral_32MX795F512L.a(spi_io_tbl_libp.o)
 .debug_abbrev  0x0000d7d2        0x1 c:/program files (x86)/microchip/xc32/v1.10/bin/../lib/gcc/pic32mx/4.5.1/../../../../pic32mx/lib/size\libmchp_peripheral_32MX795F512L.a(spi_map_tbl_libp.o)
 .debug_abbrev  0x0000d7d3       0x25 c:/program files (x86)/microchip/xc32/v1.10/bin/../lib/gcc/pic32mx/4.5.1/../../../../pic32mx/lib/size\libmchp_peripheral_32MX795F512L.a(port_set_pins_digital_in_lib.o)
 .debug_abbrev  0x0000d7f8       0x25 c:/program files (x86)/microchip/xc32/v1.10/bin/../lib/gcc/pic32mx/4.5.1/../../../../pic32mx/lib/size\libmchp_peripheral_32MX795F512L.a(port_set_pins_digital_out_lib.o)
 .debug_abbrev  0x0000d81d        0x1 c:/program files (x86)/microchip/xc32/v1.10/bin/../lib/gcc/pic32mx/4.5.1/../../../../pic32mx/lib/size\libmchp_peripheral_32MX795F512L.a(_ports_tbl_libp.o)
 .debug_abbrev  0x0000d81e       0x25 c:/program files (x86)/microchip/xc32/v1.10/bin/../lib/gcc/pic32mx/4.5.1/../../../../pic32mx/lib/size\libmchp_peripheral_32MX795F512L.a(int_enable_interrupts_lib.o)
 .debug_abbrev  0x0000d843       0x34 c:/program files (x86)/microchip/xc32/v1.10/bin/../lib/gcc/pic32mx/4.5.1/../../../../pic32mx/lib/size\libmchp_peripheral_32MX795F512L.a(_rtcc_wait_clock_off_lib.o)
 .debug_abbrev  0x0000d877       0x25 c:/program files (x86)/microchip/xc32/v1.10/bin/../lib/gcc/pic32mx/4.5.1/../../../../pic32mx/lib/size\libmchp_peripheral_32MX795F512L.a(read_core_timer_lib.o)
 .debug_abbrev  0x0000d89c      0x13d c:/program files (x86)/microchip/xc32/v1.10/bin/../lib/gcc/pic32mx/4.5.1/size\libgcc.a(_udivdi3.o)
 .debug_abbrev  0x0000d9d9       0x25 c:/program files (x86)/microchip/xc32/v1.10/bin/../lib/gcc/pic32mx/4.5.1/../../../../pic32mx/lib/size\libpic32.a(default-bootstrap-exception-handler.o)
 .debug_abbrev  0x0000d9fe       0x25 c:/program files (x86)/microchip/xc32/v1.10/bin/../lib/gcc/pic32mx/4.5.1/../../../../pic32mx/lib/size\libpic32.a(default-on-reset.o)
 .debug_abbrev  0x0000da23       0x25 c:/program files (x86)/microchip/xc32/v1.10/bin/../lib/gcc/pic32mx/4.5.1/../../../../pic32mx/lib/size\libpic32.a(default-on-bootstrap.o)
 .debug_abbrev  0x0000da48        0x1 c:/program files (x86)/microchip/xc32/v1.10/bin/../lib/gcc/pic32mx/4.5.1/../../../../pic32mx/lib/size\libpic32.a(errno.o)
 .debug_abbrev  0x0000da49       0x25 c:/program files (x86)/microchip/xc32/v1.10/bin/../lib/gcc/pic32mx/4.5.1/../../../../pic32mx/lib/size\libc.a(atoi.o)
 .debug_abbrev  0x0000da6e       0x25 c:/program files (x86)/microchip/xc32/v1.10/bin/../lib/gcc/pic32mx/4.5.1/../../../../pic32mx/lib/size\libc.a(atol.o)
 .debug_abbrev  0x0000da93        0x1 c:/program files (x86)/microchip/xc32/v1.10/bin/../lib/gcc/pic32mx/4.5.1/../../../../pic32mx/lib/size\libc.a(ctype.o)
 .debug_abbrev  0x0000da94       0x25 c:/program files (x86)/microchip/xc32/v1.10/bin/../lib/gcc/pic32mx/4.5.1/../../../../pic32mx/lib/size\libc.a(malloc.o)
 .debug_abbrev  0x0000dab9       0x25 c:/program files (x86)/microchip/xc32/v1.10/bin/../lib/gcc/pic32mx/4.5.1/../../../../pic32mx/lib/size\libc.a(rand.o)
 .debug_abbrev  0x0000dade       0x25 c:/program files (x86)/microchip/xc32/v1.10/bin/../lib/gcc/pic32mx/4.5.1/../../../../pic32mx/lib/size\libc.a(strcat.o)
 .debug_abbrev  0x0000db03       0x25 c:/program files (x86)/microchip/xc32/v1.10/bin/../lib/gcc/pic32mx/4.5.1/../../../../pic32mx/lib/size\libc.a(strchr.o)
 .debug_abbrev  0x0000db28       0x25 c:/program files (x86)/microchip/xc32/v1.10/bin/../lib/gcc/pic32mx/4.5.1/../../../../pic32mx/lib/size\libc.a(strncat.o)
 .debug_abbrev  0x0000db4d       0x25 c:/program files (x86)/microchip/xc32/v1.10/bin/../lib/gcc/pic32mx/4.5.1/../../../../pic32mx/lib/size\libc.a(strncmp.o)
 .debug_abbrev  0x0000db72       0x25 c:/program files (x86)/microchip/xc32/v1.10/bin/../lib/gcc/pic32mx/4.5.1/../../../../pic32mx/lib/size\libc.a(strncpy.o)
 .debug_abbrev  0x0000db97       0x25 c:/program files (x86)/microchip/xc32/v1.10/bin/../lib/gcc/pic32mx/4.5.1/../../../../pic32mx/lib/size\libc.a(strrchr.o)
 .debug_abbrev  0x0000dbbc       0x25 c:/program files (x86)/microchip/xc32/v1.10/bin/../lib/gcc/pic32mx/4.5.1/../../../../pic32mx/lib/size\libc.a(strstr.o)
 .debug_abbrev  0x0000dbe1       0x25 c:/program files (x86)/microchip/xc32/v1.10/bin/../lib/gcc/pic32mx/4.5.1/../../../../pic32mx/lib/size\libc.a(strtol.o)
 .debug_abbrev  0x0000dc06       0x25 c:/program files (x86)/microchip/xc32/v1.10/bin/../lib/gcc/pic32mx/4.5.1/../../../../pic32mx/lib/size\libc.a(snprintf_cdnopsuxX.eo)
 .debug_abbrev  0x0000dc2b       0x25 c:/program files (x86)/microchip/xc32/v1.10/bin/../lib/gcc/pic32mx/4.5.1/../../../../pic32mx/lib/size\libc.a(sprintf_cdnopsuxX.eo)
 .debug_abbrev  0x0000dc50       0x25 c:/program files (x86)/microchip/xc32/v1.10/bin/../lib/gcc/pic32mx/4.5.1/../../../../pic32mx/lib/size\libc.a(vsnprintf_cdnopsuxX.eo)
 .debug_abbrev  0x0000dc75       0x25 c:/program files (x86)/microchip/xc32/v1.10/bin/../lib/gcc/pic32mx/4.5.1/../../../../pic32mx/lib/size\libc.a(vsnprintf.o)
 .debug_abbrev  0x0000dc9a       0x25 c:/program files (x86)/microchip/xc32/v1.10/bin/../lib/gcc/pic32mx/4.5.1/../../../../pic32mx/lib/size\libc.a(ctypef.o)
 .debug_abbrev  0x0000dcbf       0x25 c:/program files (x86)/microchip/xc32/v1.10/bin/../lib/gcc/pic32mx/4.5.1/../../../../pic32mx/lib/size\libc.a(doprnt_cdnopsuxX.eo)
 .debug_abbrev  0x0000dce4       0x36 c:/program files (x86)/microchip/xc32/v1.10/bin/../lib/gcc/pic32mx/4.5.1/../../../../pic32mx/lib/size\libc.a(doprnt.o)
 .debug_abbrev  0x0000dd1a       0x25 c:/program files (x86)/microchip/xc32/v1.10/bin/../lib/gcc/pic32mx/4.5.1/../../../../pic32mx/lib/size\libc.a(_fputc_simple.o)
 .debug_abbrev  0x0000dd3f        0x1 c:/program files (x86)/microchip/xc32/v1.10/bin/../lib/gcc/pic32mx/4.5.1/../../../../pic32mx/lib/size\libc.a(powersf.o)
 .debug_abbrev  0x0000dd40        0x1 c:/program files (x86)/microchip/xc32/v1.10/bin/../lib/gcc/pic32mx/4.5.1/../../../../pic32mx/lib/size\libc.a(_iob.o)
 .debug_abbrev  0x0000dd41       0x25 c:/program files (x86)/microchip/xc32/v1.10/bin/../lib/gcc/pic32mx/4.5.1/../../../../pic32mx/lib/size\libc.a(_flsbuf_simple.o)
 .debug_abbrev  0x0000dd66       0x38 c:/program files (x86)/microchip/xc32/v1.10/bin/../lib/gcc/pic32mx/4.5.1/../../../../pic32mx/lib/size\libpic32.a(sbrk.o)
 .debug_abbrev  0x0000dd9e       0x25 c:/program files (x86)/microchip/xc32/v1.10/bin/../lib/gcc/pic32mx/4.5.1/../../../../pic32mx/lib/size\libpic32.a(write.o)
 .debug_abbrev  0x0000ddc3       0x25 c:/program files (x86)/microchip/xc32/v1.10/bin/../lib/gcc/pic32mx/4.5.1/../../../../pic32mx/lib/size\libpic32.a(_mon_putc.o)
 .debug_abbrev  0x0000dde8        0x1 c:/program files (x86)/microchip/xc32/v1.10/bin/../lib/gcc/pic32mx/4.5.1/../../../../pic32mx/lib/size\libpic32.a(xc32_uart.o)
 .debug_abbrev  0x0000dde9       0x32 c:/program files (x86)/microchip/xc32/v1.10/bin/../lib/gcc/pic32mx/4.5.1/../../../../pic32mx/lib/size\libe.a(_floatdisf.o)
 .debug_abbrev  0x0000de1b       0xe3 c:/program files (x86)/microchip/xc32/v1.10/bin/../lib/gcc/pic32mx/4.5.1/size\libgcc.a(_lshrdi3.o)
 .debug_abbrev  0x0000defe       0x79 c:/program files (x86)/microchip/xc32/v1.10/bin/../lib/gcc/pic32mx/4.5.1/size\libgcc.a(_floatundisf.o)
 .debug_abbrev  0x0000df77      0x15c c:/program files (x86)/microchip/xc32/v1.10/bin/../lib/gcc/pic32mx/4.5.1/size\libgcc.a(_umoddi3.o)
 .debug_abbrev  0x0000e0d3       0x61 c:/program files (x86)/microchip/xc32/v1.10/bin/../lib/gcc/pic32mx/4.5.1/size\libgcc.a(floatunsisf.o)

.debug_line     0x00000000    0x1b1c2
 *(.debug_line)
 .debug_line    0x00000000      0x1db build/default/production/_ext/1293749816/bsp.o
 .debug_line    0x000001db      0x2e4 build/default/production/_ext/101875047/hashes.o
 .debug_line    0x000004bf       0xf0 build/default/production/_ext/101875047/lfsr.o
 .debug_line    0x000005af      0x3eb build/default/production/_ext/101875047/big_int.o
 .debug_line    0x0000099a      0x14f build/default/production/_ext/101875047/big_int_helper_c32.o
 .debug_line    0x00000ae9      0x24e build/default/production/_ext/101875047/helpers.o
 .debug_line    0x00000d37        0x0 build/default/production/_ext/1472/berkeley_tcp_client_demo.o
 .debug_line    0x00000d37        0x0 build/default/production/_ext/1472/berkeley_tcp_server_demo.o
 .debug_line    0x00000d37        0x0 build/default/production/_ext/1472/berkeley_udp_client_demo.o
 .debug_line    0x00000d37      0x1c5 build/default/production/_ext/1472/generic_tcp_client.o
 .debug_line    0x00000efc      0x1c5 build/default/production/_ext/1472/generic_tcp_server.o
 .debug_line    0x000010c1      0x320 build/default/production/_ext/1472/ping_demo.o
 .debug_line    0x000013e1        0x0 build/default/production/_ext/1472/smtp_demo.o
 .debug_line    0x000013e1      0x70c build/default/production/_ext/365611741/system_services.o
 .debug_line    0x00001aed      0x45b build/default/production/_ext/365611741/system_debug.o
 .debug_line    0x00001f48      0x35d build/default/production/_ext/365611741/system_random.o
 .debug_line    0x000022a5      0x4ce build/default/production/_ext/365611741/system_command.o
 .debug_line    0x00002773      0x3bf build/default/production/_ext/365611741/system_userio.o
 .debug_line    0x00002b32      0xa84 build/default/production/_ext/97638081/sys_fs.o
 .debug_line    0x000035b6      0x5d5 build/default/production/_ext/97638081/mpfs2.o
 .debug_line    0x00003b8b      0x273 build/default/production/_ext/792872985/usart.o
 .debug_line    0x00003dfe      0x367 build/default/production/_ext/792872985/lcd.o
 .debug_line    0x00004165      0x2e9 build/default/production/_ext/792872985/drv_spi.o
 .debug_line    0x0000444e        0x0 build/default/production/_ext/792872985/db_appio.o
 .debug_line    0x0000444e      0x18e build/default/production/_ext/792872985/spi_ram.o
 .debug_line    0x000045dc      0x464 build/default/production/_ext/792872985/spi_eeprom.o
 .debug_line    0x00004a40      0x18e build/default/production/_ext/792872985/spi_flash.o
 .debug_line    0x00004bce      0x4a8 build/default/production/_ext/792872985/drv_media.o
 .debug_line    0x00005076      0x497 build/default/production/_ext/427700826/tcpip_announce.o
 .debug_line    0x0000550d      0xbf5 build/default/production/_ext/427700826/http2.o
 .debug_line    0x00006102      0x230 build/default/production/_ext/427700826/arcfour.o
 .debug_line    0x00006332      0x920 build/default/production/_ext/427700826/arp.o
 .debug_line    0x00006c52      0x230 build/default/production/_ext/427700826/berkeley_api.o
 .debug_line    0x00006e82      0x86e build/default/production/_ext/427700826/dhcp.o
 .debug_line    0x000076f0      0x29a build/default/production/_ext/427700826/dhcps.o
 .debug_line    0x0000798a      0x662 build/default/production/_ext/427700826/dns.o
 .debug_line    0x00007fec      0x230 build/default/production/_ext/427700826/dnss.o
 .debug_line    0x0000821c      0x230 build/default/production/_ext/427700826/dyn_dns.o
 .debug_line    0x0000844c      0x230 build/default/production/_ext/427700826/enc28_mac.o
 .debug_line    0x0000867c      0x230 build/default/production/_ext/427700826/enc28j60.o
 .debug_line    0x000088ac      0x230 build/default/production/_ext/427700826/encs24j600.o
 .debug_line    0x00008adc      0x230 build/default/production/_ext/427700826/encx24_mac.o
 .debug_line    0x00008d0c      0x230 build/default/production/_ext/427700826/eth_pic32_ext_phy.o
 .debug_line    0x00008f3c      0x230 build/default/production/_ext/427700826/eth_pic32_ext_phy_dp83848.o
 .debug_line    0x0000916c      0x230 build/default/production/_ext/427700826/eth_pic32_int_mac.o
 .debug_line    0x0000939c      0x230 build/default/production/_ext/427700826/ftp.o
 .debug_line    0x000095cc      0x173 build/default/production/_ext/427700826/hash_fnv.o
 .debug_line    0x0000973f      0x263 build/default/production/_ext/427700826/hash_tbl.o
 .debug_line    0x000099a2      0x411 build/default/production/_ext/427700826/icmp.o
 .debug_line    0x00009db3      0x230 build/default/production/_ext/427700826/icmpv6.o
 .debug_line    0x00009fe3      0x89f build/default/production/_ext/427700826/ipv4.o
 .debug_line    0x0000a882      0x230 build/default/production/_ext/427700826/ipv6.o
 .debug_line    0x0000aab2      0x230 build/default/production/_ext/427700826/mac_events_pic32.o
 .debug_line    0x0000ace2      0x4a3 build/default/production/_ext/427700826/nbns.o
 .debug_line    0x0000b185      0x230 build/default/production/_ext/427700826/ndp.o
 .debug_line    0x0000b3b5      0x230 build/default/production/_ext/427700826/tcpip_reboot.o
 .debug_line    0x0000b5e5      0x230 build/default/production/_ext/427700826/rsa.o
 .debug_line    0x0000b815      0x230 build/default/production/_ext/427700826/smtp.o
 .debug_line    0x0000ba45      0x230 build/default/production/_ext/427700826/snmp.o
 .debug_line    0x0000bc75      0x230 build/default/production/_ext/427700826/snmpv3.o
 .debug_line    0x0000bea5      0x230 build/default/production/_ext/427700826/snmpv3_usm.o
 .debug_line    0x0000c0d5      0x230 build/default/production/_ext/427700826/sntp.o
 .debug_line    0x0000c305      0x230 build/default/production/_ext/427700826/ssl.o
 .debug_line    0x0000c535     0x1437 build/default/production/_ext/427700826/tcp.o
 .debug_line    0x0000d96c      0x536 build/default/production/_ext/427700826/tcpip_heap_alloc.o
 .debug_line    0x0000dea2      0x230 build/default/production/_ext/427700826/tcpip_storage.o
 .debug_line    0x0000e0d2      0x230 build/default/production/_ext/427700826/telnet.o
 .debug_line    0x0000e302      0x230 build/default/production/_ext/427700826/tftpc.o
 .debug_line    0x0000e532      0xa29 build/default/production/_ext/427700826/udp.o
 .debug_line    0x0000ef5b      0x50b build/default/production/_ext/427700826/tcpip_mac_object.o
 .debug_line    0x0000f466      0xedd build/default/production/_ext/427700826/tcpip_manager.o
 .debug_line    0x00010343      0x693 build/default/production/_ext/427700826/tcpip_helpers.o
 .debug_line    0x000109d6      0x230 build/default/production/_ext/427700826/tcpip_commands.o
 .debug_line    0x00010c06      0x230 build/default/production/_ext/427700826/iperf.o
 .debug_line    0x00010e36       0xee build/default/production/_ext/427700826/tcpip_helper_c32.o
 .debug_line    0x00010f24      0x120 build/default/production/_ext/427700826/tcpip_notify.o
 .debug_line    0x00011044      0x230 build/default/production/_ext/427700826/zero_conf_helper.o
 .debug_line    0x00011274      0x2a9 build/default/production/_ext/427700826/zero_conf_link_local.o
 .debug_line    0x0001151d      0x230 build/default/production/_ext/427700826/zero_conf_multicast_dns.o
 .debug_line    0x0001174d      0x367 build/default/production/_ext/334706090/wf_tx_power.o
 .debug_line    0x00011ab4      0x3a6 build/default/production/_ext/334706090/wf_connect.o
 .debug_line    0x00011e5a      0x4ea build/default/production/_ext/334706090/wf_connection_algorithm.o
 .debug_line    0x00012344      0x3d6 build/default/production/_ext/334706090/wf_connection_manager.o
 .debug_line    0x0001271a      0x59a build/default/production/_ext/334706090/wf_connection_profile.o
 .debug_line    0x00012cb4      0x34a build/default/production/_ext/334706090/wf_easy_config.o
 .debug_line    0x00012ffe      0x2c5 build/default/production/_ext/334706090/wf_eint.o
 .debug_line    0x000132c3      0x498 build/default/production/_ext/334706090/wf_event_handler.o
 .debug_line    0x0001375b      0x3de build/default/production/_ext/334706090/wf_init.o
 .debug_line    0x00013b39      0x46f build/default/production/_ext/334706090/wf_power_save.o
 .debug_line    0x00013fa8      0x388 build/default/production/_ext/334706090/wf_scan.o
 .debug_line    0x00014330      0x364 build/default/production/_ext/334706090/wf_spi.o
 .debug_line    0x00014694      0x613 build/default/production/_ext/334706090/mrf24w_mac_pic32.o
 .debug_line    0x00014ca7      0x42d build/default/production/_ext/334706090/mrf24w_events.o
 .debug_line    0x000150d4      0x623 build/default/production/_ext/334706090/wf_debug_output.o
 .debug_line    0x000156f7      0x626 build/default/production/_ext/334706090/wf_commands.o
 .debug_line    0x00015d1d      0x230 build/default/production/_ext/334706090/wf_pbkdf2.o
 .debug_line    0x00015f4d      0x6a2 build/default/production/_ext/334706090/wf_driver_com_24g.o
 .debug_line    0x000165ef      0x5ca build/default/production/_ext/334706090/wf_driver_raw_24g.o
 .debug_line    0x00016bb9      0x6b0 build/default/production/_ext/334706090/wf_mac_24g.o
 .debug_line    0x00017269      0x402 build/default/production/_ext/334706090/wf_mgmt_msg_24g.o
 .debug_line    0x0001766b      0x5b3 build/default/production/_ext/334706090/wf_param_msg_24g.o
 .debug_line    0x00017c1e      0x3f2 build/default/production/_ext/334706090/wf_configData.o
 .debug_line    0x00018010      0x4ca build/default/production/_ext/1472/main_demo.o
 .debug_line    0x000184da        0x0 build/default/production/_ext/1472/custom_snmp_app.o
 .debug_line    0x000184da        0x0 build/default/production/_ext/1472/custom_ssl_cert.o
 .debug_line    0x000184da      0x18e build/default/production/_ext/1472/mpfs_img2.o
 .debug_line    0x00018668      0x2ac build/default/production/_ext/1472/wf_config.o
 .debug_line    0x00018914      0x81c build/default/production/_ext/1472/custom_http_app.o
 .debug_line    0x00019130      0x507 build/default/production/_ext/1472/tcp6_demo_app.o
 .debug_line    0x00019637       0x6e c:/program files (x86)/microchip/xc32/v1.10/bin/../lib/gcc/pic32mx/4.5.1/../../../../pic32mx/lib/size\libmchp_peripheral.a(open_core_timer_lib.o)
 .debug_line    0x000196a5       0xbf c:/program files (x86)/microchip/xc32/v1.10/bin/../lib/gcc/pic32mx/4.5.1/../../../../pic32mx/lib/size\libmchp_peripheral_32MX795F512L.a(soft_reset_lib.o)
 .debug_line    0x00019764       0x62 c:/program files (x86)/microchip/xc32/v1.10/bin/../lib/gcc/pic32mx/4.5.1/../../../../pic32mx/lib/size\libmchp_peripheral_32MX795F512L.a(pcache.o)
 .debug_line    0x000197c6       0x73 c:/program files (x86)/microchip/xc32/v1.10/bin/../lib/gcc/pic32mx/4.5.1/../../../../pic32mx/lib/size\libmchp_peripheral_32MX795F512L.a(int_disable_interrupts_lib.o)
 .debug_line    0x00019839       0x73 c:/program files (x86)/microchip/xc32/v1.10/bin/../lib/gcc/pic32mx/4.5.1/../../../../pic32mx/lib/size\libmchp_peripheral_32MX795F512L.a(int_restore_interrupts_lib.o)
 .debug_line    0x000198ac       0x6e c:/program files (x86)/microchip/xc32/v1.10/bin/../lib/gcc/pic32mx/4.5.1/../../../../pic32mx/lib/size\libmchp_peripheral_32MX795F512L.a(int_enable_mv_int_lib.o)
 .debug_line    0x0001991a       0x64 c:/program files (x86)/microchip/xc32/v1.10/bin/../lib/gcc/pic32mx/4.5.1/../../../../pic32mx/lib/size\libmchp_peripheral_32MX795F512L.a(int_tbl_lib.o)
 .debug_line    0x0001997e       0xda c:/program files (x86)/microchip/xc32/v1.10/bin/../lib/gcc/pic32mx/4.5.1/../../../../pic32mx/lib/size\libmchp_peripheral_32MX795F512L.a(rtcc_init_lib.o)
 .debug_line    0x00019a58       0xda c:/program files (x86)/microchip/xc32/v1.10/bin/../lib/gcc/pic32mx/4.5.1/../../../../pic32mx/lib/size\libmchp_peripheral_32MX795F512L.a(rtcc_open_lib.o)
 .debug_line    0x00019b32       0x7f c:/program files (x86)/microchip/xc32/v1.10/bin/../lib/gcc/pic32mx/4.5.1/../../../../pic32mx/lib/size\libmchp_peripheral_32MX795F512L.a(spi_chn_data_rdy_lib.o)
 .debug_line    0x00019bb1       0x7b c:/program files (x86)/microchip/xc32/v1.10/bin/../lib/gcc/pic32mx/4.5.1/../../../../pic32mx/lib/size\libmchp_peripheral_32MX795F512L.a(spi_chn_getc_lib.o)
 .debug_line    0x00019c2c       0x69 c:/program files (x86)/microchip/xc32/v1.10/bin/../lib/gcc/pic32mx/4.5.1/../../../../pic32mx/lib/size\libmchp_peripheral_32MX795F512L.a(spi_chn_open_lib.o)
 .debug_line    0x00019c95       0x7b c:/program files (x86)/microchip/xc32/v1.10/bin/../lib/gcc/pic32mx/4.5.1/../../../../pic32mx/lib/size\libmchp_peripheral_32MX795F512L.a(spi_chn_putc_lib.o)
 .debug_line    0x00019d10       0x72 c:/program files (x86)/microchip/xc32/v1.10/bin/../lib/gcc/pic32mx/4.5.1/../../../../pic32mx/lib/size\libmchp_peripheral_32MX795F512L.a(spi_chn_tx_buff_empty_lib.o)
 .debug_line    0x00019d82        0x0 c:/program files (x86)/microchip/xc32/v1.10/bin/../lib/gcc/pic32mx/4.5.1/../../../../pic32mx/lib/size\libmchp_peripheral_32MX795F512L.a(spi_io_tbl_libp.o)
 .debug_line    0x00019d82        0x0 c:/program files (x86)/microchip/xc32/v1.10/bin/../lib/gcc/pic32mx/4.5.1/../../../../pic32mx/lib/size\libmchp_peripheral_32MX795F512L.a(spi_map_tbl_libp.o)
 .debug_line    0x00019d82       0x77 c:/program files (x86)/microchip/xc32/v1.10/bin/../lib/gcc/pic32mx/4.5.1/../../../../pic32mx/lib/size\libmchp_peripheral_32MX795F512L.a(port_set_pins_digital_in_lib.o)
 .debug_line    0x00019df9       0x78 c:/program files (x86)/microchip/xc32/v1.10/bin/../lib/gcc/pic32mx/4.5.1/../../../../pic32mx/lib/size\libmchp_peripheral_32MX795F512L.a(port_set_pins_digital_out_lib.o)
 .debug_line    0x00019e71        0x0 c:/program files (x86)/microchip/xc32/v1.10/bin/../lib/gcc/pic32mx/4.5.1/../../../../pic32mx/lib/size\libmchp_peripheral_32MX795F512L.a(_ports_tbl_libp.o)
 .debug_line    0x00019e71       0x72 c:/program files (x86)/microchip/xc32/v1.10/bin/../lib/gcc/pic32mx/4.5.1/../../../../pic32mx/lib/size\libmchp_peripheral_32MX795F512L.a(int_enable_interrupts_lib.o)
 .debug_line    0x00019ee3       0xbd c:/program files (x86)/microchip/xc32/v1.10/bin/../lib/gcc/pic32mx/4.5.1/../../../../pic32mx/lib/size\libmchp_peripheral_32MX795F512L.a(_rtcc_wait_clock_off_lib.o)
 .debug_line    0x00019fa0       0x6e c:/program files (x86)/microchip/xc32/v1.10/bin/../lib/gcc/pic32mx/4.5.1/../../../../pic32mx/lib/size\libmchp_peripheral_32MX795F512L.a(read_core_timer_lib.o)
 .debug_line    0x0001a00e      0x11c c:/program files (x86)/microchip/xc32/v1.10/bin/../lib/gcc/pic32mx/4.5.1/size\libgcc.a(_udivdi3.o)
 .debug_line    0x0001a12a       0x94 c:/program files (x86)/microchip/xc32/v1.10/bin/../lib/gcc/pic32mx/4.5.1/../../../../pic32mx/lib/size\libpic32.a(default-bootstrap-exception-handler.o)
 .debug_line    0x0001a1be       0x81 c:/program files (x86)/microchip/xc32/v1.10/bin/../lib/gcc/pic32mx/4.5.1/../../../../pic32mx/lib/size\libpic32.a(default-on-reset.o)
 .debug_line    0x0001a23f       0x85 c:/program files (x86)/microchip/xc32/v1.10/bin/../lib/gcc/pic32mx/4.5.1/../../../../pic32mx/lib/size\libpic32.a(default-on-bootstrap.o)
 .debug_line    0x0001a2c4        0x0 c:/program files (x86)/microchip/xc32/v1.10/bin/../lib/gcc/pic32mx/4.5.1/../../../../pic32mx/lib/size\libpic32.a(errno.o)
 .debug_line    0x0001a2c4       0x77 c:/program files (x86)/microchip/xc32/v1.10/bin/../lib/gcc/pic32mx/4.5.1/../../../../pic32mx/lib/size\libc.a(atoi.o)
 .debug_line    0x0001a33b       0x77 c:/program files (x86)/microchip/xc32/v1.10/bin/../lib/gcc/pic32mx/4.5.1/../../../../pic32mx/lib/size\libc.a(atol.o)
 .debug_line    0x0001a3b2        0x0 c:/program files (x86)/microchip/xc32/v1.10/bin/../lib/gcc/pic32mx/4.5.1/../../../../pic32mx/lib/size\libc.a(ctype.o)
 .debug_line    0x0001a3b2       0x79 c:/program files (x86)/microchip/xc32/v1.10/bin/../lib/gcc/pic32mx/4.5.1/../../../../pic32mx/lib/size\libc.a(malloc.o)
 .debug_line    0x0001a42b       0x77 c:/program files (x86)/microchip/xc32/v1.10/bin/../lib/gcc/pic32mx/4.5.1/../../../../pic32mx/lib/size\libc.a(rand.o)
 .debug_line    0x0001a4a2       0x79 c:/program files (x86)/microchip/xc32/v1.10/bin/../lib/gcc/pic32mx/4.5.1/../../../../pic32mx/lib/size\libc.a(strcat.o)
 .debug_line    0x0001a51b       0x79 c:/program files (x86)/microchip/xc32/v1.10/bin/../lib/gcc/pic32mx/4.5.1/../../../../pic32mx/lib/size\libc.a(strchr.o)
 .debug_line    0x0001a594       0x7a c:/program files (x86)/microchip/xc32/v1.10/bin/../lib/gcc/pic32mx/4.5.1/../../../../pic32mx/lib/size\libc.a(strncat.o)
 .debug_line    0x0001a60e       0x7a c:/program files (x86)/microchip/xc32/v1.10/bin/../lib/gcc/pic32mx/4.5.1/../../../../pic32mx/lib/size\libc.a(strncmp.o)
 .debug_line    0x0001a688       0x7a c:/program files (x86)/microchip/xc32/v1.10/bin/../lib/gcc/pic32mx/4.5.1/../../../../pic32mx/lib/size\libc.a(strncpy.o)
 .debug_line    0x0001a702       0x7a c:/program files (x86)/microchip/xc32/v1.10/bin/../lib/gcc/pic32mx/4.5.1/../../../../pic32mx/lib/size\libc.a(strrchr.o)
 .debug_line    0x0001a77c       0x79 c:/program files (x86)/microchip/xc32/v1.10/bin/../lib/gcc/pic32mx/4.5.1/../../../../pic32mx/lib/size\libc.a(strstr.o)
 .debug_line    0x0001a7f5       0x79 c:/program files (x86)/microchip/xc32/v1.10/bin/../lib/gcc/pic32mx/4.5.1/../../../../pic32mx/lib/size\libc.a(strtol.o)
 .debug_line    0x0001a86e       0x7b c:/program files (x86)/microchip/xc32/v1.10/bin/../lib/gcc/pic32mx/4.5.1/../../../../pic32mx/lib/size\libc.a(snprintf_cdnopsuxX.eo)
 .debug_line    0x0001a8e9       0x7a c:/program files (x86)/microchip/xc32/v1.10/bin/../lib/gcc/pic32mx/4.5.1/../../../../pic32mx/lib/size\libc.a(sprintf_cdnopsuxX.eo)
 .debug_line    0x0001a963       0x7c c:/program files (x86)/microchip/xc32/v1.10/bin/../lib/gcc/pic32mx/4.5.1/../../../../pic32mx/lib/size\libc.a(vsnprintf_cdnopsuxX.eo)
 .debug_line    0x0001a9df       0x7c c:/program files (x86)/microchip/xc32/v1.10/bin/../lib/gcc/pic32mx/4.5.1/../../../../pic32mx/lib/size\libc.a(vsnprintf.o)
 .debug_line    0x0001aa5b       0x79 c:/program files (x86)/microchip/xc32/v1.10/bin/../lib/gcc/pic32mx/4.5.1/../../../../pic32mx/lib/size\libc.a(ctypef.o)
 .debug_line    0x0001aad4       0x79 c:/program files (x86)/microchip/xc32/v1.10/bin/../lib/gcc/pic32mx/4.5.1/../../../../pic32mx/lib/size\libc.a(doprnt_cdnopsuxX.eo)
 .debug_line    0x0001ab4d       0x79 c:/program files (x86)/microchip/xc32/v1.10/bin/../lib/gcc/pic32mx/4.5.1/../../../../pic32mx/lib/size\libc.a(doprnt.o)
 .debug_line    0x0001abc6       0x78 c:/program files (x86)/microchip/xc32/v1.10/bin/../lib/gcc/pic32mx/4.5.1/../../../../pic32mx/lib/size\libc.a(_fputc_simple.o)
 .debug_line    0x0001ac3e        0x0 c:/program files (x86)/microchip/xc32/v1.10/bin/../lib/gcc/pic32mx/4.5.1/../../../../pic32mx/lib/size\libc.a(powersf.o)
 .debug_line    0x0001ac3e        0x0 c:/program files (x86)/microchip/xc32/v1.10/bin/../lib/gcc/pic32mx/4.5.1/../../../../pic32mx/lib/size\libc.a(_iob.o)
 .debug_line    0x0001ac3e       0x79 c:/program files (x86)/microchip/xc32/v1.10/bin/../lib/gcc/pic32mx/4.5.1/../../../../pic32mx/lib/size\libc.a(_flsbuf_simple.o)
 .debug_line    0x0001acb7       0x75 c:/program files (x86)/microchip/xc32/v1.10/bin/../lib/gcc/pic32mx/4.5.1/../../../../pic32mx/lib/size\libpic32.a(sbrk.o)
 .debug_line    0x0001ad2c       0x76 c:/program files (x86)/microchip/xc32/v1.10/bin/../lib/gcc/pic32mx/4.5.1/../../../../pic32mx/lib/size\libpic32.a(write.o)
 .debug_line    0x0001ada2       0x7a c:/program files (x86)/microchip/xc32/v1.10/bin/../lib/gcc/pic32mx/4.5.1/../../../../pic32mx/lib/size\libpic32.a(_mon_putc.o)
 .debug_line    0x0001ae1c        0x0 c:/program files (x86)/microchip/xc32/v1.10/bin/../lib/gcc/pic32mx/4.5.1/../../../../pic32mx/lib/size\libpic32.a(xc32_uart.o)
 .debug_line    0x0001ae1c       0x90 c:/program files (x86)/microchip/xc32/v1.10/bin/../lib/gcc/pic32mx/4.5.1/../../../../pic32mx/lib/size\libe.a(_floatdisf.o)
 .debug_line    0x0001aeac       0xbe c:/program files (x86)/microchip/xc32/v1.10/bin/../lib/gcc/pic32mx/4.5.1/size\libgcc.a(_lshrdi3.o)
 .debug_line    0x0001af6a       0xc9 c:/program files (x86)/microchip/xc32/v1.10/bin/../lib/gcc/pic32mx/4.5.1/size\libgcc.a(_floatundisf.o)
 .debug_line    0x0001b033      0x11f c:/program files (x86)/microchip/xc32/v1.10/bin/../lib/gcc/pic32mx/4.5.1/size\libgcc.a(_umoddi3.o)
 .debug_line    0x0001b152       0x70 c:/program files (x86)/microchip/xc32/v1.10/bin/../lib/gcc/pic32mx/4.5.1/size\libgcc.a(floatunsisf.o)

.debug_frame    0x00000000     0x81d4
 *(.debug_frame)
 .debug_frame   0x00000000       0x2c build/default/production/_ext/1293749816/bsp.o
 .debug_frame   0x0000002c      0x10c build/default/production/_ext/101875047/hashes.o
 .debug_frame   0x00000138       0x48 build/default/production/_ext/101875047/lfsr.o
 .debug_frame   0x00000180      0x188 build/default/production/_ext/101875047/big_int.o
 .debug_frame   0x00000308       0xf0 build/default/production/_ext/101875047/helpers.o
 .debug_frame   0x000003f8       0x64 build/default/production/_ext/1472/ping_demo.o
 .debug_frame   0x0000045c      0x3e8 build/default/production/_ext/365611741/system_services.o
 .debug_frame   0x00000844      0x278 build/default/production/_ext/365611741/system_debug.o
 .debug_frame   0x00000abc       0xa0 build/default/production/_ext/365611741/system_random.o
 .debug_frame   0x00000b5c      0x25c build/default/production/_ext/365611741/system_command.o
 .debug_frame   0x00000db8       0xf0 build/default/production/_ext/365611741/system_userio.o
 .debug_frame   0x00000ea8      0x7a8 build/default/production/_ext/97638081/sys_fs.o
 .debug_frame   0x00001650      0x2b8 build/default/production/_ext/97638081/mpfs2.o
 .debug_frame   0x00001908       0xd8 build/default/production/_ext/792872985/usart.o
 .debug_frame   0x000019e0       0xb8 build/default/production/_ext/792872985/lcd.o
 .debug_frame   0x00001a98       0x64 build/default/production/_ext/792872985/drv_spi.o
 .debug_frame   0x00001afc      0x144 build/default/production/_ext/792872985/spi_eeprom.o
 .debug_frame   0x00001c40      0x1b4 build/default/production/_ext/792872985/drv_media.o
 .debug_frame   0x00001df4       0xd8 build/default/production/_ext/427700826/tcpip_announce.o
 .debug_frame   0x00001ecc      0x434 build/default/production/_ext/427700826/http2.o
 .debug_frame   0x00002300      0x42c build/default/production/_ext/427700826/arp.o
 .debug_frame   0x0000272c      0x240 build/default/production/_ext/427700826/dhcp.o
 .debug_frame   0x0000296c       0x64 build/default/production/_ext/427700826/dhcps.o
 .debug_frame   0x000029d0      0x148 build/default/production/_ext/427700826/dns.o
 .debug_frame   0x00002b18       0x48 build/default/production/_ext/427700826/hash_fnv.o
 .debug_frame   0x00002b60       0xf0 build/default/production/_ext/427700826/hash_tbl.o
 .debug_frame   0x00002c50       0xd4 build/default/production/_ext/427700826/icmp.o
 .debug_frame   0x00002d24      0x458 build/default/production/_ext/427700826/ipv4.o
 .debug_frame   0x0000317c       0x9c build/default/production/_ext/427700826/nbns.o
 .debug_frame   0x00003218      0x8ac build/default/production/_ext/427700826/tcp.o
 .debug_frame   0x00003ac4      0x1d0 build/default/production/_ext/427700826/tcpip_heap_alloc.o
 .debug_frame   0x00003c94      0x4e0 build/default/production/_ext/427700826/udp.o
 .debug_frame   0x00004174      0x2b0 build/default/production/_ext/427700826/tcpip_mac_object.o
 .debug_frame   0x00004424      0x8d0 build/default/production/_ext/427700826/tcpip_manager.o
 .debug_frame   0x00004cf4      0x2e8 build/default/production/_ext/427700826/tcpip_helpers.o
 .debug_frame   0x00004fdc       0x64 build/default/production/_ext/427700826/tcpip_notify.o
 .debug_frame   0x00005040       0x64 build/default/production/_ext/427700826/zero_conf_link_local.o
 .debug_frame   0x000050a4       0x64 build/default/production/_ext/334706090/wf_tx_power.o
 .debug_frame   0x00005108       0x9c build/default/production/_ext/334706090/wf_connect.o
 .debug_frame   0x000051a4      0x208 build/default/production/_ext/334706090/wf_connection_algorithm.o
 .debug_frame   0x000053ac       0xd4 build/default/production/_ext/334706090/wf_connection_manager.o
 .debug_frame   0x00005480      0x2b0 build/default/production/_ext/334706090/wf_connection_profile.o
 .debug_frame   0x00005730       0x2c build/default/production/_ext/334706090/wf_easy_config.o
 .debug_frame   0x0000575c       0x9c build/default/production/_ext/334706090/wf_eint.o
 .debug_frame   0x000057f8      0x128 build/default/production/_ext/334706090/wf_event_handler.o
 .debug_frame   0x00005920       0x9c build/default/production/_ext/334706090/wf_init.o
 .debug_frame   0x000059bc      0x1b4 build/default/production/_ext/334706090/wf_power_save.o
 .debug_frame   0x00005b70       0x64 build/default/production/_ext/334706090/wf_scan.o
 .debug_frame   0x00005bd4       0x9c build/default/production/_ext/334706090/wf_spi.o
 .debug_frame   0x00005c70      0x358 build/default/production/_ext/334706090/mrf24w_mac_pic32.o
 .debug_frame   0x00005fc8      0x144 build/default/production/_ext/334706090/mrf24w_events.o
 .debug_frame   0x0000610c      0x240 build/default/production/_ext/334706090/wf_debug_output.o
 .debug_frame   0x0000634c      0x1bc build/default/production/_ext/334706090/wf_commands.o
 .debug_frame   0x00006508      0x2b0 build/default/production/_ext/334706090/wf_driver_com_24g.o
 .debug_frame   0x000067b8      0x25c build/default/production/_ext/334706090/wf_driver_raw_24g.o
 .debug_frame   0x00006a14      0x374 build/default/production/_ext/334706090/wf_mac_24g.o
 .debug_frame   0x00006d88       0x9c build/default/production/_ext/334706090/wf_mgmt_msg_24g.o
 .debug_frame   0x00006e24      0x2e8 build/default/production/_ext/334706090/wf_param_msg_24g.o
 .debug_frame   0x0000710c       0x80 build/default/production/_ext/334706090/wf_configData.o
 .debug_frame   0x0000718c       0x84 build/default/production/_ext/1472/main_demo.o
 .debug_frame   0x00007210       0x2c build/default/production/_ext/1472/wf_config.o
 .debug_frame   0x0000723c      0x488 build/default/production/_ext/1472/custom_http_app.o
 .debug_frame   0x000076c4       0x84 build/default/production/_ext/1472/tcp6_demo_app.o
 .debug_frame   0x00007748       0x20 c:/program files (x86)/microchip/xc32/v1.10/bin/../lib/gcc/pic32mx/4.5.1/../../../../pic32mx/lib/size\libmchp_peripheral.a(open_core_timer_lib.o)
 .debug_frame   0x00007768       0x28 c:/program files (x86)/microchip/xc32/v1.10/bin/../lib/gcc/pic32mx/4.5.1/../../../../pic32mx/lib/size\libmchp_peripheral_32MX795F512L.a(soft_reset_lib.o)
 .debug_frame   0x00007790       0x30 c:/program files (x86)/microchip/xc32/v1.10/bin/../lib/gcc/pic32mx/4.5.1/../../../../pic32mx/lib/size\libmchp_peripheral_32MX795F512L.a(pcache.o)
 .debug_frame   0x000077c0       0x20 c:/program files (x86)/microchip/xc32/v1.10/bin/../lib/gcc/pic32mx/4.5.1/../../../../pic32mx/lib/size\libmchp_peripheral_32MX795F512L.a(int_disable_interrupts_lib.o)
 .debug_frame   0x000077e0       0x20 c:/program files (x86)/microchip/xc32/v1.10/bin/../lib/gcc/pic32mx/4.5.1/../../../../pic32mx/lib/size\libmchp_peripheral_32MX795F512L.a(int_restore_interrupts_lib.o)
 .debug_frame   0x00007800       0x28 c:/program files (x86)/microchip/xc32/v1.10/bin/../lib/gcc/pic32mx/4.5.1/../../../../pic32mx/lib/size\libmchp_peripheral_32MX795F512L.a(int_enable_mv_int_lib.o)
 .debug_frame   0x00007828       0xa0 c:/program files (x86)/microchip/xc32/v1.10/bin/../lib/gcc/pic32mx/4.5.1/../../../../pic32mx/lib/size\libmchp_peripheral_32MX795F512L.a(int_tbl_lib.o)
 .debug_frame   0x000078c8       0x2c c:/program files (x86)/microchip/xc32/v1.10/bin/../lib/gcc/pic32mx/4.5.1/../../../../pic32mx/lib/size\libmchp_peripheral_32MX795F512L.a(rtcc_init_lib.o)
 .debug_frame   0x000078f4       0x34 c:/program files (x86)/microchip/xc32/v1.10/bin/../lib/gcc/pic32mx/4.5.1/../../../../pic32mx/lib/size\libmchp_peripheral_32MX795F512L.a(rtcc_open_lib.o)
 .debug_frame   0x00007928       0x20 c:/program files (x86)/microchip/xc32/v1.10/bin/../lib/gcc/pic32mx/4.5.1/../../../../pic32mx/lib/size\libmchp_peripheral_32MX795F512L.a(spi_chn_data_rdy_lib.o)
 .debug_frame   0x00007948       0x30 c:/program files (x86)/microchip/xc32/v1.10/bin/../lib/gcc/pic32mx/4.5.1/../../../../pic32mx/lib/size\libmchp_peripheral_32MX795F512L.a(spi_chn_getc_lib.o)
 .debug_frame   0x00007978       0x3c c:/program files (x86)/microchip/xc32/v1.10/bin/../lib/gcc/pic32mx/4.5.1/../../../../pic32mx/lib/size\libmchp_peripheral_32MX795F512L.a(spi_chn_open_lib.o)
 .debug_frame   0x000079b4       0x40 c:/program files (x86)/microchip/xc32/v1.10/bin/../lib/gcc/pic32mx/4.5.1/../../../../pic32mx/lib/size\libmchp_peripheral_32MX795F512L.a(spi_chn_putc_lib.o)
 .debug_frame   0x000079f4       0x20 c:/program files (x86)/microchip/xc32/v1.10/bin/../lib/gcc/pic32mx/4.5.1/../../../../pic32mx/lib/size\libmchp_peripheral_32MX795F512L.a(spi_chn_tx_buff_empty_lib.o)
 .debug_frame   0x00007a14       0x20 c:/program files (x86)/microchip/xc32/v1.10/bin/../lib/gcc/pic32mx/4.5.1/../../../../pic32mx/lib/size\libmchp_peripheral_32MX795F512L.a(port_set_pins_digital_in_lib.o)
 .debug_frame   0x00007a34       0x20 c:/program files (x86)/microchip/xc32/v1.10/bin/../lib/gcc/pic32mx/4.5.1/../../../../pic32mx/lib/size\libmchp_peripheral_32MX795F512L.a(port_set_pins_digital_out_lib.o)
 .debug_frame   0x00007a54       0x20 c:/program files (x86)/microchip/xc32/v1.10/bin/../lib/gcc/pic32mx/4.5.1/../../../../pic32mx/lib/size\libmchp_peripheral_32MX795F512L.a(int_enable_interrupts_lib.o)
 .debug_frame   0x00007a74       0x44 c:/program files (x86)/microchip/xc32/v1.10/bin/../lib/gcc/pic32mx/4.5.1/../../../../pic32mx/lib/size\libmchp_peripheral_32MX795F512L.a(_rtcc_wait_clock_off_lib.o)
 .debug_frame   0x00007ab8       0x20 c:/program files (x86)/microchip/xc32/v1.10/bin/../lib/gcc/pic32mx/4.5.1/../../../../pic32mx/lib/size\libmchp_peripheral_32MX795F512L.a(read_core_timer_lib.o)
 .debug_frame   0x00007ad8       0x20 c:/program files (x86)/microchip/xc32/v1.10/bin/../lib/gcc/pic32mx/4.5.1/size\libgcc.a(_udivdi3.o)
 .debug_frame   0x00007af8       0x20 c:/program files (x86)/microchip/xc32/v1.10/bin/../lib/gcc/pic32mx/4.5.1/../../../../pic32mx/lib/size\libpic32.a(default-bootstrap-exception-handler.o)
 .debug_frame   0x00007b18       0x20 c:/program files (x86)/microchip/xc32/v1.10/bin/../lib/gcc/pic32mx/4.5.1/../../../../pic32mx/lib/size\libpic32.a(default-on-reset.o)
 .debug_frame   0x00007b38       0x20 c:/program files (x86)/microchip/xc32/v1.10/bin/../lib/gcc/pic32mx/4.5.1/../../../../pic32mx/lib/size\libpic32.a(default-on-bootstrap.o)
 .debug_frame   0x00007b58       0x20 c:/program files (x86)/microchip/xc32/v1.10/bin/../lib/gcc/pic32mx/4.5.1/../../../../pic32mx/lib/size\libc.a(atoi.o)
 .debug_frame   0x00007b78       0x20 c:/program files (x86)/microchip/xc32/v1.10/bin/../lib/gcc/pic32mx/4.5.1/../../../../pic32mx/lib/size\libc.a(atol.o)
 .debug_frame   0x00007b98       0x6c c:/program files (x86)/microchip/xc32/v1.10/bin/../lib/gcc/pic32mx/4.5.1/../../../../pic32mx/lib/size\libc.a(malloc.o)
 .debug_frame   0x00007c04       0x38 c:/program files (x86)/microchip/xc32/v1.10/bin/../lib/gcc/pic32mx/4.5.1/../../../../pic32mx/lib/size\libc.a(rand.o)
 .debug_frame   0x00007c3c       0x20 c:/program files (x86)/microchip/xc32/v1.10/bin/../lib/gcc/pic32mx/4.5.1/../../../../pic32mx/lib/size\libc.a(strcat.o)
 .debug_frame   0x00007c5c       0x20 c:/program files (x86)/microchip/xc32/v1.10/bin/../lib/gcc/pic32mx/4.5.1/../../../../pic32mx/lib/size\libc.a(strchr.o)
 .debug_frame   0x00007c7c       0x20 c:/program files (x86)/microchip/xc32/v1.10/bin/../lib/gcc/pic32mx/4.5.1/../../../../pic32mx/lib/size\libc.a(strncat.o)
 .debug_frame   0x00007c9c       0x20 c:/program files (x86)/microchip/xc32/v1.10/bin/../lib/gcc/pic32mx/4.5.1/../../../../pic32mx/lib/size\libc.a(strncmp.o)
 .debug_frame   0x00007cbc       0x20 c:/program files (x86)/microchip/xc32/v1.10/bin/../lib/gcc/pic32mx/4.5.1/../../../../pic32mx/lib/size\libc.a(strncpy.o)
 .debug_frame   0x00007cdc       0x28 c:/program files (x86)/microchip/xc32/v1.10/bin/../lib/gcc/pic32mx/4.5.1/../../../../pic32mx/lib/size\libc.a(strrchr.o)
 .debug_frame   0x00007d04       0x2c c:/program files (x86)/microchip/xc32/v1.10/bin/../lib/gcc/pic32mx/4.5.1/../../../../pic32mx/lib/size\libc.a(strstr.o)
 .debug_frame   0x00007d30       0x58 c:/program files (x86)/microchip/xc32/v1.10/bin/../lib/gcc/pic32mx/4.5.1/../../../../pic32mx/lib/size\libc.a(strtol.o)
 .debug_frame   0x00007d88       0x28 c:/program files (x86)/microchip/xc32/v1.10/bin/../lib/gcc/pic32mx/4.5.1/../../../../pic32mx/lib/size\libc.a(snprintf_cdnopsuxX.eo)
 .debug_frame   0x00007db0       0x2c c:/program files (x86)/microchip/xc32/v1.10/bin/../lib/gcc/pic32mx/4.5.1/../../../../pic32mx/lib/size\libc.a(sprintf_cdnopsuxX.eo)
 .debug_frame   0x00007ddc       0x28 c:/program files (x86)/microchip/xc32/v1.10/bin/../lib/gcc/pic32mx/4.5.1/../../../../pic32mx/lib/size\libc.a(vsnprintf_cdnopsuxX.eo)
 .debug_frame   0x00007e04       0x28 c:/program files (x86)/microchip/xc32/v1.10/bin/../lib/gcc/pic32mx/4.5.1/../../../../pic32mx/lib/size\libc.a(vsnprintf.o)
 .debug_frame   0x00007e2c      0x120 c:/program files (x86)/microchip/xc32/v1.10/bin/../lib/gcc/pic32mx/4.5.1/../../../../pic32mx/lib/size\libc.a(ctypef.o)
 .debug_frame   0x00007f4c       0x38 c:/program files (x86)/microchip/xc32/v1.10/bin/../lib/gcc/pic32mx/4.5.1/../../../../pic32mx/lib/size\libc.a(doprnt_cdnopsuxX.eo)
 .debug_frame   0x00007f84       0x74 c:/program files (x86)/microchip/xc32/v1.10/bin/../lib/gcc/pic32mx/4.5.1/../../../../pic32mx/lib/size\libc.a(doprnt.o)
 .debug_frame   0x00007ff8       0x2c c:/program files (x86)/microchip/xc32/v1.10/bin/../lib/gcc/pic32mx/4.5.1/../../../../pic32mx/lib/size\libc.a(_fputc_simple.o)
 .debug_frame   0x00008024       0x28 c:/program files (x86)/microchip/xc32/v1.10/bin/../lib/gcc/pic32mx/4.5.1/../../../../pic32mx/lib/size\libc.a(_flsbuf_simple.o)
 .debug_frame   0x0000804c       0x88 c:/program files (x86)/microchip/xc32/v1.10/bin/../lib/gcc/pic32mx/4.5.1/../../../../pic32mx/lib/size\libpic32.a(sbrk.o)
 .debug_frame   0x000080d4       0x2c c:/program files (x86)/microchip/xc32/v1.10/bin/../lib/gcc/pic32mx/4.5.1/../../../../pic32mx/lib/size\libpic32.a(write.o)
 .debug_frame   0x00008100       0x20 c:/program files (x86)/microchip/xc32/v1.10/bin/../lib/gcc/pic32mx/4.5.1/../../../../pic32mx/lib/size\libpic32.a(_mon_putc.o)
 .debug_frame   0x00008120       0x20 c:/program files (x86)/microchip/xc32/v1.10/bin/../lib/gcc/pic32mx/4.5.1/../../../../pic32mx/lib/size\libe.a(_floatdisf.o)
 .debug_frame   0x00008140       0x20 c:/program files (x86)/microchip/xc32/v1.10/bin/../lib/gcc/pic32mx/4.5.1/size\libgcc.a(_lshrdi3.o)
 .debug_frame   0x00008160       0x2c c:/program files (x86)/microchip/xc32/v1.10/bin/../lib/gcc/pic32mx/4.5.1/size\libgcc.a(_floatundisf.o)
 .debug_frame   0x0000818c       0x20 c:/program files (x86)/microchip/xc32/v1.10/bin/../lib/gcc/pic32mx/4.5.1/size\libgcc.a(_umoddi3.o)
 .debug_frame   0x000081ac       0x28 c:/program files (x86)/microchip/xc32/v1.10/bin/../lib/gcc/pic32mx/4.5.1/size\libgcc.a(floatunsisf.o)

.debug_str      0x00000000     0x9a85
 *(.debug_str)
 .debug_str     0x00000000      0x162 build/default/production/_ext/1293749816/bsp.o
 .debug_str     0x00000162       0x1a build/default/production/_ext/101875047/hashes.o
 .debug_str     0x0000017c        0x0 build/default/production/_ext/101875047/lfsr.o
 .debug_str     0x0000017c      0x12f build/default/production/_ext/101875047/big_int.o
 .debug_str     0x000002ab        0x0 build/default/production/_ext/101875047/helpers.o
 .debug_str     0x000002ab        0x0 build/default/production/_ext/1472/berkeley_tcp_client_demo.o
 .debug_str     0x000002ab        0x0 build/default/production/_ext/1472/berkeley_tcp_server_demo.o
 .debug_str     0x000002ab        0x0 build/default/production/_ext/1472/berkeley_udp_client_demo.o
 .debug_str     0x000002ab      0x156 build/default/production/_ext/1472/generic_tcp_client.o
 .debug_str     0x00000401      0x156 build/default/production/_ext/1472/generic_tcp_server.o
 .debug_str     0x00000557      0x18b build/default/production/_ext/1472/ping_demo.o
 .debug_str     0x000006e2        0x0 build/default/production/_ext/1472/smtp_demo.o
 .debug_str     0x000006e2      0x255 build/default/production/_ext/365611741/system_services.o
 .debug_str     0x00000937      0x15e build/default/production/_ext/365611741/system_debug.o
 .debug_str     0x00000a95      0x15f build/default/production/_ext/365611741/system_random.o
 .debug_str     0x00000bf4      0x127 build/default/production/_ext/365611741/system_command.o
 .debug_str     0x00000d1b      0x173 build/default/production/_ext/365611741/system_userio.o
 .debug_str     0x00000e8e      0x14f build/default/production/_ext/97638081/sys_fs.o
 .debug_str     0x00000fdd      0x135 build/default/production/_ext/97638081/mpfs2.o
 .debug_str     0x00001112      0x11a build/default/production/_ext/792872985/usart.o
 .debug_str     0x0000122c      0x17c build/default/production/_ext/792872985/lcd.o
 .debug_str     0x000013a8      0x156 build/default/production/_ext/792872985/drv_spi.o
 .debug_str     0x000014fe        0x0 build/default/production/_ext/792872985/db_appio.o
 .debug_str     0x000014fe      0x12f build/default/production/_ext/792872985/spi_ram.o
 .debug_str     0x0000162d      0x1be build/default/production/_ext/792872985/spi_eeprom.o
 .debug_str     0x000017eb      0x12f build/default/production/_ext/792872985/spi_flash.o
 .debug_str     0x0000191a      0x1c6 build/default/production/_ext/792872985/drv_media.o
 .debug_str     0x00001ae0      0x196 build/default/production/_ext/427700826/tcpip_announce.o
 .debug_str     0x00001c76      0x1d1 build/default/production/_ext/427700826/http2.o
 .debug_str     0x00001e47      0x170 build/default/production/_ext/427700826/arcfour.o
 .debug_str     0x00001fb7      0x234 build/default/production/_ext/427700826/arp.o
 .debug_str     0x000021eb      0x170 build/default/production/_ext/427700826/berkeley_api.o
 .debug_str     0x0000235b      0x1c6 build/default/production/_ext/427700826/dhcp.o
 .debug_str     0x00002521      0x170 build/default/production/_ext/427700826/dhcps.o
 .debug_str     0x00002691      0x18f build/default/production/_ext/427700826/dns.o
 .debug_str     0x00002820      0x170 build/default/production/_ext/427700826/dnss.o
 .debug_str     0x00002990      0x170 build/default/production/_ext/427700826/dyn_dns.o
 .debug_str     0x00002b00      0x170 build/default/production/_ext/427700826/enc28_mac.o
 .debug_str     0x00002c70      0x170 build/default/production/_ext/427700826/enc28j60.o
 .debug_str     0x00002de0      0x170 build/default/production/_ext/427700826/encs24j600.o
 .debug_str     0x00002f50      0x170 build/default/production/_ext/427700826/encx24_mac.o
 .debug_str     0x000030c0      0x170 build/default/production/_ext/427700826/eth_pic32_ext_phy.o
 .debug_str     0x00003230      0x170 build/default/production/_ext/427700826/eth_pic32_ext_phy_dp83848.o
 .debug_str     0x000033a0      0x170 build/default/production/_ext/427700826/eth_pic32_int_mac.o
 .debug_str     0x00003510      0x170 build/default/production/_ext/427700826/ftp.o
 .debug_str     0x00003680        0x0 build/default/production/_ext/427700826/hash_fnv.o
 .debug_str     0x00003680        0xa build/default/production/_ext/427700826/hash_tbl.o
 .debug_str     0x0000368a      0x1a8 build/default/production/_ext/427700826/icmp.o
 .debug_str     0x00003832      0x170 build/default/production/_ext/427700826/icmpv6.o
 .debug_str     0x000039a2      0x227 build/default/production/_ext/427700826/ipv4.o
 .debug_str     0x00003bc9      0x170 build/default/production/_ext/427700826/ipv6.o
 .debug_str     0x00003d39      0x170 build/default/production/_ext/427700826/mac_events_pic32.o
 .debug_str     0x00003ea9      0x1b1 build/default/production/_ext/427700826/nbns.o
 .debug_str     0x0000405a      0x170 build/default/production/_ext/427700826/ndp.o
 .debug_str     0x000041ca      0x170 build/default/production/_ext/427700826/tcpip_reboot.o
 .debug_str     0x0000433a      0x170 build/default/production/_ext/427700826/rsa.o
 .debug_str     0x000044aa      0x170 build/default/production/_ext/427700826/smtp.o
 .debug_str     0x0000461a      0x170 build/default/production/_ext/427700826/snmp.o
 .debug_str     0x0000478a      0x170 build/default/production/_ext/427700826/snmpv3.o
 .debug_str     0x000048fa      0x170 build/default/production/_ext/427700826/snmpv3_usm.o
 .debug_str     0x00004a6a      0x170 build/default/production/_ext/427700826/sntp.o
 .debug_str     0x00004bda      0x170 build/default/production/_ext/427700826/ssl.o
 .debug_str     0x00004d4a      0x26b build/default/production/_ext/427700826/tcp.o
 .debug_str     0x00004fb5      0x195 build/default/production/_ext/427700826/tcpip_heap_alloc.o
 .debug_str     0x0000514a      0x170 build/default/production/_ext/427700826/tcpip_storage.o
 .debug_str     0x000052ba      0x170 build/default/production/_ext/427700826/telnet.o
 .debug_str     0x0000542a      0x170 build/default/production/_ext/427700826/tftpc.o
 .debug_str     0x0000559a      0x247 build/default/production/_ext/427700826/udp.o
 .debug_str     0x000057e1      0x31b build/default/production/_ext/427700826/tcpip_mac_object.o
 .debug_str     0x00005afc      0x347 build/default/production/_ext/427700826/tcpip_manager.o
 .debug_str     0x00005e43      0x181 build/default/production/_ext/427700826/tcpip_helpers.o
 .debug_str     0x00005fc4      0x170 build/default/production/_ext/427700826/tcpip_commands.o
 .debug_str     0x00006134      0x170 build/default/production/_ext/427700826/iperf.o
 .debug_str     0x000062a4        0xb build/default/production/_ext/427700826/tcpip_notify.o
 .debug_str     0x000062af      0x170 build/default/production/_ext/427700826/zero_conf_helper.o
 .debug_str     0x0000641f      0x170 build/default/production/_ext/427700826/zero_conf_link_local.o
 .debug_str     0x0000658f      0x170 build/default/production/_ext/427700826/zero_conf_multicast_dns.o
 .debug_str     0x000066ff      0x178 build/default/production/_ext/334706090/wf_tx_power.o
 .debug_str     0x00006877      0x1ba build/default/production/_ext/334706090/wf_connect.o
 .debug_str     0x00006a31      0x1b2 build/default/production/_ext/334706090/wf_connection_algorithm.o
 .debug_str     0x00006be3      0x177 build/default/production/_ext/334706090/wf_connection_manager.o
 .debug_str     0x00006d5a      0x200 build/default/production/_ext/334706090/wf_connection_profile.o
 .debug_str     0x00006f5a      0x17a build/default/production/_ext/334706090/wf_easy_config.o
 .debug_str     0x000070d4      0x1a1 build/default/production/_ext/334706090/wf_eint.o
 .debug_str     0x00007275      0x1ac build/default/production/_ext/334706090/wf_event_handler.o
 .debug_str     0x00007421      0x242 build/default/production/_ext/334706090/wf_init.o
 .debug_str     0x00007663      0x1a4 build/default/production/_ext/334706090/wf_power_save.o
 .debug_str     0x00007807      0x170 build/default/production/_ext/334706090/wf_scan.o
 .debug_str     0x00007977      0x183 build/default/production/_ext/334706090/wf_spi.o
 .debug_str     0x00007afa      0x1b3 build/default/production/_ext/334706090/mrf24w_mac_pic32.o
 .debug_str     0x00007cad      0x18b build/default/production/_ext/334706090/mrf24w_events.o
 .debug_str     0x00007e38      0x2e1 build/default/production/_ext/334706090/wf_debug_output.o
 .debug_str     0x00008119      0x1bc build/default/production/_ext/334706090/wf_commands.o
 .debug_str     0x000082d5      0x170 build/default/production/_ext/334706090/wf_pbkdf2.o
 .debug_str     0x00008445      0x237 build/default/production/_ext/334706090/wf_driver_com_24g.o
 .debug_str     0x0000867c      0x22f build/default/production/_ext/334706090/wf_driver_raw_24g.o
 .debug_str     0x000088ab      0x241 build/default/production/_ext/334706090/wf_mac_24g.o
 .debug_str     0x00008aec      0x1b5 build/default/production/_ext/334706090/wf_mgmt_msg_24g.o
 .debug_str     0x00008ca1      0x1e0 build/default/production/_ext/334706090/wf_param_msg_24g.o
 .debug_str     0x00008e81      0x239 build/default/production/_ext/334706090/wf_configData.o
 .debug_str     0x000090ba      0x28a build/default/production/_ext/1472/main_demo.o
 .debug_str     0x00009344        0x0 build/default/production/_ext/1472/custom_snmp_app.o
 .debug_str     0x00009344        0x0 build/default/production/_ext/1472/custom_ssl_cert.o
 .debug_str     0x00009344      0x12f build/default/production/_ext/1472/mpfs_img2.o
 .debug_str     0x00009473      0x156 build/default/production/_ext/1472/wf_config.o
 .debug_str     0x000095c9      0x1c3 build/default/production/_ext/1472/custom_http_app.o
 .debug_str     0x0000978c      0x2f9 build/default/production/_ext/1472/tcp6_demo_app.o
 .debug_str     0x00009a85        0x0 c:/program files (x86)/microchip/xc32/v1.10/bin/../lib/gcc/pic32mx/4.5.1/../../../../pic32mx/lib/size\libmchp_peripheral.a(open_core_timer_lib.o)
 .debug_str     0x00009a85        0x0 c:/program files (x86)/microchip/xc32/v1.10/bin/../lib/gcc/pic32mx/4.5.1/../../../../pic32mx/lib/size\libmchp_peripheral_32MX795F512L.a(soft_reset_lib.o)
 .debug_str     0x00009a85        0x0 c:/program files (x86)/microchip/xc32/v1.10/bin/../lib/gcc/pic32mx/4.5.1/../../../../pic32mx/lib/size\libmchp_peripheral_32MX795F512L.a(pcache.o)
 .debug_str     0x00009a85        0x0 c:/program files (x86)/microchip/xc32/v1.10/bin/../lib/gcc/pic32mx/4.5.1/../../../../pic32mx/lib/size\libmchp_peripheral_32MX795F512L.a(int_disable_interrupts_lib.o)
 .debug_str     0x00009a85        0x0 c:/program files (x86)/microchip/xc32/v1.10/bin/../lib/gcc/pic32mx/4.5.1/../../../../pic32mx/lib/size\libmchp_peripheral_32MX795F512L.a(int_restore_interrupts_lib.o)
 .debug_str     0x00009a85        0x0 c:/program files (x86)/microchip/xc32/v1.10/bin/../lib/gcc/pic32mx/4.5.1/../../../../pic32mx/lib/size\libmchp_peripheral_32MX795F512L.a(int_enable_mv_int_lib.o)
 .debug_str     0x00009a85        0x0 c:/program files (x86)/microchip/xc32/v1.10/bin/../lib/gcc/pic32mx/4.5.1/../../../../pic32mx/lib/size\libmchp_peripheral_32MX795F512L.a(int_tbl_lib.o)
 .debug_str     0x00009a85        0x0 c:/program files (x86)/microchip/xc32/v1.10/bin/../lib/gcc/pic32mx/4.5.1/../../../../pic32mx/lib/size\libmchp_peripheral_32MX795F512L.a(rtcc_init_lib.o)
 .debug_str     0x00009a85        0x0 c:/program files (x86)/microchip/xc32/v1.10/bin/../lib/gcc/pic32mx/4.5.1/../../../../pic32mx/lib/size\libmchp_peripheral_32MX795F512L.a(rtcc_open_lib.o)
 .debug_str     0x00009a85        0x0 c:/program files (x86)/microchip/xc32/v1.10/bin/../lib/gcc/pic32mx/4.5.1/../../../../pic32mx/lib/size\libmchp_peripheral_32MX795F512L.a(spi_chn_data_rdy_lib.o)
 .debug_str     0x00009a85        0x0 c:/program files (x86)/microchip/xc32/v1.10/bin/../lib/gcc/pic32mx/4.5.1/../../../../pic32mx/lib/size\libmchp_peripheral_32MX795F512L.a(spi_chn_getc_lib.o)
 .debug_str     0x00009a85        0x0 c:/program files (x86)/microchip/xc32/v1.10/bin/../lib/gcc/pic32mx/4.5.1/../../../../pic32mx/lib/size\libmchp_peripheral_32MX795F512L.a(spi_chn_open_lib.o)
 .debug_str     0x00009a85        0x0 c:/program files (x86)/microchip/xc32/v1.10/bin/../lib/gcc/pic32mx/4.5.1/../../../../pic32mx/lib/size\libmchp_peripheral_32MX795F512L.a(spi_chn_putc_lib.o)
 .debug_str     0x00009a85        0x0 c:/program files (x86)/microchip/xc32/v1.10/bin/../lib/gcc/pic32mx/4.5.1/../../../../pic32mx/lib/size\libmchp_peripheral_32MX795F512L.a(spi_chn_tx_buff_empty_lib.o)
 .debug_str     0x00009a85        0x0 c:/program files (x86)/microchip/xc32/v1.10/bin/../lib/gcc/pic32mx/4.5.1/../../../../pic32mx/lib/size\libmchp_peripheral_32MX795F512L.a(spi_io_tbl_libp.o)
 .debug_str     0x00009a85        0x0 c:/program files (x86)/microchip/xc32/v1.10/bin/../lib/gcc/pic32mx/4.5.1/../../../../pic32mx/lib/size\libmchp_peripheral_32MX795F512L.a(spi_map_tbl_libp.o)
 .debug_str     0x00009a85        0x0 c:/program files (x86)/microchip/xc32/v1.10/bin/../lib/gcc/pic32mx/4.5.1/../../../../pic32mx/lib/size\libmchp_peripheral_32MX795F512L.a(port_set_pins_digital_in_lib.o)
 .debug_str     0x00009a85        0x0 c:/program files (x86)/microchip/xc32/v1.10/bin/../lib/gcc/pic32mx/4.5.1/../../../../pic32mx/lib/size\libmchp_peripheral_32MX795F512L.a(port_set_pins_digital_out_lib.o)
 .debug_str     0x00009a85        0x0 c:/program files (x86)/microchip/xc32/v1.10/bin/../lib/gcc/pic32mx/4.5.1/../../../../pic32mx/lib/size\libmchp_peripheral_32MX795F512L.a(_ports_tbl_libp.o)
 .debug_str     0x00009a85        0x0 c:/program files (x86)/microchip/xc32/v1.10/bin/../lib/gcc/pic32mx/4.5.1/../../../../pic32mx/lib/size\libmchp_peripheral_32MX795F512L.a(int_enable_interrupts_lib.o)
 .debug_str     0x00009a85        0x0 c:/program files (x86)/microchip/xc32/v1.10/bin/../lib/gcc/pic32mx/4.5.1/../../../../pic32mx/lib/size\libmchp_peripheral_32MX795F512L.a(_rtcc_wait_clock_off_lib.o)
 .debug_str     0x00009a85        0x0 c:/program files (x86)/microchip/xc32/v1.10/bin/../lib/gcc/pic32mx/4.5.1/../../../../pic32mx/lib/size\libmchp_peripheral_32MX795F512L.a(read_core_timer_lib.o)
 .debug_str     0x00009a85        0x0 c:/program files (x86)/microchip/xc32/v1.10/bin/../lib/gcc/pic32mx/4.5.1/size\libgcc.a(_udivdi3.o)
 .debug_str     0x00009a85        0x0 c:/program files (x86)/microchip/xc32/v1.10/bin/../lib/gcc/pic32mx/4.5.1/../../../../pic32mx/lib/size\libpic32.a(default-bootstrap-exception-handler.o)
 .debug_str     0x00009a85        0x0 c:/program files (x86)/microchip/xc32/v1.10/bin/../lib/gcc/pic32mx/4.5.1/../../../../pic32mx/lib/size\libpic32.a(default-on-reset.o)
 .debug_str     0x00009a85        0x0 c:/program files (x86)/microchip/xc32/v1.10/bin/../lib/gcc/pic32mx/4.5.1/../../../../pic32mx/lib/size\libpic32.a(default-on-bootstrap.o)
 .debug_str     0x00009a85        0x0 c:/program files (x86)/microchip/xc32/v1.10/bin/../lib/gcc/pic32mx/4.5.1/../../../../pic32mx/lib/size\libpic32.a(errno.o)
 .debug_str     0x00009a85        0x0 c:/program files (x86)/microchip/xc32/v1.10/bin/../lib/gcc/pic32mx/4.5.1/../../../../pic32mx/lib/size\libc.a(atoi.o)
 .debug_str     0x00009a85        0x0 c:/program files (x86)/microchip/xc32/v1.10/bin/../lib/gcc/pic32mx/4.5.1/../../../../pic32mx/lib/size\libc.a(atol.o)
 .debug_str     0x00009a85        0x0 c:/program files (x86)/microchip/xc32/v1.10/bin/../lib/gcc/pic32mx/4.5.1/../../../../pic32mx/lib/size\libc.a(ctype.o)
 .debug_str     0x00009a85        0x0 c:/program files (x86)/microchip/xc32/v1.10/bin/../lib/gcc/pic32mx/4.5.1/../../../../pic32mx/lib/size\libc.a(malloc.o)
 .debug_str     0x00009a85        0x0 c:/program files (x86)/microchip/xc32/v1.10/bin/../lib/gcc/pic32mx/4.5.1/../../../../pic32mx/lib/size\libc.a(rand.o)
 .debug_str     0x00009a85        0x0 c:/program files (x86)/microchip/xc32/v1.10/bin/../lib/gcc/pic32mx/4.5.1/../../../../pic32mx/lib/size\libc.a(strcat.o)
 .debug_str     0x00009a85        0x0 c:/program files (x86)/microchip/xc32/v1.10/bin/../lib/gcc/pic32mx/4.5.1/../../../../pic32mx/lib/size\libc.a(strchr.o)
 .debug_str     0x00009a85        0x0 c:/program files (x86)/microchip/xc32/v1.10/bin/../lib/gcc/pic32mx/4.5.1/../../../../pic32mx/lib/size\libc.a(strncat.o)
 .debug_str     0x00009a85        0x0 c:/program files (x86)/microchip/xc32/v1.10/bin/../lib/gcc/pic32mx/4.5.1/../../../../pic32mx/lib/size\libc.a(strncmp.o)
 .debug_str     0x00009a85        0x0 c:/program files (x86)/microchip/xc32/v1.10/bin/../lib/gcc/pic32mx/4.5.1/../../../../pic32mx/lib/size\libc.a(strncpy.o)
 .debug_str     0x00009a85        0x0 c:/program files (x86)/microchip/xc32/v1.10/bin/../lib/gcc/pic32mx/4.5.1/../../../../pic32mx/lib/size\libc.a(strrchr.o)
 .debug_str     0x00009a85        0x0 c:/program files (x86)/microchip/xc32/v1.10/bin/../lib/gcc/pic32mx/4.5.1/../../../../pic32mx/lib/size\libc.a(strstr.o)
 .debug_str     0x00009a85        0x0 c:/program files (x86)/microchip/xc32/v1.10/bin/../lib/gcc/pic32mx/4.5.1/../../../../pic32mx/lib/size\libc.a(strtol.o)
 .debug_str     0x00009a85        0x0 c:/program files (x86)/microchip/xc32/v1.10/bin/../lib/gcc/pic32mx/4.5.1/../../../../pic32mx/lib/size\libc.a(snprintf_cdnopsuxX.eo)
 .debug_str     0x00009a85        0x0 c:/program files (x86)/microchip/xc32/v1.10/bin/../lib/gcc/pic32mx/4.5.1/../../../../pic32mx/lib/size\libc.a(sprintf_cdnopsuxX.eo)
 .debug_str     0x00009a85        0x0 c:/program files (x86)/microchip/xc32/v1.10/bin/../lib/gcc/pic32mx/4.5.1/../../../../pic32mx/lib/size\libc.a(vsnprintf_cdnopsuxX.eo)
 .debug_str     0x00009a85        0x0 c:/program files (x86)/microchip/xc32/v1.10/bin/../lib/gcc/pic32mx/4.5.1/../../../../pic32mx/lib/size\libc.a(vsnprintf.o)
 .debug_str     0x00009a85        0x0 c:/program files (x86)/microchip/xc32/v1.10/bin/../lib/gcc/pic32mx/4.5.1/../../../../pic32mx/lib/size\libc.a(ctypef.o)
 .debug_str     0x00009a85        0x0 c:/program files (x86)/microchip/xc32/v1.10/bin/../lib/gcc/pic32mx/4.5.1/../../../../pic32mx/lib/size\libc.a(doprnt_cdnopsuxX.eo)
 .debug_str     0x00009a85        0x0 c:/program files (x86)/microchip/xc32/v1.10/bin/../lib/gcc/pic32mx/4.5.1/../../../../pic32mx/lib/size\libc.a(doprnt.o)
 .debug_str     0x00009a85        0x0 c:/program files (x86)/microchip/xc32/v1.10/bin/../lib/gcc/pic32mx/4.5.1/../../../../pic32mx/lib/size\libc.a(_fputc_simple.o)
 .debug_str     0x00009a85        0x0 c:/program files (x86)/microchip/xc32/v1.10/bin/../lib/gcc/pic32mx/4.5.1/../../../../pic32mx/lib/size\libc.a(powersf.o)
 .debug_str     0x00009a85        0x0 c:/program files (x86)/microchip/xc32/v1.10/bin/../lib/gcc/pic32mx/4.5.1/../../../../pic32mx/lib/size\libc.a(_iob.o)
 .debug_str     0x00009a85        0x0 c:/program files (x86)/microchip/xc32/v1.10/bin/../lib/gcc/pic32mx/4.5.1/../../../../pic32mx/lib/size\libc.a(_flsbuf_simple.o)
 .debug_str     0x00009a85        0x0 c:/program files (x86)/microchip/xc32/v1.10/bin/../lib/gcc/pic32mx/4.5.1/../../../../pic32mx/lib/size\libpic32.a(sbrk.o)
 .debug_str     0x00009a85        0x0 c:/program files (x86)/microchip/xc32/v1.10/bin/../lib/gcc/pic32mx/4.5.1/../../../../pic32mx/lib/size\libpic32.a(write.o)
 .debug_str     0x00009a85        0x0 c:/program files (x86)/microchip/xc32/v1.10/bin/../lib/gcc/pic32mx/4.5.1/../../../../pic32mx/lib/size\libpic32.a(_mon_putc.o)
 .debug_str     0x00009a85        0x0 c:/program files (x86)/microchip/xc32/v1.10/bin/../lib/gcc/pic32mx/4.5.1/../../../../pic32mx/lib/size\libpic32.a(xc32_uart.o)
 .debug_str     0x00009a85        0x0 c:/program files (x86)/microchip/xc32/v1.10/bin/../lib/gcc/pic32mx/4.5.1/../../../../pic32mx/lib/size\libe.a(_floatdisf.o)
 .debug_str     0x00009a85        0x0 c:/program files (x86)/microchip/xc32/v1.10/bin/../lib/gcc/pic32mx/4.5.1/size\libgcc.a(_lshrdi3.o)
 .debug_str     0x00009a85        0x0 c:/program files (x86)/microchip/xc32/v1.10/bin/../lib/gcc/pic32mx/4.5.1/size\libgcc.a(_floatundisf.o)
 .debug_str     0x00009a85        0x0 c:/program files (x86)/microchip/xc32/v1.10/bin/../lib/gcc/pic32mx/4.5.1/size\libgcc.a(_umoddi3.o)
 .debug_str     0x00009a85        0x0 c:/program files (x86)/microchip/xc32/v1.10/bin/../lib/gcc/pic32mx/4.5.1/size\libgcc.a(floatunsisf.o)

.debug_loc      0x00000000     0x16cc
 *(.debug_loc)
 .debug_loc     0x00000000      0xaaf c:/program files (x86)/microchip/xc32/v1.10/bin/../lib/gcc/pic32mx/4.5.1/size\libgcc.a(_udivdi3.o)
 .debug_loc     0x00000aaf       0x5f c:/program files (x86)/microchip/xc32/v1.10/bin/../lib/gcc/pic32mx/4.5.1/size\libgcc.a(_lshrdi3.o)
 .debug_loc     0x00000b0e       0xc9 c:/program files (x86)/microchip/xc32/v1.10/bin/../lib/gcc/pic32mx/4.5.1/size\libgcc.a(_floatundisf.o)
 .debug_loc     0x00000bd7      0xa98 c:/program files (x86)/microchip/xc32/v1.10/bin/../lib/gcc/pic32mx/4.5.1/size\libgcc.a(_umoddi3.o)
 .debug_loc     0x0000166f       0x5d c:/program files (x86)/microchip/xc32/v1.10/bin/../lib/gcc/pic32mx/4.5.1/size\libgcc.a(floatunsisf.o)

.debug_macinfo
 *(.debug_macinfo)

.debug_weaknames
 *(.debug_weaknames)

.debug_funcnames
 *(.debug_funcnames)

.debug_typenames
 *(.debug_typenames)

.debug_varnames
 *(.debug_varnames)

.debug_pubtypes
                0x00000000     0xb013
 *(.debug_pubtypes)
 .debug_pubtypes
                0x00000000      0x120 build/default/production/_ext/1293749816/bsp.o
 .debug_pubtypes
                0x00000120       0x6d build/default/production/_ext/101875047/hashes.o
 .debug_pubtypes
                0x0000018d       0x3e build/default/production/_ext/101875047/lfsr.o
 .debug_pubtypes
                0x000001cb      0x13a build/default/production/_ext/101875047/big_int.o
 .debug_pubtypes
                0x00000305       0x68 build/default/production/_ext/101875047/helpers.o
 .debug_pubtypes
                0x0000036d       0xf4 build/default/production/_ext/1472/generic_tcp_client.o
 .debug_pubtypes
                0x00000461       0xf4 build/default/production/_ext/1472/generic_tcp_server.o
 .debug_pubtypes
                0x00000555      0x17a build/default/production/_ext/1472/ping_demo.o
 .debug_pubtypes
                0x000006cf      0x2a9 build/default/production/_ext/365611741/system_services.o
 .debug_pubtypes
                0x00000978      0x1a8 build/default/production/_ext/365611741/system_debug.o
 .debug_pubtypes
                0x00000b20      0x14c build/default/production/_ext/365611741/system_random.o
 .debug_pubtypes
                0x00000c6c      0x1c6 build/default/production/_ext/365611741/system_command.o
 .debug_pubtypes
                0x00000e32      0x1fe build/default/production/_ext/365611741/system_userio.o
 .debug_pubtypes
                0x00001030      0x1ab build/default/production/_ext/97638081/sys_fs.o
 .debug_pubtypes
                0x000011db      0x192 build/default/production/_ext/97638081/mpfs2.o
 .debug_pubtypes
                0x0000136d      0x1a7 build/default/production/_ext/792872985/usart.o
 .debug_pubtypes
                0x00001514      0x174 build/default/production/_ext/792872985/lcd.o
 .debug_pubtypes
                0x00001688      0x131 build/default/production/_ext/792872985/drv_spi.o
 .debug_pubtypes
                0x000017b9       0xe7 build/default/production/_ext/792872985/spi_ram.o
 .debug_pubtypes
                0x000018a0      0x17e build/default/production/_ext/792872985/spi_eeprom.o
 .debug_pubtypes
                0x00001a1e       0xe7 build/default/production/_ext/792872985/spi_flash.o
 .debug_pubtypes
                0x00001b05      0x29a build/default/production/_ext/792872985/drv_media.o
 .debug_pubtypes
                0x00001d9f      0x32f build/default/production/_ext/427700826/tcpip_announce.o
 .debug_pubtypes
                0x000020ce      0x36f build/default/production/_ext/427700826/http2.o
 .debug_pubtypes
                0x0000243d      0x12c build/default/production/_ext/427700826/arcfour.o
 .debug_pubtypes
                0x00002569      0x483 build/default/production/_ext/427700826/arp.o
 .debug_pubtypes
                0x000029ec      0x12c build/default/production/_ext/427700826/berkeley_api.o
 .debug_pubtypes
                0x00002b18      0x392 build/default/production/_ext/427700826/dhcp.o
 .debug_pubtypes
                0x00002eaa      0x141 build/default/production/_ext/427700826/dhcps.o
 .debug_pubtypes
                0x00002feb      0x34b build/default/production/_ext/427700826/dns.o
 .debug_pubtypes
                0x00003336      0x12c build/default/production/_ext/427700826/dnss.o
 .debug_pubtypes
                0x00003462      0x12c build/default/production/_ext/427700826/dyn_dns.o
 .debug_pubtypes
                0x0000358e      0x12c build/default/production/_ext/427700826/enc28_mac.o
 .debug_pubtypes
                0x000036ba      0x12c build/default/production/_ext/427700826/enc28j60.o
 .debug_pubtypes
                0x000037e6      0x12c build/default/production/_ext/427700826/encs24j600.o
 .debug_pubtypes
                0x00003912      0x12c build/default/production/_ext/427700826/encx24_mac.o
 .debug_pubtypes
                0x00003a3e      0x12c build/default/production/_ext/427700826/eth_pic32_ext_phy.o
 .debug_pubtypes
                0x00003b6a      0x12c build/default/production/_ext/427700826/eth_pic32_ext_phy_dp83848.o
 .debug_pubtypes
                0x00003c96      0x12c build/default/production/_ext/427700826/eth_pic32_int_mac.o
 .debug_pubtypes
                0x00003dc2      0x12c build/default/production/_ext/427700826/ftp.o
 .debug_pubtypes
                0x00003eee       0x3a build/default/production/_ext/427700826/hash_fnv.o
 .debug_pubtypes
                0x00003f28       0xe1 build/default/production/_ext/427700826/hash_tbl.o
 .debug_pubtypes
                0x00004009      0x360 build/default/production/_ext/427700826/icmp.o
 .debug_pubtypes
                0x00004369      0x12c build/default/production/_ext/427700826/icmpv6.o
 .debug_pubtypes
                0x00004495      0x399 build/default/production/_ext/427700826/ipv4.o
 .debug_pubtypes
                0x0000482e      0x12c build/default/production/_ext/427700826/ipv6.o
 .debug_pubtypes
                0x0000495a      0x12c build/default/production/_ext/427700826/mac_events_pic32.o
 .debug_pubtypes
                0x00004a86      0x3f7 build/default/production/_ext/427700826/nbns.o
 .debug_pubtypes
                0x00004e7d      0x12c build/default/production/_ext/427700826/ndp.o
 .debug_pubtypes
                0x00004fa9      0x12c build/default/production/_ext/427700826/tcpip_reboot.o
 .debug_pubtypes
                0x000050d5      0x12c build/default/production/_ext/427700826/rsa.o
 .debug_pubtypes
                0x00005201      0x12c build/default/production/_ext/427700826/smtp.o
 .debug_pubtypes
                0x0000532d      0x12c build/default/production/_ext/427700826/snmp.o
 .debug_pubtypes
                0x00005459      0x12c build/default/production/_ext/427700826/snmpv3.o
 .debug_pubtypes
                0x00005585      0x12c build/default/production/_ext/427700826/snmpv3_usm.o
 .debug_pubtypes
                0x000056b1      0x12c build/default/production/_ext/427700826/sntp.o
 .debug_pubtypes
                0x000057dd      0x12c build/default/production/_ext/427700826/ssl.o
 .debug_pubtypes
                0x00005909      0x4a1 build/default/production/_ext/427700826/tcp.o
 .debug_pubtypes
                0x00005daa      0x203 build/default/production/_ext/427700826/tcpip_heap_alloc.o
 .debug_pubtypes
                0x00005fad      0x12c build/default/production/_ext/427700826/tcpip_storage.o
 .debug_pubtypes
                0x000060d9      0x12c build/default/production/_ext/427700826/telnet.o
 .debug_pubtypes
                0x00006205      0x12c build/default/production/_ext/427700826/tftpc.o
 .debug_pubtypes
                0x00006331      0x44b build/default/production/_ext/427700826/udp.o
 .debug_pubtypes
                0x0000677c      0x238 build/default/production/_ext/427700826/tcpip_mac_object.o
 .debug_pubtypes
                0x000069b4      0x5c4 build/default/production/_ext/427700826/tcpip_manager.o
 .debug_pubtypes
                0x00006f78      0x262 build/default/production/_ext/427700826/tcpip_helpers.o
 .debug_pubtypes
                0x000071da      0x12c build/default/production/_ext/427700826/tcpip_commands.o
 .debug_pubtypes
                0x00007306      0x12c build/default/production/_ext/427700826/iperf.o
 .debug_pubtypes
                0x00007432       0x6c build/default/production/_ext/427700826/tcpip_notify.o
 .debug_pubtypes
                0x0000749e      0x12c build/default/production/_ext/427700826/zero_conf_helper.o
 .debug_pubtypes
                0x000075ca      0x141 build/default/production/_ext/427700826/zero_conf_link_local.o
 .debug_pubtypes
                0x0000770b      0x12c build/default/production/_ext/427700826/zero_conf_multicast_dns.o
 .debug_pubtypes
                0x00007837      0x155 build/default/production/_ext/334706090/wf_tx_power.o
 .debug_pubtypes
                0x0000798c      0x20c build/default/production/_ext/334706090/wf_connect.o
 .debug_pubtypes
                0x00007b98      0x1f9 build/default/production/_ext/334706090/wf_connection_algorithm.o
 .debug_pubtypes
                0x00007d91      0x17b build/default/production/_ext/334706090/wf_connection_manager.o
 .debug_pubtypes
                0x00007f0c      0x27f build/default/production/_ext/334706090/wf_connection_profile.o
 .debug_pubtypes
                0x0000818b      0x1c0 build/default/production/_ext/334706090/wf_easy_config.o
 .debug_pubtypes
                0x0000834b      0x185 build/default/production/_ext/334706090/wf_eint.o
 .debug_pubtypes
                0x000084d0      0x21b build/default/production/_ext/334706090/wf_event_handler.o
 .debug_pubtypes
                0x000086eb      0x22c build/default/production/_ext/334706090/wf_init.o
 .debug_pubtypes
                0x00008917      0x1bf build/default/production/_ext/334706090/wf_power_save.o
 .debug_pubtypes
                0x00008ad6      0x171 build/default/production/_ext/334706090/wf_scan.o
 .debug_pubtypes
                0x00008c47      0x16c build/default/production/_ext/334706090/wf_spi.o
 .debug_pubtypes
                0x00008db3      0x343 build/default/production/_ext/334706090/mrf24w_mac_pic32.o
 .debug_pubtypes
                0x000090f6      0x1e2 build/default/production/_ext/334706090/mrf24w_events.o
 .debug_pubtypes
                0x000092d8      0x295 build/default/production/_ext/334706090/wf_debug_output.o
 .debug_pubtypes
                0x0000956d      0x2b8 build/default/production/_ext/334706090/wf_commands.o
 .debug_pubtypes
                0x00009825      0x12c build/default/production/_ext/334706090/wf_pbkdf2.o
 .debug_pubtypes
                0x00009951      0x25c build/default/production/_ext/334706090/wf_driver_com_24g.o
 .debug_pubtypes
                0x00009bad      0x16a build/default/production/_ext/334706090/wf_driver_raw_24g.o
 .debug_pubtypes
                0x00009d17      0x295 build/default/production/_ext/334706090/wf_mac_24g.o
 .debug_pubtypes
                0x00009fac      0x17e build/default/production/_ext/334706090/wf_mgmt_msg_24g.o
 .debug_pubtypes
                0x0000a12a      0x21b build/default/production/_ext/334706090/wf_param_msg_24g.o
 .debug_pubtypes
                0x0000a345      0x217 build/default/production/_ext/334706090/wf_configData.o
 .debug_pubtypes
                0x0000a55c      0x2fa build/default/production/_ext/1472/main_demo.o
 .debug_pubtypes
                0x0000a856       0xe7 build/default/production/_ext/1472/mpfs_img2.o
 .debug_pubtypes
                0x0000a93d      0x111 build/default/production/_ext/1472/wf_config.o
 .debug_pubtypes
                0x0000aa4e      0x1e5 build/default/production/_ext/1472/custom_http_app.o
 .debug_pubtypes
                0x0000ac33      0x258 build/default/production/_ext/1472/tcp6_demo_app.o
 .debug_pubtypes
                0x0000ae8b       0x59 c:/program files (x86)/microchip/xc32/v1.10/bin/../lib/gcc/pic32mx/4.5.1/size\libgcc.a(_udivdi3.o)
 .debug_pubtypes
                0x0000aee4       0x62 c:/program files (x86)/microchip/xc32/v1.10/bin/../lib/gcc/pic32mx/4.5.1/size\libgcc.a(_lshrdi3.o)
 .debug_pubtypes
                0x0000af46       0x40 c:/program files (x86)/microchip/xc32/v1.10/bin/../lib/gcc/pic32mx/4.5.1/size\libgcc.a(_floatundisf.o)
 .debug_pubtypes
                0x0000af86       0x59 c:/program files (x86)/microchip/xc32/v1.10/bin/../lib/gcc/pic32mx/4.5.1/size\libgcc.a(_umoddi3.o)
 .debug_pubtypes
                0x0000afdf       0x34 c:/program files (x86)/microchip/xc32/v1.10/bin/../lib/gcc/pic32mx/4.5.1/size\libgcc.a(floatunsisf.o)

.debug_ranges   0x00000000     0x2898
 *(.debug_ranges)
 .debug_ranges  0x00000000       0x10 build/default/production/_ext/1293749816/bsp.o
 .debug_ranges  0x00000010       0x50 build/default/production/_ext/101875047/hashes.o
 .debug_ranges  0x00000060       0x18 build/default/production/_ext/101875047/lfsr.o
 .debug_ranges  0x00000078       0x70 build/default/production/_ext/101875047/big_int.o
 .debug_ranges  0x000000e8       0x48 build/default/production/_ext/101875047/helpers.o
 .debug_ranges  0x00000130       0x20 build/default/production/_ext/1472/ping_demo.o
 .debug_ranges  0x00000150      0x150 build/default/production/_ext/365611741/system_services.o
 .debug_ranges  0x000002a0       0xb8 build/default/production/_ext/365611741/system_debug.o
 .debug_ranges  0x00000358       0x30 build/default/production/_ext/365611741/system_random.o
 .debug_ranges  0x00000388       0xb0 build/default/production/_ext/365611741/system_command.o
 .debug_ranges  0x00000438       0x48 build/default/production/_ext/365611741/system_userio.o
 .debug_ranges  0x00000480      0x230 build/default/production/_ext/97638081/sys_fs.o
 .debug_ranges  0x000006b0       0xc8 build/default/production/_ext/97638081/mpfs2.o
 .debug_ranges  0x00000778       0x40 build/default/production/_ext/792872985/usart.o
 .debug_ranges  0x000007b8       0x38 build/default/production/_ext/792872985/lcd.o
 .debug_ranges  0x000007f0       0x20 build/default/production/_ext/792872985/drv_spi.o
 .debug_ranges  0x00000810       0x60 build/default/production/_ext/792872985/spi_eeprom.o
 .debug_ranges  0x00000870       0x80 build/default/production/_ext/792872985/drv_media.o
 .debug_ranges  0x000008f0       0x40 build/default/production/_ext/427700826/tcpip_announce.o
 .debug_ranges  0x00000930      0x130 build/default/production/_ext/427700826/http2.o
 .debug_ranges  0x00000a60      0x128 build/default/production/_ext/427700826/arp.o
 .debug_ranges  0x00000b88       0xa0 build/default/production/_ext/427700826/dhcp.o
 .debug_ranges  0x00000c28       0x20 build/default/production/_ext/427700826/dhcps.o
 .debug_ranges  0x00000c48       0x60 build/default/production/_ext/427700826/dns.o
 .debug_ranges  0x00000ca8       0x18 build/default/production/_ext/427700826/hash_fnv.o
 .debug_ranges  0x00000cc0       0x48 build/default/production/_ext/427700826/hash_tbl.o
 .debug_ranges  0x00000d08       0x40 build/default/production/_ext/427700826/icmp.o
 .debug_ranges  0x00000d48      0x140 build/default/production/_ext/427700826/ipv4.o
 .debug_ranges  0x00000e88       0x30 build/default/production/_ext/427700826/nbns.o
 .debug_ranges  0x00000eb8      0x290 build/default/production/_ext/427700826/tcp.o
 .debug_ranges  0x00001148       0x88 build/default/production/_ext/427700826/tcpip_heap_alloc.o
 .debug_ranges  0x000011d0      0x160 build/default/production/_ext/427700826/udp.o
 .debug_ranges  0x00001330       0xc8 build/default/production/_ext/427700826/tcpip_mac_object.o
 .debug_ranges  0x000013f8      0x288 build/default/production/_ext/427700826/tcpip_manager.o
 .debug_ranges  0x00001680       0xd8 build/default/production/_ext/427700826/tcpip_helpers.o
 .debug_ranges  0x00001758       0x20 build/default/production/_ext/427700826/tcpip_notify.o
 .debug_ranges  0x00001778       0x20 build/default/production/_ext/427700826/zero_conf_link_local.o
 .debug_ranges  0x00001798       0x20 build/default/production/_ext/334706090/wf_tx_power.o
 .debug_ranges  0x000017b8       0x30 build/default/production/_ext/334706090/wf_connect.o
 .debug_ranges  0x000017e8       0x98 build/default/production/_ext/334706090/wf_connection_algorithm.o
 .debug_ranges  0x00001880       0x40 build/default/production/_ext/334706090/wf_connection_manager.o
 .debug_ranges  0x000018c0       0xc8 build/default/production/_ext/334706090/wf_connection_profile.o
 .debug_ranges  0x00001988       0x10 build/default/production/_ext/334706090/wf_easy_config.o
 .debug_ranges  0x00001998       0x30 build/default/production/_ext/334706090/wf_eint.o
 .debug_ranges  0x000019c8       0x58 build/default/production/_ext/334706090/wf_event_handler.o
 .debug_ranges  0x00001a20       0x30 build/default/production/_ext/334706090/wf_init.o
 .debug_ranges  0x00001a50       0x80 build/default/production/_ext/334706090/wf_power_save.o
 .debug_ranges  0x00001ad0       0x20 build/default/production/_ext/334706090/wf_scan.o
 .debug_ranges  0x00001af0       0x30 build/default/production/_ext/334706090/wf_spi.o
 .debug_ranges  0x00001b20       0xf8 build/default/production/_ext/334706090/mrf24w_mac_pic32.o
 .debug_ranges  0x00001c18       0x60 build/default/production/_ext/334706090/mrf24w_events.o
 .debug_ranges  0x00001c78       0xa8 build/default/production/_ext/334706090/wf_debug_output.o
 .debug_ranges  0x00001d20       0x80 build/default/production/_ext/334706090/wf_commands.o
 .debug_ranges  0x00001da0       0xc8 build/default/production/_ext/334706090/wf_driver_com_24g.o
 .debug_ranges  0x00001e68       0xb0 build/default/production/_ext/334706090/wf_driver_raw_24g.o
 .debug_ranges  0x00001f18      0x100 build/default/production/_ext/334706090/wf_mac_24g.o
 .debug_ranges  0x00002018       0x30 build/default/production/_ext/334706090/wf_mgmt_msg_24g.o
 .debug_ranges  0x00002048       0xd8 build/default/production/_ext/334706090/wf_param_msg_24g.o
 .debug_ranges  0x00002120       0x28 build/default/production/_ext/334706090/wf_configData.o
 .debug_ranges  0x00002148       0x28 build/default/production/_ext/1472/main_demo.o
 .debug_ranges  0x00002170       0x10 build/default/production/_ext/1472/wf_config.o
 .debug_ranges  0x00002180      0x148 build/default/production/_ext/1472/custom_http_app.o
 .debug_ranges  0x000022c8       0x28 build/default/production/_ext/1472/tcp6_demo_app.o
 .debug_ranges  0x000022f0       0x10 c:/program files (x86)/microchip/xc32/v1.10/bin/../lib/gcc/pic32mx/4.5.1/../../../../pic32mx/lib/size\libmchp_peripheral.a(open_core_timer_lib.o)
 .debug_ranges  0x00002300       0x10 c:/program files (x86)/microchip/xc32/v1.10/bin/../lib/gcc/pic32mx/4.5.1/../../../../pic32mx/lib/size\libmchp_peripheral_32MX795F512L.a(soft_reset_lib.o)
 .debug_ranges  0x00002310       0x18 c:/program files (x86)/microchip/xc32/v1.10/bin/../lib/gcc/pic32mx/4.5.1/../../../../pic32mx/lib/size\libmchp_peripheral_32MX795F512L.a(pcache.o)
 .debug_ranges  0x00002328       0x10 c:/program files (x86)/microchip/xc32/v1.10/bin/../lib/gcc/pic32mx/4.5.1/../../../../pic32mx/lib/size\libmchp_peripheral_32MX795F512L.a(int_disable_interrupts_lib.o)
 .debug_ranges  0x00002338       0x10 c:/program files (x86)/microchip/xc32/v1.10/bin/../lib/gcc/pic32mx/4.5.1/../../../../pic32mx/lib/size\libmchp_peripheral_32MX795F512L.a(int_restore_interrupts_lib.o)
 .debug_ranges  0x00002348       0x10 c:/program files (x86)/microchip/xc32/v1.10/bin/../lib/gcc/pic32mx/4.5.1/../../../../pic32mx/lib/size\libmchp_peripheral_32MX795F512L.a(int_enable_mv_int_lib.o)
 .debug_ranges  0x00002358       0x50 c:/program files (x86)/microchip/xc32/v1.10/bin/../lib/gcc/pic32mx/4.5.1/../../../../pic32mx/lib/size\libmchp_peripheral_32MX795F512L.a(int_tbl_lib.o)
 .debug_ranges  0x000023a8       0x10 c:/program files (x86)/microchip/xc32/v1.10/bin/../lib/gcc/pic32mx/4.5.1/../../../../pic32mx/lib/size\libmchp_peripheral_32MX795F512L.a(rtcc_init_lib.o)
 .debug_ranges  0x000023b8       0x10 c:/program files (x86)/microchip/xc32/v1.10/bin/../lib/gcc/pic32mx/4.5.1/../../../../pic32mx/lib/size\libmchp_peripheral_32MX795F512L.a(rtcc_open_lib.o)
 .debug_ranges  0x000023c8       0x10 c:/program files (x86)/microchip/xc32/v1.10/bin/../lib/gcc/pic32mx/4.5.1/../../../../pic32mx/lib/size\libmchp_peripheral_32MX795F512L.a(spi_chn_data_rdy_lib.o)
 .debug_ranges  0x000023d8       0x18 c:/program files (x86)/microchip/xc32/v1.10/bin/../lib/gcc/pic32mx/4.5.1/../../../../pic32mx/lib/size\libmchp_peripheral_32MX795F512L.a(spi_chn_getc_lib.o)
 .debug_ranges  0x000023f0       0x10 c:/program files (x86)/microchip/xc32/v1.10/bin/../lib/gcc/pic32mx/4.5.1/../../../../pic32mx/lib/size\libmchp_peripheral_32MX795F512L.a(spi_chn_open_lib.o)
 .debug_ranges  0x00002400       0x20 c:/program files (x86)/microchip/xc32/v1.10/bin/../lib/gcc/pic32mx/4.5.1/../../../../pic32mx/lib/size\libmchp_peripheral_32MX795F512L.a(spi_chn_putc_lib.o)
 .debug_ranges  0x00002420       0x10 c:/program files (x86)/microchip/xc32/v1.10/bin/../lib/gcc/pic32mx/4.5.1/../../../../pic32mx/lib/size\libmchp_peripheral_32MX795F512L.a(spi_chn_tx_buff_empty_lib.o)
 .debug_ranges  0x00002430       0x10 c:/program files (x86)/microchip/xc32/v1.10/bin/../lib/gcc/pic32mx/4.5.1/../../../../pic32mx/lib/size\libmchp_peripheral_32MX795F512L.a(port_set_pins_digital_in_lib.o)
 .debug_ranges  0x00002440       0x10 c:/program files (x86)/microchip/xc32/v1.10/bin/../lib/gcc/pic32mx/4.5.1/../../../../pic32mx/lib/size\libmchp_peripheral_32MX795F512L.a(port_set_pins_digital_out_lib.o)
 .debug_ranges  0x00002450       0x10 c:/program files (x86)/microchip/xc32/v1.10/bin/../lib/gcc/pic32mx/4.5.1/../../../../pic32mx/lib/size\libmchp_peripheral_32MX795F512L.a(int_enable_interrupts_lib.o)
 .debug_ranges  0x00002460       0x18 c:/program files (x86)/microchip/xc32/v1.10/bin/../lib/gcc/pic32mx/4.5.1/../../../../pic32mx/lib/size\libmchp_peripheral_32MX795F512L.a(_rtcc_wait_clock_off_lib.o)
 .debug_ranges  0x00002478       0x10 c:/program files (x86)/microchip/xc32/v1.10/bin/../lib/gcc/pic32mx/4.5.1/../../../../pic32mx/lib/size\libmchp_peripheral_32MX795F512L.a(read_core_timer_lib.o)
 .debug_ranges  0x00002488       0xc0 c:/program files (x86)/microchip/xc32/v1.10/bin/../lib/gcc/pic32mx/4.5.1/size\libgcc.a(_udivdi3.o)
 .debug_ranges  0x00002548       0x10 c:/program files (x86)/microchip/xc32/v1.10/bin/../lib/gcc/pic32mx/4.5.1/../../../../pic32mx/lib/size\libpic32.a(default-bootstrap-exception-handler.o)
 .debug_ranges  0x00002558       0x10 c:/program files (x86)/microchip/xc32/v1.10/bin/../lib/gcc/pic32mx/4.5.1/../../../../pic32mx/lib/size\libpic32.a(default-on-reset.o)
 .debug_ranges  0x00002568       0x10 c:/program files (x86)/microchip/xc32/v1.10/bin/../lib/gcc/pic32mx/4.5.1/../../../../pic32mx/lib/size\libpic32.a(default-on-bootstrap.o)
 .debug_ranges  0x00002578       0x10 c:/program files (x86)/microchip/xc32/v1.10/bin/../lib/gcc/pic32mx/4.5.1/../../../../pic32mx/lib/size\libc.a(atoi.o)
 .debug_ranges  0x00002588       0x10 c:/program files (x86)/microchip/xc32/v1.10/bin/../lib/gcc/pic32mx/4.5.1/../../../../pic32mx/lib/size\libc.a(atol.o)
 .debug_ranges  0x00002598       0x20 c:/program files (x86)/microchip/xc32/v1.10/bin/../lib/gcc/pic32mx/4.5.1/../../../../pic32mx/lib/size\libc.a(malloc.o)
 .debug_ranges  0x000025b8       0x18 c:/program files (x86)/microchip/xc32/v1.10/bin/../lib/gcc/pic32mx/4.5.1/../../../../pic32mx/lib/size\libc.a(rand.o)
 .debug_ranges  0x000025d0       0x10 c:/program files (x86)/microchip/xc32/v1.10/bin/../lib/gcc/pic32mx/4.5.1/../../../../pic32mx/lib/size\libc.a(strcat.o)
 .debug_ranges  0x000025e0       0x10 c:/program files (x86)/microchip/xc32/v1.10/bin/../lib/gcc/pic32mx/4.5.1/../../../../pic32mx/lib/size\libc.a(strchr.o)
 .debug_ranges  0x000025f0       0x10 c:/program files (x86)/microchip/xc32/v1.10/bin/../lib/gcc/pic32mx/4.5.1/../../../../pic32mx/lib/size\libc.a(strncat.o)
 .debug_ranges  0x00002600       0x10 c:/program files (x86)/microchip/xc32/v1.10/bin/../lib/gcc/pic32mx/4.5.1/../../../../pic32mx/lib/size\libc.a(strncmp.o)
 .debug_ranges  0x00002610       0x10 c:/program files (x86)/microchip/xc32/v1.10/bin/../lib/gcc/pic32mx/4.5.1/../../../../pic32mx/lib/size\libc.a(strncpy.o)
 .debug_ranges  0x00002620       0x10 c:/program files (x86)/microchip/xc32/v1.10/bin/../lib/gcc/pic32mx/4.5.1/../../../../pic32mx/lib/size\libc.a(strrchr.o)
 .debug_ranges  0x00002630       0x10 c:/program files (x86)/microchip/xc32/v1.10/bin/../lib/gcc/pic32mx/4.5.1/../../../../pic32mx/lib/size\libc.a(strstr.o)
 .debug_ranges  0x00002640       0x18 c:/program files (x86)/microchip/xc32/v1.10/bin/../lib/gcc/pic32mx/4.5.1/../../../../pic32mx/lib/size\libc.a(strtol.o)
 .debug_ranges  0x00002658       0x10 c:/program files (x86)/microchip/xc32/v1.10/bin/../lib/gcc/pic32mx/4.5.1/../../../../pic32mx/lib/size\libc.a(snprintf_cdnopsuxX.eo)
 .debug_ranges  0x00002668       0x10 c:/program files (x86)/microchip/xc32/v1.10/bin/../lib/gcc/pic32mx/4.5.1/../../../../pic32mx/lib/size\libc.a(sprintf_cdnopsuxX.eo)
 .debug_ranges  0x00002678       0x10 c:/program files (x86)/microchip/xc32/v1.10/bin/../lib/gcc/pic32mx/4.5.1/../../../../pic32mx/lib/size\libc.a(vsnprintf_cdnopsuxX.eo)
 .debug_ranges  0x00002688       0x10 c:/program files (x86)/microchip/xc32/v1.10/bin/../lib/gcc/pic32mx/4.5.1/../../../../pic32mx/lib/size\libc.a(vsnprintf.o)
 .debug_ranges  0x00002698       0x90 c:/program files (x86)/microchip/xc32/v1.10/bin/../lib/gcc/pic32mx/4.5.1/../../../../pic32mx/lib/size\libc.a(ctypef.o)
 .debug_ranges  0x00002728       0x10 c:/program files (x86)/microchip/xc32/v1.10/bin/../lib/gcc/pic32mx/4.5.1/../../../../pic32mx/lib/size\libc.a(doprnt_cdnopsuxX.eo)
 .debug_ranges  0x00002738       0x20 c:/program files (x86)/microchip/xc32/v1.10/bin/../lib/gcc/pic32mx/4.5.1/../../../../pic32mx/lib/size\libc.a(doprnt.o)
 .debug_ranges  0x00002758       0x10 c:/program files (x86)/microchip/xc32/v1.10/bin/../lib/gcc/pic32mx/4.5.1/../../../../pic32mx/lib/size\libc.a(_fputc_simple.o)
 .debug_ranges  0x00002768       0x10 c:/program files (x86)/microchip/xc32/v1.10/bin/../lib/gcc/pic32mx/4.5.1/../../../../pic32mx/lib/size\libc.a(_flsbuf_simple.o)
 .debug_ranges  0x00002778       0x30 c:/program files (x86)/microchip/xc32/v1.10/bin/../lib/gcc/pic32mx/4.5.1/../../../../pic32mx/lib/size\libpic32.a(sbrk.o)
 .debug_ranges  0x000027a8       0x10 c:/program files (x86)/microchip/xc32/v1.10/bin/../lib/gcc/pic32mx/4.5.1/../../../../pic32mx/lib/size\libpic32.a(write.o)
 .debug_ranges  0x000027b8       0x10 c:/program files (x86)/microchip/xc32/v1.10/bin/../lib/gcc/pic32mx/4.5.1/../../../../pic32mx/lib/size\libpic32.a(_mon_putc.o)
 .debug_ranges  0x000027c8       0x10 c:/program files (x86)/microchip/xc32/v1.10/bin/../lib/gcc/pic32mx/4.5.1/../../../../pic32mx/lib/size\libe.a(_floatdisf.o)
 .debug_ranges  0x000027d8       0xc0 c:/program files (x86)/microchip/xc32/v1.10/bin/../lib/gcc/pic32mx/4.5.1/size\libgcc.a(_umoddi3.o)

.gnu.attributes
                0x00000000       0x10
 *(.gnu.attributes)
 .gnu.attributes
                0x00000000       0x10 build/default/production/_ext/1293749816/bsp.o
 .gnu.attributes
                0x00000010       0x10 build/default/production/_ext/101875047/hashes.o
 .gnu.attributes
                0x00000020       0x10 build/default/production/_ext/101875047/lfsr.o
 .gnu.attributes
                0x00000030       0x10 build/default/production/_ext/101875047/big_int.o
 .gnu.attributes
                0x00000040       0x10 build/default/production/_ext/101875047/helpers.o
 .gnu.attributes
                0x00000050       0x10 build/default/production/_ext/1472/berkeley_tcp_client_demo.o
 .gnu.attributes
                0x00000060       0x10 build/default/production/_ext/1472/berkeley_tcp_server_demo.o
 .gnu.attributes
                0x00000070       0x10 build/default/production/_ext/1472/berkeley_udp_client_demo.o
 .gnu.attributes
                0x00000080       0x10 build/default/production/_ext/1472/generic_tcp_client.o
 .gnu.attributes
                0x00000090       0x10 build/default/production/_ext/1472/generic_tcp_server.o
 .gnu.attributes
                0x000000a0       0x10 build/default/production/_ext/1472/ping_demo.o
 .gnu.attributes
                0x000000b0       0x10 build/default/production/_ext/1472/smtp_demo.o
 .gnu.attributes
                0x000000c0       0x10 build/default/production/_ext/365611741/system_services.o
 .gnu.attributes
                0x000000d0       0x10 build/default/production/_ext/365611741/system_debug.o
 .gnu.attributes
                0x000000e0       0x10 build/default/production/_ext/365611741/system_random.o
 .gnu.attributes
                0x000000f0       0x10 build/default/production/_ext/365611741/system_command.o
 .gnu.attributes
                0x00000100       0x10 build/default/production/_ext/365611741/system_userio.o
 .gnu.attributes
                0x00000110       0x10 build/default/production/_ext/97638081/sys_fs.o
 .gnu.attributes
                0x00000120       0x10 build/default/production/_ext/97638081/mpfs2.o
 .gnu.attributes
                0x00000130       0x10 build/default/production/_ext/792872985/usart.o
 .gnu.attributes
                0x00000140       0x10 build/default/production/_ext/792872985/lcd.o
 .gnu.attributes
                0x00000150       0x10 build/default/production/_ext/792872985/drv_spi.o
 .gnu.attributes
                0x00000160       0x10 build/default/production/_ext/792872985/db_appio.o
 .gnu.attributes
                0x00000170       0x10 build/default/production/_ext/792872985/spi_ram.o
 .gnu.attributes
                0x00000180       0x10 build/default/production/_ext/792872985/spi_eeprom.o
 .gnu.attributes
                0x00000190       0x10 build/default/production/_ext/792872985/spi_flash.o
 .gnu.attributes
                0x000001a0       0x10 build/default/production/_ext/792872985/drv_media.o
 .gnu.attributes
                0x000001b0       0x10 build/default/production/_ext/427700826/tcpip_announce.o
 .gnu.attributes
                0x000001c0       0x10 build/default/production/_ext/427700826/http2.o
 .gnu.attributes
                0x000001d0       0x10 build/default/production/_ext/427700826/arcfour.o
 .gnu.attributes
                0x000001e0       0x10 build/default/production/_ext/427700826/arp.o
 .gnu.attributes
                0x000001f0       0x10 build/default/production/_ext/427700826/berkeley_api.o
 .gnu.attributes
                0x00000200       0x10 build/default/production/_ext/427700826/dhcp.o
 .gnu.attributes
                0x00000210       0x10 build/default/production/_ext/427700826/dhcps.o
 .gnu.attributes
                0x00000220       0x10 build/default/production/_ext/427700826/dns.o
 .gnu.attributes
                0x00000230       0x10 build/default/production/_ext/427700826/dnss.o
 .gnu.attributes
                0x00000240       0x10 build/default/production/_ext/427700826/dyn_dns.o
 .gnu.attributes
                0x00000250       0x10 build/default/production/_ext/427700826/enc28_mac.o
 .gnu.attributes
                0x00000260       0x10 build/default/production/_ext/427700826/enc28j60.o
 .gnu.attributes
                0x00000270       0x10 build/default/production/_ext/427700826/encs24j600.o
 .gnu.attributes
                0x00000280       0x10 build/default/production/_ext/427700826/encx24_mac.o
 .gnu.attributes
                0x00000290       0x10 build/default/production/_ext/427700826/eth_pic32_ext_phy.o
 .gnu.attributes
                0x000002a0       0x10 build/default/production/_ext/427700826/eth_pic32_ext_phy_dp83848.o
 .gnu.attributes
                0x000002b0       0x10 build/default/production/_ext/427700826/eth_pic32_int_mac.o
 .gnu.attributes
                0x000002c0       0x10 build/default/production/_ext/427700826/ftp.o
 .gnu.attributes
                0x000002d0       0x10 build/default/production/_ext/427700826/hash_fnv.o
 .gnu.attributes
                0x000002e0       0x10 build/default/production/_ext/427700826/hash_tbl.o
 .gnu.attributes
                0x000002f0       0x10 build/default/production/_ext/427700826/icmp.o
 .gnu.attributes
                0x00000300       0x10 build/default/production/_ext/427700826/icmpv6.o
 .gnu.attributes
                0x00000310       0x10 build/default/production/_ext/427700826/ipv4.o
 .gnu.attributes
                0x00000320       0x10 build/default/production/_ext/427700826/ipv6.o
 .gnu.attributes
                0x00000330       0x10 build/default/production/_ext/427700826/mac_events_pic32.o
 .gnu.attributes
                0x00000340       0x10 build/default/production/_ext/427700826/nbns.o
 .gnu.attributes
                0x00000350       0x10 build/default/production/_ext/427700826/ndp.o
 .gnu.attributes
                0x00000360       0x10 build/default/production/_ext/427700826/tcpip_reboot.o
 .gnu.attributes
                0x00000370       0x10 build/default/production/_ext/427700826/rsa.o
 .gnu.attributes
                0x00000380       0x10 build/default/production/_ext/427700826/smtp.o
 .gnu.attributes
                0x00000390       0x10 build/default/production/_ext/427700826/snmp.o
 .gnu.attributes
                0x000003a0       0x10 build/default/production/_ext/427700826/snmpv3.o
 .gnu.attributes
                0x000003b0       0x10 build/default/production/_ext/427700826/snmpv3_usm.o
 .gnu.attributes
                0x000003c0       0x10 build/default/production/_ext/427700826/sntp.o
 .gnu.attributes
                0x000003d0       0x10 build/default/production/_ext/427700826/ssl.o
 .gnu.attributes
                0x000003e0       0x10 build/default/production/_ext/427700826/tcp.o
 .gnu.attributes
                0x000003f0       0x10 build/default/production/_ext/427700826/tcpip_heap_alloc.o
 .gnu.attributes
                0x00000400       0x10 build/default/production/_ext/427700826/tcpip_storage.o
 .gnu.attributes
                0x00000410       0x10 build/default/production/_ext/427700826/telnet.o
 .gnu.attributes
                0x00000420       0x10 build/default/production/_ext/427700826/tftpc.o
 .gnu.attributes
                0x00000430       0x10 build/default/production/_ext/427700826/udp.o
 .gnu.attributes
                0x00000440       0x10 build/default/production/_ext/427700826/tcpip_mac_object.o
 .gnu.attributes
                0x00000450       0x10 build/default/production/_ext/427700826/tcpip_manager.o
 .gnu.attributes
                0x00000460       0x10 build/default/production/_ext/427700826/tcpip_helpers.o
 .gnu.attributes
                0x00000470       0x10 build/default/production/_ext/427700826/tcpip_commands.o
 .gnu.attributes
                0x00000480       0x10 build/default/production/_ext/427700826/iperf.o
 .gnu.attributes
                0x00000490       0x10 build/default/production/_ext/427700826/tcpip_notify.o
 .gnu.attributes
                0x000004a0       0x10 build/default/production/_ext/427700826/zero_conf_helper.o
 .gnu.attributes
                0x000004b0       0x10 build/default/production/_ext/427700826/zero_conf_link_local.o
 .gnu.attributes
                0x000004c0       0x10 build/default/production/_ext/427700826/zero_conf_multicast_dns.o
 .gnu.attributes
                0x000004d0       0x10 build/default/production/_ext/334706090/wf_tx_power.o
 .gnu.attributes
                0x000004e0       0x10 build/default/production/_ext/334706090/wf_connect.o
 .gnu.attributes
                0x000004f0       0x10 build/default/production/_ext/334706090/wf_connection_algorithm.o
 .gnu.attributes
                0x00000500       0x10 build/default/production/_ext/334706090/wf_connection_manager.o
 .gnu.attributes
                0x00000510       0x10 build/default/production/_ext/334706090/wf_connection_profile.o
 .gnu.attributes
                0x00000520       0x10 build/default/production/_ext/334706090/wf_easy_config.o
 .gnu.attributes
                0x00000530       0x10 build/default/production/_ext/334706090/wf_eint.o
 .gnu.attributes
                0x00000540       0x10 build/default/production/_ext/334706090/wf_event_handler.o
 .gnu.attributes
                0x00000550       0x10 build/default/production/_ext/334706090/wf_init.o
 .gnu.attributes
                0x00000560       0x10 build/default/production/_ext/334706090/wf_power_save.o
 .gnu.attributes
                0x00000570       0x10 build/default/production/_ext/334706090/wf_scan.o
 .gnu.attributes
                0x00000580       0x10 build/default/production/_ext/334706090/wf_spi.o
 .gnu.attributes
                0x00000590       0x10 build/default/production/_ext/334706090/mrf24w_mac_pic32.o
 .gnu.attributes
                0x000005a0       0x10 build/default/production/_ext/334706090/mrf24w_events.o
 .gnu.attributes
                0x000005b0       0x10 build/default/production/_ext/334706090/wf_debug_output.o
 .gnu.attributes
                0x000005c0       0x10 build/default/production/_ext/334706090/wf_commands.o
 .gnu.attributes
                0x000005d0       0x10 build/default/production/_ext/334706090/wf_pbkdf2.o
 .gnu.attributes
                0x000005e0       0x10 build/default/production/_ext/334706090/wf_driver_com_24g.o
 .gnu.attributes
                0x000005f0       0x10 build/default/production/_ext/334706090/wf_driver_raw_24g.o
 .gnu.attributes
                0x00000600       0x10 build/default/production/_ext/334706090/wf_mac_24g.o
 .gnu.attributes
                0x00000610       0x10 build/default/production/_ext/334706090/wf_mgmt_msg_24g.o
 .gnu.attributes
                0x00000620       0x10 build/default/production/_ext/334706090/wf_param_msg_24g.o
 .gnu.attributes
                0x00000630       0x10 build/default/production/_ext/334706090/wf_configData.o
 .gnu.attributes
                0x00000640       0x10 build/default/production/_ext/1472/main_demo.o
 .gnu.attributes
                0x00000650       0x10 build/default/production/_ext/1472/custom_snmp_app.o
 .gnu.attributes
                0x00000660       0x10 build/default/production/_ext/1472/custom_ssl_cert.o
 .gnu.attributes
                0x00000670       0x10 build/default/production/_ext/1472/mpfs_img2.o
 .gnu.attributes
                0x00000680       0x10 build/default/production/_ext/1472/wf_config.o
 .gnu.attributes
                0x00000690       0x10 build/default/production/_ext/1472/custom_http_app.o
 .gnu.attributes
                0x000006a0       0x10 build/default/production/_ext/1472/tcp6_demo_app.o
 .gnu.attributes
                0x000006b0       0x10 c:/program files (x86)/microchip/xc32/v1.10/bin/../lib/gcc/pic32mx/4.5.1/../../../../pic32mx/lib/size\libmchp_peripheral.a(open_core_timer_lib.o)
 .gnu.attributes
                0x000006c0       0x10 c:/program files (x86)/microchip/xc32/v1.10/bin/../lib/gcc/pic32mx/4.5.1/../../../../pic32mx/lib/size\libmchp_peripheral_32MX795F512L.a(soft_reset_lib.o)
 .gnu.attributes
                0x000006d0       0x10 c:/program files (x86)/microchip/xc32/v1.10/bin/../lib/gcc/pic32mx/4.5.1/../../../../pic32mx/lib/size\libmchp_peripheral_32MX795F512L.a(pcache.o)
 .gnu.attributes
                0x000006e0       0x10 c:/program files (x86)/microchip/xc32/v1.10/bin/../lib/gcc/pic32mx/4.5.1/../../../../pic32mx/lib/size\libmchp_peripheral_32MX795F512L.a(int_disable_interrupts_lib.o)
 .gnu.attributes
                0x000006f0       0x10 c:/program files (x86)/microchip/xc32/v1.10/bin/../lib/gcc/pic32mx/4.5.1/../../../../pic32mx/lib/size\libmchp_peripheral_32MX795F512L.a(int_restore_interrupts_lib.o)
 .gnu.attributes
                0x00000700       0x10 c:/program files (x86)/microchip/xc32/v1.10/bin/../lib/gcc/pic32mx/4.5.1/../../../../pic32mx/lib/size\libmchp_peripheral_32MX795F512L.a(int_enable_mv_int_lib.o)
 .gnu.attributes
                0x00000710       0x10 c:/program files (x86)/microchip/xc32/v1.10/bin/../lib/gcc/pic32mx/4.5.1/../../../../pic32mx/lib/size\libmchp_peripheral_32MX795F512L.a(int_tbl_lib.o)
 .gnu.attributes
                0x00000720       0x10 c:/program files (x86)/microchip/xc32/v1.10/bin/../lib/gcc/pic32mx/4.5.1/../../../../pic32mx/lib/size\libmchp_peripheral_32MX795F512L.a(rtcc_init_lib.o)
 .gnu.attributes
                0x00000730       0x10 c:/program files (x86)/microchip/xc32/v1.10/bin/../lib/gcc/pic32mx/4.5.1/../../../../pic32mx/lib/size\libmchp_peripheral_32MX795F512L.a(rtcc_open_lib.o)
 .gnu.attributes
                0x00000740       0x10 c:/program files (x86)/microchip/xc32/v1.10/bin/../lib/gcc/pic32mx/4.5.1/../../../../pic32mx/lib/size\libmchp_peripheral_32MX795F512L.a(spi_chn_data_rdy_lib.o)
 .gnu.attributes
                0x00000750       0x10 c:/program files (x86)/microchip/xc32/v1.10/bin/../lib/gcc/pic32mx/4.5.1/../../../../pic32mx/lib/size\libmchp_peripheral_32MX795F512L.a(spi_chn_getc_lib.o)
 .gnu.attributes
                0x00000760       0x10 c:/program files (x86)/microchip/xc32/v1.10/bin/../lib/gcc/pic32mx/4.5.1/../../../../pic32mx/lib/size\libmchp_peripheral_32MX795F512L.a(spi_chn_open_lib.o)
 .gnu.attributes
                0x00000770       0x10 c:/program files (x86)/microchip/xc32/v1.10/bin/../lib/gcc/pic32mx/4.5.1/../../../../pic32mx/lib/size\libmchp_peripheral_32MX795F512L.a(spi_chn_putc_lib.o)
 .gnu.attributes
                0x00000780       0x10 c:/program files (x86)/microchip/xc32/v1.10/bin/../lib/gcc/pic32mx/4.5.1/../../../../pic32mx/lib/size\libmchp_peripheral_32MX795F512L.a(spi_chn_tx_buff_empty_lib.o)
 .gnu.attributes
                0x00000790       0x10 c:/program files (x86)/microchip/xc32/v1.10/bin/../lib/gcc/pic32mx/4.5.1/../../../../pic32mx/lib/size\libmchp_peripheral_32MX795F512L.a(spi_io_tbl_libp.o)
 .gnu.attributes
                0x000007a0       0x10 c:/program files (x86)/microchip/xc32/v1.10/bin/../lib/gcc/pic32mx/4.5.1/../../../../pic32mx/lib/size\libmchp_peripheral_32MX795F512L.a(spi_map_tbl_libp.o)
 .gnu.attributes
                0x000007b0       0x10 c:/program files (x86)/microchip/xc32/v1.10/bin/../lib/gcc/pic32mx/4.5.1/../../../../pic32mx/lib/size\libmchp_peripheral_32MX795F512L.a(port_set_pins_digital_in_lib.o)
 .gnu.attributes
                0x000007c0       0x10 c:/program files (x86)/microchip/xc32/v1.10/bin/../lib/gcc/pic32mx/4.5.1/../../../../pic32mx/lib/size\libmchp_peripheral_32MX795F512L.a(port_set_pins_digital_out_lib.o)
 .gnu.attributes
                0x000007d0       0x10 c:/program files (x86)/microchip/xc32/v1.10/bin/../lib/gcc/pic32mx/4.5.1/../../../../pic32mx/lib/size\libmchp_peripheral_32MX795F512L.a(_ports_tbl_libp.o)
 .gnu.attributes
                0x000007e0       0x10 c:/program files (x86)/microchip/xc32/v1.10/bin/../lib/gcc/pic32mx/4.5.1/../../../../pic32mx/lib/size\libmchp_peripheral_32MX795F512L.a(int_enable_interrupts_lib.o)
 .gnu.attributes
                0x000007f0       0x10 c:/program files (x86)/microchip/xc32/v1.10/bin/../lib/gcc/pic32mx/4.5.1/../../../../pic32mx/lib/size\libmchp_peripheral_32MX795F512L.a(_rtcc_wait_clock_off_lib.o)
 .gnu.attributes
                0x00000800       0x10 c:/program files (x86)/microchip/xc32/v1.10/bin/../lib/gcc/pic32mx/4.5.1/../../../../pic32mx/lib/size\libmchp_peripheral_32MX795F512L.a(read_core_timer_lib.o)
 .gnu.attributes
                0x00000810       0x10 c:/program files (x86)/microchip/xc32/v1.10/bin/../lib/gcc/pic32mx/4.5.1/size\libgcc.a(_udivdi3.o)
 .gnu.attributes
                0x00000820       0x10 c:/program files (x86)/microchip/xc32/v1.10/bin/../lib/gcc/pic32mx/4.5.1/../../../../pic32mx/lib/size\libpic32.a(default-bootstrap-exception-handler.o)
 .gnu.attributes
                0x00000830       0x10 c:/program files (x86)/microchip/xc32/v1.10/bin/../lib/gcc/pic32mx/4.5.1/../../../../pic32mx/lib/size\libpic32.a(default-on-reset.o)
 .gnu.attributes
                0x00000840       0x10 c:/program files (x86)/microchip/xc32/v1.10/bin/../lib/gcc/pic32mx/4.5.1/../../../../pic32mx/lib/size\libpic32.a(default-on-bootstrap.o)
 .gnu.attributes
                0x00000850       0x10 c:/program files (x86)/microchip/xc32/v1.10/bin/../lib/gcc/pic32mx/4.5.1/../../../../pic32mx/lib/size\libpic32.a(errno.o)
 .gnu.attributes
                0x00000860       0x10 c:/program files (x86)/microchip/xc32/v1.10/bin/../lib/gcc/pic32mx/4.5.1/../../../../pic32mx/lib/size\libc.a(atoi.o)
 .gnu.attributes
                0x00000870       0x10 c:/program files (x86)/microchip/xc32/v1.10/bin/../lib/gcc/pic32mx/4.5.1/../../../../pic32mx/lib/size\libc.a(atol.o)
 .gnu.attributes
                0x00000880       0x10 c:/program files (x86)/microchip/xc32/v1.10/bin/../lib/gcc/pic32mx/4.5.1/../../../../pic32mx/lib/size\libc.a(ctype.o)
 .gnu.attributes
                0x00000890       0x10 c:/program files (x86)/microchip/xc32/v1.10/bin/../lib/gcc/pic32mx/4.5.1/../../../../pic32mx/lib/size\libc.a(malloc.o)
 .gnu.attributes
                0x000008a0       0x10 c:/program files (x86)/microchip/xc32/v1.10/bin/../lib/gcc/pic32mx/4.5.1/../../../../pic32mx/lib/size\libc.a(rand.o)
 .gnu.attributes
                0x000008b0       0x10 c:/program files (x86)/microchip/xc32/v1.10/bin/../lib/gcc/pic32mx/4.5.1/../../../../pic32mx/lib/size\libc.a(strcat.o)
 .gnu.attributes
                0x000008c0       0x10 c:/program files (x86)/microchip/xc32/v1.10/bin/../lib/gcc/pic32mx/4.5.1/../../../../pic32mx/lib/size\libc.a(strchr.o)
 .gnu.attributes
                0x000008d0       0x10 c:/program files (x86)/microchip/xc32/v1.10/bin/../lib/gcc/pic32mx/4.5.1/../../../../pic32mx/lib/size\libc.a(strncat.o)
 .gnu.attributes
                0x000008e0       0x10 c:/program files (x86)/microchip/xc32/v1.10/bin/../lib/gcc/pic32mx/4.5.1/../../../../pic32mx/lib/size\libc.a(strncmp.o)
 .gnu.attributes
                0x000008f0       0x10 c:/program files (x86)/microchip/xc32/v1.10/bin/../lib/gcc/pic32mx/4.5.1/../../../../pic32mx/lib/size\libc.a(strncpy.o)
 .gnu.attributes
                0x00000900       0x10 c:/program files (x86)/microchip/xc32/v1.10/bin/../lib/gcc/pic32mx/4.5.1/../../../../pic32mx/lib/size\libc.a(strrchr.o)
 .gnu.attributes
                0x00000910       0x10 c:/program files (x86)/microchip/xc32/v1.10/bin/../lib/gcc/pic32mx/4.5.1/../../../../pic32mx/lib/size\libc.a(strstr.o)
 .gnu.attributes
                0x00000920       0x10 c:/program files (x86)/microchip/xc32/v1.10/bin/../lib/gcc/pic32mx/4.5.1/../../../../pic32mx/lib/size\libc.a(strtol.o)
 .gnu.attributes
                0x00000930       0x10 c:/program files (x86)/microchip/xc32/v1.10/bin/../lib/gcc/pic32mx/4.5.1/../../../../pic32mx/lib/size\libc.a(snprintf_cdnopsuxX.eo)
 .gnu.attributes
                0x00000940       0x10 c:/program files (x86)/microchip/xc32/v1.10/bin/../lib/gcc/pic32mx/4.5.1/../../../../pic32mx/lib/size\libc.a(sprintf_cdnopsuxX.eo)
 .gnu.attributes
                0x00000950       0x10 c:/program files (x86)/microchip/xc32/v1.10/bin/../lib/gcc/pic32mx/4.5.1/../../../../pic32mx/lib/size\libc.a(vsnprintf_cdnopsuxX.eo)
 .gnu.attributes
                0x00000960       0x10 c:/program files (x86)/microchip/xc32/v1.10/bin/../lib/gcc/pic32mx/4.5.1/../../../../pic32mx/lib/size\libc.a(vsnprintf.o)
 .gnu.attributes
                0x00000970       0x10 c:/program files (x86)/microchip/xc32/v1.10/bin/../lib/gcc/pic32mx/4.5.1/../../../../pic32mx/lib/size\libc.a(ctypef.o)
 .gnu.attributes
                0x00000980       0x10 c:/program files (x86)/microchip/xc32/v1.10/bin/../lib/gcc/pic32mx/4.5.1/../../../../pic32mx/lib/size\libc.a(doprnt_cdnopsuxX.eo)
 .gnu.attributes
                0x00000990       0x10 c:/program files (x86)/microchip/xc32/v1.10/bin/../lib/gcc/pic32mx/4.5.1/../../../../pic32mx/lib/size\libc.a(doprnt.o)
 .gnu.attributes
                0x000009a0       0x10 c:/program files (x86)/microchip/xc32/v1.10/bin/../lib/gcc/pic32mx/4.5.1/../../../../pic32mx/lib/size\libc.a(_fputc_simple.o)
 .gnu.attributes
                0x000009b0       0x10 c:/program files (x86)/microchip/xc32/v1.10/bin/../lib/gcc/pic32mx/4.5.1/../../../../pic32mx/lib/size\libc.a(powersf.o)
 .gnu.attributes
                0x000009c0       0x10 c:/program files (x86)/microchip/xc32/v1.10/bin/../lib/gcc/pic32mx/4.5.1/../../../../pic32mx/lib/size\libc.a(_iob.o)
 .gnu.attributes
                0x000009d0       0x10 c:/program files (x86)/microchip/xc32/v1.10/bin/../lib/gcc/pic32mx/4.5.1/../../../../pic32mx/lib/size\libc.a(_flsbuf_simple.o)
 .gnu.attributes
                0x000009e0       0x10 c:/program files (x86)/microchip/xc32/v1.10/bin/../lib/gcc/pic32mx/4.5.1/../../../../pic32mx/lib/size\libpic32.a(sbrk.o)
 .gnu.attributes
                0x000009f0       0x10 c:/program files (x86)/microchip/xc32/v1.10/bin/../lib/gcc/pic32mx/4.5.1/../../../../pic32mx/lib/size\libpic32.a(write.o)
 .gnu.attributes
                0x00000a00       0x10 c:/program files (x86)/microchip/xc32/v1.10/bin/../lib/gcc/pic32mx/4.5.1/../../../../pic32mx/lib/size\libpic32.a(_mon_putc.o)
 .gnu.attributes
                0x00000a10       0x10 c:/program files (x86)/microchip/xc32/v1.10/bin/../lib/gcc/pic32mx/4.5.1/../../../../pic32mx/lib/size\libpic32.a(xc32_uart.o)
 .gnu.attributes
                0x00000a20       0x10 c:/program files (x86)/microchip/xc32/v1.10/bin/../lib/gcc/pic32mx/4.5.1/../../../../pic32mx/lib/size\libe.a(_floatdisf.o)
 .gnu.attributes
                0x00000a30       0x10 c:/program files (x86)/microchip/xc32/v1.10/bin/../lib/gcc/pic32mx/4.5.1/size\libgcc.a(_lshrdi3.o)
 .gnu.attributes
                0x00000a40       0x10 c:/program files (x86)/microchip/xc32/v1.10/bin/../lib/gcc/pic32mx/4.5.1/size\libgcc.a(_floatundisf.o)
 .gnu.attributes
                0x00000a50       0x10 c:/program files (x86)/microchip/xc32/v1.10/bin/../lib/gcc/pic32mx/4.5.1/size\libgcc.a(_umoddi3.o)
 .gnu.attributes
                0x00000a60       0x10 c:/program files (x86)/microchip/xc32/v1.10/bin/../lib/gcc/pic32mx/4.5.1/size\libgcc.a(floatunsisf.o)
LOAD c:/program files (x86)/microchip/xc32/v1.10/bin/../lib/gcc/pic32mx/4.5.1/size\libgcc.a
START GROUP
LOAD c:/program files (x86)/microchip/xc32/v1.10/bin/../lib/gcc/pic32mx/4.5.1/../../../../pic32mx/lib/size\libpic32.a
LOAD c:/program files (x86)/microchip/xc32/v1.10/bin/../lib/gcc/pic32mx/4.5.1/../../../../pic32mx/lib/size\libdebug.a
LOAD c:/program files (x86)/microchip/xc32/v1.10/bin/../lib/gcc/pic32mx/4.5.1/../../../../pic32mx/lib/size\libm.a
LOAD c:/program files (x86)/microchip/xc32/v1.10/bin/../lib/gcc/pic32mx/4.5.1/../../../../pic32mx/lib/size\libe.a
LOAD c:/program files (x86)/microchip/xc32/v1.10/bin/../lib/gcc/pic32mx/4.5.1/../../../../pic32mx/lib/size\libdsp.a
LOAD c:/program files (x86)/microchip/xc32/v1.10/bin/../lib/gcc/pic32mx/4.5.1/size\libgcc.a
LOAD c:/program files (x86)/microchip/xc32/v1.10/bin/../lib/gcc/pic32mx/4.5.1/../../../../pic32mx/lib/size\libpic32.a
LOAD c:/program files (x86)/microchip/xc32/v1.10/bin/../lib/gcc/pic32mx/4.5.1/../../../../pic32mx/lib/size\libc.a
LOAD c:/program files (x86)/microchip/xc32/v1.10/bin/../lib/gcc/pic32mx/4.5.1/../../../../pic32mx/lib/size\libpic32.a
END GROUP
LOAD c:/program files (x86)/microchip/xc32/v1.10/bin/../lib/gcc/pic32mx/4.5.1/size\libgcc.a
OUTPUT(dist/default/production/tcp6_demo_app_wifi.X.production.elf elf32-tradlittlemips)
LOAD stack
LOAD data_init

.reginfo        0x9d000000       0x18
 .reginfo       0x9d000000       0x18 c:/program files (x86)/microchip/xc32/v1.10/bin/../lib/gcc/pic32mx/4.5.1/../../../../pic32mx/lib/size/crt0.o

.stack          0xa0007a48      0x800
 .stack         0xa0007a48      0x800 stack

.bss            0xa0002190      0x210
 .bss           0xa0002190      0x210 build/default/production/_ext/97638081/sys_fs.o

.data           0xa00023a0      0x174
 .data          0xa00023a0      0x174 build/default/production/_ext/334706090/wf_debug_output.o
                0xa00023a0                connectionFailureStrings
                0xa00023f0                deauthDisssocReasonCodes
                0xa0002454                statusCodes

.bss            0xa0002514      0x248
 .bss           0xa0002514       0xd8 build/default/production/_ext/97638081/mpfs2.o
 .bss           0xa00025ec       0x68 build/default/production/_ext/365611741/system_command.o
 .bss           0xa0002654       0x5c build/default/production/_ext/365611741/system_random.o
 .bss           0xa00026b0       0x5c build/default/production/_ext/1472/custom_http_app.o
 .bss           0xa000270c       0x50 build/default/production/_ext/365611741/system_userio.o

.data           0xa000275c       0x44
 .data          0xa000275c       0x44 build/default/production/_ext/1472/tcp6_demo_app.o
                0xa000275c                b64

.bss            0xa00027a0       0x6c
 .bss           0xa00027a0       0x40 c:/program files (x86)/microchip/xc32/v1.10/bin/../lib/gcc/pic32mx/4.5.1/../../../../pic32mx/lib/size\libc.a(_iob.o)
                0xa00027a0                _sibuf
                0xa00027c0                _sobuf
 .bss           0xa00027e0       0x1c c:/program files (x86)/microchip/xc32/v1.10/bin/../lib/gcc/pic32mx/4.5.1/../../../../pic32mx/lib/size\libpic32.a(sbrk.o)
 .bss           0xa00027fc       0x10 c:/program files (x86)/microchip/xc32/v1.10/bin/../lib/gcc/pic32mx/4.5.1/../../../../pic32mx/lib/size\libc.a(malloc.o)
                0xa00027fc                __allocs

.bss            0xa0002810       0x10
 .bss           0xa0002810       0x10 c:/program files (x86)/microchip/xc32/v1.10/bin/../lib/gcc/pic32mx/4.5.1/../../../../pic32mx/lib/size\libc.a(rand.o)

.text.HTTPProcess
                0x9d000020     0x1804
 .text.HTTPProcess
                0x9d000020     0x1804 build/default/production/_ext/427700826/http2.o

.text._TcpHandleSeg
                0x9d001824     0x17e0
 .text._TcpHandleSeg
                0x9d001824     0x17e0 build/default/production/_ext/427700826/tcp.o

.text.vfprintf  0x9d003004     0x15b4
 .text.vfprintf
                0x9d003004     0x15b4 c:/program files (x86)/microchip/xc32/v1.10/bin/../lib/gcc/pic32mx/4.5.1/../../../../pic32mx/lib/size\libc.a(doprnt.o)
                0x9d003004                vfprintf

.text.DNSClientTask
                0x9d0045b8     0x1144
 .text.DNSClientTask
                0x9d0045b8     0x1144 build/default/production/_ext/427700826/dns.o
                0x9d0045b8                DNSClientTask

.rodata         0x9d0056fc     0x1088
 .rodata        0x9d0056fc     0x1088 build/default/production/_ext/334706090/wf_debug_output.o

.text.tcp6_demo_app_tasks
                0x9d006784      0xfd8
 .text.tcp6_demo_app_tasks
                0x9d006784      0xfd8 build/default/production/_ext/1472/tcp6_demo_app.o
                0x9d006784                tcp6_demo_app_tasks

.text.DHCPTask  0x9d00775c      0xa74
 .text.DHCPTask
                0x9d00775c      0xa74 build/default/production/_ext/427700826/dhcp.o
                0x9d00775c                DHCPTask

.text._TcpSend  0x9d0081d0      0xa50
 .text._TcpSend
                0x9d0081d0      0xa50 build/default/production/_ext/427700826/tcp.o

.text.TCPAdjustFIFOSize
                0x9d008c20      0x974
 .text.TCPAdjustFIFOSize
                0x9d008c20      0x974 build/default/production/_ext/427700826/tcp.o
                0x9d008c20                TCPAdjustFIFOSize

.rodata         0x9d009594      0x8f4
 .rodata        0x9d009594      0x8f4 build/default/production/_ext/427700826/http2.o

.text           0x9d009e88      0x8ec
 .text          0x9d009e88      0x8ec c:/program files (x86)/microchip/xc32/v1.10/bin/../lib/gcc/pic32mx/4.5.1/../../../../pic32mx/lib/size\libm.a(fp32.o)
                0x9d009e88                __subsf3
                0x9d009e88                fpsub
                0x9d009e90                fpadd
                0x9d009e90                __addsf3
                0x9d00a0fc                fpmul
                0x9d00a0fc                __mulsf3
                0x9d00a2b4                fpdiv
                0x9d00a2b4                __divsf3
                0x9d00a4e0                litofp
                0x9d00a4e0                sitofp
                0x9d00a4e0                __floatsisf
                0x9d00a53c                uitofp
                0x9d00a53c                ultofp
                0x9d00a588                fptosi
                0x9d00a588                fptoli
                0x9d00a588                __fixsfsi
                0x9d00a600                __fixunssfsi
                0x9d00a600                fptoul
                0x9d00a600                fptoui
                0x9d00a674                __eqsf2
                0x9d00a674                __nesf2
                0x9d00a674                __lesf2
                0x9d00a674                __ltsf2
                0x9d00a674                fpcmp
                0x9d00a674                __gtsf2
                0x9d00a674                __gesf2
                0x9d00a708                fpfabs
                0x9d00a708                fabsf
                0x9d00a718                __negsf2
                0x9d00a728                fpnan
                0x9d00a728                nanf

.text._vfprintf_cdnopsuxX
                0x9d00a774      0x8c4
 .text._vfprintf_cdnopsuxX
                0x9d00a774      0x8c4 c:/program files (x86)/microchip/xc32/v1.10/bin/../lib/gcc/pic32mx/4.5.1/../../../../pic32mx/lib/size\libc.a(doprnt_cdnopsuxX.eo)
                0x9d00a774                _vfprintf_cdnopuxX
                0x9d00a774                _vfprintf_cdnopsuxX

.text.TCPTick   0x9d00b038      0x8b8
 .text.TCPTick  0x9d00b038      0x8b8 build/default/production/_ext/427700826/tcp.o
                0x9d00b038                TCPTick

.rodata         0x9d00b8f0      0x7d4
 .rodata        0x9d00b8f0      0x7d4 c:/program files (x86)/microchip/xc32/v1.10/bin/../lib/gcc/pic32mx/4.5.1/../../../../pic32mx/lib/size\libmchp_peripheral_32MX795F512L.a(int_tbl_lib.o)
                0x9d00b8f0                __IntSrcTbl
                0x9d00be0c                __IntVectorTbl

.text._DHCPReceive
                0x9d00c0c4      0x748
 .text._DHCPReceive
                0x9d00c0c4      0x748 build/default/production/_ext/427700826/dhcp.o

.dinit          0x9d00c80c      0x748
 .dinit         0x9d00c80c      0x748 data_init

.text.NBNSTask  0x9d00cf54      0x740
 .text.NBNSTask
                0x9d00cf54      0x740 build/default/production/_ext/427700826/nbns.o
                0x9d00cf54                NBNSTask

.text.HTTPPrint
                0x9d00d694      0x6ac
 .text.HTTPPrint
                0x9d00d694      0x6ac build/default/production/_ext/427700826/http2.o
                0x9d00d694                HTTPPrint

.text.HTTPPostConfig
                0x9d00dd40      0x694
 .text.HTTPPostConfig
                0x9d00dd40      0x694 build/default/production/_ext/1472/custom_http_app.o

.text._DHCPSend
                0x9d00e3d4      0x5c8
 .text._DHCPSend
                0x9d00e3d4      0x5c8 build/default/production/_ext/427700826/dhcp.o

.text.TCPFindArray
                0x9d00e99c      0x578
 .text.TCPFindArray
                0x9d00e99c      0x578 build/default/production/_ext/427700826/tcp.o
                0x9d00e99c                TCPFindArray

.text.SHA1HashBlock
                0x9d00ef14      0x4fc
 .text.SHA1HashBlock
                0x9d00ef14      0x4fc build/default/production/_ext/101875047/hashes.o

.text.SYS_Initialize
                0x9d00f410      0x4f0
 .text.SYS_Initialize
                0x9d00f410      0x4f0 build/default/production/_ext/365611741/system_services.o
                0x9d00f410                SYS_Initialize

.text.TCPIP_ANNOUNCE_Send
                0x9d00f900      0x490
 .text.TCPIP_ANNOUNCE_Send
                0x9d00f900      0x490 build/default/production/_ext/427700826/tcpip_announce.o
                0x9d00f900                TCPIP_ANNOUNCE_Send

.text._TCPIP_HEAP_Free
                0x9d00fd90      0x490
 .text._TCPIP_HEAP_Free
                0x9d00fd90      0x490 build/default/production/_ext/427700826/tcpip_heap_alloc.o
                0x9d00fd90                _TCPIP_HEAP_Free

.text.TCPIP_STACK_Init
                0x9d010220      0x468
 .text.TCPIP_STACK_Init
                0x9d010220      0x468 build/default/production/_ext/427700826/tcpip_manager.o
                0x9d010220                TCPIP_STACK_Init

.text           0x9d010688      0x8ac
 .text          0x9d010688      0x464 c:/program files (x86)/microchip/xc32/v1.10/bin/../lib/gcc/pic32mx/4.5.1/size\libgcc.a(_umoddi3.o)
                0x9d010688                __umoddi3
 .text          0x9d010aec      0x448 c:/program files (x86)/microchip/xc32/v1.10/bin/../lib/gcc/pic32mx/4.5.1/size\libgcc.a(_udivdi3.o)
                0x9d010aec                __udivdi3

.rodata         0x9d010f34      0x43c
 .rodata        0x9d010f34      0x43c build/default/production/_ext/1472/tcp6_demo_app.o
                0x9d010f34                Version
                0x9d010f38                CompileDate
                0x9d010f44                CompileTime
                0x9d011054                HTTP_TRANSACTION_LIST

.text.TCPIP_STACK_BringNetUp
                0x9d011370      0x438
 .text.TCPIP_STACK_BringNetUp
                0x9d011370      0x438 build/default/production/_ext/427700826/tcpip_manager.o

.text.CommandHelp
                0x9d0117a8      0x428
 .text.CommandHelp
                0x9d0117a8      0x428 build/default/production/_ext/365611741/system_command.o

.text.TCPOpen   0x9d011bd0      0x420
 .text.TCPOpen  0x9d011bd0      0x420 build/default/production/_ext/427700826/tcp.o

.text.HTTPExecuteGet
                0x9d011ff0      0x414
 .text.HTTPExecuteGet
                0x9d011ff0      0x414 build/default/production/_ext/1472/custom_http_app.o
                0x9d011ff0                HTTPExecuteGet

.text.HTTPMPFSUpload
                0x9d012404      0x410
 .text.HTTPMPFSUpload
                0x9d012404      0x410 build/default/production/_ext/427700826/http2.o

.text.MPFSSeek  0x9d012814      0x400
 .text.MPFSSeek
                0x9d012814      0x400 build/default/production/_ext/97638081/mpfs2.o
                0x9d012814                MPFSSeek

.rodata         0x9d012c14      0x3f8
 .rodata        0x9d012c14      0x3f8 build/default/production/_ext/427700826/tcpip_manager.o

.text.ARPInitialize
                0x9d01300c      0x3f4
 .text.ARPInitialize
                0x9d01300c      0x3f4 build/default/production/_ext/427700826/arp.o
                0x9d01300c                ARPInitialize

.text._TcpFindMatchingSocket
                0x9d013400      0x3e8
 .text._TcpFindMatchingSocket
                0x9d013400      0x3e8 build/default/production/_ext/427700826/tcp.o

.text           0x9d0137e8      0x3dc
 .text          0x9d0137e8      0x3dc c:/program files (x86)/microchip/xc32/v1.10/bin/../lib/gcc/pic32mx/4.5.1/../../../../pic32mx/lib/size\libm.a(fpmod32.o)
                0x9d0137e8                fmodf
                0x9d0137e8                fpfmod
                0x9d01392c                frexpf
                0x9d01392c                fpfrexp
                0x9d0139b0                __mchp_ldexpf
                0x9d0139b0                fpldexp
                0x9d013af4                fpmodf
                0x9d013af4                modff

.text.TCPIP_HELPER_StringToIPAddress
                0x9d013bc4      0x3b8
 .text.TCPIP_HELPER_StringToIPAddress
                0x9d013bc4      0x3b8 build/default/production/_ext/427700826/tcpip_helpers.o
                0x9d013bc4                TCPIP_HELPER_StringToIPAddress

.text.WFProcessMgmtIndicateMsg
                0x9d013f7c      0x3b0
 .text.WFProcessMgmtIndicateMsg
                0x9d013f7c      0x3b0 build/default/production/_ext/334706090/wf_event_handler.o
                0x9d013f7c                WFProcessMgmtIndicateMsg

.text.FindMatchingSocket
                0x9d01432c      0x3a0
 .text.FindMatchingSocket
                0x9d01432c      0x3a0 build/default/production/_ext/427700826/udp.o

.text.TCPIP_Helper_Base64Decode
                0x9d0146cc      0x394
 .text.TCPIP_Helper_Base64Decode
                0x9d0146cc      0x394 build/default/production/_ext/427700826/tcpip_helpers.o
                0x9d0146cc                TCPIP_Helper_Base64Decode

.text.OutputSecurityMode
                0x9d014a60      0x38c
 .text.OutputSecurityMode
                0x9d014a60      0x38c build/default/production/_ext/334706090/wf_debug_output.o

.text.TCPIP_STACK_Task
                0x9d014dec      0x35c
 .text.TCPIP_STACK_Task
                0x9d014dec      0x35c build/default/production/_ext/427700826/tcpip_manager.o
                0x9d014dec                TCPIP_STACK_Task

.text._SYS_COMMAND_TASK
                0x9d015148      0x354
 .text._SYS_COMMAND_TASK
                0x9d015148      0x354 build/default/production/_ext/365611741/system_command.o
                0x9d015148                _SYS_COMMAND_TASK

.text.HTTPPostMD5
                0x9d01549c      0x340
 .text.HTTPPostMD5
                0x9d01549c      0x340 build/default/production/_ext/1472/custom_http_app.o

.text.UDPOpen   0x9d0157dc      0x334
 .text.UDPOpen  0x9d0157dc      0x334 build/default/production/_ext/427700826/udp.o

.text.main      0x9d015b10      0x328
 .text.main     0x9d015b10      0x328 build/default/production/_ext/1472/main_demo.o
                0x9d015b10                main

.text.MPFSOpen  0x9d015e38      0x31c
 .text.MPFSOpen
                0x9d015e38      0x31c build/default/production/_ext/97638081/mpfs2.o
                0x9d015e38                MPFSOpen

.text.OutputConnectionFailedMsg
                0x9d016154      0x31c
 .text.OutputConnectionFailedMsg
                0x9d016154      0x31c build/default/production/_ext/334706090/wf_debug_output.o

.text.HTTPInit  0x9d016470      0x318
 .text.HTTPInit
                0x9d016470      0x318 build/default/production/_ext/427700826/http2.o
                0x9d016470                HTTPInit

.text.UDPInit   0x9d016788      0x318
 .text.UDPInit  0x9d016788      0x318 build/default/production/_ext/427700826/udp.o
                0x9d016788                UDPInit

.text.ARPTask   0x9d016aa0      0x310
 .text.ARPTask  0x9d016aa0      0x310 build/default/production/_ext/427700826/arp.o
                0x9d016aa0                ARPTask

.text.TCPIP_IPV4_PutArrayHelper
                0x9d016db0      0x310
 .text.TCPIP_IPV4_PutArrayHelper
                0x9d016db0      0x310 build/default/production/_ext/427700826/ipv4.o
                0x9d016db0                TCPIP_IPV4_PutArrayHelper

.text.SYS_FS_mount
                0x9d0170c0      0x2e0
 .text.SYS_FS_mount
                0x9d0170c0      0x2e0 build/default/production/_ext/97638081/sys_fs.o
                0x9d0170c0                SYS_FS_mount

.text.tcp6_demo_app_init
                0x9d0173a0      0x2d8
 .text.tcp6_demo_app_init
                0x9d0173a0      0x2d8 build/default/production/_ext/1472/tcp6_demo_app.o
                0x9d0173a0                tcp6_demo_app_init

.text.MD5HashBlock
                0x9d017678      0x2c8
 .text.MD5HashBlock
                0x9d017678      0x2c8 build/default/production/_ext/101875047/hashes.o

.text.ProcessEscSequence
                0x9d017940      0x2c8
 .text.ProcessEscSequence
                0x9d017940      0x2c8 build/default/production/_ext/365611741/system_command.o

.text.DoWrite   0x9d017c08      0x2c4
 .text.DoWrite  0x9d017c08      0x2c4 build/default/production/_ext/792872985/spi_eeprom.o

.text.HTTPReadTo
                0x9d017ecc      0x2c4
 .text.HTTPReadTo
                0x9d017ecc      0x2c4 build/default/production/_ext/427700826/http2.o

.text.MPFSGetArray
                0x9d018190      0x2bc
 .text.MPFSGetArray
                0x9d018190      0x2bc build/default/production/_ext/97638081/mpfs2.o
                0x9d018190                MPFSGetArray

.text.ICMPProcess
                0x9d01844c      0x2ac
 .text.ICMPProcess
                0x9d01844c      0x2ac build/default/production/_ext/427700826/icmp.o
                0x9d01844c                ICMPProcess

.text.MD5Calculate
                0x9d0186f8      0x2a8
 .text.MD5Calculate
                0x9d0186f8      0x2a8 build/default/production/_ext/101875047/hashes.o
                0x9d0186f8                MD5Calculate

.text.TCPPutArray
                0x9d0189a0      0x2a8
 .text.TCPPutArray
                0x9d0189a0      0x2a8 build/default/production/_ext/427700826/tcp.o
                0x9d0189a0                TCPPutArray

.text.ParseCmdBuffer
                0x9d018c48      0x2a4
 .text.ParseCmdBuffer
                0x9d018c48      0x2a4 build/default/production/_ext/365611741/system_command.o

.text.DRV_MEDIA_Open
                0x9d018eec      0x294
 .text.DRV_MEDIA_Open
                0x9d018eec      0x294 build/default/production/_ext/792872985/drv_media.o
                0x9d018eec                DRV_MEDIA_Open

.rodata         0x9d019180      0x28c
 .rodata        0x9d019180      0x28c build/default/production/_ext/365611741/system_command.o
                0x9d019190                sysConsoleApi

.text.Wifi_Connect
                0x9d01940c      0x284
 .text.Wifi_Connect
                0x9d01940c      0x284 build/default/production/_ext/334706090/wf_connect.o
                0x9d01940c                Wifi_Connect

.text.UDPProcessIPv4
                0x9d019690      0x27c
 .text.UDPProcessIPv4
                0x9d019690      0x27c build/default/production/_ext/427700826/udp.o
                0x9d019690                UDPProcessIPv4

.text.SyncENCPtrRAWState
                0x9d01990c      0x278
 .text.SyncENCPtrRAWState
                0x9d01990c      0x278 build/default/production/_ext/334706090/wf_mac_24g.o

.text.GetMaxSegSizeOption
                0x9d019b84      0x274
 .text.GetMaxSegSizeOption
                0x9d019b84      0x274 build/default/production/_ext/427700826/tcp.o

.text.MPFSGet   0x9d019df8      0x270
 .text.MPFSGet  0x9d019df8      0x270 build/default/production/_ext/97638081/mpfs2.o
                0x9d019df8                MPFSGet

.text.WriteAnalogRegisterBitBang
                0x9d01a068      0x270
 .text.WriteAnalogRegisterBitBang
                0x9d01a068      0x270 build/default/production/_ext/334706090/wf_driver_com_24g.o

.text.XEEReadArray
                0x9d01a2d8      0x268
 .text.XEEReadArray
                0x9d01a2d8      0x268 build/default/production/_ext/792872985/spi_eeprom.o
                0x9d01a2d8                XEEReadArray

.text.TCPIP_IPV4_CalculatePayloadChecksum
                0x9d01a540      0x268
 .text.TCPIP_IPV4_CalculatePayloadChecksum
                0x9d01a540      0x268 build/default/production/_ext/427700826/ipv4.o
                0x9d01a540                TCPIP_IPV4_CalculatePayloadChecksum

.text.HTTPSendFile
                0x9d01a7a8      0x264
 .text.HTTPSendFile
                0x9d01a7a8      0x264 build/default/production/_ext/427700826/http2.o

.text.TCPGetArray
                0x9d01aa0c      0x264
 .text.TCPGetArray
                0x9d01aa0c      0x264 build/default/production/_ext/427700826/tcp.o
                0x9d01aa0c                TCPGetArray

.text.SYS_GENERATE_RANDOM_DWORD
                0x9d01ac70      0x25c
 .text.SYS_GENERATE_RANDOM_DWORD
                0x9d01ac70      0x25c build/default/production/_ext/365611741/system_random.o
                0x9d01ac70                SYS_GENERATE_RANDOM_DWORD

.text.SYS_CLK_OscClockGet
                0x9d01aecc      0x258
 .text.SYS_CLK_OscClockGet
                0x9d01aecc      0x258 build/default/production/_ext/365611741/system_services.o
                0x9d01aecc                SYS_CLK_OscClockGet

.text.TCPIP_IPV4_CopyTxPacketStruct
                0x9d01b124      0x250
 .text.TCPIP_IPV4_CopyTxPacketStruct
                0x9d01b124      0x250 build/default/production/_ext/427700826/ipv4.o
                0x9d01b124                TCPIP_IPV4_CopyTxPacketStruct

.text           0x9d01b374      0x248
 .text          0x9d01b374      0x248 build/default/production/_ext/427700826/tcpip_helper_c32.o
                0x9d01b374                TCPIP_HELPER_htonl
                0x9d01b380                TCPIP_HELPER_htons
                0x9d01b38c                TCPIP_Helper_CalcIPChecksum

.text.LoadDefaultConfig
                0x9d01b5bc      0x244
 .text.LoadDefaultConfig
                0x9d01b5bc      0x244 build/default/production/_ext/427700826/tcpip_manager.o

.text.malloc    0x9d01b800      0x244
 .text.malloc   0x9d01b800      0x244 c:/program files (x86)/microchip/xc32/v1.10/bin/../lib/gcc/pic32mx/4.5.1/../../../../pic32mx/lib/size\libc.a(malloc.o)
                0x9d01b800                malloc

.text.ProcessTCPIPMacEvents
                0x9d01ba44      0x240
 .text.ProcessTCPIPMacEvents
                0x9d01ba44      0x240 build/default/production/_ext/427700826/tcpip_manager.o

.rodata         0x9d01bc84      0x238
 .rodata        0x9d01bc84      0x238 build/default/production/_ext/365611741/system_services.o
                0x9d01bc94                MEDIA_STORAGE_WIFI_STORAGE_PARTITION
                0x9d01bcb0                MEDIA_STORAGE_TCPIP_STORAGE_PARTITION
                0x9d01bcc4                MEDIA_STORAGE_MPFS_IMAGE_PARTITION
                0x9d01bcd8                MEDIA_STORAGE_CONFIGURATION

.text.LCD_UPDATE_OFFSET
                0x9d01bebc      0x230
 .text.LCD_UPDATE_OFFSET
                0x9d01bebc      0x230 build/default/production/_ext/792872985/lcd.o
                0x9d01bebc                LCD_UPDATE_OFFSET

.text.ARPEntryRemoveNet
                0x9d01c0ec      0x224
 .text.ARPEntryRemoveNet
                0x9d01c0ec      0x224 build/default/production/_ext/427700826/arp.o
                0x9d01c0ec                ARPEntryRemoveNet

.text.TCPIP_IPV4_GetDataSegmentByType
                0x9d01c310      0x224
 .text.TCPIP_IPV4_GetDataSegmentByType
                0x9d01c310      0x224 build/default/production/_ext/427700826/ipv4.o
                0x9d01c310                TCPIP_IPV4_GetDataSegmentByType

.text.__floatdisf
                0x9d01c534      0x21c
 .text.__floatdisf
                0x9d01c534      0x21c c:/program files (x86)/microchip/xc32/v1.10/bin/../lib/gcc/pic32mx/4.5.1/../../../../pic32mx/lib/size\libe.a(_floatdisf.o)
                0x9d01c534                __floatdisf

.text.HTTPHeaderParseCookie
                0x9d01c750      0x214
 .text.HTTPHeaderParseCookie
                0x9d01c750      0x214 build/default/production/_ext/427700826/http2.o

.text.TCPInit   0x9d01c964      0x20c
 .text.TCPInit  0x9d01c964      0x20c build/default/production/_ext/427700826/tcp.o
                0x9d01c964                TCPInit

.text.DHCPInit  0x9d01cb70      0x204
 .text.DHCPInit
                0x9d01cb70      0x204 build/default/production/_ext/427700826/dhcp.o
                0x9d01cb70                DHCPInit

.text.HTTPIncFile
                0x9d01cd74      0x200
 .text.HTTPIncFile
                0x9d01cd74      0x200 build/default/production/_ext/427700826/http2.o
                0x9d01cd74                HTTPIncFile

.text._TcpDisconnect
                0x9d01cf74      0x200
 .text._TcpDisconnect
                0x9d01cf74      0x200 build/default/production/_ext/427700826/tcp.o

.text.UDPTask   0x9d01d174      0x200
 .text.UDPTask  0x9d01d174      0x200 build/default/production/_ext/427700826/udp.o
                0x9d01d174                UDPTask

.text.SYS_USERIO_SetLED
                0x9d01d374      0x1f8
 .text.SYS_USERIO_SetLED
                0x9d01d374      0x1f8 build/default/production/_ext/365611741/system_userio.o
                0x9d01d374                SYS_USERIO_SetLED

.text.TCPIP_ANNOUNCE_Task
                0x9d01d56c      0x1f8
 .text.TCPIP_ANNOUNCE_Task
                0x9d01d56c      0x1f8 build/default/production/_ext/427700826/tcpip_announce.o
                0x9d01d56c                TCPIP_ANNOUNCE_Task

.text.SYS_FS_chdir
                0x9d01d764      0x1f4
 .text.SYS_FS_chdir
                0x9d01d764      0x1f4 build/default/production/_ext/97638081/sys_fs.o
                0x9d01d764                SYS_FS_chdir

.text.ARPProcess
                0x9d01d958      0x1f4
 .text.ARPProcess
                0x9d01d958      0x1f4 build/default/production/_ext/427700826/arp.o
                0x9d01d958                ARPProcess

.text.TCPIP_IPV4_Flush
                0x9d01db4c      0x1ec
 .text.TCPIP_IPV4_Flush
                0x9d01db4c      0x1ec build/default/production/_ext/427700826/ipv4.o
                0x9d01db4c                TCPIP_IPV4_Flush

.text.SYS_FS_ExtractFirstFilename
                0x9d01dd38      0x1e8
 .text.SYS_FS_ExtractFirstFilename
                0x9d01dd38      0x1e8 build/default/production/_ext/97638081/sys_fs.o

.text.SYS_FS_initialize
                0x9d01df20      0x1e8
 .text.SYS_FS_initialize
                0x9d01df20      0x1e8 build/default/production/_ext/97638081/sys_fs.o
                0x9d01df20                SYS_FS_initialize

.rodata         0x9d01e108      0x1e8
 .rodata        0x9d01e108      0x1e8 build/default/production/_ext/1472/main_demo.o
                0x9d01e108                arpConfigData
                0x9d01e128                dhcpConfigData
                0x9d01e138                httpConfigData
                0x9d01e144                macPIC32INTConfigData
                0x9d01e154                mac97J60ConfigData
                0x9d01e154                tcpConfigData
                0x9d01e154                macMRF24WConfigData
                0x9d01e154                macENCJ600ConfigData
                0x9d01e154                macENCJ60ConfigData
                0x9d01e15c                udpConfigData
                0x9d01e1b4                TCPIP_HOSTS_CONFIGURATION
                0x9d01e1dc                TCPIP_STACK_MODULE_CONFIG_TBL

.text._TCPIP_HEAP_Malloc
                0x9d01e2f0      0x1e0
 .text._TCPIP_HEAP_Malloc
                0x9d01e2f0      0x1e0 build/default/production/_ext/427700826/tcpip_heap_alloc.o
                0x9d01e2f0                _TCPIP_HEAP_Malloc

.rodata         0x9d01e4d0      0x1e0
 .rodata        0x9d01e4d0      0x1e0 build/default/production/_ext/1472/custom_http_app.o
                0x9d01e5fc                HTML_UP_ARROW
                0x9d01e600                HTML_DOWN_ARROW

.text.StringToArgs
                0x9d01e6b0      0x1dc
 .text.StringToArgs
                0x9d01e6b0      0x1dc build/default/production/_ext/365611741/system_command.o

.text.HTTPURLDecode
                0x9d01e88c      0x1dc
 .text.HTTPURLDecode
                0x9d01e88c      0x1dc build/default/production/_ext/427700826/http2.o
                0x9d01e88c                HTTPURLDecode

.text.TCPProcessIPv4
                0x9d01ea68      0x1dc
 .text.TCPProcessIPv4
                0x9d01ea68      0x1dc build/default/production/_ext/427700826/tcp.o
                0x9d01ea68                TCPProcessIPv4

.text.TCPIP_IPV4_IsTxPutReady
                0x9d01ec44      0x1d8
 .text.TCPIP_IPV4_IsTxPutReady
                0x9d01ec44      0x1d8 build/default/production/_ext/427700826/ipv4.o
                0x9d01ec44                TCPIP_IPV4_IsTxPutReady

.text.HTTPHeaderParseAuthorization
                0x9d01ee1c      0x1d4
 .text.HTTPHeaderParseAuthorization
                0x9d01ee1c      0x1d4 build/default/production/_ext/427700826/http2.o

.text.UDPv4IsTxPutReady
                0x9d01eff0      0x1d4
 .text.UDPv4IsTxPutReady
                0x9d01eff0      0x1d4 build/default/production/_ext/427700826/udp.o

.text._TCPIsPutReady
                0x9d01f1c4      0x1cc
 .text._TCPIsPutReady
                0x9d01f1c4      0x1cc build/default/production/_ext/427700826/tcp.o

.text.UDPDeInit
                0x9d01f390      0x1cc
 .text.UDPDeInit
                0x9d01f390      0x1cc build/default/production/_ext/427700826/udp.o
                0x9d01f390                UDPDeInit

.text.strtoul   0x9d01f55c      0x1cc
 .text.strtoul  0x9d01f55c      0x1cc c:/program files (x86)/microchip/xc32/v1.10/bin/../lib/gcc/pic32mx/4.5.1/../../../../pic32mx/lib/size\libc.a(strtol.o)
                0x9d01f55c                strtoul

.text.SYS_USERIO_ReadIO
                0x9d01f728      0x1c8
 .text.SYS_USERIO_ReadIO
                0x9d01f728      0x1c8 build/default/production/_ext/365611741/system_userio.o

.text._TcpSocketSetIdleState
                0x9d01f8f0      0x1c8
 .text._TcpSocketSetIdleState
                0x9d01f8f0      0x1c8 build/default/production/_ext/427700826/tcp.o

.text.HTTPPrint_ledSelected
                0x9d01fab8      0x1c4
 .text.HTTPPrint_ledSelected
                0x9d01fab8      0x1c4 build/default/production/_ext/1472/custom_http_app.o
                0x9d01fab8                HTTPPrint_ledSelected

.text.TCPSetOptions
                0x9d01fc7c      0x1b8
 .text.TCPSetOptions
                0x9d01fc7c      0x1b8 build/default/production/_ext/427700826/tcp.o
                0x9d01fc7c                TCPSetOptions

.text.MRF24W_MACGetHeader
                0x9d01fe34      0x1b8
 .text.MRF24W_MACGetHeader
                0x9d01fe34      0x1b8 build/default/production/_ext/334706090/wf_mac_24g.o
                0x9d01fe34                MRF24W_MACGetHeader

.text.HTTPPrint_uploadedmd5
                0x9d01ffec      0x1b8
 .text.HTTPPrint_uploadedmd5
                0x9d01ffec      0x1b8 build/default/production/_ext/1472/custom_http_app.o
                0x9d01ffec                HTTPPrint_uploadedmd5

.text.WF_ProcessEvent
                0x9d0201a4      0x1b4
 .text.WF_ProcessEvent
                0x9d0201a4      0x1b4 build/default/production/_ext/1472/wf_config.o
                0x9d0201a4                WF_ProcessEvent

.text._SystemTickIntHandler
                0x9d020358      0x1b0
 .text._SystemTickIntHandler
                0x9d020358      0x1b0 build/default/production/_ext/365611741/system_services.o
                0x9d020358                _SystemTickIntHandler

.text.isNotifyApp
                0x9d020508      0x1a8
 .text.isNotifyApp
                0x9d020508      0x1a8 build/default/production/_ext/334706090/wf_event_handler.o

.text.DisplayNodeMsg
                0x9d0206b0      0x1a0
 .text.DisplayNodeMsg
                0x9d0206b0      0x1a0 build/default/production/_ext/365611741/system_command.o

.text.HTTPPrint_led
                0x9d020850      0x1a0
 .text.HTTPPrint_led
                0x9d020850      0x1a0 build/default/production/_ext/1472/custom_http_app.o
                0x9d020850                HTTPPrint_led

.text           0x9d0209f0      0x1a0
 .text          0x9d0209f0      0x1a0 c:/program files (x86)/microchip/xc32/v1.10/bin/../lib/gcc/pic32mx/4.5.1/../../../../pic32mx/lib/size\libpic32.a(strcpy.o)
                0x9d0209f0                strcpy

.text._TcpCloseSocket
                0x9d020b90      0x198
 .text._TcpCloseSocket
                0x9d020b90      0x198 build/default/production/_ext/427700826/tcp.o

.text.NBNSGetName
                0x9d020d28      0x194
 .text.NBNSGetName
                0x9d020d28      0x194 build/default/production/_ext/427700826/nbns.o

.text._Sys_Ext1_Isr
                0x9d020ebc      0x190
 .text._Sys_Ext1_Isr
                0x9d020ebc      0x190 build/default/production/_ext/365611741/system_services.o
                0x9d020ebc                _Sys_Ext1_Isr

.text._Sys_Ext3_Isr
                0x9d02104c      0x190
 .text._Sys_Ext3_Isr
                0x9d02104c      0x190 build/default/production/_ext/365611741/system_services.o
                0x9d02104c                _Sys_Ext3_Isr

.text._Sys_CN_Isr
                0x9d0211dc      0x190
 .text._Sys_CN_Isr
                0x9d0211dc      0x190 build/default/production/_ext/365611741/system_services.o
                0x9d0211dc                _Sys_CN_Isr

.text.MRF24W_ChipReset
                0x9d02136c      0x190
 .text.MRF24W_ChipReset
                0x9d02136c      0x190 build/default/production/_ext/334706090/wf_driver_com_24g.o
                0x9d02136c                MRF24W_ChipReset

.text.RawMove   0x9d0214fc      0x190
 .text.RawMove  0x9d0214fc      0x190 build/default/production/_ext/334706090/wf_driver_raw_24g.o

.text.TCPIP_HELPER_StringToMACAddress
                0x9d02168c      0x18c
 .text.TCPIP_HELPER_StringToMACAddress
                0x9d02168c      0x18c build/default/production/_ext/427700826/tcpip_helpers.o
                0x9d02168c                TCPIP_HELPER_StringToMACAddress

.text.WaitForRawMoveComplete
                0x9d021818      0x18c
 .text.WaitForRawMoveComplete
                0x9d021818      0x18c build/default/production/_ext/334706090/wf_driver_raw_24g.o

.text.DRV_MEDIA_Initialize
                0x9d0219a4      0x188
 .text.DRV_MEDIA_Initialize
                0x9d0219a4      0x188 build/default/production/_ext/792872985/drv_media.o
                0x9d0219a4                DRV_MEDIA_Initialize

.text.UDPGetArray
                0x9d021b2c      0x188
 .text.UDPGetArray
                0x9d021b2c      0x188 build/default/production/_ext/427700826/udp.o
                0x9d021b2c                UDPGetArray

.text.OutputBeaconTimeout
                0x9d021cb4      0x188
 .text.OutputBeaconTimeout
                0x9d021cb4      0x188 build/default/production/_ext/334706090/wf_debug_output.o

.text.HTTPServer
                0x9d021e3c      0x180
 .text.HTTPServer
                0x9d021e3c      0x180 build/default/production/_ext/427700826/http2.o
                0x9d021e3c                HTTPServer

.text._OAHashFindBkt
                0x9d021fbc      0x180
 .text._OAHashFindBkt
                0x9d021fbc      0x180 build/default/production/_ext/427700826/hash_tbl.o

.text.ARPIsResolved
                0x9d02213c      0x178
 .text.ARPIsResolved
                0x9d02213c      0x178 build/default/production/_ext/427700826/arp.o
                0x9d02213c                ARPIsResolved

.text.TCPIP_IPV4_AllocateTxPacket
                0x9d0222b4      0x178
 .text.TCPIP_IPV4_AllocateTxPacket
                0x9d0222b4      0x178 build/default/production/_ext/427700826/ipv4.o
                0x9d0222b4                TCPIP_IPV4_AllocateTxPacket

.text.TCPIP_HEAP_Create
                0x9d02242c      0x178
 .text.TCPIP_HEAP_Create
                0x9d02242c      0x178 build/default/production/_ext/427700826/tcpip_heap_alloc.o
                0x9d02242c                TCPIP_HEAP_Create

.text.HTTPPostLCD
                0x9d0225a4      0x178
 .text.HTTPPostLCD
                0x9d0225a4      0x178 build/default/production/_ext/1472/custom_http_app.o

.text.MPFSOpenID
                0x9d02271c      0x174
 .text.MPFSOpenID
                0x9d02271c      0x174 build/default/production/_ext/97638081/mpfs2.o
                0x9d02271c                MPFSOpenID

.text.SYS_FS_IsLegalDirString
                0x9d022890      0x170
 .text.SYS_FS_IsLegalDirString
                0x9d022890      0x170 build/default/production/_ext/97638081/sys_fs.o
                0x9d022890                SYS_FS_IsLegalDirString

.text.LCD_INIT  0x9d022a00      0x170
 .text.LCD_INIT
                0x9d022a00      0x170 build/default/production/_ext/792872985/lcd.o
                0x9d022a00                LCD_INIT

.text._ARPProbeAddress
                0x9d022b70      0x170
 .text._ARPProbeAddress
                0x9d022b70      0x170 build/default/production/_ext/427700826/arp.o

.text.SpiChnOpen
                0x9d022ce0      0x170
 .text.SpiChnOpen
                0x9d022ce0      0x170 c:/program files (x86)/microchip/xc32/v1.10/bin/../lib/gcc/pic32mx/4.5.1/../../../../pic32mx/lib/size\libmchp_peripheral_32MX795F512L.a(spi_chn_open_lib.o)
                0x9d022ce0                SpiChnOpen

.text.stricmppgm2ram
                0x9d022e50      0x16c
 .text.stricmppgm2ram
                0x9d022e50      0x16c build/default/production/_ext/101875047/helpers.o
                0x9d022e50                stricmppgm2ram

.text.OAHashLookUpInsert
                0x9d022fbc      0x16c
 .text.OAHashLookUpInsert
                0x9d022fbc      0x16c build/default/production/_ext/427700826/hash_tbl.o
                0x9d022fbc                OAHashLookUpInsert

.text.UDPv4Flush
                0x9d023128      0x16c
 .text.UDPv4Flush
                0x9d023128      0x16c build/default/production/_ext/427700826/udp.o

.text.WFHardwareInit
                0x9d023294      0x168
 .text.WFHardwareInit
                0x9d023294      0x168 build/default/production/_ext/334706090/wf_driver_com_24g.o
                0x9d023294                WFHardwareInit

.text           0x9d0233fc      0x2d0
 .text          0x9d0233fc      0x168 c:/program files (x86)/microchip/xc32/v1.10/bin/../lib/gcc/pic32mx/4.5.1/../../../../pic32mx/lib/size\libpic32.a(memcpy.o)
                0x9d0233fc                memcpy
 .text          0x9d023564      0x168 c:/program files (x86)/microchip/xc32/v1.10/bin/../lib/gcc/pic32mx/4.5.1/../../../../pic32mx/lib/size\libpic32.a(strlen.o)
                0x9d023564                strlen

.text.USART_INIT
                0x9d0236cc      0x164
 .text.USART_INIT
                0x9d0236cc      0x164 build/default/production/_ext/792872985/usart.o
                0x9d0236cc                USART_INIT

.text.XEEIsBusy
                0x9d023830      0x164
 .text.XEEIsBusy
                0x9d023830      0x164 build/default/production/_ext/792872985/spi_eeprom.o
                0x9d023830                XEEIsBusy

.text.RawSetIndex
                0x9d023994      0x164
 .text.RawSetIndex
                0x9d023994      0x164 build/default/production/_ext/334706090/wf_driver_raw_24g.o
                0x9d023994                RawSetIndex

.text.SYS_TICK_TimerDelete
                0x9d023af8      0x160
 .text.SYS_TICK_TimerDelete
                0x9d023af8      0x160 build/default/production/_ext/365611741/system_services.o
                0x9d023af8                SYS_TICK_TimerDelete

.text.DRV_SPI_TxRx
                0x9d023c58      0x160
 .text.DRV_SPI_TxRx
                0x9d023c58      0x160 build/default/production/_ext/792872985/drv_spi.o
                0x9d023c58                DRV_SPI_TxRx

.text.DNSPutString
                0x9d023db8      0x160
 .text.DNSPutString
                0x9d023db8      0x160 build/default/production/_ext/427700826/dns.o

.text.TCPIP_IPV4_TransmitPacket
                0x9d023f18      0x160
 .text.TCPIP_IPV4_TransmitPacket
                0x9d023f18      0x160 build/default/production/_ext/427700826/ipv4.o
                0x9d023f18                TCPIP_IPV4_TransmitPacket

.text.UDPBind   0x9d024078      0x160
 .text.UDPBind  0x9d024078      0x160 build/default/production/_ext/427700826/udp.o
                0x9d024078                UDPBind

.text.WFEintHandler
                0x9d0241d8      0x160
 .text.WFEintHandler
                0x9d0241d8      0x160 build/default/production/_ext/334706090/wf_driver_com_24g.o
                0x9d0241d8                WFEintHandler

.text.encodeblock
                0x9d024338      0x160
 .text.encodeblock
                0x9d024338      0x160 build/default/production/_ext/1472/tcp6_demo_app.o
                0x9d024338                encodeblock

.text.ARP_SendIfPkt
                0x9d024498      0x15c
 .text.ARP_SendIfPkt
                0x9d024498      0x15c build/default/production/_ext/427700826/arp.o

.text.TCPIP_IPV4_GetHeader
                0x9d0245f4      0x15c
 .text.TCPIP_IPV4_GetHeader
                0x9d0245f4      0x15c build/default/production/_ext/427700826/ipv4.o
                0x9d0245f4                TCPIP_IPV4_GetHeader

.text.DRV_MEDIA_Read
                0x9d024750      0x158
 .text.DRV_MEDIA_Read
                0x9d024750      0x158 build/default/production/_ext/792872985/drv_media.o
                0x9d024750                DRV_MEDIA_Read

.text.HTTPPrint_config_mac
                0x9d0248a8      0x158
 .text.HTTPPrint_config_mac
                0x9d0248a8      0x158 build/default/production/_ext/1472/custom_http_app.o
                0x9d0248a8                HTTPPrint_config_mac

.text.ProcessInterruptServiceResult
                0x9d024a00      0x154
 .text.ProcessInterruptServiceResult
                0x9d024a00      0x154 build/default/production/_ext/334706090/wf_driver_com_24g.o

.rodata         0x9d024b54      0x150
 .rodata        0x9d024b54      0x150 build/default/production/_ext/365611741/system_debug.o

.text._TCPIPStackIsLocalNetwork
                0x9d024ca4      0x150
 .text._TCPIPStackIsLocalNetwork
                0x9d024ca4      0x150 build/default/production/_ext/427700826/tcpip_manager.o
                0x9d024ca4                _TCPIPStackIsLocalNetwork

.text.TCPIP_Helper_CalcMACBufferIPChecksum
                0x9d024df4      0x150
 .text.TCPIP_Helper_CalcMACBufferIPChecksum
                0x9d024df4      0x150 build/default/production/_ext/427700826/tcpip_helpers.o
                0x9d024df4                TCPIP_Helper_CalcMACBufferIPChecksum

.text.OutputChannelList
                0x9d024f44      0x150
 .text.OutputChannelList
                0x9d024f44      0x150 build/default/production/_ext/334706090/wf_debug_output.o

.text.UDPSocketSetNet
                0x9d025094      0x14c
 .text.UDPSocketSetNet
                0x9d025094      0x14c build/default/production/_ext/427700826/udp.o
                0x9d025094                UDPSocketSetNet

.text._sbrk_init
                0x9d0251e0      0x14c
 .text._sbrk_init
                0x9d0251e0      0x14c c:/program files (x86)/microchip/xc32/v1.10/bin/../lib/gcc/pic32mx/4.5.1/../../../../pic32mx/lib/size\libpic32.a(sbrk.o)
                0x9d0251e0                _sbrk_init

.text._SYS_CMDIO_DELETE
                0x9d02532c      0x148
 .text._SYS_CMDIO_DELETE
                0x9d02532c      0x148 build/default/production/_ext/365611741/system_command.o
                0x9d02532c                _SYS_CMDIO_DELETE

.text.TCPIP_STACK_DeInit
                0x9d025474      0x148
 .text.TCPIP_STACK_DeInit
                0x9d025474      0x148 build/default/production/_ext/427700826/tcpip_manager.o
                0x9d025474                TCPIP_STACK_DeInit

.text.OutputConnectionTempLostMsg
                0x9d0255bc      0x148
 .text.OutputConnectionTempLostMsg
                0x9d0255bc      0x148 build/default/production/_ext/334706090/wf_debug_output.o

.text.OutputConnectionPermLostMsg
                0x9d025704      0x148
 .text.OutputConnectionPermLostMsg
                0x9d025704      0x148 build/default/production/_ext/334706090/wf_debug_output.o

.text.SendMgmtMsg
                0x9d02584c      0x148
 .text.SendMgmtMsg
                0x9d02584c      0x148 build/default/production/_ext/334706090/wf_mgmt_msg_24g.o
                0x9d02584c                SendMgmtMsg

.text.OAHashLookUp
                0x9d025994      0x144
 .text.OAHashLookUp
                0x9d025994      0x144 build/default/production/_ext/427700826/hash_tbl.o
                0x9d025994                OAHashLookUp

.text.scale     0x9d025ad8      0x144
 .text.scale    0x9d025ad8      0x144 c:/program files (x86)/microchip/xc32/v1.10/bin/../lib/gcc/pic32mx/4.5.1/../../../../pic32mx/lib/size\libc.a(doprnt.o)

.rodata         0x9d025c1c      0x140
 .rodata        0x9d025c1c      0x140 build/default/production/_ext/101875047/hashes.o

.text._WF_OutputConnectionContext
                0x9d025d5c      0x140
 .text._WF_OutputConnectionContext
                0x9d025d5c      0x140 build/default/production/_ext/334706090/wf_debug_output.o
                0x9d025d5c                _WF_OutputConnectionContext

.text.PowerSaveTask
                0x9d025e9c      0x140
 .text.PowerSaveTask
                0x9d025e9c      0x140 build/default/production/_ext/334706090/wf_driver_com_24g.o
                0x9d025e9c                PowerSaveTask

.text.UDPIsGetReady
                0x9d025fdc      0x13c
 .text.UDPIsGetReady
                0x9d025fdc      0x13c build/default/production/_ext/427700826/udp.o
                0x9d025fdc                UDPIsGetReady

.text.WF_SetMultiCastFilter
                0x9d026118      0x13c
 .text.WF_SetMultiCastFilter
                0x9d026118      0x13c build/default/production/_ext/334706090/wf_param_msg_24g.o
                0x9d026118                WF_SetMultiCastFilter

.text._ARPUpdateEntry
                0x9d026254      0x138
 .text._ARPUpdateEntry
                0x9d026254      0x138 build/default/production/_ext/427700826/arp.o

.text.TCPIP_IPV4_QueuedPacketTransmitTask
                0x9d02638c      0x138
 .text.TCPIP_IPV4_QueuedPacketTransmitTask
                0x9d02638c      0x138 build/default/production/_ext/427700826/ipv4.o

.text.HTTPPrint_btn
                0x9d0264c4      0x138
 .text.HTTPPrint_btn
                0x9d0264c4      0x138 build/default/production/_ext/1472/custom_http_app.o
                0x9d0264c4                HTTPPrint_btn

.text._general_exception_handler
                0x9d0265fc      0x134
 .text._general_exception_handler
                0x9d0265fc      0x134 build/default/production/_ext/365611741/system_debug.o
                0x9d0265fc                _general_exception_handler

.text.SYS_USERIO_Initialize
                0x9d026730      0x134
 .text.SYS_USERIO_Initialize
                0x9d026730      0x134 build/default/production/_ext/365611741/system_userio.o
                0x9d026730                SYS_USERIO_Initialize

.text.SYS_FS_FSFromAbsPath
                0x9d026864      0x134
 .text.SYS_FS_FSFromAbsPath
                0x9d026864      0x134 build/default/production/_ext/97638081/sys_fs.o

.text.TCPIP_IPV4_InsertIPPacketSegment
                0x9d026998      0x134
 .text.TCPIP_IPV4_InsertIPPacketSegment
                0x9d026998      0x134 build/default/production/_ext/427700826/ipv4.o
                0x9d026998                TCPIP_IPV4_InsertIPPacketSegment

.text.SetSecurity
                0x9d026acc      0x134
 .text.SetSecurity
                0x9d026acc      0x134 build/default/production/_ext/334706090/wf_connection_profile.o

.text.fputc     0x9d026c00      0x134
 .text.fputc    0x9d026c00      0x134 c:/program files (x86)/microchip/xc32/v1.10/bin/../lib/gcc/pic32mx/4.5.1/../../../../pic32mx/lib/size\libc.a(_fputc_simple.o)
                0x9d026c00                fputc

.text.DRV_MEDIA_Write
                0x9d026d34      0x130
 .text.DRV_MEDIA_Write
                0x9d026d34      0x130 build/default/production/_ext/792872985/drv_media.o
                0x9d026d34                DRV_MEDIA_Write

.text.UDPSetBcastIPV4Address
                0x9d026e64      0x130
 .text.UDPSetBcastIPV4Address
                0x9d026e64      0x130 build/default/production/_ext/427700826/udp.o
                0x9d026e64                UDPSetBcastIPV4Address

.text.realloc   0x9d026f94      0x130
 .text.realloc  0x9d026f94      0x130 c:/program files (x86)/microchip/xc32/v1.10/bin/../lib/gcc/pic32mx/4.5.1/../../../../pic32mx/lib/size\libc.a(malloc.o)
                0x9d026f94                realloc

.text.uitoa     0x9d0270c4      0x12c
 .text.uitoa    0x9d0270c4      0x12c build/default/production/_ext/101875047/helpers.o
                0x9d0270c4                uitoa

.text.WF_ConfigDataLoad
                0x9d0271f0      0x12c
 .text.WF_ConfigDataLoad
                0x9d0271f0      0x12c build/default/production/_ext/334706090/wf_init.o
                0x9d0271f0                WF_ConfigDataLoad

.text.DNSBeginUsage
                0x9d02731c      0x128
 .text.DNSBeginUsage
                0x9d02731c      0x128 build/default/production/_ext/427700826/dns.o
                0x9d02731c                DNSBeginUsage

.text.HTTPDeInit
                0x9d027444      0x124
 .text.HTTPDeInit
                0x9d027444      0x124 build/default/production/_ext/427700826/http2.o
                0x9d027444                HTTPDeInit

.text.TCPIP_IPV4_Initialize
                0x9d027568      0x124
 .text.TCPIP_IPV4_Initialize
                0x9d027568      0x124 build/default/production/_ext/427700826/ipv4.o
                0x9d027568                TCPIP_IPV4_Initialize

.text._TCPSendWinIncUpdate
                0x9d02768c      0x124
 .text._TCPSendWinIncUpdate
                0x9d02768c      0x124 build/default/production/_ext/427700826/tcp.o

.text.UDPOpenServer
                0x9d0277b0      0x124
 .text.UDPOpenServer
                0x9d0277b0      0x124 build/default/production/_ext/427700826/udp.o
                0x9d0277b0                UDPOpenServer

.text.WaitForMgmtResponse
                0x9d0278d4      0x124
 .text.WaitForMgmtResponse
                0x9d0278d4      0x124 build/default/production/_ext/334706090/wf_mgmt_msg_24g.o
                0x9d0278d4                WaitForMgmtResponse

.text.strtol    0x9d0279f8      0x124
 .text.strtol   0x9d0279f8      0x124 c:/program files (x86)/microchip/xc32/v1.10/bin/../lib/gcc/pic32mx/4.5.1/../../../../pic32mx/lib/size\libc.a(strtol.o)
                0x9d0279f8                strtol

.text.TCPIP_IPV4_QueuePacket
                0x9d027b1c      0x120
 .text.TCPIP_IPV4_QueuePacket
                0x9d027b1c      0x120 build/default/production/_ext/427700826/ipv4.o

.text.TCPOpenServer
                0x9d027c3c      0x120
 .text.TCPOpenServer
                0x9d027c3c      0x120 build/default/production/_ext/427700826/tcp.o
                0x9d027c3c                TCPOpenServer

.text           0x9d027d5c      0x120
 .text          0x9d027d5c      0x120 c:/program files (x86)/microchip/xc32/v1.10/bin/../lib/gcc/pic32mx/4.5.1/../../../../pic32mx/lib/size\libpic32.a(strcmp.o)
                0x9d027d5c                strcmp

.text.fround    0x9d027e7c      0x120
 .text.fround   0x9d027e7c      0x120 c:/program files (x86)/microchip/xc32/v1.10/bin/../lib/gcc/pic32mx/4.5.1/../../../../pic32mx/lib/size\libc.a(doprnt.o)

.text.SHA1AddData
                0x9d027f9c      0x11c
 .text.SHA1AddData
                0x9d027f9c      0x11c build/default/production/_ext/101875047/hashes.o
                0x9d027f9c                SHA1AddData

.text.b64_encode
                0x9d0280b8      0x11c
 .text.b64_encode
                0x9d0280b8      0x11c build/default/production/_ext/1472/tcp6_demo_app.o
                0x9d0280b8                b64_encode

.text.BSP_Initialize
                0x9d0281d4      0x114
 .text.BSP_Initialize
                0x9d0281d4      0x114 build/default/production/_ext/1293749816/bsp.o
                0x9d0281d4                BSP_Initialize

.text.TCPIP_IPV4_PutHeader
                0x9d0282e8      0x114
 .text.TCPIP_IPV4_PutHeader
                0x9d0282e8      0x114 build/default/production/_ext/427700826/ipv4.o
                0x9d0282e8                TCPIP_IPV4_PutHeader

.text.DisplayIPValue
                0x9d0283fc      0x114
 .text.DisplayIPValue
                0x9d0283fc      0x114 build/default/production/_ext/1472/main_demo.o
                0x9d0283fc                DisplayIPValue

.text.MD5AddData
                0x9d028510      0x110
 .text.MD5AddData
                0x9d028510      0x110 build/default/production/_ext/101875047/hashes.o
                0x9d028510                MD5AddData

.text.WiFiAsyncTask
                0x9d028620      0x110
 .text.WiFiAsyncTask
                0x9d028620      0x110 build/default/production/_ext/334706090/wf_event_handler.o
                0x9d028620                WiFiAsyncTask

.text.WF_PsPollEnable
                0x9d028730      0x110
 .text.WF_PsPollEnable
                0x9d028730      0x110 build/default/production/_ext/334706090/wf_power_save.o
                0x9d028730                WF_PsPollEnable

.text._flsbuf   0x9d028840      0x110
 .text._flsbuf  0x9d028840      0x110 c:/program files (x86)/microchip/xc32/v1.10/bin/../lib/gcc/pic32mx/4.5.1/../../../../pic32mx/lib/size\libc.a(_flsbuf_simple.o)
                0x9d028840                _flsbuf

.text._TcpSwapHeader
                0x9d028950      0x10c
 .text._TcpSwapHeader
                0x9d028950      0x10c build/default/production/_ext/427700826/tcp.o

.text.TCPIP_STACK_BringNetDown
                0x9d028a5c      0x108
 .text.TCPIP_STACK_BringNetDown
                0x9d028a5c      0x108 build/default/production/_ext/427700826/tcpip_manager.o

.text.OutputNetworkType
                0x9d028b64      0x108
 .text.OutputNetworkType
                0x9d028b64      0x108 build/default/production/_ext/334706090/wf_debug_output.o

.text._DHCPClose
                0x9d028c6c      0x104
 .text._DHCPClose
                0x9d028c6c      0x104 build/default/production/_ext/427700826/dhcp.o

.text.WF_ScanContextGet
                0x9d028d70      0x104
 .text.WF_ScanContextGet
                0x9d028d70      0x104 build/default/production/_ext/334706090/wf_connection_algorithm.o
                0x9d028d70                WF_ScanContextGet

.rodata         0x9d028e74      0x208
 .rodata        0x9d028e74      0x104 build/default/production/_ext/1472/wf_config.o
 .rodata        0x9d028f78      0x104 c:/program files (x86)/microchip/xc32/v1.10/bin/../lib/gcc/pic32mx/4.5.1/../../../../pic32mx/lib/size\libc.a(ctype.o)
                0x9d028f78                _ctype

.text.hexatob   0x9d02907c      0x100
 .text.hexatob  0x9d02907c      0x100 build/default/production/_ext/101875047/helpers.o
                0x9d02907c                hexatob

.text.MPFSGetFilename
                0x9d02917c       0xfc
 .text.MPFSGetFilename
                0x9d02917c       0xfc build/default/production/_ext/97638081/mpfs2.o
                0x9d02917c                MPFSGetFilename

.text.WaitForMgmtResponseAndReadData
                0x9d029278       0xfc
 .text.WaitForMgmtResponseAndReadData
                0x9d029278       0xfc build/default/production/_ext/334706090/wf_mgmt_msg_24g.o
                0x9d029278                WaitForMgmtResponseAndReadData

.text.HTTPExecutePost
                0x9d029374       0xfc
 .text.HTTPExecutePost
                0x9d029374       0xfc build/default/production/_ext/1472/custom_http_app.o
                0x9d029374                HTTPExecutePost

.text.SYS_FS_IsAbsolutePath
                0x9d029470       0xf8
 .text.SYS_FS_IsAbsolutePath
                0x9d029470       0xf8 build/default/production/_ext/97638081/sys_fs.o

.text._TCPIPStackAddressServiceEvent
                0x9d029568       0xf8
 .text._TCPIPStackAddressServiceEvent
                0x9d029568       0xf8 build/default/production/_ext/427700826/tcpip_manager.o
                0x9d029568                _TCPIPStackAddressServiceEvent

.text.SingleListRemoveNode
                0x9d029660       0xf8
 .text.SingleListRemoveNode
                0x9d029660       0xf8 build/default/production/_ext/427700826/tcpip_helpers.o
                0x9d029660                SingleListRemoveNode

.text.WF_Init   0x9d029758       0xf8
 .text.WF_Init  0x9d029758       0xf8 build/default/production/_ext/334706090/wf_init.o
                0x9d029758                WF_Init

.text.SYS_USERIO_DeviceDebounce
                0x9d029850       0xf4
 .text.SYS_USERIO_DeviceDebounce
                0x9d029850       0xf4 build/default/production/_ext/365611741/system_userio.o
                0x9d029850                SYS_USERIO_DeviceDebounce

.text.UDPSetSourceIPAddress
                0x9d029944       0xf4
 .text.UDPSetSourceIPAddress
                0x9d029944       0xf4 build/default/production/_ext/427700826/udp.o
                0x9d029944                UDPSetSourceIPAddress

.text.UDPSetDestinationIPAddress
                0x9d029a38       0xf4
 .text.UDPSetDestinationIPAddress
                0x9d029a38       0xf4 build/default/production/_ext/427700826/udp.o
                0x9d029a38                UDPSetDestinationIPAddress

.text.WF_SecurityGet
                0x9d029b2c       0xf4
 .text.WF_SecurityGet
                0x9d029b2c       0xf4 build/default/production/_ext/334706090/wf_connection_profile.o
                0x9d029b2c                WF_SecurityGet

.text.MRF24W_MACInitialize
                0x9d029c20       0xf4
 .text.MRF24W_MACInitialize
                0x9d029c20       0xf4 build/default/production/_ext/334706090/mrf24w_mac_pic32.o
                0x9d029c20                MRF24W_MACInitialize

.text._ARPAddCompleteEntry
                0x9d029d14       0xf0
 .text._ARPAddCompleteEntry
                0x9d029d14       0xf0 build/default/production/_ext/427700826/arp.o

.text.UDPDiscard
                0x9d029e04       0xf0
 .text.UDPDiscard
                0x9d029e04       0xf0 build/default/production/_ext/427700826/udp.o
                0x9d029e04                UDPDiscard

.text.WF_ScanContextSet
                0x9d029ef4       0xf0
 .text.WF_ScanContextSet
                0x9d029ef4       0xf0 build/default/production/_ext/334706090/wf_connection_algorithm.o
                0x9d029ef4                WF_ScanContextSet

.text.NBNSPutName
                0x9d029fe4       0xec
 .text.NBNSPutName
                0x9d029fe4       0xec build/default/production/_ext/427700826/nbns.o

.text.TCPIsPutReady
                0x9d02a0d0       0xec
 .text.TCPIsPutReady
                0x9d02a0d0       0xec build/default/production/_ext/427700826/tcp.o
                0x9d02a0d0                TCPIsPutReady

.text._TCPIP_HEAP_CallocDebug
                0x9d02a1bc       0xec
 .text._TCPIP_HEAP_CallocDebug
                0x9d02a1bc       0xec build/default/production/_ext/427700826/tcpip_heap_alloc.o
                0x9d02a1bc                _TCPIP_HEAP_CallocDebug

.text.AllocateDataTxBuffer
                0x9d02a2a8       0xec
 .text.AllocateDataTxBuffer
                0x9d02a2a8       0xec build/default/production/_ext/334706090/wf_driver_raw_24g.o
                0x9d02a2a8                AllocateDataTxBuffer

.text.HTTPReadPostValue
                0x9d02a394       0xe8
 .text.HTTPReadPostValue
                0x9d02a394       0xe8 build/default/production/_ext/427700826/http2.o
                0x9d02a394                HTTPReadPostValue

.text.DNSIsResolved
                0x9d02a47c       0xe8
 .text.DNSIsResolved
                0x9d02a47c       0xe8 build/default/production/_ext/427700826/dns.o
                0x9d02a47c                DNSIsResolved

.text.TCPIP_IPV4_PutUpperLayerHeader
                0x9d02a564       0xe8
 .text.TCPIP_IPV4_PutUpperLayerHeader
                0x9d02a564       0xe8 build/default/production/_ext/427700826/ipv4.o
                0x9d02a564                TCPIP_IPV4_PutUpperLayerHeader

.text.UDPSetRxOffset
                0x9d02a64c       0xe8
 .text.UDPSetRxOffset
                0x9d02a64c       0xe8 build/default/production/_ext/427700826/udp.o
                0x9d02a64c                UDPSetRxOffset

.text.ProcessTCPIPTickEvent
                0x9d02a734       0xe8
 .text.ProcessTCPIPTickEvent
                0x9d02a734       0xe8 build/default/production/_ext/427700826/tcpip_manager.o

.text.WF_GetDeviceInfo
                0x9d02a81c       0xe8
 .text.WF_GetDeviceInfo
                0x9d02a81c       0xe8 build/default/production/_ext/334706090/wf_param_msg_24g.o
                0x9d02a81c                WF_GetDeviceInfo

.rodata         0x9d02a908       0xe8
 .rodata        0x9d02a908       0xe8 c:/program files (x86)/microchip/xc32/v1.10/bin/../lib/gcc/pic32mx/4.5.1/../../../../pic32mx/lib/size\libc.a(doprnt.o)

.text.LCD_WRITE
                0x9d02a9f0       0xe4
 .text.LCD_WRITE
                0x9d02a9f0       0xe4 build/default/production/_ext/792872985/lcd.o
                0x9d02a9f0                LCD_WRITE

.text.TCPIP_IPV4_ResetTransmitPacketState
                0x9d02aad4       0xe4
 .text.TCPIP_IPV4_ResetTransmitPacketState
                0x9d02aad4       0xe4 build/default/production/_ext/427700826/ipv4.o
                0x9d02aad4                TCPIP_IPV4_ResetTransmitPacketState

.text.TCPIP_IPV4_AllocateDataSegmentHeader
                0x9d02abb8       0xe4
 .text.TCPIP_IPV4_AllocateDataSegmentHeader
                0x9d02abb8       0xe4 build/default/production/_ext/427700826/ipv4.o
                0x9d02abb8                TCPIP_IPV4_AllocateDataSegmentHeader

.text.TCPDeInit
                0x9d02ac9c       0xe4
 .text.TCPDeInit
                0x9d02ac9c       0xe4 build/default/production/_ext/427700826/tcp.o
                0x9d02ac9c                TCPDeInit

.text.TCPIP_HEAP_Delete
                0x9d02ad80       0xe4
 .text.TCPIP_HEAP_Delete
                0x9d02ad80       0xe4 build/default/production/_ext/427700826/tcpip_heap_alloc.o
                0x9d02ad80                TCPIP_HEAP_Delete

.text.SYS_TICK_TimerCreate
                0x9d02ae64       0xe0
 .text.SYS_TICK_TimerCreate
                0x9d02ae64       0xe0 build/default/production/_ext/365611741/system_services.o
                0x9d02ae64                SYS_TICK_TimerCreate

.text._SYS_CMDIO_ADD
                0x9d02af44       0xe0
 .text._SYS_CMDIO_ADD
                0x9d02af44       0xe0 build/default/production/_ext/365611741/system_command.o
                0x9d02af44                _SYS_CMDIO_ADD

.text._ARPSetEntry
                0x9d02b024       0xe0
 .text._ARPSetEntry
                0x9d02b024       0xe0 build/default/production/_ext/427700826/arp.o

.text.ARPResolve
                0x9d02b104       0xe0
 .text.ARPResolve
                0x9d02b104       0xe0 build/default/production/_ext/427700826/arp.o
                0x9d02b104                ARPResolve

.text.UDPOpenClient
                0x9d02b1e4       0xe0
 .text.UDPOpenClient
                0x9d02b1e4       0xe0 build/default/production/_ext/427700826/udp.o
                0x9d02b1e4                UDPOpenClient

.text.UDPPutArray
                0x9d02b2c4       0xe0
 .text.UDPPutArray
                0x9d02b2c4       0xe0 build/default/production/_ext/427700826/udp.o
                0x9d02b2c4                UDPPutArray

.text.TCPIPMacEventCB
                0x9d02b3a4       0xe0
 .text.TCPIPMacEventCB
                0x9d02b3a4       0xe0 build/default/production/_ext/427700826/tcpip_manager.o

.text._SYS_ERROR_PRINT
                0x9d02b484       0xdc
 .text._SYS_ERROR_PRINT
                0x9d02b484       0xdc build/default/production/_ext/365611741/system_debug.o
                0x9d02b484                _SYS_ERROR_PRINT

.text.HTTPHeaderParseContentLength
                0x9d02b560       0xdc
 .text.HTTPHeaderParseContentLength
                0x9d02b560       0xdc build/default/production/_ext/427700826/http2.o

.text.ARPHashDeleteEntry
                0x9d02b63c       0xdc
 .text.ARPHashDeleteEntry
                0x9d02b63c       0xdc build/default/production/_ext/427700826/arp.o
                0x9d02b63c                ARPHashDeleteEntry

.text.DHCPConnectionHandler
                0x9d02b718       0xdc
 .text.DHCPConnectionHandler
                0x9d02b718       0xdc build/default/production/_ext/427700826/dhcp.o
                0x9d02b718                DHCPConnectionHandler

.text._TcpCleanup
                0x9d02b7f4       0xdc
 .text._TcpCleanup
                0x9d02b7f4       0xdc build/default/production/_ext/427700826/tcp.o

.text.TCPOpenClient
                0x9d02b8d0       0xdc
 .text.TCPOpenClient
                0x9d02b8d0       0xdc build/default/production/_ext/427700826/tcp.o
                0x9d02b8d0                TCPOpenClient

.text.TcpAllocateEphemeralPort
                0x9d02b9ac       0xdc
 .text.TcpAllocateEphemeralPort
                0x9d02b9ac       0xdc build/default/production/_ext/427700826/tcp.o

.text.UdpAllocateEphemeralPort
                0x9d02ba88       0xdc
 .text.UdpAllocateEphemeralPort
                0x9d02ba88       0xdc build/default/production/_ext/427700826/udp.o

.text.OutputTxMode
                0x9d02bb64       0xdc
 .text.OutputTxMode
                0x9d02bb64       0xdc build/default/production/_ext/334706090/wf_debug_output.o

.text.MACIFService
                0x9d02bc40       0xdc
 .text.MACIFService
                0x9d02bc40       0xdc build/default/production/_ext/334706090/wf_mac_24g.o

.text.DHCPEnable
                0x9d02bd1c       0xd8
 .text.DHCPEnable
                0x9d02bd1c       0xd8 build/default/production/_ext/427700826/dhcp.o
                0x9d02bd1c                DHCPEnable

.text.TCPIP_IPV4_GetPseudoHeaderChecksum
                0x9d02bdf4       0xd8
 .text.TCPIP_IPV4_GetPseudoHeaderChecksum
                0x9d02bdf4       0xd8 build/default/production/_ext/427700826/ipv4.o
                0x9d02bdf4                TCPIP_IPV4_GetPseudoHeaderChecksum

.text._TcpAbort
                0x9d02becc       0xd8
 .text._TcpAbort
                0x9d02becc       0xd8 build/default/production/_ext/427700826/tcp.o

.text._TCPIP_HEAP_MallocDebug
                0x9d02bfa4       0xd8
 .text._TCPIP_HEAP_MallocDebug
                0x9d02bfa4       0xd8 build/default/production/_ext/427700826/tcpip_heap_alloc.o
                0x9d02bfa4                _TCPIP_HEAP_MallocDebug

.text._SYS_RANDOM_INIT
                0x9d02c07c       0xd4
 .text._SYS_RANDOM_INIT
                0x9d02c07c       0xd4 build/default/production/_ext/365611741/system_random.o
                0x9d02c07c                _SYS_RANDOM_INIT

.text.TCPIP_ANNOUNCE_Init
                0x9d02c150       0xd4
 .text.TCPIP_ANNOUNCE_Init
                0x9d02c150       0xd4 build/default/production/_ext/427700826/tcpip_announce.o
                0x9d02c150                TCPIP_ANNOUNCE_Init

.text.TCPClose  0x9d02c224       0xd4
 .text.TCPClose
                0x9d02c224       0xd4 build/default/production/_ext/427700826/tcp.o
                0x9d02c224                TCPClose

.text.OutputDomain
                0x9d02c2f8       0xd4
 .text.OutputDomain
                0x9d02c2f8       0xd4 build/default/production/_ext/334706090/wf_debug_output.o

.text.AllocateMgmtTxBuffer
                0x9d02c3cc       0xd4
 .text.AllocateMgmtTxBuffer
                0x9d02c3cc       0xd4 build/default/production/_ext/334706090/wf_driver_raw_24g.o
                0x9d02c3cc                AllocateMgmtTxBuffer

.text           0x9d02c4a0       0xd4
 .text          0x9d02c4a0       0xd4 c:/program files (x86)/microchip/xc32/v1.10/bin/../lib/gcc/pic32mx/4.5.1/size\libgcc.a(_floatundisf.o)
                0x9d02c4a0                __floatundisf

.text._LoadFATRecord
                0x9d02c574       0xd0
 .text._LoadFATRecord
                0x9d02c574       0xd0 build/default/production/_ext/97638081/mpfs2.o

.text.HTTPGetArg
                0x9d02c644       0xd0
 .text.HTTPGetArg
                0x9d02c644       0xd0 build/default/production/_ext/427700826/http2.o
                0x9d02c644                HTTPGetArg

.text._ARPDeleteResources
                0x9d02c714       0xd0
 .text._ARPDeleteResources
                0x9d02c714       0xd0 build/default/production/_ext/427700826/arp.o

.text.fnv_32_hash
                0x9d02c7e4       0xd0
 .text.fnv_32_hash
                0x9d02c7e4       0xd0 build/default/production/_ext/427700826/hash_fnv.o
                0x9d02c7e4                fnv_32_hash

.text._TcpSocketInitialize
                0x9d02c8b4       0xd0
 .text._TcpSocketInitialize
                0x9d02c8b4       0xd0 build/default/production/_ext/427700826/tcp.o

.text.UDPSetOptions
                0x9d02c984       0xd0
 .text.UDPSetOptions
                0x9d02c984       0xd0 build/default/production/_ext/427700826/udp.o
                0x9d02c984                UDPSetOptions

.text.TCPIP_STACK_RegisterHandler
                0x9d02ca54       0xd0
 .text.TCPIP_STACK_RegisterHandler
                0x9d02ca54       0xd0 build/default/production/_ext/427700826/tcpip_manager.o
                0x9d02ca54                TCPIP_STACK_RegisterHandler

.text.DhcpConfigTask
                0x9d02cb24       0xd0
 .text.DhcpConfigTask
                0x9d02cb24       0xd0 build/default/production/_ext/334706090/wf_connection_profile.o
                0x9d02cb24                DhcpConfigTask

.text.OutputDeviceInfo
                0x9d02cbf4       0xd0
 .text.OutputDeviceInfo
                0x9d02cbf4       0xd0 build/default/production/_ext/334706090/wf_debug_output.o

.text.MRF24W_MACPutHeader
                0x9d02ccc4       0xd0
 .text.MRF24W_MACPutHeader
                0x9d02ccc4       0xd0 build/default/production/_ext/334706090/wf_mac_24g.o
                0x9d02ccc4                MRF24W_MACPutHeader

.text.general_exception
                0x9d02cd94       0xd0
 .text.general_exception
                0x9d02cd94       0xd0 c:/program files (x86)/microchip/xc32/v1.10/bin/../lib/gcc/pic32mx/4.5.1/../../../../pic32mx/lib/size\libpic32.a(general-exception.o)
                0x9d02cd94                _general_exception_context

.rodata         0x9d02ce68       0xd0
 .rodata        0x9d02ce68       0xd0 c:/program files (x86)/microchip/xc32/v1.10/bin/../lib/gcc/pic32mx/4.5.1/../../../../pic32mx/lib/size\libc.a(doprnt_cdnopsuxX.eo)

.text.DRV_MEDIA_WriteSetOffset
                0x9d02cf38       0xcc
 .text.DRV_MEDIA_WriteSetOffset
                0x9d02cf38       0xcc build/default/production/_ext/792872985/drv_media.o
                0x9d02cf38                DRV_MEDIA_WriteSetOffset

.text.HTTPSetMediaWriteHeader
                0x9d02d004       0xcc
 .text.HTTPSetMediaWriteHeader
                0x9d02d004       0xcc build/default/production/_ext/427700826/http2.o

.text.TCPIP_IPV4_SetPayload
                0x9d02d0d0       0xcc
 .text.TCPIP_IPV4_SetPayload
                0x9d02d0d0       0xcc build/default/production/_ext/427700826/ipv4.o
                0x9d02d0d0                TCPIP_IPV4_SetPayload

.text.MPFSInit  0x9d02d19c       0xc8
 .text.MPFSInit
                0x9d02d19c       0xc8 build/default/production/_ext/97638081/mpfs2.o
                0x9d02d19c                MPFSInit

.text.DNSRetry  0x9d02d264       0xc8
 .text.DNSRetry
                0x9d02d264       0xc8 build/default/production/_ext/427700826/dns.o

.text.DNSDiscardName
                0x9d02d32c       0xc8
 .text.DNSDiscardName
                0x9d02d32c       0xc8 build/default/production/_ext/427700826/dns.o

.text.UDPClose  0x9d02d3f4       0xc8
 .text.UDPClose
                0x9d02d3f4       0xc8 build/default/production/_ext/427700826/udp.o
                0x9d02d3f4                UDPClose

.text.UDPSetTxOffset
                0x9d02d4bc       0xc8
 .text.UDPSetTxOffset
                0x9d02d4bc       0xc8 build/default/production/_ext/427700826/udp.o
                0x9d02d4bc                UDPSetTxOffset

.text.InitNetConfig
                0x9d02d584       0xc8
 .text.InitNetConfig
                0x9d02d584       0xc8 build/default/production/_ext/427700826/tcpip_manager.o

.text.TCPIP_Helper_FormatNetBIOSName
                0x9d02d64c       0xc8
 .text.TCPIP_Helper_FormatNetBIOSName
                0x9d02d64c       0xc8 build/default/production/_ext/427700826/tcpip_helpers.o
                0x9d02d64c                TCPIP_Helper_FormatNetBIOSName

.text.OutputDemoHeader
                0x9d02d714       0xc8
 .text.OutputDemoHeader
                0x9d02d714       0xc8 build/default/production/_ext/334706090/wf_debug_output.o
                0x9d02d714                OutputDemoHeader

.text.HostInterruptRegInit
                0x9d02d7dc       0xc8
 .text.HostInterruptRegInit
                0x9d02d7dc       0xc8 build/default/production/_ext/334706090/wf_driver_com_24g.o

.text.HTTPPrintIP
                0x9d02d8a4       0xc8
 .text.HTTPPrintIP
                0x9d02d8a4       0xc8 build/default/production/_ext/1472/custom_http_app.o
                0x9d02d8a4                HTTPPrintIP

.text.CmdAddHead
                0x9d02d96c       0xc4
 .text.CmdAddHead
                0x9d02d96c       0xc4 build/default/production/_ext/365611741/system_command.o

.text._DHCPEnable
                0x9d02da30       0xc4
 .text._DHCPEnable
                0x9d02da30       0xc4 build/default/production/_ext/427700826/dhcp.o

.text.MRF24W_MACGetArray
                0x9d02daf4       0xc4
 .text.MRF24W_MACGetArray
                0x9d02daf4       0xc4 build/default/production/_ext/334706090/wf_mac_24g.o
                0x9d02daf4                MRF24W_MACGetArray

.text.SYS_TICK_Initialize
                0x9d02dbb8       0xc0
 .text.SYS_TICK_Initialize
                0x9d02dbb8       0xc0 build/default/production/_ext/365611741/system_services.o
                0x9d02dbb8                SYS_TICK_Initialize

.text.LowLevel_CPGetElement
                0x9d02dc78       0xc0
 .text.LowLevel_CPGetElement
                0x9d02dc78       0xc0 build/default/production/_ext/334706090/wf_connection_profile.o

.text.ProcessMgmtRxMsg
                0x9d02dd38       0xc0
 .text.ProcessMgmtRxMsg
                0x9d02dd38       0xc0 build/default/production/_ext/334706090/wf_driver_com_24g.o

.text.SYS_INT_DynamicRegister
                0x9d02ddf8       0xbc
 .text.SYS_INT_DynamicRegister
                0x9d02ddf8       0xbc build/default/production/_ext/365611741/system_services.o
                0x9d02ddf8                SYS_INT_DynamicRegister

.text._SYS_COMMAND_INIT
                0x9d02deb4       0xbc
 .text._SYS_COMMAND_INIT
                0x9d02deb4       0xbc build/default/production/_ext/365611741/system_command.o
                0x9d02deb4                _SYS_COMMAND_INIT

.text.MPFSGetEndAddr
                0x9d02df70       0xbc
 .text.MPFSGetEndAddr
                0x9d02df70       0xbc build/default/production/_ext/97638081/mpfs2.o
                0x9d02df70                MPFSGetEndAddr

.text._ARPRemoveEntry
                0x9d02e02c       0xbc
 .text._ARPRemoveEntry
                0x9d02e02c       0xbc build/default/production/_ext/427700826/arp.o

.text.OAHashRemoveAll
                0x9d02e0e8       0xbc
 .text.OAHashRemoveAll
                0x9d02e0e8       0xbc build/default/production/_ext/427700826/hash_tbl.o
                0x9d02e0e8                OAHashRemoveAll

.text.UDPDiscardNet
                0x9d02e1a4       0xbc
 .text.UDPDiscardNet
                0x9d02e1a4       0xbc build/default/production/_ext/427700826/udp.o
                0x9d02e1a4                UDPDiscardNet

.text.TCPIP_Helper_StringToPowerMode
                0x9d02e260       0xbc
 .text.TCPIP_Helper_StringToPowerMode
                0x9d02e260       0xbc build/default/production/_ext/427700826/tcpip_helpers.o
                0x9d02e260                TCPIP_Helper_StringToPowerMode

.text.LowLevel_CAGetElement
                0x9d02e31c       0xbc
 .text.LowLevel_CAGetElement
                0x9d02e31c       0xbc build/default/production/_ext/334706090/wf_connection_algorithm.o

.text.MRF24W_MACEventSetNotifyHandler
                0x9d02e3d8       0xbc
 .text.MRF24W_MACEventSetNotifyHandler
                0x9d02e3d8       0xbc build/default/production/_ext/334706090/mrf24w_events.o
                0x9d02e3d8                MRF24W_MACEventSetNotifyHandler

.text.OutputMacAddress
                0x9d02e494       0xbc
 .text.OutputMacAddress
                0x9d02e494       0xbc build/default/production/_ext/334706090/wf_debug_output.o

.text._SYS_DEBUG_INIT
                0x9d02e550       0xb8
 .text._SYS_DEBUG_INIT
                0x9d02e550       0xb8 build/default/production/_ext/365611741/system_debug.o
                0x9d02e550                _SYS_DEBUG_INIT

.text._SYS_CONSOLE_INIT
                0x9d02e608       0xb8
 .text._SYS_CONSOLE_INIT
                0x9d02e608       0xb8 build/default/production/_ext/365611741/system_debug.o
                0x9d02e608                _SYS_CONSOLE_INIT

.text.XEEInit   0x9d02e6c0       0xb8
 .text.XEEInit  0x9d02e6c0       0xb8 build/default/production/_ext/792872985/spi_eeprom.o
                0x9d02e6c0                XEEInit

.text.TCPv4AllocateTxPacketStruct
                0x9d02e778       0xb8
 .text.TCPv4AllocateTxPacketStruct
                0x9d02e778       0xb8 build/default/production/_ext/427700826/tcp.o

.text._TCPIsGetReady
                0x9d02e830       0xb8
 .text._TCPIsGetReady
                0x9d02e830       0xb8 build/default/production/_ext/427700826/tcp.o

.text.UDPGetTxCount
                0x9d02e8e8       0xb8
 .text.UDPGetTxCount
                0x9d02e8e8       0xb8 build/default/production/_ext/427700826/udp.o
                0x9d02e8e8                UDPGetTxCount

.text.OutputScanType
                0x9d02e9a0       0xb8
 .text.OutputScanType
                0x9d02e9a0       0xb8 build/default/production/_ext/334706090/wf_debug_output.o

.text.RawGetByte
                0x9d02ea58       0xb8
 .text.RawGetByte
                0x9d02ea58       0xb8 build/default/production/_ext/334706090/wf_driver_raw_24g.o
                0x9d02ea58                RawGetByte

.text.RawSetByte
                0x9d02eb10       0xb8
 .text.RawSetByte
                0x9d02eb10       0xb8 build/default/production/_ext/334706090/wf_driver_raw_24g.o
                0x9d02eb10                RawSetByte

.text.MPFSGetFlags
                0x9d02ebc8       0xb4
 .text.MPFSGetFlags
                0x9d02ebc8       0xb4 build/default/production/_ext/97638081/mpfs2.o
                0x9d02ebc8                MPFSGetFlags

.text.MPFSGetSize
                0x9d02ec7c       0xb4
 .text.MPFSGetSize
                0x9d02ec7c       0xb4 build/default/production/_ext/97638081/mpfs2.o
                0x9d02ec7c                MPFSGetSize

.text.MPFSGetStartAddr
                0x9d02ed30       0xb4
 .text.MPFSGetStartAddr
                0x9d02ed30       0xb4 build/default/production/_ext/97638081/mpfs2.o
                0x9d02ed30                MPFSGetStartAddr

.text._TcpMac2RamCopy
                0x9d02ede4       0xb4
 .text._TcpMac2RamCopy
                0x9d02ede4       0xb4 build/default/production/_ext/427700826/tcp.o

.text.UDPv4AllocateTxPacketStruct
                0x9d02ee98       0xb4
 .text.UDPv4AllocateTxPacketStruct
                0x9d02ee98       0xb4 build/default/production/_ext/427700826/udp.o

.text.UDPIsTxPutReady
                0x9d02ef4c       0xb4
 .text.UDPIsTxPutReady
                0x9d02ef4c       0xb4 build/default/production/_ext/427700826/udp.o
                0x9d02ef4c                UDPIsTxPutReady

.text.WF_SsidSet
                0x9d02f000       0xb4
 .text.WF_SsidSet
                0x9d02f000       0xb4 build/default/production/_ext/334706090/wf_connection_profile.o
                0x9d02f000                WF_SsidSet

.text.MRF24W_MACEventInit
                0x9d02f0b4       0xb4
 .text.MRF24W_MACEventInit
                0x9d02f0b4       0xb4 build/default/production/_ext/334706090/mrf24w_events.o
                0x9d02f0b4                MRF24W_MACEventInit

.text._mon_putc
                0x9d02f168       0xb4
 .text._mon_putc
                0x9d02f168       0xb4 c:/program files (x86)/microchip/xc32/v1.10/bin/../lib/gcc/pic32mx/4.5.1/../../../../pic32mx/lib/size\libpic32.a(_mon_putc.o)
                0x9d02f168                _mon_putc

.text.CommandQuit
                0x9d02f21c       0xb0
 .text.CommandQuit
                0x9d02f21c       0xb0 build/default/production/_ext/365611741/system_command.o

.text.CmdRemoveTail
                0x9d02f2cc       0xb0
 .text.CmdRemoveTail
                0x9d02f2cc       0xb0 build/default/production/_ext/365611741/system_command.o

.text.Delay10us
                0x9d02f37c       0xb0
 .text.Delay10us
                0x9d02f37c       0xb0 build/default/production/_ext/792872985/lcd.o
                0x9d02f37c                Delay10us

.text.TCPIP_ANNOUNCE_DeInit
                0x9d02f42c       0xb0
 .text.TCPIP_ANNOUNCE_DeInit
                0x9d02f42c       0xb0 build/default/production/_ext/427700826/tcpip_announce.o
                0x9d02f42c                TCPIP_ANNOUNCE_DeInit

.text._ARPRemoveCacheEntries
                0x9d02f4dc       0xb0
 .text._ARPRemoveCacheEntries
                0x9d02f4dc       0xb0 build/default/production/_ext/427700826/arp.o

.text._ARPNotifyClients
                0x9d02f58c       0xb0
 .text._ARPNotifyClients
                0x9d02f58c       0xb0 build/default/production/_ext/427700826/arp.o

.text._Tcpv4AckFnc
                0x9d02f63c       0xb0
 .text._Tcpv4AckFnc
                0x9d02f63c       0xb0 build/default/production/_ext/427700826/tcp.o

.text._TCPIPStackSetNetAddress
                0x9d02f6ec       0xb0
 .text._TCPIPStackSetNetAddress
                0x9d02f6ec       0xb0 build/default/production/_ext/427700826/tcpip_manager.o
                0x9d02f6ec                _TCPIPStackSetNetAddress

.text._TCPIPStackIsBcastAddress
                0x9d02f79c       0xb0
 .text._TCPIPStackIsBcastAddress
                0x9d02f79c       0xb0 build/default/production/_ext/427700826/tcpip_manager.o
                0x9d02f79c                _TCPIPStackIsBcastAddress

.text.HostInterrupt2RegInit
                0x9d02f84c       0xb0
 .text.HostInterrupt2RegInit
                0x9d02f84c       0xb0 build/default/production/_ext/334706090/wf_driver_com_24g.o

.rodata         0x9d02f8fc       0xac
 .rodata        0x9d02f8fc       0xac build/default/production/_ext/427700826/tcp.o

.text.TCPIsConnected
                0x9d02f9a8       0xac
 .text.TCPIsConnected
                0x9d02f9a8       0xac build/default/production/_ext/427700826/tcp.o
                0x9d02f9a8                TCPIsConnected

.text.HTTPPrint_cookiename
                0x9d02fa54       0xac
 .text.HTTPPrint_cookiename
                0x9d02fa54       0xac build/default/production/_ext/1472/custom_http_app.o
                0x9d02fa54                HTTPPrint_cookiename

.text._SYS_ERROR
                0x9d02fb00       0xa8
 .text._SYS_ERROR
                0x9d02fb00       0xa8 build/default/production/_ext/365611741/system_debug.o
                0x9d02fb00                _SYS_ERROR

.text.ARPDeinitialize
                0x9d02fba8       0xa8
 .text.ARPDeinitialize
                0x9d02fba8       0xa8 build/default/production/_ext/427700826/arp.o
                0x9d02fba8                ARPDeinitialize

.text._TCPIPStackStringToMACId
                0x9d02fc50       0xa8
 .text._TCPIPStackStringToMACId
                0x9d02fc50       0xa8 build/default/production/_ext/427700826/tcpip_manager.o
                0x9d02fc50                _TCPIPStackStringToMACId

.text.WFConfigureLowPowerMode
                0x9d02fcf8       0xa8
 .text.WFConfigureLowPowerMode
                0x9d02fcf8       0xa8 build/default/production/_ext/334706090/wf_power_save.o
                0x9d02fcf8                WFConfigureLowPowerMode

.text.WF_OutputConnectionDebugMsg
                0x9d02fda0       0xa8
 .text.WF_OutputConnectionDebugMsg
                0x9d02fda0       0xa8 build/default/production/_ext/334706090/wf_debug_output.o
                0x9d02fda0                WF_OutputConnectionDebugMsg

.text           0x9d02fe48       0xa8
 .text          0x9d02fe48       0xa8 c:/program files (x86)/microchip/xc32/v1.10/bin/../lib/gcc/pic32mx/4.5.1/../../../../pic32mx/lib/size\libpic32.a(memset.o)
                0x9d02fe48                memset

.text._Validate
                0x9d02fef0       0xa4
 .text._Validate
                0x9d02fef0       0xa4 build/default/production/_ext/97638081/mpfs2.o

.text.XEEWriteArray
                0x9d02ff94       0xa4
 .text.XEEWriteArray
                0x9d02ff94       0xa4 build/default/production/_ext/792872985/spi_eeprom.o
                0x9d02ff94                XEEWriteArray

.text.DNSResolve
                0x9d030038       0xa4
 .text.DNSResolve
                0x9d030038       0xa4 build/default/production/_ext/427700826/dns.o
                0x9d030038                DNSResolve

.text._ICMPAllocateTxPacketStruct
                0x9d0300dc       0xa4
 .text._ICMPAllocateTxPacketStruct
                0x9d0300dc       0xa4 build/default/production/_ext/427700826/icmp.o

.text.TCPIP_IPV4_DeInitialize
                0x9d030180       0xa4
 .text.TCPIP_IPV4_DeInitialize
                0x9d030180       0xa4 build/default/production/_ext/427700826/ipv4.o
                0x9d030180                TCPIP_IPV4_DeInitialize

.text._UdpSocketDcpt
                0x9d030224       0xa4
 .text._UdpSocketDcpt
                0x9d030224       0xa4 build/default/production/_ext/427700826/udp.o

.text._TCPIPStackNetByAddress
                0x9d0302c8       0xa4
 .text._TCPIPStackNetByAddress
                0x9d0302c8       0xa4 build/default/production/_ext/427700826/tcpip_manager.o
                0x9d0302c8                _TCPIPStackNetByAddress

.text.WF_ReconnectModeSet
                0x9d03036c       0xa4
 .text.WF_ReconnectModeSet
                0x9d03036c       0xa4 build/default/production/_ext/334706090/wf_connection_algorithm.o
                0x9d03036c                WF_ReconnectModeSet

.text.WF_LibInitialize
                0x9d030410       0xa4
 .text.WF_LibInitialize
                0x9d030410       0xa4 build/default/production/_ext/334706090/wf_init.o
                0x9d030410                WF_LibInitialize

.text.HTTPPrint_hellomsg
                0x9d0304b4       0xa4
 .text.HTTPPrint_hellomsg
                0x9d0304b4       0xa4 build/default/production/_ext/1472/custom_http_app.o
                0x9d0304b4                HTTPPrint_hellomsg

.text._sbrk     0x9d030558       0xa4
 .text._sbrk    0x9d030558       0xa4 c:/program files (x86)/microchip/xc32/v1.10/bin/../lib/gcc/pic32mx/4.5.1/../../../../pic32mx/lib/size\libpic32.a(sbrk.o)
                0x9d030558                _sbrk

.text.USART_GETS
                0x9d0305fc       0xa0
 .text.USART_GETS
                0x9d0305fc       0xa0 build/default/production/_ext/792872985/usart.o
                0x9d0305fc                USART_GETS

.text.XEEWrite  0x9d03069c       0xa0
 .text.XEEWrite
                0x9d03069c       0xa0 build/default/production/_ext/792872985/spi_eeprom.o
                0x9d03069c                XEEWrite

.text._DHCPDiscard
                0x9d03073c       0xa0
 .text._DHCPDiscard
                0x9d03073c       0xa0 build/default/production/_ext/427700826/dhcp.o

.text._DHCPNotifyClients
                0x9d0307dc       0xa0
 .text._DHCPNotifyClients
                0x9d0307dc       0xa0 build/default/production/_ext/427700826/dhcp.o

.text.HTTPPrint_builddate
                0x9d03087c       0xa0
 .text.HTTPPrint_builddate
                0x9d03087c       0xa0 build/default/production/_ext/1472/custom_http_app.o
                0x9d03087c                HTTPPrint_builddate

.rodata         0x9d03091c       0xa0
 .rodata        0x9d03091c       0xa0 c:/program files (x86)/microchip/xc32/v1.10/bin/../lib/gcc/pic32mx/4.5.1/../../../../pic32mx/lib/size\libmchp_peripheral_32MX795F512L.a(spi_io_tbl_libp.o)
                0x9d03091c                _SpiIoTbl

.text.strupr    0x9d0309bc       0x9c
 .text.strupr   0x9d0309bc       0x9c build/default/production/_ext/101875047/helpers.o
                0x9d0309bc                strupr

.text.MPFSDeinit
                0x9d030a58       0x9c
 .text.MPFSDeinit
                0x9d030a58       0x9c build/default/production/_ext/97638081/mpfs2.o
                0x9d030a58                MPFSDeinit

.text.ANNOUNCE_Notify
                0x9d030af4       0x9c
 .text.ANNOUNCE_Notify
                0x9d030af4       0x9c build/default/production/_ext/427700826/tcpip_announce.o

.text.DHCPRegisterHandler
                0x9d030b90       0x9c
 .text.DHCPRegisterHandler
                0x9d030b90       0x9c build/default/production/_ext/427700826/dhcp.o
                0x9d030b90                DHCPRegisterHandler

.text._TcpSocketKill
                0x9d030c2c       0x9c
 .text._TcpSocketKill
                0x9d030c2c       0x9c build/default/production/_ext/427700826/tcp.o

.text.TCPIsAvailablePort
                0x9d030cc8       0x9c
 .text.TCPIsAvailablePort
                0x9d030cc8       0x9c build/default/production/_ext/427700826/tcp.o

.text.UdpIsAvailablePort
                0x9d030d64       0x9c
 .text.UdpIsAvailablePort
                0x9d030d64       0x9c build/default/production/_ext/427700826/udp.o

.text._TCPIPStackMacIdToNet
                0x9d030e00       0x9c
 .text._TCPIPStackMacIdToNet
                0x9d030e00       0x9c build/default/production/_ext/427700826/tcpip_manager.o
                0x9d030e00                _TCPIPStackMacIdToNet

.text.SingleListRemoveHead
                0x9d030e9c       0x9c
 .text.SingleListRemoveHead
                0x9d030e9c       0x9c build/default/production/_ext/427700826/tcpip_helpers.o
                0x9d030e9c                SingleListRemoveHead

.text.SetWpsSecurity
                0x9d030f38       0x9c
 .text.SetWpsSecurity
                0x9d030f38       0x9c build/default/production/_ext/334706090/wf_connect.o

.text.WF_SpiTxRx
                0x9d030fd4       0x9c
 .text.WF_SpiTxRx
                0x9d030fd4       0x9c build/default/production/_ext/334706090/wf_spi.o
                0x9d030fd4                WF_SpiTxRx

.text.OutputIpAddress
                0x9d031070       0x9c
 .text.OutputIpAddress
                0x9d031070       0x9c build/default/production/_ext/334706090/wf_debug_output.o

.text.GetSpiPortWithBitBang
                0x9d03110c       0x9c
 .text.GetSpiPortWithBitBang
                0x9d03110c       0x9c build/default/production/_ext/334706090/wf_driver_com_24g.o

.text.HTTPPrint_ddns_status_msg
                0x9d0311a8       0x9c
 .text.HTTPPrint_ddns_status_msg
                0x9d0311a8       0x9c build/default/production/_ext/1472/custom_http_app.o
                0x9d0311a8                HTTPPrint_ddns_status_msg

.text._SYS_DEBUG_OPEN
                0x9d031244       0x98
 .text._SYS_DEBUG_OPEN
                0x9d031244       0x98 build/default/production/_ext/365611741/system_debug.o
                0x9d031244                _SYS_DEBUG_OPEN

.text._SYS_ASSERT
                0x9d0312dc       0x98
 .text._SYS_ASSERT
                0x9d0312dc       0x98 build/default/production/_ext/365611741/system_debug.o
                0x9d0312dc                _SYS_ASSERT

.text._SYS_CONSOLE_OPEN
                0x9d031374       0x98
 .text._SYS_CONSOLE_OPEN
                0x9d031374       0x98 build/default/production/_ext/365611741/system_debug.o
                0x9d031374                _SYS_CONSOLE_OPEN

.text.DelayMs   0x9d03140c       0x98
 .text.DelayMs  0x9d03140c       0x98 build/default/production/_ext/792872985/lcd.o
                0x9d03140c                DelayMs

.text.TCPIP_STACK_VerifyPktIf
                0x9d0314a4       0x98
 .text.TCPIP_STACK_VerifyPktIf
                0x9d0314a4       0x98 build/default/production/_ext/427700826/tcpip_manager.o

.text.WF_ReconnectModeGet
                0x9d03153c       0x98
 .text.WF_ReconnectModeGet
                0x9d03153c       0x98 build/default/production/_ext/334706090/wf_connection_algorithm.o
                0x9d03153c                WF_ReconnectModeGet

.text.WF_ChannelListGet
                0x9d0315d4       0x98
 .text.WF_ChannelListGet
                0x9d0315d4       0x98 build/default/production/_ext/334706090/wf_connection_algorithm.o
                0x9d0315d4                WF_ChannelListGet

.text           0x9d03166c       0x98
 .text          0x9d03166c       0x98 c:/program files (x86)/microchip/xc32/v1.10/bin/../lib/gcc/pic32mx/4.5.1/../../../../pic32mx/lib/size\libpic32.a(memcmp.o)
                0x9d03166c                memcmp

.text.HTTPHeaderParseLookup
                0x9d031704       0x94
 .text.HTTPHeaderParseLookup
                0x9d031704       0x94 build/default/production/_ext/427700826/http2.o

.text.TCPWasReset
                0x9d031798       0x94
 .text.TCPWasReset
                0x9d031798       0x94 build/default/production/_ext/427700826/tcp.o
                0x9d031798                TCPWasReset

.text.TCP_PutArray
                0x9d03182c       0x94
 .text.TCP_PutArray
                0x9d03182c       0x94 build/default/production/_ext/427700826/tcp.o

.text.SingleListAddTail
                0x9d0318c0       0x94
 .text.SingleListAddTail
                0x9d0318c0       0x94 build/default/production/_ext/427700826/tcpip_helpers.o
                0x9d0318c0                SingleListAddTail

.text.LowLevel_CPSetElement
                0x9d031954       0x94
 .text.LowLevel_CPSetElement
                0x9d031954       0x94 build/default/production/_ext/334706090/wf_connection_profile.o

.text.MRF24W_SetUserEvents
                0x9d0319e8       0x94
 .text.MRF24W_SetUserEvents
                0x9d0319e8       0x94 build/default/production/_ext/334706090/mrf24w_events.o
                0x9d0319e8                MRF24W_SetUserEvents

.text.RawMountRxBuffer
                0x9d031a7c       0x94
 .text.RawMountRxBuffer
                0x9d031a7c       0x94 build/default/production/_ext/334706090/wf_driver_raw_24g.o
                0x9d031a7c                RawMountRxBuffer

.text.MRF24W_MACCalcRxChecksum
                0x9d031b10       0x94
 .text.MRF24W_MACCalcRxChecksum
                0x9d031b10       0x94 build/default/production/_ext/334706090/wf_mac_24g.o
                0x9d031b10                MRF24W_MACCalcRxChecksum

.text.USART_PRINT
                0x9d031ba4       0x90
 .text.USART_PRINT
                0x9d031ba4       0x90 build/default/production/_ext/792872985/usart.o
                0x9d031ba4                USART_PRINT

.text._HttpCleanup
                0x9d031c34       0x90
 .text._HttpCleanup
                0x9d031c34       0x90 build/default/production/_ext/427700826/http2.o

.text.DHCPIsBound
                0x9d031cc4       0x90
 .text.DHCPIsBound
                0x9d031cc4       0x90 build/default/production/_ext/427700826/dhcp.o
                0x9d031cc4                DHCPIsBound

.text.TCPIP_IPV4_FreePacketData
                0x9d031d54       0x90
 .text.TCPIP_IPV4_FreePacketData
                0x9d031d54       0x90 build/default/production/_ext/427700826/ipv4.o
                0x9d031d54                TCPIP_IPV4_FreePacketData

.text.NBNSDeInit
                0x9d031de4       0x90
 .text.NBNSDeInit
                0x9d031de4       0x90 build/default/production/_ext/427700826/nbns.o
                0x9d031de4                NBNSDeInit

.text.TCPDiscard
                0x9d031e74       0x90
 .text.TCPDiscard
                0x9d031e74       0x90 build/default/production/_ext/427700826/tcp.o
                0x9d031e74                TCPDiscard

.text.TCP_SetPayload
                0x9d031f04       0x90
 .text.TCP_SetPayload
                0x9d031f04       0x90 build/default/production/_ext/427700826/tcp.o

.text.UDPRemoteBind
                0x9d031f94       0x90
 .text.UDPRemoteBind
                0x9d031f94       0x90 build/default/production/_ext/427700826/udp.o
                0x9d031f94                UDPRemoteBind

.text._TCPIPStackIsNetBcastAddress
                0x9d032024       0x90
 .text._TCPIPStackIsNetBcastAddress
                0x9d032024       0x90 build/default/production/_ext/427700826/tcpip_manager.o
                0x9d032024                _TCPIPStackIsNetBcastAddress

.text.OutputSsid
                0x9d0320b4       0x90
 .text.OutputSsid
                0x9d0320b4       0x90 build/default/production/_ext/334706090/wf_debug_output.o

.text.ReadWFArray
                0x9d032144       0x90
 .text.ReadWFArray
                0x9d032144       0x90 build/default/production/_ext/334706090/wf_driver_com_24g.o
                0x9d032144                ReadWFArray

.text.SendGetParamMsg
                0x9d0321d4       0x90
 .text.SendGetParamMsg
                0x9d0321d4       0x90 build/default/production/_ext/334706090/wf_param_msg_24g.o
                0x9d0321d4                SendGetParamMsg

.text.atol      0x9d032264       0x90
 .text.atol     0x9d032264       0x90 c:/program files (x86)/microchip/xc32/v1.10/bin/../lib/gcc/pic32mx/4.5.1/../../../../pic32mx/lib/size\libc.a(atol.o)
                0x9d032264                atol

.text.HTTPReadPostName
                0x9d0322f4       0x8c
 .text.HTTPReadPostName
                0x9d0322f4       0x8c build/default/production/_ext/427700826/http2.o
                0x9d0322f4                HTTPReadPostName

.text.SwapARPPacket
                0x9d032380       0x8c
 .text.SwapARPPacket
                0x9d032380       0x8c build/default/production/_ext/427700826/arp.o

.text.DHCPDisable
                0x9d03240c       0x8c
 .text.DHCPDisable
                0x9d03240c       0x8c build/default/production/_ext/427700826/dhcp.o
                0x9d03240c                DHCPDisable

.text.DNSClientInit
                0x9d032498       0x8c
 .text.DNSClientInit
                0x9d032498       0x8c build/default/production/_ext/427700826/dns.o
                0x9d032498                DNSClientInit

.text.SwapIPV4Header
                0x9d032524       0x8c
 .text.SwapIPV4Header
                0x9d032524       0x8c build/default/production/_ext/427700826/ipv4.o

.text.UDPFlush  0x9d0325b0       0x8c
 .text.UDPFlush
                0x9d0325b0       0x8c build/default/production/_ext/427700826/udp.o
                0x9d0325b0                UDPFlush

.text.LowLevel_CASetElement
                0x9d03263c       0x8c
 .text.LowLevel_CASetElement
                0x9d03263c       0x8c build/default/production/_ext/334706090/wf_connection_algorithm.o

.text.HTTPNeedsAuth
                0x9d0326c8       0x8c
 .text.HTTPNeedsAuth
                0x9d0326c8       0x8c build/default/production/_ext/1472/custom_http_app.o
                0x9d0326c8                HTTPNeedsAuth

.text.HTTPPrint_status_ok
                0x9d032754       0x8c
 .text.HTTPPrint_status_ok
                0x9d032754       0x8c build/default/production/_ext/1472/custom_http_app.o
                0x9d032754                HTTPPrint_status_ok

.text.HTTPPrint_status_fail
                0x9d0327e0       0x8c
 .text.HTTPPrint_status_fail
                0x9d0327e0       0x8c build/default/production/_ext/1472/custom_http_app.o
                0x9d0327e0                HTTPPrint_status_fail

.text.write     0x9d03286c       0x8c
 .text.write    0x9d03286c       0x8c c:/program files (x86)/microchip/xc32/v1.10/bin/../lib/gcc/pic32mx/4.5.1/../../../../pic32mx/lib/size\libpic32.a(write.o)
                0x9d03286c                write

.text.SHA1Initialize
                0x9d0328f8       0x88
 .text.SHA1Initialize
                0x9d0328f8       0x88 build/default/production/_ext/101875047/hashes.o
                0x9d0328f8                SHA1Initialize

.text._SysGetCDevEntry
                0x9d032980       0x88
 .text._SysGetCDevEntry
                0x9d032980       0x88 build/default/production/_ext/365611741/system_debug.o

.text.DHCPDeInit
                0x9d032a08       0x88
 .text.DHCPDeInit
                0x9d032a08       0x88 build/default/production/_ext/427700826/dhcp.o
                0x9d032a08                DHCPDeInit

.text.TCP_IsTxPutReady
                0x9d032a90       0x88
 .text.TCP_IsTxPutReady
                0x9d032a90       0x88 build/default/production/_ext/427700826/tcp.o

.text.TCP_PutHeader
                0x9d032b18       0x88
 .text.TCP_PutHeader
                0x9d032b18       0x88 build/default/production/_ext/427700826/tcp.o

.text._TCPIPStackIpAddToNet
                0x9d032ba0       0x88
 .text._TCPIPStackIpAddToNet
                0x9d032ba0       0x88 build/default/production/_ext/427700826/tcpip_manager.o
                0x9d032ba0                _TCPIPStackIpAddToNet

.text._TCPIPStackMACIdToString
                0x9d032c28       0x88
 .text._TCPIPStackMACIdToString
                0x9d032c28       0x88 build/default/production/_ext/427700826/tcpip_manager.o
                0x9d032c28                _TCPIPStackMACIdToString

.text.TCPIP_STACK_NetBcastAddress
                0x9d032cb0       0x88
 .text.TCPIP_STACK_NetBcastAddress
                0x9d032cb0       0x88 build/default/production/_ext/427700826/tcpip_manager.o
                0x9d032cb0                TCPIP_STACK_NetBcastAddress

.text.WF_EintInit
                0x9d032d38       0x88
 .text.WF_EintInit
                0x9d032d38       0x88 build/default/production/_ext/334706090/wf_eint.o
                0x9d032d38                WF_EintInit

.text.Read16BitWFRegister
                0x9d032dc0       0x88
 .text.Read16BitWFRegister
                0x9d032dc0       0x88 build/default/production/_ext/334706090/wf_driver_com_24g.o
                0x9d032dc0                Read16BitWFRegister

.text.Write16BitWFRegister
                0x9d032e48       0x88
 .text.Write16BitWFRegister
                0x9d032e48       0x88 build/default/production/_ext/334706090/wf_driver_com_24g.o
                0x9d032e48                Write16BitWFRegister

.text.WriteWFArray
                0x9d032ed0       0x88
 .text.WriteWFArray
                0x9d032ed0       0x88 build/default/production/_ext/334706090/wf_driver_com_24g.o
                0x9d032ed0                WriteWFArray

.text.SendSetParamMsg
                0x9d032f58       0x88
 .text.SendSetParamMsg
                0x9d032f58       0x88 build/default/production/_ext/334706090/wf_param_msg_24g.o
                0x9d032f58                SendSetParamMsg

.text.LFSRSeedRand
                0x9d032fe0       0x84
 .text.LFSRSeedRand
                0x9d032fe0       0x84 build/default/production/_ext/101875047/lfsr.o
                0x9d032fe0                LFSRSeedRand

.text._SYS_CONSOLE_PRINT
                0x9d033064       0x84
 .text._SYS_CONSOLE_PRINT
                0x9d033064       0x84 build/default/production/_ext/365611741/system_debug.o
                0x9d033064                _SYS_CONSOLE_PRINT

.text.DRV_MEDIA_ReadSetOffset
                0x9d0330e8       0x84
 .text.DRV_MEDIA_ReadSetOffset
                0x9d0330e8       0x84 build/default/production/_ext/792872985/drv_media.o
                0x9d0330e8                DRV_MEDIA_ReadSetOffset

.text.OAHashInit
                0x9d03316c       0x84
 .text.OAHashInit
                0x9d03316c       0x84 build/default/production/_ext/427700826/hash_tbl.o
                0x9d03316c                OAHashInit

.text._TCPIP_HEAP_Calloc
                0x9d0331f0       0x84
 .text._TCPIP_HEAP_Calloc
                0x9d0331f0       0x84 build/default/production/_ext/427700826/tcpip_heap_alloc.o
                0x9d0331f0                _TCPIP_HEAP_Calloc

.text.TcpipStackFindModuleData
                0x9d033274       0x84
 .text.TcpipStackFindModuleData
                0x9d033274       0x84 build/default/production/_ext/427700826/tcpip_manager.o

.text.TcpipStackFindMacModule
                0x9d0332f8       0x84
 .text.TcpipStackFindMacModule
                0x9d0332f8       0x84 build/default/production/_ext/427700826/tcpip_manager.o

.text.mrf24w_MACPowerMode
                0x9d03337c       0x84
 .text.mrf24w_MACPowerMode
                0x9d03337c       0x84 build/default/production/_ext/334706090/mrf24w_mac_pic32.o

.text.MRF24W_ISR
                0x9d033400       0x84
 .text.MRF24W_ISR
                0x9d033400       0x84 build/default/production/_ext/334706090/mrf24w_events.o
                0x9d033400                MRF24W_ISR

.rodata         0x9d033484       0x84
 .rodata        0x9d033484       0x84 build/default/production/_ext/334706090/wf_driver_raw_24g.o
                0x9d0334c4                g_RawAccessOutOfBoundsMask

.text.HTTPCheckAuth
                0x9d033508       0x84
 .text.HTTPCheckAuth
                0x9d033508       0x84 build/default/production/_ext/1472/custom_http_app.o
                0x9d033508                HTTPCheckAuth

.text.atoi      0x9d03358c       0x84
 .text.atoi     0x9d03358c       0x84 c:/program files (x86)/microchip/xc32/v1.10/bin/../lib/gcc/pic32mx/4.5.1/../../../../pic32mx/lib/size\libc.a(atoi.o)
                0x9d03358c                atoi

.text.TCPIP_IPV4_FlushDataSegments
                0x9d033610       0x80
 .text.TCPIP_IPV4_FlushDataSegments
                0x9d033610       0x80 build/default/production/_ext/427700826/ipv4.o
                0x9d033610                TCPIP_IPV4_FlushDataSegments

.text.TCPDisconnect
                0x9d033690       0x80
 .text.TCPDisconnect
                0x9d033690       0x80 build/default/production/_ext/427700826/tcp.o
                0x9d033690                TCPDisconnect

.text.TCP_IsTxReady
                0x9d033710       0x80
 .text.TCP_IsTxReady
                0x9d033710       0x80 build/default/production/_ext/427700826/tcp.o

.text.TCP_CopyTxPacketStruct
                0x9d033790       0x80
 .text.TCP_CopyTxPacketStruct
                0x9d033790       0x80 build/default/production/_ext/427700826/tcp.o

.text._Udpv4AckFnc
                0x9d033810       0x80
 .text._Udpv4AckFnc
                0x9d033810       0x80 build/default/production/_ext/427700826/udp.o

.text.SetWpaSecurity
                0x9d033890       0x80
 .text.SetWpaSecurity
                0x9d033890       0x80 build/default/production/_ext/334706090/wf_connect.o

.text.ValidateConfig
                0x9d033910       0x80
 .text.ValidateConfig
                0x9d033910       0x80 build/default/production/_ext/334706090/wf_debug_output.o
                0x9d033910                ValidateConfig

.text.ScratchMount
                0x9d033990       0x80
 .text.ScratchMount
                0x9d033990       0x80 build/default/production/_ext/334706090/wf_driver_raw_24g.o
                0x9d033990                ScratchMount

.text.ProcessNotification
                0x9d033a10       0x80
 .text.ProcessNotification
                0x9d033a10       0x80 build/default/production/_ext/1472/main_demo.o

.text._SYS_CMDIO_GET_HANDLE
                0x9d033a90       0x7c
 .text._SYS_CMDIO_GET_HANDLE
                0x9d033a90       0x7c build/default/production/_ext/365611741/system_command.o
                0x9d033a90                _SYS_CMDIO_GET_HANDLE

.text.SYS_FS_setdefdir
                0x9d033b0c       0x7c
 .text.SYS_FS_setdefdir
                0x9d033b0c       0x7c build/default/production/_ext/97638081/sys_fs.o
                0x9d033b0c                SYS_FS_setdefdir

.text.TCPFind   0x9d033b88       0x7c
 .text.TCPFind  0x9d033b88       0x7c build/default/production/_ext/427700826/tcp.o
                0x9d033b88                TCPFind

.text.TCP_Flush
                0x9d033c04       0x7c
 .text.TCP_Flush
                0x9d033c04       0x7c build/default/production/_ext/427700826/tcp.o

.text._TCPIPStackAddressServiceSelect
                0x9d033c80       0x7c
 .text._TCPIPStackAddressServiceSelect
                0x9d033c80       0x7c build/default/production/_ext/427700826/tcpip_manager.o
                0x9d033c80                _TCPIPStackAddressServiceSelect

.text.MRF24W_MACGetConfig
                0x9d033cfc       0x7c
 .text.MRF24W_MACGetConfig
                0x9d033cfc       0x7c build/default/production/_ext/334706090/mrf24w_mac_pic32.o
                0x9d033cfc                MRF24W_MACGetConfig

.text.DeallocateDataRxBuffer
                0x9d033d78       0x7c
 .text.DeallocateDataRxBuffer
                0x9d033d78       0x7c build/default/production/_ext/334706090/wf_driver_raw_24g.o
                0x9d033d78                DeallocateDataRxBuffer

.text.HTTPPrint_config_dhcpchecked
                0x9d033df4       0x7c
 .text.HTTPPrint_config_dhcpchecked
                0x9d033df4       0x7c build/default/production/_ext/1472/custom_http_app.o
                0x9d033df4                HTTPPrint_config_dhcpchecked

.text.LFSRRand  0x9d033e70       0x78
 .text.LFSRRand
                0x9d033e70       0x78 build/default/production/_ext/101875047/lfsr.o
                0x9d033e70                LFSRRand

.text.SYS_TICK_TimerSetRate
                0x9d033ee8       0x78
 .text.SYS_TICK_TimerSetRate
                0x9d033ee8       0x78 build/default/production/_ext/365611741/system_services.o
                0x9d033ee8                SYS_TICK_TimerSetRate

.text.DHCPDeRegisterHandler
                0x9d033f60       0x78
 .text.DHCPDeRegisterHandler
                0x9d033f60       0x78 build/default/production/_ext/427700826/dhcp.o
                0x9d033f60                DHCPDeRegisterHandler

.text.DNSClientDeInit
                0x9d033fd8       0x78
 .text.DNSClientDeInit
                0x9d033fd8       0x78 build/default/production/_ext/427700826/dns.o
                0x9d033fd8                DNSClientDeInit

.text.SetWepSecurity
                0x9d034050       0x78
 .text.SetWepSecurity
                0x9d034050       0x78 build/default/production/_ext/334706090/wf_connect.o

.text.ResetPll  0x9d0340c8       0x78
 .text.ResetPll
                0x9d0340c8       0x78 build/default/production/_ext/334706090/wf_driver_com_24g.o

.text.SendRAWDataFrame
                0x9d034140       0x78
 .text.SendRAWDataFrame
                0x9d034140       0x78 build/default/production/_ext/334706090/wf_driver_raw_24g.o
                0x9d034140                SendRAWDataFrame

.text.MRF24W_MACFlush
                0x9d0341b8       0x78
 .text.MRF24W_MACFlush
                0x9d0341b8       0x78 build/default/production/_ext/334706090/wf_mac_24g.o
                0x9d0341b8                MRF24W_MACFlush

.text.SoftReset
                0x9d034230       0x78
 .text.SoftReset
                0x9d034230       0x78 c:/program files (x86)/microchip/xc32/v1.10/bin/../lib/gcc/pic32mx/4.5.1/../../../../pic32mx/lib/size\libmchp_peripheral_32MX795F512L.a(soft_reset_lib.o)
                0x9d034230                SoftReset

.text.rand      0x9d0342a8       0x78
 .text.rand     0x9d0342a8       0x78 c:/program files (x86)/microchip/xc32/v1.10/bin/../lib/gcc/pic32mx/4.5.1/../../../../pic32mx/lib/size\libc.a(rand.o)
                0x9d0342a8                rand

.text.strstr    0x9d034320       0x78
 .text.strstr   0x9d034320       0x78 c:/program files (x86)/microchip/xc32/v1.10/bin/../lib/gcc/pic32mx/4.5.1/../../../../pic32mx/lib/size\libc.a(strstr.o)
                0x9d034320                strstr

.text.MD5Initialize
                0x9d034398       0x74
 .text.MD5Initialize
                0x9d034398       0x74 build/default/production/_ext/101875047/hashes.o
                0x9d034398                MD5Initialize

.text.SYS_RANDOM_ADD
                0x9d03440c       0x74
 .text.SYS_RANDOM_ADD
                0x9d03440c       0x74 build/default/production/_ext/365611741/system_random.o
                0x9d03440c                SYS_RANDOM_ADD

.text.CommandCleanup
                0x9d034480       0x74
 .text.CommandCleanup
                0x9d034480       0x74 build/default/production/_ext/365611741/system_command.o

.text.SYS_FS_IsLegalDirChar
                0x9d0344f4       0x74
 .text.SYS_FS_IsLegalDirChar
                0x9d0344f4       0x74 build/default/production/_ext/97638081/sys_fs.o
                0x9d0344f4                SYS_FS_IsLegalDirChar

.text.TCPIP_IPV4_SetTxBuffer
                0x9d034568       0x74
 .text.TCPIP_IPV4_SetTxBuffer
                0x9d034568       0x74 build/default/production/_ext/427700826/ipv4.o
                0x9d034568                TCPIP_IPV4_SetTxBuffer

.text.TCP_GetUpperLayerHeaderPtr
                0x9d0345dc       0x74
 .text.TCP_GetUpperLayerHeaderPtr
                0x9d0345dc       0x74 build/default/production/_ext/427700826/tcp.o

.text.TCP_IsPacketQueued
                0x9d034650       0x74
 .text.TCP_IsPacketQueued
                0x9d034650       0x74 build/default/production/_ext/427700826/tcp.o

.text.TCP_ResetTransmitPacketState
                0x9d0346c4       0x74
 .text.TCP_ResetTransmitPacketState
                0x9d0346c4       0x74 build/default/production/_ext/427700826/tcp.o

.text._TCPIP_HEAP_FreeDebug
                0x9d034738       0x74
 .text._TCPIP_HEAP_FreeDebug
                0x9d034738       0x74 build/default/production/_ext/427700826/tcpip_heap_alloc.o
                0x9d034738                _TCPIP_HEAP_FreeDebug

.text.UDPIsConnected
                0x9d0347ac       0x74
 .text.UDPIsConnected
                0x9d0347ac       0x74 build/default/production/_ext/427700826/udp.o
                0x9d0347ac                UDPIsConnected

.text._TCPIPStackIsAddressOfNet
                0x9d034820       0x74
 .text._TCPIPStackIsAddressOfNet
                0x9d034820       0x74 build/default/production/_ext/427700826/tcpip_manager.o
                0x9d034820                _TCPIPStackIsAddressOfNet

.text.WF_PsPollDisable
                0x9d034894       0x74
 .text.WF_PsPollDisable
                0x9d034894       0x74 build/default/production/_ext/334706090/wf_power_save.o
                0x9d034894                WF_PsPollDisable

.text.EnsureWFisAwake
                0x9d034908       0x74
 .text.EnsureWFisAwake
                0x9d034908       0x74 build/default/production/_ext/334706090/wf_power_save.o
                0x9d034908                EnsureWFisAwake

.text.RawRead   0x9d03497c       0x74
 .text.RawRead  0x9d03497c       0x74 build/default/production/_ext/334706090/wf_driver_raw_24g.o
                0x9d03497c                RawRead

.text.RawWrite  0x9d0349f0       0x74
 .text.RawWrite
                0x9d0349f0       0x74 build/default/production/_ext/334706090/wf_driver_raw_24g.o
                0x9d0349f0                RawWrite

.text.RawInit   0x9d034a64       0x74
 .text.RawInit  0x9d034a64       0x74 build/default/production/_ext/334706090/wf_mac_24g.o
                0x9d034a64                RawInit

.text.HTTPPrint_pot
                0x9d034ad8       0x74
 .text.HTTPPrint_pot
                0x9d034ad8       0x74 build/default/production/_ext/1472/custom_http_app.o
                0x9d034ad8                HTTPPrint_pot

.text.HTTPPrint_config_hostname
                0x9d034b4c       0x74
 .text.HTTPPrint_config_hostname
                0x9d034b4c       0x74 build/default/production/_ext/1472/custom_http_app.o
                0x9d034b4c                HTTPPrint_config_hostname

.text.SYS_INT_SourceRestore
                0x9d034bc0       0x70
 .text.SYS_INT_SourceRestore
                0x9d034bc0       0x70 build/default/production/_ext/365611741/system_services.o
                0x9d034bc0                SYS_INT_SourceRestore

.text._sys_CONSOLE_PRINT
                0x9d034c30       0x70
 .text._sys_CONSOLE_PRINT
                0x9d034c30       0x70 build/default/production/_ext/365611741/system_command.o

.text._ARPDeleteCache
                0x9d034ca0       0x70
 .text._ARPDeleteCache
                0x9d034ca0       0x70 build/default/production/_ext/427700826/arp.o

.text.ICMPInitialize
                0x9d034d10       0x70
 .text.ICMPInitialize
                0x9d034d10       0x70 build/default/production/_ext/427700826/icmp.o
                0x9d034d10                ICMPInitialize

.text.TCPIP_IPV4_SingleListFree
                0x9d034d80       0x70
 .text.TCPIP_IPV4_SingleListFree
                0x9d034d80       0x70 build/default/production/_ext/427700826/ipv4.o
                0x9d034d80                TCPIP_IPV4_SingleListFree

.text.NBNSInit  0x9d034df0       0x70
 .text.NBNSInit
                0x9d034df0       0x70 build/default/production/_ext/427700826/nbns.o
                0x9d034df0                NBNSInit

.text.TCPPutString
                0x9d034e60       0x70
 .text.TCPPutString
                0x9d034e60       0x70 build/default/production/_ext/427700826/tcp.o
                0x9d034e60                TCPPutString

.text.WF_Connect
                0x9d034ed0       0x70
 .text.WF_Connect
                0x9d034ed0       0x70 build/default/production/_ext/334706090/wf_connection_manager.o
                0x9d034ed0                WF_Connect

.text.MRF24W_MACOpen
                0x9d034f40       0x70
 .text.MRF24W_MACOpen
                0x9d034f40       0x70 build/default/production/_ext/334706090/mrf24w_mac_pic32.o
                0x9d034f40                MRF24W_MACOpen

.text.Write8BitWFRegister
                0x9d034fb0       0x70
 .text.Write8BitWFRegister
                0x9d034fb0       0x70 build/default/production/_ext/334706090/wf_driver_com_24g.o
                0x9d034fb0                Write8BitWFRegister

.text.HTTPPrint_config_ip
                0x9d035020       0x70
 .text.HTTPPrint_config_ip
                0x9d035020       0x70 build/default/production/_ext/1472/custom_http_app.o
                0x9d035020                HTTPPrint_config_ip

.text.HTTPPrint_config_gw
                0x9d035090       0x70
 .text.HTTPPrint_config_gw
                0x9d035090       0x70 build/default/production/_ext/1472/custom_http_app.o
                0x9d035090                HTTPPrint_config_gw

.text.HTTPPrint_config_subnet
                0x9d035100       0x70
 .text.HTTPPrint_config_subnet
                0x9d035100       0x70 build/default/production/_ext/1472/custom_http_app.o
                0x9d035100                HTTPPrint_config_subnet

.text.HTTPPrint_config_dns1
                0x9d035170       0x70
 .text.HTTPPrint_config_dns1
                0x9d035170       0x70 build/default/production/_ext/1472/custom_http_app.o
                0x9d035170                HTTPPrint_config_dns1

.text.HTTPPrint_config_dns2
                0x9d0351e0       0x70
 .text.HTTPPrint_config_dns2
                0x9d0351e0       0x70 build/default/production/_ext/1472/custom_http_app.o
                0x9d0351e0                HTTPPrint_config_dns2

.text.CommandReset
                0x9d035250       0x6c
 .text.CommandReset
                0x9d035250       0x6c build/default/production/_ext/365611741/system_command.o

.text.MPFSGetPosition
                0x9d0352bc       0x6c
 .text.MPFSGetPosition
                0x9d0352bc       0x6c build/default/production/_ext/97638081/mpfs2.o
                0x9d0352bc                MPFSGetPosition

.text._ARPRefreshEntry
                0x9d035328       0x6c
 .text._ARPRefreshEntry
                0x9d035328       0x6c build/default/production/_ext/427700826/arp.o

.text._TCPGetRxFIFOFree
                0x9d035394       0x6c
 .text._TCPGetRxFIFOFree
                0x9d035394       0x6c build/default/production/_ext/427700826/tcp.o

.text.TcpClientIpv4RemoteHash
                0x9d035400       0x6c
 .text.TcpClientIpv4RemoteHash
                0x9d035400       0x6c build/default/production/_ext/427700826/tcp.o

.text.TCPIP_HEAP_FreeSize
                0x9d03546c       0x6c
 .text.TCPIP_HEAP_FreeSize
                0x9d03546c       0x6c build/default/production/_ext/427700826/tcpip_heap_alloc.o
                0x9d03546c                TCPIP_HEAP_FreeSize

.rodata         0x9d0354d8       0x6c
 .rodata        0x9d0354d8       0x6c build/default/production/_ext/427700826/udp.o

.text.ProcessTCPIPMacGeneric
                0x9d035544       0x6c
 .text.ProcessTCPIPMacGeneric
                0x9d035544       0x6c build/default/production/_ext/427700826/tcpip_manager.o

.text.TCPIP_STACK_NetGatewayAddress
                0x9d0355b0       0x6c
 .text.TCPIP_STACK_NetGatewayAddress
                0x9d0355b0       0x6c build/default/production/_ext/427700826/tcpip_manager.o
                0x9d0355b0                TCPIP_STACK_NetGatewayAddress

.text.TCPIP_STACK_NetPriDNSAddress
                0x9d03561c       0x6c
 .text.TCPIP_STACK_NetPriDNSAddress
                0x9d03561c       0x6c build/default/production/_ext/427700826/tcpip_manager.o
                0x9d03561c                TCPIP_STACK_NetPriDNSAddress

.text.TCPIP_STACK_NetSecondDNSAddress
                0x9d035688       0x6c
 .text.TCPIP_STACK_NetSecondDNSAddress
                0x9d035688       0x6c build/default/production/_ext/427700826/tcpip_manager.o
                0x9d035688                TCPIP_STACK_NetSecondDNSAddress

.text.TCPIP_STACK_NetBIOSName
                0x9d0356f4       0x6c
 .text.TCPIP_STACK_NetBIOSName
                0x9d0356f4       0x6c build/default/production/_ext/427700826/tcpip_manager.o
                0x9d0356f4                TCPIP_STACK_NetBIOSName

.text.TCPIP_STACK_FilterRxPkt
                0x9d035760       0x6c
 .text.TCPIP_STACK_FilterRxPkt
                0x9d035760       0x6c build/default/production/_ext/427700826/tcpip_manager.o

.text.TCPIP_NotificationRemove
                0x9d0357cc       0x6c
 .text.TCPIP_NotificationRemove
                0x9d0357cc       0x6c build/default/production/_ext/427700826/tcpip_notify.o
                0x9d0357cc                TCPIP_NotificationRemove

.text.SendPowerModeMsg
                0x9d035838       0x6c
 .text.SendPowerModeMsg
                0x9d035838       0x6c build/default/production/_ext/334706090/wf_power_save.o

.text.Read8BitWFRegister
                0x9d0358a4       0x6c
 .text.Read8BitWFRegister
                0x9d0358a4       0x6c build/default/production/_ext/334706090/wf_driver_com_24g.o
                0x9d0358a4                Read8BitWFRegister

.text.MRF24W_MACInit
                0x9d035910       0x6c
 .text.MRF24W_MACInit
                0x9d035910       0x6c build/default/production/_ext/334706090/wf_mac_24g.o
                0x9d035910                MRF24W_MACInit

.text.MPFSClose
                0x9d03597c       0x68
 .text.MPFSClose
                0x9d03597c       0x68 build/default/production/_ext/97638081/mpfs2.o
                0x9d03597c                MPFSClose

.text.OAHashGetEntry
                0x9d0359e4       0x68
 .text.OAHashGetEntry
                0x9d0359e4       0x68 build/default/production/_ext/427700826/hash_tbl.o
                0x9d0359e4                OAHashGetEntry

.text.TCPIP_IPV4_FreePacket
                0x9d035a4c       0x68
 .text.TCPIP_IPV4_FreePacket
                0x9d035a4c       0x68 build/default/production/_ext/427700826/ipv4.o
                0x9d035a4c                TCPIP_IPV4_FreePacket

.text._TcpSocketBind
                0x9d035ab4       0x68
 .text._TcpSocketBind
                0x9d035ab4       0x68 build/default/production/_ext/427700826/tcp.o

.text._TcpSocketChk
                0x9d035b1c       0x68
 .text._TcpSocketChk
                0x9d035b1c       0x68 build/default/production/_ext/427700826/tcp.o

.text._TcpFlush
                0x9d035b84       0x68
 .text._TcpFlush
                0x9d035b84       0x68 build/default/production/_ext/427700826/tcp.o

.text.TCPIsGetReady
                0x9d035bec       0x68
 .text.TCPIsGetReady
                0x9d035bec       0x68 build/default/production/_ext/427700826/tcp.o
                0x9d035bec                TCPIsGetReady

.text.TCPGetRxFIFOFree
                0x9d035c54       0x68
 .text.TCPGetRxFIFOFree
                0x9d035c54       0x68 build/default/production/_ext/427700826/tcp.o
                0x9d035c54                TCPGetRxFIFOFree

.text._UdpSocketBind
                0x9d035cbc       0x68
 .text._UdpSocketBind
                0x9d035cbc       0x68 build/default/production/_ext/427700826/udp.o

.text.MACPutHeader
                0x9d035d24       0x68
 .text.MACPutHeader
                0x9d035d24       0x68 build/default/production/_ext/427700826/tcpip_mac_object.o
                0x9d035d24                MACPutHeader

.text.TCPIP_STACK_IxToNet
                0x9d035d8c       0x68
 .text.TCPIP_STACK_IxToNet
                0x9d035d8c       0x68 build/default/production/_ext/427700826/tcpip_manager.o
                0x9d035d8c                TCPIP_STACK_IxToNet

.text.TCPIP_STACK_NetName
                0x9d035df4       0x68
 .text.TCPIP_STACK_NetName
                0x9d035df4       0x68 build/default/production/_ext/427700826/tcpip_manager.o
                0x9d035df4                TCPIP_STACK_NetName

.text.TCPIP_NotificationAdd
                0x9d035e5c       0x68
 .text.TCPIP_NotificationAdd
                0x9d035e5c       0x68 build/default/production/_ext/427700826/tcpip_notify.o
                0x9d035e5c                TCPIP_NotificationAdd

.rodata         0x9d035ec4       0x68
 .rodata        0x9d035ec4       0x68 build/default/production/_ext/334706090/mrf24w_mac_pic32.o

.text.MRF24W_MACEventDeInit
                0x9d035f2c       0x68
 .text.MRF24W_MACEventDeInit
                0x9d035f2c       0x68 build/default/production/_ext/334706090/mrf24w_events.o
                0x9d035f2c                MRF24W_MACEventDeInit

.text.RawCalculateChecksum
                0x9d035f94       0x68
 .text.RawCalculateChecksum
                0x9d035f94       0x68 build/default/production/_ext/334706090/wf_driver_raw_24g.o
                0x9d035f94                RawCalculateChecksum

.text.MRF24W_MACPutArray
                0x9d035ffc       0x68
 .text.MRF24W_MACPutArray
                0x9d035ffc       0x68 build/default/production/_ext/334706090/wf_mac_24g.o
                0x9d035ffc                MRF24W_MACPutArray

.rodata         0x9d036064       0x68
 .rodata        0x9d036064       0x68 c:/program files (x86)/microchip/xc32/v1.10/bin/../lib/gcc/pic32mx/4.5.1/../../../../pic32mx/lib/size\libc.a(powersf.o)
                0x9d036064                _powers_f
                0x9d036098                _npowers_f

.text.btohexa_high
                0x9d0360cc       0x64
 .text.btohexa_high
                0x9d0360cc       0x64 build/default/production/_ext/101875047/helpers.o
                0x9d0360cc                btohexa_high

.text.btohexa_low
                0x9d036130       0x64
 .text.btohexa_low
                0x9d036130       0x64 build/default/production/_ext/101875047/helpers.o
                0x9d036130                btohexa_low

.text.DRV_MEDIA_ReadByte
                0x9d036194       0x64
 .text.DRV_MEDIA_ReadByte
                0x9d036194       0x64 build/default/production/_ext/792872985/drv_media.o
                0x9d036194                DRV_MEDIA_ReadByte

.text.DHCPIsEnabled
                0x9d0361f8       0x64
 .text.DHCPIsEnabled
                0x9d0361f8       0x64 build/default/production/_ext/427700826/dhcp.o
                0x9d0361f8                DHCPIsEnabled

.text.TCPIP_IPV4_GetDataSegmentContentsByType
                0x9d03625c       0x64
 .text.TCPIP_IPV4_GetDataSegmentContentsByType
                0x9d03625c       0x64 build/default/production/_ext/427700826/ipv4.o
                0x9d03625c                TCPIP_IPV4_GetDataSegmentContentsByType

.text.TCPSocketGetNet
                0x9d0362c0       0x64
 .text.TCPSocketGetNet
                0x9d0362c0       0x64 build/default/production/_ext/427700826/tcp.o
                0x9d0362c0                TCPSocketGetNet

.text._TCPIPStackIsNetLinked
                0x9d036324       0x64
 .text._TCPIPStackIsNetLinked
                0x9d036324       0x64 build/default/production/_ext/427700826/tcpip_manager.o
                0x9d036324                _TCPIPStackIsNetLinked

.text.TCPIP_NotificationRemoveAll
                0x9d036388       0x64
 .text.TCPIP_NotificationRemoveAll
                0x9d036388       0x64 build/default/production/_ext/427700826/tcpip_notify.o
                0x9d036388                TCPIP_NotificationRemoveAll

.text.WF_CPCreate
                0x9d0363ec       0x64
 .text.WF_CPCreate
                0x9d0363ec       0x64 build/default/production/_ext/334706090/wf_connection_profile.o
                0x9d0363ec                WF_CPCreate

.text.MRF24W_MACEventSetNotifyEvents
                0x9d036450       0x64
 .text.MRF24W_MACEventSetNotifyEvents
                0x9d036450       0x64 build/default/production/_ext/334706090/mrf24w_events.o
                0x9d036450                MRF24W_MACEventSetNotifyEvents

.text._sprintf_cdnopsuxX
                0x9d0364b4       0x64
 .text._sprintf_cdnopsuxX
                0x9d0364b4       0x64 c:/program files (x86)/microchip/xc32/v1.10/bin/../lib/gcc/pic32mx/4.5.1/../../../../pic32mx/lib/size\libc.a(sprintf_cdnopsuxX.eo)
                0x9d0364b4                _sprintf_cdnopuxX
                0x9d0364b4                _sprintf_cdnopsuxX

.text.SYS_DRIVERS_Initialize
                0x9d036518       0x60
 .text.SYS_DRIVERS_Initialize
                0x9d036518       0x60 build/default/production/_ext/365611741/system_services.o
                0x9d036518                SYS_DRIVERS_Initialize

.text.USART_PUTC
                0x9d036578       0x60
 .text.USART_PUTC
                0x9d036578       0x60 build/default/production/_ext/792872985/usart.o
                0x9d036578                USART_PUTC

.text.HTTPReleaseMedia
                0x9d0365d8       0x60
 .text.HTTPReleaseMedia
                0x9d0365d8       0x60 build/default/production/_ext/427700826/http2.o

.text.ICMPDeinitialize
                0x9d036638       0x60
 .text.ICMPDeinitialize
                0x9d036638       0x60 build/default/production/_ext/427700826/icmp.o
                0x9d036638                ICMPDeinitialize

.text.TCPIP_IPV4_SetRxBuffer
                0x9d036698       0x60
 .text.TCPIP_IPV4_SetRxBuffer
                0x9d036698       0x60 build/default/production/_ext/427700826/ipv4.o
                0x9d036698                TCPIP_IPV4_SetRxBuffer

.text.TCP_FreePacket
                0x9d0366f8       0x60
 .text.TCP_FreePacket
                0x9d0366f8       0x60 build/default/production/_ext/427700826/tcp.o

.text.MACCalcRxChecksum
                0x9d036758       0x60
 .text.MACCalcRxChecksum
                0x9d036758       0x60 build/default/production/_ext/427700826/tcpip_mac_object.o
                0x9d036758                MACCalcRxChecksum

.rodata         0x9d0367b8       0x60
 .rodata        0x9d0367b8       0x60 build/default/production/_ext/427700826/tcpip_helpers.o

.text.MRF24W_MACDeinitialize
                0x9d036818       0x60
 .text.MRF24W_MACDeinitialize
                0x9d036818       0x60 build/default/production/_ext/334706090/mrf24w_mac_pic32.o
                0x9d036818                MRF24W_MACDeinitialize

.text.mrf24w_MACSetRXHashTableEntry
                0x9d036878       0x60
 .text.mrf24w_MACSetRXHashTableEntry
                0x9d036878       0x60 build/default/production/_ext/334706090/mrf24w_mac_pic32.o

.text.WiFi_EintTask
                0x9d0368d8       0x60
 .text.WiFi_EintTask
                0x9d0368d8       0x60 build/default/production/_ext/334706090/wf_driver_com_24g.o
                0x9d0368d8                WiFi_EintTask

.text.HTTPPrint_rebootaddr
                0x9d036938       0x60
 .text.HTTPPrint_rebootaddr
                0x9d036938       0x60 build/default/production/_ext/1472/custom_http_app.o
                0x9d036938                HTTPPrint_rebootaddr

.text.SYS_INT_SourceDisable
                0x9d036998       0x5c
 .text.SYS_INT_SourceDisable
                0x9d036998       0x5c build/default/production/_ext/365611741/system_services.o
                0x9d036998                SYS_INT_SourceDisable

.text.SYS_INT_PrioritySet
                0x9d0369f4       0x5c
 .text.SYS_INT_PrioritySet
                0x9d0369f4       0x5c build/default/production/_ext/365611741/system_services.o
                0x9d0369f4                SYS_INT_PrioritySet

.text.SYS_INT_SubprioritySet
                0x9d036a50       0x5c
 .text.SYS_INT_SubprioritySet
                0x9d036a50       0x5c build/default/production/_ext/365611741/system_services.o
                0x9d036a50                SYS_INT_SubprioritySet

.text.MPFSGetLong
                0x9d036aac       0x5c
 .text.MPFSGetLong
                0x9d036aac       0x5c build/default/production/_ext/97638081/mpfs2.o
                0x9d036aac                MPFSGetLong

.text.USART_OPEN
                0x9d036b08       0x5c
 .text.USART_OPEN
                0x9d036b08       0x5c build/default/production/_ext/792872985/usart.o
                0x9d036b08                USART_OPEN

.text._DHCPCleanup
                0x9d036b64       0x5c
 .text._DHCPCleanup
                0x9d036b64       0x5c build/default/production/_ext/427700826/dhcp.o

.text.OAHashRemoveEntry
                0x9d036bc0       0x5c
 .text.OAHashRemoveEntry
                0x9d036bc0       0x5c build/default/production/_ext/427700826/hash_tbl.o
                0x9d036bc0                OAHashRemoveEntry

.text.TCPFlush  0x9d036c1c       0x5c
 .text.TCPFlush
                0x9d036c1c       0x5c build/default/production/_ext/427700826/tcp.o
                0x9d036c1c                TCPFlush

.text.MACGetArray
                0x9d036c78       0x5c
 .text.MACGetArray
                0x9d036c78       0x5c build/default/production/_ext/427700826/tcpip_mac_object.o
                0x9d036c78                MACGetArray

.text.MACPutArray
                0x9d036cd4       0x5c
 .text.MACPutArray
                0x9d036cd4       0x5c build/default/production/_ext/427700826/tcpip_mac_object.o
                0x9d036cd4                MACPutArray

.text.MACEventSetNotifyHandler
                0x9d036d30       0x5c
 .text.MACEventSetNotifyHandler
                0x9d036d30       0x5c build/default/production/_ext/427700826/tcpip_mac_object.o
                0x9d036d30                MACEventSetNotifyHandler

.text._TCPIPStackNetAddress
                0x9d036d8c       0x5c
 .text._TCPIPStackNetAddress
                0x9d036d8c       0x5c build/default/production/_ext/427700826/tcpip_manager.o
                0x9d036d8c                _TCPIPStackNetAddress

.text._TCPIPStackNetMask
                0x9d036de8       0x5c
 .text._TCPIPStackNetMask
                0x9d036de8       0x5c build/default/production/_ext/427700826/tcpip_manager.o
                0x9d036de8                _TCPIPStackNetMask

.text._TCPIPStackNetMacAddress
                0x9d036e44       0x5c
 .text._TCPIPStackNetMacAddress
                0x9d036e44       0x5c build/default/production/_ext/427700826/tcpip_manager.o
                0x9d036e44                _TCPIPStackNetMacAddress

.text.SetListenInterval
                0x9d036ea0       0x5c
 .text.SetListenInterval
                0x9d036ea0       0x5c build/default/production/_ext/334706090/wf_connection_algorithm.o
                0x9d036ea0                SetListenInterval

.text.SetDtimInterval
                0x9d036efc       0x5c
 .text.SetDtimInterval
                0x9d036efc       0x5c build/default/production/_ext/334706090/wf_connection_algorithm.o
                0x9d036efc                SetDtimInterval

.text.WF_SecurityWepSet
                0x9d036f58       0x5c
 .text.WF_SecurityWepSet
                0x9d036f58       0x5c build/default/production/_ext/334706090/wf_connection_profile.o
                0x9d036f58                WF_SecurityWepSet

.text.WF_SecurityWpaSet
                0x9d036fb4       0x5c
 .text.WF_SecurityWpaSet
                0x9d036fb4       0x5c build/default/production/_ext/334706090/wf_connection_profile.o
                0x9d036fb4                WF_SecurityWpaSet

.text.WF_SecurityWpsSet
                0x9d037010       0x5c
 .text.WF_SecurityWpsSet
                0x9d037010       0x5c build/default/production/_ext/334706090/wf_connection_profile.o
                0x9d037010                WF_SecurityWpsSet

.text.WF_EintIsPending
                0x9d03706c       0x5c
 .text.WF_EintIsPending
                0x9d03706c       0x5c build/default/production/_ext/334706090/wf_eint.o
                0x9d03706c                WF_EintIsPending

.text.ConfigureSpiMRF24W
                0x9d0370c8       0x5c
 .text.ConfigureSpiMRF24W
                0x9d0370c8       0x5c build/default/production/_ext/334706090/wf_spi.o

.text.mrf24w_MACPutHeader
                0x9d037124       0x5c
 .text.mrf24w_MACPutHeader
                0x9d037124       0x5c build/default/production/_ext/334706090/mrf24w_mac_pic32.o

.text.SignalWiFiConnectionChanged
                0x9d037180       0x5c
 .text.SignalWiFiConnectionChanged
                0x9d037180       0x5c build/default/production/_ext/334706090/wf_driver_com_24g.o
                0x9d037180                SignalWiFiConnectionChanged

.text.WF_StartGratuitousArp
                0x9d0371dc       0x5c
 .text.WF_StartGratuitousArp
                0x9d0371dc       0x5c build/default/production/_ext/334706090/wf_mac_24g.o
                0x9d0371dc                WF_StartGratuitousArp

.text.MRF24W_MACIsTxReady
                0x9d037238       0x5c
 .text.MRF24W_MACIsTxReady
                0x9d037238       0x5c build/default/production/_ext/334706090/wf_mac_24g.o
                0x9d037238                MRF24W_MACIsTxReady

.text.SYS_INT_SourceEnable
                0x9d037294       0x58
 .text.SYS_INT_SourceEnable
                0x9d037294       0x58 build/default/production/_ext/365611741/system_services.o
                0x9d037294                SYS_INT_SourceEnable

.text.USART_GETC
                0x9d0372ec       0x58
 .text.USART_GETC
                0x9d0372ec       0x58 build/default/production/_ext/792872985/usart.o
                0x9d0372ec                USART_GETC

.text.LCD_ERASE
                0x9d037344       0x58
 .text.LCD_ERASE
                0x9d037344       0x58 build/default/production/_ext/792872985/lcd.o
                0x9d037344                LCD_ERASE

.text.WaitForDataByte
                0x9d03739c       0x58
 .text.WaitForDataByte
                0x9d03739c       0x58 build/default/production/_ext/792872985/drv_spi.o

.text._XEEFlashInit
                0x9d0373f4       0x58
 .text._XEEFlashInit
                0x9d0373f4       0x58 build/default/production/_ext/792872985/drv_media.o

.text.ARPHashKeyHash
                0x9d03744c       0x58
 .text.ARPHashKeyHash
                0x9d03744c       0x58 build/default/production/_ext/427700826/arp.o
                0x9d03744c                ARPHashKeyHash

.text._TcpipHeapHandleToDcpt
                0x9d0374a4       0x58
 .text._TcpipHeapHandleToDcpt
                0x9d0374a4       0x58 build/default/production/_ext/427700826/tcpip_heap_alloc.o

.text._TCPIPStackIsNetUp
                0x9d0374fc       0x58
 .text._TCPIPStackIsNetUp
                0x9d0374fc       0x58 build/default/production/_ext/427700826/tcpip_manager.o
                0x9d0374fc                _TCPIPStackIsNetUp

.text.WF_NetworkTypeSet
                0x9d037554       0x58
 .text.WF_NetworkTypeSet
                0x9d037554       0x58 build/default/production/_ext/334706090/wf_connection_profile.o
                0x9d037554                WF_NetworkTypeSet

.text.mrf24w_MACCalcRxChecksum
                0x9d0375ac       0x58
 .text.mrf24w_MACCalcRxChecksum
                0x9d0375ac       0x58 build/default/production/_ext/334706090/mrf24w_mac_pic32.o

.text.MRF24W_MACCalcIPBufferChecksum
                0x9d037604       0x58
 .text.MRF24W_MACCalcIPBufferChecksum
                0x9d037604       0x58 build/default/production/_ext/334706090/wf_mac_24g.o
                0x9d037604                MRF24W_MACCalcIPBufferChecksum

.text.HTTPPrint_ddns_status
                0x9d03765c       0x58
 .text.HTTPPrint_ddns_status
                0x9d03765c       0x58 build/default/production/_ext/1472/custom_http_app.o
                0x9d03765c                HTTPPrint_ddns_status

.text.HTTPPrint_smtps_en
                0x9d0376b4       0x58
 .text.HTTPPrint_smtps_en
                0x9d0376b4       0x58 build/default/production/_ext/1472/custom_http_app.o
                0x9d0376b4                HTTPPrint_smtps_en

.text.HTTPPrint_snmp_en
                0x9d03770c       0x58
 .text.HTTPPrint_snmp_en
                0x9d03770c       0x58 build/default/production/_ext/1472/custom_http_app.o
                0x9d03770c                HTTPPrint_snmp_en

.text.SYS_INT_SourceStatusClear
                0x9d037764       0x54
 .text.SYS_INT_SourceStatusClear
                0x9d037764       0x54 build/default/production/_ext/365611741/system_services.o
                0x9d037764                SYS_INT_SourceStatusClear

.text._SYS_CONSOLE_PUTC
                0x9d0377b8       0x54
 .text._SYS_CONSOLE_PUTC
                0x9d0377b8       0x54 build/default/production/_ext/365611741/system_debug.o
                0x9d0377b8                _SYS_CONSOLE_PUTC

.text._SYS_OUT_MESSAGE_OFFSET
                0x9d03780c       0x54
 .text._SYS_OUT_MESSAGE_OFFSET
                0x9d03780c       0x54 build/default/production/_ext/365611741/system_debug.o
                0x9d03780c                _SYS_OUT_MESSAGE_OFFSET

.text._ICMPAckPacket
                0x9d037860       0x54
 .text._ICMPAckPacket
                0x9d037860       0x54 build/default/production/_ext/427700826/icmp.o

.text._TcpDiscardTx
                0x9d0378b4       0x54
 .text._TcpDiscardTx
                0x9d0378b4       0x54 build/default/production/_ext/427700826/tcp.o

.text.TCPPut    0x9d037908       0x54
 .text.TCPPut   0x9d037908       0x54 build/default/production/_ext/427700826/tcp.o
                0x9d037908                TCPPut

.text._UdpSocketInit
                0x9d03795c       0x54
 .text._UdpSocketInit
                0x9d03795c       0x54 build/default/production/_ext/427700826/udp.o

.text.UDPPut    0x9d0379b0       0x54
 .text.UDPPut   0x9d0379b0       0x54 build/default/production/_ext/427700826/udp.o
                0x9d0379b0                UDPPut

.text.MACGetHeader
                0x9d037a04       0x54
 .text.MACGetHeader
                0x9d037a04       0x54 build/default/production/_ext/427700826/tcpip_mac_object.o
                0x9d037a04                MACGetHeader

.text.MACSetReadPtrInRx
                0x9d037a58       0x54
 .text.MACSetReadPtrInRx
                0x9d037a58       0x54 build/default/production/_ext/427700826/tcpip_mac_object.o
                0x9d037a58                MACSetReadPtrInRx

.text.MACCalcIPBufferChecksum
                0x9d037aac       0x54
 .text.MACCalcIPBufferChecksum
                0x9d037aac       0x54 build/default/production/_ext/427700826/tcpip_mac_object.o
                0x9d037aac                MACCalcIPBufferChecksum

.text.MACEventSetNotifyEvents
                0x9d037b00       0x54
 .text.MACEventSetNotifyEvents
                0x9d037b00       0x54 build/default/production/_ext/427700826/tcpip_mac_object.o
                0x9d037b00                MACEventSetNotifyEvents

.text.MACEventAck
                0x9d037b54       0x54
 .text.MACEventAck
                0x9d037b54       0x54 build/default/production/_ext/427700826/tcpip_mac_object.o
                0x9d037b54                MACEventAck

.text._TCPIPStackAddressServiceCanStart
                0x9d037ba8       0x54
 .text._TCPIPStackAddressServiceCanStart
                0x9d037ba8       0x54 build/default/production/_ext/427700826/tcpip_manager.o
                0x9d037ba8                _TCPIPStackAddressServiceCanStart

.text._TCPIPStackAddressServiceSetDefault
                0x9d037bfc       0x54
 .text._TCPIPStackAddressServiceSetDefault
                0x9d037bfc       0x54 build/default/production/_ext/427700826/tcpip_manager.o
                0x9d037bfc                _TCPIPStackAddressServiceSetDefault

.text.mrf24w_MACDeinitialize
                0x9d037c50       0x54
 .text.mrf24w_MACDeinitialize
                0x9d037c50       0x54 build/default/production/_ext/334706090/mrf24w_mac_pic32.o

.text.GratuitousArpHandler
                0x9d037ca4       0x54
 .text.GratuitousArpHandler
                0x9d037ca4       0x54 build/default/production/_ext/334706090/wf_mac_24g.o

.text.HTTPPrint_version
                0x9d037cf8       0x54
 .text.HTTPPrint_version
                0x9d037cf8       0x54 build/default/production/_ext/1472/custom_http_app.o
                0x9d037cf8                HTTPPrint_version

.rodata         0x9d037d4c       0x54
 .rodata        0x9d037d4c       0x54 c:/program files (x86)/microchip/xc32/v1.10/bin/../lib/gcc/pic32mx/4.5.1/../../../../pic32mx/lib/size\libmchp_peripheral_32MX795F512L.a(_ports_tbl_libp.o)
                0x9d037d4c                PortRegTbl

.text._vsnprintf_cdnopsuxX
                0x9d037da0       0x54
 .text._vsnprintf_cdnopsuxX
                0x9d037da0       0x54 c:/program files (x86)/microchip/xc32/v1.10/bin/../lib/gcc/pic32mx/4.5.1/../../../../pic32mx/lib/size\libc.a(vsnprintf_cdnopsuxX.eo)
                0x9d037da0                _vsnprintf_cdnopsuxX

.text.vsnprintf
                0x9d037df4       0x54
 .text.vsnprintf
                0x9d037df4       0x54 c:/program files (x86)/microchip/xc32/v1.10/bin/../lib/gcc/pic32mx/4.5.1/../../../../pic32mx/lib/size\libc.a(vsnprintf.o)
                0x9d037df4                vsnprintf

.text._SYS_CONSOLE_MESSAGE
                0x9d037e48       0x50
 .text._SYS_CONSOLE_MESSAGE
                0x9d037e48       0x50 build/default/production/_ext/365611741/system_debug.o
                0x9d037e48                _SYS_CONSOLE_MESSAGE

.text._TCPIP_AnnounceCleanup
                0x9d037e98       0x50
 .text._TCPIP_AnnounceCleanup
                0x9d037e98       0x50 build/default/production/_ext/427700826/tcpip_announce.o

.text.HTTPPrint_
                0x9d037ee8       0x50
 .text.HTTPPrint_
                0x9d037ee8       0x50 build/default/production/_ext/427700826/http2.o
                0x9d037ee8                HTTPPrint_

.text.ARPHashKeyCompare
                0x9d037f38       0x50
 .text.ARPHashKeyCompare
                0x9d037f38       0x50 build/default/production/_ext/427700826/arp.o
                0x9d037f38                ARPHashKeyCompare

.text._DNSReleaseSocket
                0x9d037f88       0x50
 .text._DNSReleaseSocket
                0x9d037f88       0x50 build/default/production/_ext/427700826/dns.o

.text.WF_SpiInit
                0x9d037fd8       0x50
 .text.WF_SpiInit
                0x9d037fd8       0x50 build/default/production/_ext/334706090/wf_spi.o
                0x9d037fd8                WF_SpiInit

.text.mrf24w_MACEventSetNotifyHandler
                0x9d038028       0x50
 .text.mrf24w_MACEventSetNotifyHandler
                0x9d038028       0x50 build/default/production/_ext/334706090/mrf24w_mac_pic32.o

.text.MRF24W_GetTrafficEvents
                0x9d038078       0x50
 .text.MRF24W_GetTrafficEvents
                0x9d038078       0x50 build/default/production/_ext/334706090/mrf24w_events.o
                0x9d038078                MRF24W_GetTrafficEvents

.text.MRF24W_GetMgmtEvents
                0x9d0380c8       0x50
 .text.MRF24W_GetMgmtEvents
                0x9d0380c8       0x50 build/default/production/_ext/334706090/mrf24w_events.o
                0x9d0380c8                MRF24W_GetMgmtEvents

.text.SignalDHCPSuccessful
                0x9d038118       0x50
 .text.SignalDHCPSuccessful
                0x9d038118       0x50 build/default/production/_ext/334706090/wf_driver_com_24g.o
                0x9d038118                SignalDHCPSuccessful

.text.InitGratuitousArp
                0x9d038168       0x50
 .text.InitGratuitousArp
                0x9d038168       0x50 build/default/production/_ext/334706090/wf_mac_24g.o
                0x9d038168                InitGratuitousArp

.text.MRF24W_MACSetWritePtr
                0x9d0381b8       0x50
 .text.MRF24W_MACSetWritePtr
                0x9d0381b8       0x50 build/default/production/_ext/334706090/wf_mac_24g.o
                0x9d0381b8                MRF24W_MACSetWritePtr

.text.MRF24W_MACSetReadPtr
                0x9d038208       0x50
 .text.MRF24W_MACSetReadPtr
                0x9d038208       0x50 build/default/production/_ext/334706090/wf_mac_24g.o
                0x9d038208                MRF24W_MACSetReadPtr

.text.MRF24W_MACSetBaseReadPtr
                0x9d038258       0x50
 .text.MRF24W_MACSetBaseReadPtr
                0x9d038258       0x50 build/default/production/_ext/334706090/wf_mac_24g.o
                0x9d038258                MRF24W_MACSetBaseReadPtr

.text.StackNotification
                0x9d0382a8       0x50
 .text.StackNotification
                0x9d0382a8       0x50 build/default/production/_ext/1472/main_demo.o

.text.DRV_SPI_Initialize
                0x9d0382f8       0x4c
 .text.DRV_SPI_Initialize
                0x9d0382f8       0x4c build/default/production/_ext/792872985/drv_spi.o
                0x9d0382f8                DRV_SPI_Initialize

.text.TCPGet    0x9d038344       0x4c
 .text.TCPGet   0x9d038344       0x4c build/default/production/_ext/427700826/tcp.o
                0x9d038344                TCPGet

.text.UDPGet    0x9d038390       0x4c
 .text.UDPGet   0x9d038390       0x4c build/default/production/_ext/427700826/udp.o
                0x9d038390                UDPGet

.text.MACSetWritePtr
                0x9d0383dc       0x4c
 .text.MACSetWritePtr
                0x9d0383dc       0x4c build/default/production/_ext/427700826/tcpip_mac_object.o
                0x9d0383dc                MACSetWritePtr

.text.MACSetReadPtr
                0x9d038428       0x4c
 .text.MACSetReadPtr
                0x9d038428       0x4c build/default/production/_ext/427700826/tcpip_mac_object.o
                0x9d038428                MACSetReadPtr

.text.MACEventGetPending
                0x9d038474       0x4c
 .text.MACEventGetPending
                0x9d038474       0x4c build/default/production/_ext/427700826/tcpip_mac_object.o
                0x9d038474                MACEventGetPending

.text.WF_ChannelListSet
                0x9d0384c0       0x4c
 .text.WF_ChannelListSet
                0x9d0384c0       0x4c build/default/production/_ext/334706090/wf_connection_algorithm.o
                0x9d0384c0                WF_ChannelListSet

.text.WF_EintEnable
                0x9d03850c       0x4c
 .text.WF_EintEnable
                0x9d03850c       0x4c build/default/production/_ext/334706090/wf_eint.o
                0x9d03850c                WF_EintEnable

.text.DhcpEventHandler
                0x9d038558       0x4c
 .text.DhcpEventHandler
                0x9d038558       0x4c build/default/production/_ext/334706090/wf_event_handler.o
                0x9d038558                DhcpEventHandler

.rodata         0x9d0385a4       0x4c
 .rodata        0x9d0385a4       0x4c build/default/production/_ext/334706090/wf_init.o

.text.mrf24w_MACPutArray
                0x9d0385f0       0x4c
 .text.mrf24w_MACPutArray
                0x9d0385f0       0x4c build/default/production/_ext/334706090/mrf24w_mac_pic32.o

.text.mrf24w_MACGetArray
                0x9d03863c       0x4c
 .text.mrf24w_MACGetArray
                0x9d03863c       0x4c build/default/production/_ext/334706090/mrf24w_mac_pic32.o

.text.MRF24W_MACEventAck
                0x9d038688       0x4c
 .text.MRF24W_MACEventAck
                0x9d038688       0x4c build/default/production/_ext/334706090/mrf24w_events.o
                0x9d038688                MRF24W_MACEventAck

.text.SendRAWManagementFrame
                0x9d0386d4       0x4c
 .text.SendRAWManagementFrame
                0x9d0386d4       0x4c build/default/production/_ext/334706090/wf_driver_raw_24g.o
                0x9d0386d4                SendRAWManagementFrame

.text.ScratchUnmount
                0x9d038720       0x4c
 .text.ScratchUnmount
                0x9d038720       0x4c build/default/production/_ext/334706090/wf_driver_raw_24g.o
                0x9d038720                ScratchUnmount

.text.MRF24W_MACSetReadPtrInRx
                0x9d03876c       0x4c
 .text.MRF24W_MACSetReadPtrInRx
                0x9d03876c       0x4c build/default/production/_ext/334706090/wf_mac_24g.o
                0x9d03876c                MRF24W_MACSetReadPtrInRx

.text.WiFiMemory_write
                0x9d0387b8       0x4c
 .text.WiFiMemory_write
                0x9d0387b8       0x4c build/default/production/_ext/334706090/wf_configData.o
                0x9d0387b8                WiFiMemory_write

.text.INTEnable
                0x9d038804       0x4c
 .text.INTEnable
                0x9d038804       0x4c c:/program files (x86)/microchip/xc32/v1.10/bin/../lib/gcc/pic32mx/4.5.1/../../../../pic32mx/lib/size\libmchp_peripheral_32MX795F512L.a(int_tbl_lib.o)
                0x9d038804                INTEnable

.text.strncat   0x9d038850       0x4c
 .text.strncat  0x9d038850       0x4c c:/program files (x86)/microchip/xc32/v1.10/bin/../lib/gcc/pic32mx/4.5.1/../../../../pic32mx/lib/size\libc.a(strncat.o)
                0x9d038850                strncat

.text           0x9d03889c       0x4c
 .text          0x9d03889c       0x4c c:/program files (x86)/microchip/xc32/v1.10/bin/../lib/gcc/pic32mx/4.5.1/size\libgcc.a(floatunsisf.o)
                0x9d03889c                __floatunsisf

.text.SYS_CLK_PeripheralClockGet
                0x9d0388e8       0x48
 .text.SYS_CLK_PeripheralClockGet
                0x9d0388e8       0x48 build/default/production/_ext/365611741/system_services.o
                0x9d0388e8                SYS_CLK_PeripheralClockGet

.text._SYS_CONSOLE_DATA_RDY
                0x9d038930       0x48
 .text._SYS_CONSOLE_DATA_RDY
                0x9d038930       0x48 build/default/production/_ext/365611741/system_debug.o
                0x9d038930                _SYS_CONSOLE_DATA_RDY

.text._SYS_CONSOLE_GETC
                0x9d038978       0x48
 .text._SYS_CONSOLE_GETC
                0x9d038978       0x48 build/default/production/_ext/365611741/system_debug.o
                0x9d038978                _SYS_CONSOLE_GETC

.text._SYS_OUT_MESSAGE_LINE
                0x9d0389c0       0x48
 .text._SYS_OUT_MESSAGE_LINE
                0x9d0389c0       0x48 build/default/production/_ext/365611741/system_debug.o
                0x9d0389c0                _SYS_OUT_MESSAGE_LINE

.rodata         0x9d038a08       0x48
 .rodata        0x9d038a08       0x48 build/default/production/_ext/97638081/sys_fs.o

.text.MPFSGetID
                0x9d038a50       0x48
 .text.MPFSGetID
                0x9d038a50       0x48 build/default/production/_ext/97638081/mpfs2.o
                0x9d038a50                MPFSGetID

.text.HTTPCurConnectionByteCountDec
                0x9d038a98       0x48
 .text.HTTPCurConnectionByteCountDec
                0x9d038a98       0x48 build/default/production/_ext/427700826/http2.o
                0x9d038a98                HTTPCurConnectionByteCountDec

.text.ARPHashKeyCopy
                0x9d038ae0       0x48
 .text.ARPHashKeyCopy
                0x9d038ae0       0x48 build/default/production/_ext/427700826/arp.o
                0x9d038ae0                ARPHashKeyCopy

.text.DNSEndUsage
                0x9d038b28       0x48
 .text.DNSEndUsage
                0x9d038b28       0x48 build/default/production/_ext/427700826/dns.o
                0x9d038b28                DNSEndUsage

.text.TCPIP_IPV4_SetSourceAddress
                0x9d038b70       0x48
 .text.TCPIP_IPV4_SetSourceAddress
                0x9d038b70       0x48 build/default/production/_ext/427700826/ipv4.o
                0x9d038b70                TCPIP_IPV4_SetSourceAddress

.text.TCPIP_STACK_NetAddress
                0x9d038bb8       0x48
 .text.TCPIP_STACK_NetAddress
                0x9d038bb8       0x48 build/default/production/_ext/427700826/tcpip_manager.o
                0x9d038bb8                TCPIP_STACK_NetAddress

.text.TCPIP_STACK_NetMask
                0x9d038c00       0x48
 .text.TCPIP_STACK_NetMask
                0x9d038c00       0x48 build/default/production/_ext/427700826/tcpip_manager.o
                0x9d038c00                TCPIP_STACK_NetMask

.text.TCPIP_STACK_NetMacAddress
                0x9d038c48       0x48
 .text.TCPIP_STACK_NetMacAddress
                0x9d038c48       0x48 build/default/production/_ext/427700826/tcpip_manager.o
                0x9d038c48                TCPIP_STACK_NetMacAddress

.text.isEventNotifyBitSet
                0x9d038c90       0x48
 .text.isEventNotifyBitSet
                0x9d038c90       0x48 build/default/production/_ext/334706090/wf_event_handler.o

.text.mrf24w_MACCalcIPBufferChecksum
                0x9d038cd8       0x48
 .text.mrf24w_MACCalcIPBufferChecksum
                0x9d038cd8       0x48 build/default/production/_ext/334706090/mrf24w_mac_pic32.o

.text.mrf24w_MACEventSetNotifyEvents
                0x9d038d20       0x48
 .text.mrf24w_MACEventSetNotifyEvents
                0x9d038d20       0x48 build/default/production/_ext/334706090/mrf24w_mac_pic32.o

.text.mrf24w_MACEventClearNotifyEvents
                0x9d038d68       0x48
 .text.mrf24w_MACEventClearNotifyEvents
                0x9d038d68       0x48 build/default/production/_ext/334706090/mrf24w_mac_pic32.o

.text.mrf24w_MACEventAck
                0x9d038db0       0x48
 .text.mrf24w_MACEventAck
                0x9d038db0       0x48 build/default/production/_ext/334706090/mrf24w_mac_pic32.o

.text.MRF24W_MACEventClearNotifyEvents
                0x9d038df8       0x48
 .text.MRF24W_MACEventClearNotifyEvents
                0x9d038df8       0x48 build/default/production/_ext/334706090/mrf24w_events.o
                0x9d038df8                MRF24W_MACEventClearNotifyEvents

.text.OutputPowerSaveMode
                0x9d038e40       0x48
 .text.OutputPowerSaveMode
                0x9d038e40       0x48 build/default/production/_ext/334706090/wf_debug_output.o

.text.WFEnableMRF24WMode
                0x9d038e88       0x48
 .text.WFEnableMRF24WMode
                0x9d038e88       0x48 build/default/production/_ext/334706090/wf_param_msg_24g.o
                0x9d038e88                WFEnableMRF24WMode

.text.strncpy   0x9d038ed0       0x48
 .text.strncpy  0x9d038ed0       0x48 c:/program files (x86)/microchip/xc32/v1.10/bin/../lib/gcc/pic32mx/4.5.1/../../../../pic32mx/lib/size\libc.a(strncpy.o)
                0x9d038ed0                strncpy

.text.sbrk      0x9d038f18       0x48
 .text.sbrk     0x9d038f18       0x48 c:/program files (x86)/microchip/xc32/v1.10/bin/../lib/gcc/pic32mx/4.5.1/../../../../pic32mx/lib/size\libpic32.a(sbrk.o)
                0x9d038f18                sbrk

.text.SYS_CLK_ClockGet
                0x9d038f60       0x44
 .text.SYS_CLK_ClockGet
                0x9d038f60       0x44 build/default/production/_ext/365611741/system_services.o
                0x9d038f60                SYS_CLK_ClockGet

.text._SYS_OUT_MESSAGE
                0x9d038fa4       0x44
 .text._SYS_OUT_MESSAGE
                0x9d038fa4       0x44 build/default/production/_ext/365611741/system_debug.o
                0x9d038fa4                _SYS_OUT_MESSAGE

.text._sys_CONSOLE_PUTC
                0x9d038fe8       0x44
 .text._sys_CONSOLE_PUTC
                0x9d038fe8       0x44 build/default/production/_ext/365611741/system_command.o

.text.USART_DATA_RDY
                0x9d03902c       0x44
 .text.USART_DATA_RDY
                0x9d03902c       0x44 build/default/production/_ext/792872985/usart.o
                0x9d03902c                USART_DATA_RDY

.text.TCPIP_IPV4_SetPacketIPProtocol
                0x9d039070       0x44
 .text.TCPIP_IPV4_SetPacketIPProtocol
                0x9d039070       0x44 build/default/production/_ext/427700826/ipv4.o
                0x9d039070                TCPIP_IPV4_SetPacketIPProtocol

.text.MACClose  0x9d0390b4       0x44
 .text.MACClose
                0x9d0390b4       0x44 build/default/production/_ext/427700826/tcpip_mac_object.o
                0x9d0390b4                MACClose

.text.MACDiscardRx
                0x9d0390f8       0x44
 .text.MACDiscardRx
                0x9d0390f8       0x44 build/default/production/_ext/427700826/tcpip_mac_object.o
                0x9d0390f8                MACDiscardRx

.text.MACIsTxReady
                0x9d03913c       0x44
 .text.MACIsTxReady
                0x9d03913c       0x44 build/default/production/_ext/427700826/tcpip_mac_object.o
                0x9d03913c                MACIsTxReady

.text.MACFlush  0x9d039180       0x44
 .text.MACFlush
                0x9d039180       0x44 build/default/production/_ext/427700826/tcpip_mac_object.o
                0x9d039180                MACFlush

.text.MACCheckLink
                0x9d0391c4       0x44
 .text.MACCheckLink
                0x9d0391c4       0x44 build/default/production/_ext/427700826/tcpip_mac_object.o
                0x9d0391c4                MACCheckLink

.text.MACGetTxBaseAddr
                0x9d039208       0x44
 .text.MACGetTxBaseAddr
                0x9d039208       0x44 build/default/production/_ext/427700826/tcpip_mac_object.o
                0x9d039208                MACGetTxBaseAddr

.text.TCPIP_STACK_NetHandle
                0x9d03924c       0x44
 .text.TCPIP_STACK_NetHandle
                0x9d03924c       0x44 build/default/production/_ext/427700826/tcpip_manager.o
                0x9d03924c                TCPIP_STACK_NetHandle

.text._TCPIPStackNetIx
                0x9d039290       0x44
 .text._TCPIPStackNetIx
                0x9d039290       0x44 build/default/production/_ext/427700826/tcpip_manager.o
                0x9d039290                _TCPIPStackNetIx

.text._TCPIPStackSetGatewayAddress
                0x9d0392d4       0x44
 .text._TCPIPStackSetGatewayAddress
                0x9d0392d4       0x44 build/default/production/_ext/427700826/tcpip_manager.o
                0x9d0392d4                _TCPIPStackSetGatewayAddress

.text._TCPIPStackSetPriDNSAddress
                0x9d039318       0x44
 .text._TCPIPStackSetPriDNSAddress
                0x9d039318       0x44 build/default/production/_ext/427700826/tcpip_manager.o
                0x9d039318                _TCPIPStackSetPriDNSAddress

.text._TCPIPStackSetSecondDNSAddress
                0x9d03935c       0x44
 .text._TCPIPStackSetSecondDNSAddress
                0x9d03935c       0x44 build/default/production/_ext/427700826/tcpip_manager.o
                0x9d03935c                _TCPIPStackSetSecondDNSAddress

.text._TCPIPStackNetToMac
                0x9d0393a0       0x44
 .text._TCPIPStackNetToMac
                0x9d0393a0       0x44 build/default/production/_ext/427700826/tcpip_manager.o
                0x9d0393a0                _TCPIPStackNetToMac

.text.SingleListInit
                0x9d0393e4       0x44
 .text.SingleListInit
                0x9d0393e4       0x44 build/default/production/_ext/427700826/tcpip_helpers.o
                0x9d0393e4                SingleListInit

.text.WF_ConnectContextGet
                0x9d039428       0x44
 .text.WF_ConnectContextGet
                0x9d039428       0x44 build/default/production/_ext/334706090/wf_connection_manager.o
                0x9d039428                WF_ConnectContextGet

.rodata         0x9d03946c       0x44
 .rodata        0x9d03946c       0x44 build/default/production/_ext/334706090/wf_connection_profile.o

.text.WF_NetworkTypeGet
                0x9d0394b0       0x44
 .text.WF_NetworkTypeGet
                0x9d0394b0       0x44 build/default/production/_ext/334706090/wf_connection_profile.o
                0x9d0394b0                WF_NetworkTypeGet

.text.WF_WepKeyTypeGet
                0x9d0394f4       0x44
 .text.WF_WepKeyTypeGet
                0x9d0394f4       0x44 build/default/production/_ext/334706090/wf_connection_profile.o
                0x9d0394f4                WF_WepKeyTypeGet

.text.mrf24w_MACGetHeader
                0x9d039538       0x44
 .text.mrf24w_MACGetHeader
                0x9d039538       0x44 build/default/production/_ext/334706090/mrf24w_mac_pic32.o

.text.mrf24w_MACSetReadPtrInRx
                0x9d03957c       0x44
 .text.mrf24w_MACSetReadPtrInRx
                0x9d03957c       0x44 build/default/production/_ext/334706090/mrf24w_mac_pic32.o

.text.WiFi_GratuitousArpTask
                0x9d0395c0       0x44
 .text.WiFi_GratuitousArpTask
                0x9d0395c0       0x44 build/default/production/_ext/334706090/wf_mac_24g.o
                0x9d0395c0                WiFi_GratuitousArpTask

.text.MRF24W_MACProcess
                0x9d039604       0x44
 .text.MRF24W_MACProcess
                0x9d039604       0x44 build/default/production/_ext/334706090/wf_mac_24g.o
                0x9d039604                MRF24W_MACProcess

.text.RawGetMgmtRxBuffer
                0x9d039648       0x44
 .text.RawGetMgmtRxBuffer
                0x9d039648       0x44 build/default/production/_ext/334706090/wf_mac_24g.o
                0x9d039648                RawGetMgmtRxBuffer

.text.WF_SetWPATimeout
                0x9d03968c       0x44
 .text.WF_SetWPATimeout
                0x9d03968c       0x44 build/default/production/_ext/334706090/wf_param_msg_24g.o
                0x9d03968c                WF_SetWPATimeout

.text.WF_SetTxMode
                0x9d0396d0       0x44
 .text.WF_SetTxMode
                0x9d0396d0       0x44 build/default/production/_ext/334706090/wf_param_msg_24g.o
                0x9d0396d0                WF_SetTxMode

.text.WF_SetTxDataConfirm
                0x9d039714       0x44
 .text.WF_SetTxDataConfirm
                0x9d039714       0x44 build/default/production/_ext/334706090/wf_param_msg_24g.o
                0x9d039714                WF_SetTxDataConfirm

.text.WiFiMemory_read
                0x9d039758       0x44
 .text.WiFiMemory_read
                0x9d039758       0x44 build/default/production/_ext/334706090/wf_configData.o
                0x9d039758                WiFiMemory_read

.text.strncmp   0x9d03979c       0x44
 .text.strncmp  0x9d03979c       0x44 c:/program files (x86)/microchip/xc32/v1.10/bin/../lib/gcc/pic32mx/4.5.1/../../../../pic32mx/lib/size\libc.a(strncmp.o)
                0x9d03979c                strncmp

.text           0x9d0397e0       0x44
 .text          0x9d0397e0       0x44 c:/program files (x86)/microchip/xc32/v1.10/bin/../lib/gcc/pic32mx/4.5.1/size\libgcc.a(_lshrdi3.o)
                0x9d0397e0                __lshrdi3

.text.XEEEndWrite
                0x9d039824       0x40
 .text.XEEEndWrite
                0x9d039824       0x40 build/default/production/_ext/792872985/spi_eeprom.o
                0x9d039824                XEEEndWrite

.text.HTTPCurConnectionPostSmSet
                0x9d039864       0x40
 .text.HTTPCurConnectionPostSmSet
                0x9d039864       0x40 build/default/production/_ext/427700826/http2.o
                0x9d039864                HTTPCurConnectionPostSmSet

.text.HTTPCurConnectionHasArgsSet
                0x9d0398a4       0x40
 .text.HTTPCurConnectionHasArgsSet
                0x9d0398a4       0x40 build/default/production/_ext/427700826/http2.o
                0x9d0398a4                HTTPCurConnectionHasArgsSet

.text.TCPIP_IPV4_Task
                0x9d0398e4       0x40
 .text.TCPIP_IPV4_Task
                0x9d0398e4       0x40 build/default/production/_ext/427700826/ipv4.o
                0x9d0398e4                TCPIP_IPV4_Task

.text.UDPResetHeader
                0x9d039924       0x40
 .text.UDPResetHeader
                0x9d039924       0x40 build/default/production/_ext/427700826/udp.o
                0x9d039924                UDPResetHeader

.text.WF_CASetEventNotificationAction
                0x9d039964       0x40
 .text.WF_CASetEventNotificationAction
                0x9d039964       0x40 build/default/production/_ext/334706090/wf_connection_algorithm.o
                0x9d039964                WF_CASetEventNotificationAction

.text.WF_SecurityOpenSet
                0x9d0399a4       0x40
 .text.WF_SecurityOpenSet
                0x9d0399a4       0x40 build/default/production/_ext/334706090/wf_connection_profile.o
                0x9d0399a4                WF_SecurityOpenSet

.text.WF_ConfigDataSave
                0x9d0399e4       0x40
 .text.WF_ConfigDataSave
                0x9d0399e4       0x40 build/default/production/_ext/334706090/wf_init.o
                0x9d0399e4                WF_ConfigDataSave

.text.MRF24W_MACConnect
                0x9d039a24       0x40
 .text.MRF24W_MACConnect
                0x9d039a24       0x40 build/default/production/_ext/334706090/mrf24w_mac_pic32.o
                0x9d039a24                MRF24W_MACConnect

.text.mrf24w_MACEventGetPending
                0x9d039a64       0x40
 .text.mrf24w_MACEventGetPending
                0x9d039a64       0x40 build/default/production/_ext/334706090/mrf24w_mac_pic32.o

.text.DeallocateMgmtRxBuffer
                0x9d039aa4       0x40
 .text.DeallocateMgmtRxBuffer
                0x9d039aa4       0x40 build/default/production/_ext/334706090/wf_driver_raw_24g.o
                0x9d039aa4                DeallocateMgmtRxBuffer

.text.MRF24W_MACDiscardRx
                0x9d039ae4       0x40
 .text.MRF24W_MACDiscardRx
                0x9d039ae4       0x40 build/default/production/_ext/334706090/wf_mac_24g.o
                0x9d039ae4                MRF24W_MACDiscardRx

.text.WF_GetTxMode
                0x9d039b24       0x40
 .text.WF_GetTxMode
                0x9d039b24       0x40 build/default/production/_ext/334706090/wf_param_msg_24g.o
                0x9d039b24                WF_GetTxMode

.text.WF_MacAddressSet
                0x9d039b64       0x40
 .text.WF_MacAddressSet
                0x9d039b64       0x40 build/default/production/_ext/334706090/wf_param_msg_24g.o
                0x9d039b64                WF_MacAddressSet

.text.WF_MacAddressGet
                0x9d039ba4       0x40
 .text.WF_MacAddressGet
                0x9d039ba4       0x40 build/default/production/_ext/334706090/wf_param_msg_24g.o
                0x9d039ba4                WF_MacAddressGet

.text.WF_RegionalDomainGet
                0x9d039be4       0x40
 .text.WF_RegionalDomainGet
                0x9d039be4       0x40 build/default/production/_ext/334706090/wf_param_msg_24g.o
                0x9d039be4                WF_RegionalDomainGet

.text.SpiChnDataRdy
                0x9d039c24       0x40
 .text.SpiChnDataRdy
                0x9d039c24       0x40 c:/program files (x86)/microchip/xc32/v1.10/bin/../lib/gcc/pic32mx/4.5.1/../../../../pic32mx/lib/size\libmchp_peripheral_32MX795F512L.a(spi_chn_data_rdy_lib.o)
                0x9d039c24                SpiChnDataRdy

.text._sys_CONSOLE_MESSAGE
                0x9d039c64       0x3c
 .text._sys_CONSOLE_MESSAGE
                0x9d039c64       0x3c build/default/production/_ext/365611741/system_command.o

.text.DRV_MEDIA_WriteFlush
                0x9d039ca0       0x3c
 .text.DRV_MEDIA_WriteFlush
                0x9d039ca0       0x3c build/default/production/_ext/792872985/drv_media.o
                0x9d039ca0                DRV_MEDIA_WriteFlush

.text.HTTPCurConnectionCallbackPosSet
                0x9d039cdc       0x3c
 .text.HTTPCurConnectionCallbackPosSet
                0x9d039cdc       0x3c build/default/production/_ext/427700826/http2.o
                0x9d039cdc                HTTPCurConnectionCallbackPosSet

.text.HTTPCurConnectionStatusSet
                0x9d039d18       0x3c
 .text.HTTPCurConnectionStatusSet
                0x9d039d18       0x3c build/default/production/_ext/427700826/http2.o
                0x9d039d18                HTTPCurConnectionStatusSet

.text._ARPDeleteClients
                0x9d039d54       0x3c
 .text._ARPDeleteClients
                0x9d039d54       0x3c build/default/production/_ext/427700826/arp.o

.text.ARPTmoHandler
                0x9d039d90       0x3c
 .text.ARPTmoHandler
                0x9d039d90       0x3c build/default/production/_ext/427700826/arp.o

.text.TCPIP_IPV4_GetUpperLayerHeaderPtr
                0x9d039dcc       0x3c
 .text.TCPIP_IPV4_GetUpperLayerHeaderPtr
                0x9d039dcc       0x3c build/default/production/_ext/427700826/ipv4.o
                0x9d039dcc                TCPIP_IPV4_GetUpperLayerHeaderPtr

.text.TCPIP_IPV4_GetPayloadLength
                0x9d039e08       0x3c
 .text.TCPIP_IPV4_GetPayloadLength
                0x9d039e08       0x3c build/default/production/_ext/427700826/ipv4.o
                0x9d039e08                TCPIP_IPV4_GetPayloadLength

.rodata         0x9d039e44       0x3c
 .rodata        0x9d039e44       0x3c build/default/production/_ext/427700826/tcpip_heap_alloc.o

.text.WifiAsyncSetEventPending
                0x9d039e80       0x3c
 .text.WifiAsyncSetEventPending
                0x9d039e80       0x3c build/default/production/_ext/334706090/wf_event_handler.o
                0x9d039e80                WifiAsyncSetEventPending

.text.mrf24w_MACSetWritePtr
                0x9d039ebc       0x3c
 .text.mrf24w_MACSetWritePtr
                0x9d039ebc       0x3c build/default/production/_ext/334706090/mrf24w_mac_pic32.o

.text.mrf24w_MACSetReadPtr
                0x9d039ef8       0x3c
 .text.mrf24w_MACSetReadPtr
                0x9d039ef8       0x3c build/default/production/_ext/334706090/mrf24w_mac_pic32.o

.text.mrf24w_MACSetBaseReadPtr
                0x9d039f34       0x3c
 .text.mrf24w_MACSetBaseReadPtr
                0x9d039f34       0x3c build/default/production/_ext/334706090/mrf24w_mac_pic32.o

.text.PORTSetPinsDigitalIn
                0x9d039f70       0x3c
 .text.PORTSetPinsDigitalIn
                0x9d039f70       0x3c c:/program files (x86)/microchip/xc32/v1.10/bin/../lib/gcc/pic32mx/4.5.1/../../../../pic32mx/lib/size\libmchp_peripheral_32MX795F512L.a(port_set_pins_digital_in_lib.o)
                0x9d039f70                PORTSetPinsDigitalIn

.text.PORTSetPinsDigitalOut
                0x9d039fac       0x3c
 .text.PORTSetPinsDigitalOut
                0x9d039fac       0x3c c:/program files (x86)/microchip/xc32/v1.10/bin/../lib/gcc/pic32mx/4.5.1/../../../../pic32mx/lib/size\libmchp_peripheral_32MX795F512L.a(port_set_pins_digital_out_lib.o)
                0x9d039fac                PORTSetPinsDigitalOut

.text           0x9d039fe8       0x38
 .text          0x9d039fe8       0x38 c:/program files (x86)/microchip/xc32/v1.10/bin/../lib/gcc/pic32mx/4.5.1/../../../../pic32mx/lib/size/crt0.o
                0x9d03a014                __crt0_exit

.text.SYS_Tasks
                0x9d03a020       0x38
 .text.SYS_Tasks
                0x9d03a020       0x38 build/default/production/_ext/365611741/system_services.o
                0x9d03a020                SYS_Tasks

.text._SYS_OUT_INIT
                0x9d03a058       0x38
 .text._SYS_OUT_INIT
                0x9d03a058       0x38 build/default/production/_ext/365611741/system_debug.o
                0x9d03a058                _SYS_OUT_INIT

.text.DRV_MEDIA_Close
                0x9d03a090       0x38
 .text.DRV_MEDIA_Close
                0x9d03a090       0x38 build/default/production/_ext/792872985/drv_media.o
                0x9d03a090                DRV_MEDIA_Close

.text._OAHashProbeStep
                0x9d03a0c8       0x38
 .text._OAHashProbeStep
                0x9d03a0c8       0x38 build/default/production/_ext/427700826/hash_tbl.o

.rodata         0x9d03a100       0x38
 .rodata        0x9d03a100       0x38 build/default/production/_ext/334706090/wf_event_handler.o

.text.RenewDhcp
                0x9d03a138       0x38
 .text.RenewDhcp
                0x9d03a138       0x38 build/default/production/_ext/334706090/wf_event_handler.o

.text.mrf24w_MACClose
                0x9d03a170       0x38
 .text.mrf24w_MACClose
                0x9d03a170       0x38 build/default/production/_ext/334706090/mrf24w_mac_pic32.o

.rodata         0x9d03a1a8       0x70
 .rodata        0x9d03a1a8       0x38 build/default/production/_ext/334706090/wf_driver_com_24g.o
 .rodata        0x9d03a1e0       0x38 build/default/production/_ext/334706090/wf_param_msg_24g.o

.text.INTSetVectorPriority
                0x9d03a218       0x38
 .text.INTSetVectorPriority
                0x9d03a218       0x38 c:/program files (x86)/microchip/xc32/v1.10/bin/../lib/gcc/pic32mx/4.5.1/../../../../pic32mx/lib/size\libmchp_peripheral_32MX795F512L.a(int_tbl_lib.o)
                0x9d03a218                INTSetVectorPriority

.text.INTSetVectorSubPriority
                0x9d03a250       0x38
 .text.INTSetVectorSubPriority
                0x9d03a250       0x38 c:/program files (x86)/microchip/xc32/v1.10/bin/../lib/gcc/pic32mx/4.5.1/../../../../pic32mx/lib/size\libmchp_peripheral_32MX795F512L.a(int_tbl_lib.o)
                0x9d03a250                INTSetVectorSubPriority

.text._sys_CONSOLE_DATA_RDY
                0x9d03a288       0x34
 .text._sys_CONSOLE_DATA_RDY
                0x9d03a288       0x34 build/default/production/_ext/365611741/system_command.o

.text._sys_CONSOLE_GETC
                0x9d03a2bc       0x34
 .text._sys_CONSOLE_GETC
                0x9d03a2bc       0x34 build/default/production/_ext/365611741/system_command.o

.text.XEEBeginWrite
                0x9d03a2f0       0x34
 .text.XEEBeginWrite
                0x9d03a2f0       0x34 build/default/production/_ext/792872985/spi_eeprom.o
                0x9d03a2f0                XEEBeginWrite

.text.DRV_MEDIA_ClientStatus
                0x9d03a324       0x34
 .text.DRV_MEDIA_ClientStatus
                0x9d03a324       0x34 build/default/production/_ext/792872985/drv_media.o
                0x9d03a324                DRV_MEDIA_ClientStatus

.text.HTTPCurConnectionFileGet
                0x9d03a358       0x34
 .text.HTTPCurConnectionFileGet
                0x9d03a358       0x34 build/default/production/_ext/427700826/http2.o
                0x9d03a358                HTTPCurConnectionFileGet

.text.HTTPCurConnectionPostSmGet
                0x9d03a38c       0x34
 .text.HTTPCurConnectionPostSmGet
                0x9d03a38c       0x34 build/default/production/_ext/427700826/http2.o
                0x9d03a38c                HTTPCurConnectionPostSmGet

.text.HTTPCurConnectionDataBufferGet
                0x9d03a3c0       0x34
 .text.HTTPCurConnectionDataBufferGet
                0x9d03a3c0       0x34 build/default/production/_ext/427700826/http2.o
                0x9d03a3c0                HTTPCurConnectionDataBufferGet

.text.HTTPCurConnectionByteCountGet
                0x9d03a3f4       0x34
 .text.HTTPCurConnectionByteCountGet
                0x9d03a3f4       0x34 build/default/production/_ext/427700826/http2.o
                0x9d03a3f4                HTTPCurConnectionByteCountGet

.text.HTTPCurConnectionSocketGet
                0x9d03a428       0x34
 .text.HTTPCurConnectionSocketGet
                0x9d03a428       0x34 build/default/production/_ext/427700826/http2.o
                0x9d03a428                HTTPCurConnectionSocketGet

.text.TCPIP_IPV4_SetDestAddress
                0x9d03a45c       0x34
 .text.TCPIP_IPV4_SetDestAddress
                0x9d03a45c       0x34 build/default/production/_ext/427700826/ipv4.o
                0x9d03a45c                TCPIP_IPV4_SetDestAddress

.text.TCPIP_IPV4_GetDestAddress
                0x9d03a490       0x34
 .text.TCPIP_IPV4_GetDestAddress
                0x9d03a490       0x34 build/default/production/_ext/427700826/ipv4.o
                0x9d03a490                TCPIP_IPV4_GetDestAddress

.text.TCPIP_IPV4_GetSourceAddress
                0x9d03a4c4       0x34
 .text.TCPIP_IPV4_GetSourceAddress
                0x9d03a4c4       0x34 build/default/production/_ext/427700826/ipv4.o
                0x9d03a4c4                TCPIP_IPV4_GetSourceAddress

.text.ProcessTCPIPMacErrorEvents
                0x9d03a4f8       0x34
 .text.ProcessTCPIPMacErrorEvents
                0x9d03a4f8       0x34 build/default/production/_ext/427700826/tcpip_manager.o

.rodata         0x9d03a52c       0x34
 .rodata        0x9d03a52c       0x34 build/default/production/_ext/334706090/wf_connect.o

.text.WF_EintIsDisabled
                0x9d03a560       0x34
 .text.WF_EintIsDisabled
                0x9d03a560       0x34 build/default/production/_ext/334706090/wf_eint.o
                0x9d03a560                WF_EintIsDisabled

.text.WF_DeInit
                0x9d03a594       0x34
 .text.WF_DeInit
                0x9d03a594       0x34 build/default/production/_ext/334706090/wf_init.o
                0x9d03a594                WF_DeInit

.text.WF_SpiDisableChipSelect
                0x9d03a5c8       0x34
 .text.WF_SpiDisableChipSelect
                0x9d03a5c8       0x34 build/default/production/_ext/334706090/wf_spi.o
                0x9d03a5c8                WF_SpiDisableChipSelect

.text.mrf24w_MACGetReadPtrInRx
                0x9d03a5fc       0x34
 .text.mrf24w_MACGetReadPtrInRx
                0x9d03a5fc       0x34 build/default/production/_ext/334706090/mrf24w_mac_pic32.o

.text.mrf24w_MACIsTxReady
                0x9d03a630       0x34
 .text.mrf24w_MACIsTxReady
                0x9d03a630       0x34 build/default/production/_ext/334706090/mrf24w_mac_pic32.o

.text.mrf24w_MACFlush
                0x9d03a664       0x34
 .text.mrf24w_MACFlush
                0x9d03a664       0x34 build/default/production/_ext/334706090/mrf24w_mac_pic32.o

.text.mrf24w_MACDiscardRx
                0x9d03a698       0x34
 .text.mrf24w_MACDiscardRx
                0x9d03a698       0x34 build/default/production/_ext/334706090/mrf24w_mac_pic32.o

.text.mrf24w_MACCheckLink
                0x9d03a6cc       0x34
 .text.mrf24w_MACCheckLink
                0x9d03a6cc       0x34 build/default/production/_ext/334706090/mrf24w_mac_pic32.o

.text.SetNetworkConfig
                0x9d03a700       0x34
 .text.SetNetworkConfig
                0x9d03a700       0x34 build/default/production/_ext/334706090/wf_mac_24g.o
                0x9d03a700                SetNetworkConfig

.rodata         0x9d03a734       0x34
 .rodata        0x9d03a734       0x34 build/default/production/_ext/334706090/wf_mgmt_msg_24g.o

.text.HTTPPrint_reboot
                0x9d03a768       0x34
 .text.HTTPPrint_reboot
                0x9d03a768       0x34 build/default/production/_ext/1472/custom_http_app.o
                0x9d03a768                HTTPPrint_reboot

.text.INTEnableSystemMultiVectoredInt
                0x9d03a79c       0x34
 .text.INTEnableSystemMultiVectoredInt
                0x9d03a79c       0x34 c:/program files (x86)/microchip/xc32/v1.10/bin/../lib/gcc/pic32mx/4.5.1/../../../../pic32mx/lib/size\libmchp_peripheral_32MX795F512L.a(int_enable_mv_int_lib.o)
                0x9d03a79c                INTEnableSystemMultiVectoredInt

.text.SYS_USERIO_Tasks
                0x9d03a7d0       0x30
 .text.SYS_USERIO_Tasks
                0x9d03a7d0       0x30 build/default/production/_ext/365611741/system_userio.o
                0x9d03a7d0                SYS_USERIO_Tasks

.text.SYS_FS_mpfs2fs_Init
                0x9d03a800       0x30
 .text.SYS_FS_mpfs2fs_Init
                0x9d03a800       0x30 build/default/production/_ext/97638081/sys_fs.o
                0x9d03a800                SYS_FS_mpfs2fs_Init

.text.TCPIP_IPV4_TmoHandler
                0x9d03a830       0x30
 .text.TCPIP_IPV4_TmoHandler
                0x9d03a830       0x30 build/default/production/_ext/427700826/ipv4.o
                0x9d03a830                TCPIP_IPV4_TmoHandler

.text._TcpTmoHandler
                0x9d03a860       0x30
 .text._TcpTmoHandler
                0x9d03a860       0x30 build/default/production/_ext/427700826/tcp.o

.text.TCPIP_STACK_TickHandler
                0x9d03a890       0x30
 .text.TCPIP_STACK_TickHandler
                0x9d03a890       0x30 build/default/production/_ext/427700826/tcpip_manager.o

.text.SetEventNotificationMask
                0x9d03a8c0       0x30
 .text.SetEventNotificationMask
                0x9d03a8c0       0x30 build/default/production/_ext/334706090/wf_connection_algorithm.o

.text.SetLogicalConnectionState
                0x9d03a8f0       0x30
 .text.SetLogicalConnectionState
                0x9d03a8f0       0x30 build/default/production/_ext/334706090/wf_connection_manager.o
                0x9d03a8f0                SetLogicalConnectionState

.text.SetAppPowerSaveMode
                0x9d03a920       0x30
 .text.SetAppPowerSaveMode
                0x9d03a920       0x30 build/default/production/_ext/334706090/wf_power_save.o
                0x9d03a920                SetAppPowerSaveMode

.text.WF_GetPowerSaveState
                0x9d03a950       0x30
 .text.WF_GetPowerSaveState
                0x9d03a950       0x30 build/default/production/_ext/334706090/wf_power_save.o
                0x9d03a950                WF_GetPowerSaveState

.text.SetPowerSaveState
                0x9d03a980       0x30
 .text.SetPowerSaveState
                0x9d03a980       0x30 build/default/production/_ext/334706090/wf_power_save.o

.text.WF_SpiEnableChipSelect
                0x9d03a9b0       0x30
 .text.WF_SpiEnableChipSelect
                0x9d03a9b0       0x30 build/default/production/_ext/334706090/wf_spi.o
                0x9d03a9b0                WF_SpiEnableChipSelect

.rodata         0x9d03a9e0       0x30
 .rodata        0x9d03a9e0       0x30 build/default/production/_ext/334706090/wf_mac_24g.o

.text.MRF24W_MACCheckLink
                0x9d03aa10       0x30
 .text.MRF24W_MACCheckLink
                0x9d03aa10       0x30 build/default/production/_ext/334706090/wf_mac_24g.o
                0x9d03aa10                MRF24W_MACCheckLink

.text.strcat    0x9d03aa40       0x30
 .text.strcat   0x9d03aa40       0x30 c:/program files (x86)/microchip/xc32/v1.10/bin/../lib/gcc/pic32mx/4.5.1/../../../../pic32mx/lib/size\libc.a(strcat.o)
                0x9d03aa40                strcat

.text.SYS_WDT_Clear
                0x9d03aa70       0x2c
 .text.SYS_WDT_Clear
                0x9d03aa70       0x2c build/default/production/_ext/365611741/system_services.o
                0x9d03aa70                SYS_WDT_Clear

.text.TCPIP_ANNOUNCE_TaskPending
                0x9d03aa9c       0x2c
 .text.TCPIP_ANNOUNCE_TaskPending
                0x9d03aa9c       0x2c build/default/production/_ext/427700826/tcpip_announce.o
                0x9d03aa9c                TCPIP_ANNOUNCE_TaskPending

.text.ARPTaskPending
                0x9d03aac8       0x2c
 .text.ARPTaskPending
                0x9d03aac8       0x2c build/default/production/_ext/427700826/arp.o
                0x9d03aac8                ARPTaskPending

.text.TCPIP_IPV4_TaskPending
                0x9d03aaf4       0x2c
 .text.TCPIP_IPV4_TaskPending
                0x9d03aaf4       0x2c build/default/production/_ext/427700826/ipv4.o
                0x9d03aaf4                TCPIP_IPV4_TaskPending

.text.TCPTaskPending
                0x9d03ab20       0x2c
 .text.TCPTaskPending
                0x9d03ab20       0x2c build/default/production/_ext/427700826/tcp.o
                0x9d03ab20                TCPTaskPending

.text.WF_EintDisable
                0x9d03ab4c       0x2c
 .text.WF_EintDisable
                0x9d03ab4c       0x2c build/default/production/_ext/334706090/wf_eint.o
                0x9d03ab4c                WF_EintDisable

.text.WiFiAsyncTaskPending
                0x9d03ab78       0x2c
 .text.WiFiAsyncTaskPending
                0x9d03ab78       0x2c build/default/production/_ext/334706090/wf_event_handler.o
                0x9d03ab78                WiFiAsyncTaskPending

.rodata         0x9d03aba4       0x2c
 .rodata        0x9d03aba4       0x2c build/default/production/_ext/334706090/wf_spi.o

.text.MRF24W_MACEventGetPending
                0x9d03abd0       0x2c
 .text.MRF24W_MACEventGetPending
                0x9d03abd0       0x2c build/default/production/_ext/334706090/mrf24w_events.o
                0x9d03abd0                MRF24W_MACEventGetPending

.text.HTTPPrint_read_comm
                0x9d03abfc       0x2c
 .text.HTTPPrint_read_comm
                0x9d03abfc       0x2c build/default/production/_ext/1472/custom_http_app.o
                0x9d03abfc                HTTPPrint_read_comm

.text.HTTPPrint_write_comm
                0x9d03ac28       0x2c
 .text.HTTPPrint_write_comm
                0x9d03ac28       0x2c build/default/production/_ext/1472/custom_http_app.o
                0x9d03ac28                HTTPPrint_write_comm

.text.HTTPPrint_ddns_service
                0x9d03ac54       0x2c
 .text.HTTPPrint_ddns_service
                0x9d03ac54       0x2c build/default/production/_ext/1472/custom_http_app.o
                0x9d03ac54                HTTPPrint_ddns_service

.text.strchr    0x9d03ac80       0x2c
 .text.strchr   0x9d03ac80       0x2c c:/program files (x86)/microchip/xc32/v1.10/bin/../lib/gcc/pic32mx/4.5.1/../../../../pic32mx/lib/size\libc.a(strchr.o)
                0x9d03ac80                strchr

.text._stub_sbd_memlayout
                0x9d03acac       0x2c
 .text._stub_sbd_memlayout
                0x9d03acac       0x2c c:/program files (x86)/microchip/xc32/v1.10/bin/../lib/gcc/pic32mx/4.5.1/../../../../pic32mx/lib/size\libpic32.a(sbrk.o)
                0x9d03acac                _stub_sbd_memlayout
                0x9d03acac                _sbd_memlayout

.text.SYS_FS_GenError
                0x9d03acd8       0x28
 .text.SYS_FS_GenError
                0x9d03acd8       0x28 build/default/production/_ext/97638081/sys_fs.o

.rodata         0x9d03ad00       0x28
 .rodata        0x9d03ad00       0x28 build/default/production/_ext/792872985/usart.o

.text.DHCPServerDisable
                0x9d03ad28       0x28
 .text.DHCPServerDisable
                0x9d03ad28       0x28 build/default/production/_ext/427700826/dhcps.o
                0x9d03ad28                DHCPServerDisable

.text.DHCPServerEnable
                0x9d03ad50       0x28
 .text.DHCPServerEnable
                0x9d03ad50       0x28 build/default/production/_ext/427700826/dhcps.o
                0x9d03ad50                DHCPServerEnable

.text.ZCLLEnable
                0x9d03ad78       0x28
 .text.ZCLLEnable
                0x9d03ad78       0x28 build/default/production/_ext/427700826/zero_conf_link_local.o
                0x9d03ad78                ZCLLEnable

.text.SetSleepNeeded
                0x9d03ada0       0x28
 .text.SetSleepNeeded
                0x9d03ada0       0x28 build/default/production/_ext/334706090/wf_power_save.o
                0x9d03ada0                SetSleepNeeded

.text.mrf24w_MACGetTxBaseAddr
                0x9d03adc8       0x28
 .text.mrf24w_MACGetTxBaseAddr
                0x9d03adc8       0x28 build/default/production/_ext/334706090/mrf24w_mac_pic32.o

.text.WF_OutputConnectionContext
                0x9d03adf0       0x28
 .text.WF_OutputConnectionContext
                0x9d03adf0       0x28 build/default/production/_ext/334706090/wf_debug_output.o
                0x9d03adf0                WF_OutputConnectionContext

.text.SetDhcpProgressState
                0x9d03ae18       0x28
 .text.SetDhcpProgressState
                0x9d03ae18       0x28 build/default/production/_ext/334706090/wf_driver_com_24g.o
                0x9d03ae18                SetDhcpProgressState

.text.SignalMgmtConfirmReceivedEvent
                0x9d03ae40       0x28
 .text.SignalMgmtConfirmReceivedEvent
                0x9d03ae40       0x28 build/default/production/_ext/334706090/wf_mgmt_msg_24g.o
                0x9d03ae40                SignalMgmtConfirmReceivedEvent

.text.INTClearFlag
                0x9d03ae68       0x28
 .text.INTClearFlag
                0x9d03ae68       0x28 c:/program files (x86)/microchip/xc32/v1.10/bin/../lib/gcc/pic32mx/4.5.1/../../../../pic32mx/lib/size\libmchp_peripheral_32MX795F512L.a(int_tbl_lib.o)
                0x9d03ae68                INTClearFlag

.text.TCPIP_STACK_GetDefaultNet
                0x9d03ae90       0x24
 .text.TCPIP_STACK_GetDefaultNet
                0x9d03ae90       0x24 build/default/production/_ext/427700826/tcpip_manager.o
                0x9d03ae90                TCPIP_STACK_GetDefaultNet

.text.TCPIP_STACK_NetworksNo
                0x9d03aeb4       0x24
 .text.TCPIP_STACK_NetworksNo
                0x9d03aeb4       0x24 build/default/production/_ext/427700826/tcpip_manager.o
                0x9d03aeb4                TCPIP_STACK_NetworksNo

.text.GetEventNotificationMask
                0x9d03aed8       0x24
 .text.GetEventNotificationMask
                0x9d03aed8       0x24 build/default/production/_ext/334706090/wf_connection_algorithm.o
                0x9d03aed8                GetEventNotificationMask

.text.WFisConnected
                0x9d03aefc       0x24
 .text.WFisConnected
                0x9d03aefc       0x24 build/default/production/_ext/334706090/wf_connection_manager.o
                0x9d03aefc                WFisConnected

.text.GetWiFiNetworkType
                0x9d03af20       0x24
 .text.GetWiFiNetworkType
                0x9d03af20       0x24 build/default/production/_ext/334706090/wf_connection_profile.o
                0x9d03af20                GetWiFiNetworkType

.text.WifiAsyncClearAllEvents
                0x9d03af44       0x24
 .text.WifiAsyncClearAllEvents
                0x9d03af44       0x24 build/default/production/_ext/334706090/wf_event_handler.o
                0x9d03af44                WifiAsyncClearAllEvents

.text.isSleepNeeded
                0x9d03af68       0x24
 .text.isSleepNeeded
                0x9d03af68       0x24 build/default/production/_ext/334706090/wf_power_save.o
                0x9d03af68                isSleepNeeded

.text.ClearSleepNeeded
                0x9d03af8c       0x24
 .text.ClearSleepNeeded
                0x9d03af8c       0x24 build/default/production/_ext/334706090/wf_power_save.o
                0x9d03af8c                ClearSleepNeeded

.text.GetAppPowerSaveMode
                0x9d03afb0       0x24
 .text.GetAppPowerSaveMode
                0x9d03afb0       0x24 build/default/production/_ext/334706090/wf_power_save.o
                0x9d03afb0                GetAppPowerSaveMode

.text.InitPowerSaveTask
                0x9d03afd4       0x24
 .text.InitPowerSaveTask
                0x9d03afd4       0x24 build/default/production/_ext/334706090/wf_driver_com_24g.o
                0x9d03afd4                InitPowerSaveTask

.text.isDhcpInProgress
                0x9d03aff8       0x24
 .text.isDhcpInProgress
                0x9d03aff8       0x24 build/default/production/_ext/334706090/wf_driver_com_24g.o

.text.GetReadPtrRawWindow
                0x9d03b01c       0x24
 .text.GetReadPtrRawWindow
                0x9d03b01c       0x24 build/default/production/_ext/334706090/wf_mac_24g.o
                0x9d03b01c                GetReadPtrRawWindow

.text.GetNetworkConfig
                0x9d03b040       0x24
 .text.GetNetworkConfig
                0x9d03b040       0x24 build/default/production/_ext/334706090/wf_mac_24g.o
                0x9d03b040                GetNetworkConfig

.text.MRF24W_MACGetReadPtrInRx
                0x9d03b064       0x24
 .text.MRF24W_MACGetReadPtrInRx
                0x9d03b064       0x24 build/default/production/_ext/334706090/wf_mac_24g.o
                0x9d03b064                MRF24W_MACGetReadPtrInRx

.text.HTTPPrint_lcdtext
                0x9d03b088       0x24
 .text.HTTPPrint_lcdtext
                0x9d03b088       0x24 build/default/production/_ext/1472/custom_http_app.o
                0x9d03b088                HTTPPrint_lcdtext

.text.HTTPPrint_ddns_user
                0x9d03b0ac       0x24
 .text.HTTPPrint_ddns_user
                0x9d03b0ac       0x24 build/default/production/_ext/1472/custom_http_app.o
                0x9d03b0ac                HTTPPrint_ddns_user

.text.HTTPPrint_ddns_pass
                0x9d03b0d0       0x24
 .text.HTTPPrint_ddns_pass
                0x9d03b0d0       0x24 build/default/production/_ext/1472/custom_http_app.o
                0x9d03b0d0                HTTPPrint_ddns_pass

.text.HTTPPrint_ddns_host
                0x9d03b0f4       0x24
 .text.HTTPPrint_ddns_host
                0x9d03b0f4       0x24 build/default/production/_ext/1472/custom_http_app.o
                0x9d03b0f4                HTTPPrint_ddns_host

.text.free      0x9d03b118       0x24
 .text.free     0x9d03b118       0x24 c:/program files (x86)/microchip/xc32/v1.10/bin/../lib/gcc/pic32mx/4.5.1/../../../../pic32mx/lib/size\libc.a(malloc.o)
                0x9d03b118                free

.text._snprintf_cdnopsuxX
                0x9d03b13c       0x24
 .text._snprintf_cdnopsuxX
                0x9d03b13c       0x24 c:/program files (x86)/microchip/xc32/v1.10/bin/../lib/gcc/pic32mx/4.5.1/../../../../pic32mx/lib/size\libc.a(snprintf_cdnopsuxX.eo)
                0x9d03b13c                _snprintf_cdnopsuxX

.text.toupper   0x9d03b160       0x24
 .text.toupper  0x9d03b160       0x24 c:/program files (x86)/microchip/xc32/v1.10/bin/../lib/gcc/pic32mx/4.5.1/../../../../pic32mx/lib/size\libc.a(ctypef.o)
                0x9d03b160                toupper

.rodata         0x9d03b184       0x20
 .rodata        0x9d03b184       0x20 build/default/production/_ext/427700826/arp.o

.text.SetEapSecurity
                0x9d03b1a4       0x20
 .text.SetEapSecurity
                0x9d03b1a4       0x20 build/default/production/_ext/334706090/wf_connect.o

.text.MRF24W_MACPowerDown
                0x9d03b1c4       0x20
 .text.MRF24W_MACPowerDown
                0x9d03b1c4       0x20 build/default/production/_ext/334706090/wf_mac_24g.o
                0x9d03b1c4                MRF24W_MACPowerDown

.text.MRF24W_MACPowerUp
                0x9d03b1e4       0x20
 .text.MRF24W_MACPowerUp
                0x9d03b1e4       0x20 build/default/production/_ext/334706090/wf_mac_24g.o
                0x9d03b1e4                MRF24W_MACPowerUp

.text.SpiChnReadC
                0x9d03b204       0x20
 .text.SpiChnReadC
                0x9d03b204       0x20 c:/program files (x86)/microchip/xc32/v1.10/bin/../lib/gcc/pic32mx/4.5.1/../../../../pic32mx/lib/size\libmchp_peripheral_32MX795F512L.a(spi_chn_getc_lib.o)
                0x9d03b204                SpiChnReadC

.text.SpiChnWriteC
                0x9d03b224       0x20
 .text.SpiChnWriteC
                0x9d03b224       0x20 c:/program files (x86)/microchip/xc32/v1.10/bin/../lib/gcc/pic32mx/4.5.1/../../../../pic32mx/lib/size\libmchp_peripheral_32MX795F512L.a(spi_chn_putc_lib.o)
                0x9d03b224                SpiChnWriteC

.text.SpiChnTxBuffEmpty
                0x9d03b244       0x20
 .text.SpiChnTxBuffEmpty
                0x9d03b244       0x20 c:/program files (x86)/microchip/xc32/v1.10/bin/../lib/gcc/pic32mx/4.5.1/../../../../pic32mx/lib/size\libmchp_peripheral_32MX795F512L.a(spi_chn_tx_buff_empty_lib.o)
                0x9d03b244                SpiChnTxBuffEmpty

.text.INTRestoreInterrupts
                0x9d03b264       0x1c
 .text.INTRestoreInterrupts
                0x9d03b264       0x1c c:/program files (x86)/microchip/xc32/v1.10/bin/../lib/gcc/pic32mx/4.5.1/../../../../pic32mx/lib/size\libmchp_peripheral_32MX795F512L.a(int_restore_interrupts_lib.o)
                0x9d03b264                INTRestoreInterrupts

.text.srand     0x9d03b280       0x1c
 .text.srand    0x9d03b280       0x1c c:/program files (x86)/microchip/xc32/v1.10/bin/../lib/gcc/pic32mx/4.5.1/../../../../pic32mx/lib/size\libc.a(rand.o)
                0x9d03b280                srand

.text.SYS_Reboot
                0x9d03b29c       0x18
 .text.SYS_Reboot
                0x9d03b29c       0x18 build/default/production/_ext/365611741/system_services.o
                0x9d03b29c                SYS_Reboot

.text.CheKseg0CacheOn
                0x9d03b2b4       0x18
 .text.CheKseg0CacheOn
                0x9d03b2b4       0x18 c:/program files (x86)/microchip/xc32/v1.10/bin/../lib/gcc/pic32mx/4.5.1/../../../../pic32mx/lib/size\libmchp_peripheral_32MX795F512L.a(pcache.o)
                0x9d03b2b4                CheKseg0CacheOn

.text           0x9d03b2cc       0x18
 .text          0x9d03b2cc       0x18 c:/program files (x86)/microchip/xc32/v1.10/bin/../lib/gcc/pic32mx/4.5.1/../../../../pic32mx/lib/size\libpic32.a(default-nmi-handler.o)
                0x9d03b2cc                _nmi_handler

.rodata         0x9d03b2e4       0x34
 .rodata        0x9d03b2e4       0x14 c:/program files (x86)/microchip/xc32/v1.10/bin/../lib/gcc/pic32mx/4.5.1/../../../../pic32mx/lib/size\libmchp_peripheral_32MX795F512L.a(spi_map_tbl_libp.o)
                0x9d03b2e4                _SpiMapTbl
 .rodata        0x9d03b2f8       0x10 build/default/production/_ext/97638081/mpfs2.o
 .rodata        0x9d03b308       0x10 build/default/production/_ext/427700826/dhcp.o

.text.OpenCoreTimer
                0x9d03b318        0xc
 .text.OpenCoreTimer
                0x9d03b318        0xc c:/program files (x86)/microchip/xc32/v1.10/bin/../lib/gcc/pic32mx/4.5.1/../../../../pic32mx/lib/size\libmchp_peripheral.a(open_core_timer_lib.o)
                0x9d03b318                OpenCoreTimer

.text._bootstrap_exception_handler
                0x9d03b324        0xc
 .text._bootstrap_exception_handler
                0x9d03b324        0xc c:/program files (x86)/microchip/xc32/v1.10/bin/../lib/gcc/pic32mx/4.5.1/../../../../pic32mx/lib/size\libpic32.a(default-bootstrap-exception-handler.o)
                0x9d03b324                _bootstrap_exception_handler

.text.INTDisableInterrupts
                0x9d03b330        0x8
 .text.INTDisableInterrupts
                0x9d03b330        0x8 c:/program files (x86)/microchip/xc32/v1.10/bin/../lib/gcc/pic32mx/4.5.1/../../../../pic32mx/lib/size\libmchp_peripheral_32MX795F512L.a(int_disable_interrupts_lib.o)
                0x9d03b330                INTDisableInterrupts

.text.INTEnableInterrupts
                0x9d03b338        0x8
 .text.INTEnableInterrupts
                0x9d03b338        0x8 c:/program files (x86)/microchip/xc32/v1.10/bin/../lib/gcc/pic32mx/4.5.1/../../../../pic32mx/lib/size\libmchp_peripheral_32MX795F512L.a(int_enable_interrupts_lib.o)
                0x9d03b338                INTEnableInterrupts

.text._on_reset
                0x9d03b340        0x8
 .text._on_reset
                0x9d03b340        0x8 c:/program files (x86)/microchip/xc32/v1.10/bin/../lib/gcc/pic32mx/4.5.1/../../../../pic32mx/lib/size\libpic32.a(default-on-reset.o)
                0x9d03b340                _on_reset

.text._on_bootstrap
                0x9d03b348        0x8
 .text._on_bootstrap
                0x9d03b348        0x8 c:/program files (x86)/microchip/xc32/v1.10/bin/../lib/gcc/pic32mx/4.5.1/../../../../pic32mx/lib/size\libpic32.a(default-on-bootstrap.o)
                0x9d03b348                _on_bootstrap

.rodata         0x9d03b350        0x8
 .rodata        0x9d03b350        0x8 c:/program files (x86)/microchip/xc32/v1.10/bin/../lib/gcc/pic32mx/4.5.1/size\libgcc.a(_floatundisf.o)

.rodata         0x9d02a904        0x4
 .rodata        0x9d02a904        0x4 build/default/production/_ext/427700826/tcpip_announce.o
